 jpackage

 Timestamp is ffffffff (Sun Feb  7 06:28:15 2106)

 Preferred load address is 10000000

 Start         Length     Name                   Class
 0001:00000000 00000030H .text$di                CODE
 0001:00000030 0000bf2eH .text$mn                CODE
 0001:0000bf5e 000017f9H .text$x                 CODE
 0001:0000d757 0000002bH .text$yd                CODE
 0002:00000000 00000320H .idata$5                DATA
 0002:00000320 00000004H .00cfg                  DATA
 0002:00000324 00000004H .CRT$XCA                DATA
 0002:00000328 00000004H .CRT$XCL                DATA
 0002:0000032c 0000000cH .CRT$XCU                DATA
 0002:00000338 00000004H .CRT$XCZ                DATA
 0002:0000033c 00000004H .CRT$XIA                DATA
 0002:00000340 00000004H .CRT$XIZ                DATA
 0002:00000344 00000004H .CRT$XPA                DATA
 0002:00000348 00000004H .CRT$XPZ                DATA
 0002:0000034c 00000004H .CRT$XTA                DATA
 0002:00000350 00000008H .CRT$XTZ                DATA
 0002:00000354 00000000H .gfids$y                DATA
 0002:00000358 00001620H .rdata                  DATA
 0002:00001978 00000e24H .rdata$r                DATA
 0002:0000279c 0000018cH .rdata$sxdata           DATA
 0002:00002928 0000030cH .rdata$zzzdbg           DATA
 0002:00002c34 00000004H .rtc$IAA                DATA
 0002:00002c38 00000004H .rtc$IZZ                DATA
 0002:00002c3c 00000004H .rtc$TAA                DATA
 0002:00002c40 00000008H .rtc$TZZ                DATA
 0002:00002c48 00001d38H .xdata$x                DATA
 0002:00004980 00000308H .edata                  DATA
 0002:00004c88 000000dcH .idata$2                DATA
 0002:00004d64 00000014H .idata$3                DATA
 0002:00004d78 00000320H .idata$4                DATA
 0002:00005098 00001e3cH .idata$6                DATA
 0003:00000000 00000248H .data                   DATA
 0003:00000248 00000820H .data$r                 DATA
 0003:00000a68 000003a4H .bss                    DATA
 0004:00000000 00000060H .rsrc$01                DATA
 0004:00000060 00000328H .rsrc$02                DATA

  Address         Publics by Value              Rva+Base       Lib:Object

 0000:00000000       ___guard_eh_cont_count     00000000     <absolute>
 0000:00000000       ___arm64x_redirection_metadata 00000000     <absolute>
 0000:00000000       ___guard_fids_count        00000000     <absolute>
 0000:00000000       ___guard_longjmp_table     00000000     <absolute>
 0000:00000000       ___hybrid_code_map_count   00000000     <absolute>
 0000:00000000       ___arm64x_extra_rfe_table_size 00000000     <absolute>
 0000:00000000       ___volatile_metadata       00000000     <absolute>
 0000:00000000       ___arm64x_extra_rfe_table  00000000     <absolute>
 0000:00000000       ___arm64x_native_entrypoint 00000000     <absolute>
 0000:00000000       ___guard_iat_count         00000000     <absolute>
 0000:00000000       ___AbsoluteZero            00000000     <absolute>
 0000:00000000       ___dynamic_value_reloc_table 00000000     <absolute>
 0000:00000000       ___guard_longjmp_count     00000000     <absolute>
 0000:00000000       ___guard_fids_table        00000000     <absolute>
 0000:00000000       ___x64_code_ranges_to_entry_points 00000000     <absolute>
 0000:00000000       ___x64_code_ranges_to_entry_points_count 00000000     <absolute>
 0000:00000000       ___hybrid_code_map         00000000     <absolute>
 0000:00000000       ___guard_iat_table         00000000     <absolute>
 0000:00000000       ___enclave_config          00000000     <absolute>
 0000:00000000       ___arm64x_redirection_metadata_count 00000000     <absolute>
 0000:00000000       ___hybrid_auxiliary_iat    00000000     <absolute>
 0000:00000000       ___guard_eh_cont_table     00000000     <absolute>
 0000:00000063       ___safe_se_handler_count   00000063     <absolute>
 0000:00000100       ___guard_flags             00000100     <absolute>
 0000:00000000       ___ImageBase               10000000     <linker-defined>
 0001:00000030       ??$?6DU?$char_traits@D@std@@V?$allocator@D@1@@std@@YAAAV?$basic_ostream@DU?$char_traits@D@std@@@0@AAV10@ABV?$basic_string@DU?$char_traits@D@std@@V?$allocator@D@2@@0@@Z 10001030 f i ErrorHandling.obj
 0001:0000004f       ??$?6GU?$char_traits@G@std@@@std@@YAAAV?$basic_ostream@GU?$char_traits@G@std@@@0@AAV10@PBD@Z 1000104f f i ErrorHandling.obj
 0001:0000026b       ??$?6GU?$char_traits@G@std@@@std@@YAAAV?$basic_ostream@GU?$char_traits@G@std@@@0@AAV10@PBG@Z 1000126b f i ErrorHandling.obj
 0001:000003e6       ??$?6GU?$char_traits@G@std@@V?$allocator@G@1@@std@@YAAAV?$basic_ostream@GU?$char_traits@G@std@@@0@AAV10@ABV?$basic_string@GU?$char_traits@G@std@@V?$allocator@G@2@@0@@Z 100013e6 f i ErrorHandling.obj
 0001:00000405       ??$?6PBD@any@tstrings@@QAEAAV01@PBD@Z 10001405 f i ErrorHandling.obj
 0001:0000041a       ??$?6U?$char_traits@D@std@@@std@@YAAAV?$basic_ostream@DU?$char_traits@D@std@@@0@AAV10@PBD@Z 1000141a f i ErrorHandling.obj
 0001:0000058c       ??$_Allocate@$07U_Default_allocate_traits@std@@$0A@@std@@YAPAXI@Z 1000158c f i ErrorHandling.obj
 0001:000005ae       ??$_Allocate_manually_vector_aligned@U_Default_allocate_traits@std@@@std@@YAPAXI@Z 100015ae f i ErrorHandling.obj
 0001:000005da       ??$_Deallocate@$07$0A@@std@@YAXPAXI@Z 100015da f i ErrorHandling.obj
 0001:00000606       ??$_Insert_string@DU?$char_traits@D@std@@I@std@@YAAAV?$basic_ostream@DU?$char_traits@D@std@@@0@AAV10@QBDI@Z 10001606 f i ErrorHandling.obj
 0001:00000741       ??$_Insert_string@GU?$char_traits@G@std@@I@std@@YAAAV?$basic_ostream@GU?$char_traits@G@std@@@0@AAV10@QBGI@Z 10001741 f i ErrorHandling.obj
 0001:00000884       ??$_Reallocate_for@V<lambda_2b7e716477254df52771775b37436d39>@@PBG@?$basic_string@GU?$char_traits@G@std@@V?$allocator@G@2@@std@@AAEAAV01@IV<lambda_2b7e716477254df52771775b37436d39>@@PBG@Z 10001884 f i ErrorHandling.obj
 0001:000008fe       ??$_Reallocate_for@V<lambda_9366063389c5f42a00a5088cf24e69de>@@PBD@?$basic_string@DU?$char_traits@D@std@@V?$allocator@D@2@@std@@AAEAAV01@IV<lambda_9366063389c5f42a00a5088cf24e69de>@@PBD@Z 100018fe f i ErrorHandling.obj
 0001:0000096a       ??$_Traits_find_ch@U?$char_traits@D@std@@@std@@YAIQBDIID@Z 1000196a f i ErrorHandling.obj
 0001:0000099d       ??$_Traits_find_last_of@U?$char_traits@D@std@@@std@@YAIQBDII0IU?$integral_constant@_N$00@0@@Z 1000199d f i ErrorHandling.obj
 0001:00000a4b       ??$find_if@V?$_String_const_iterator@V?$_String_val@U?$_Simple_types@D@std@@@std@@@std@@P6A_NH@Z@std@@YA?AV?$_String_const_iterator@V?$_String_val@U?$_Simple_types@D@std@@@std@@@0@V10@V10@P6A_NH@Z@Z 10001a4b f i ErrorHandling.obj
 0001:00000a72       ??$find_if@V?$reverse_iterator@V?$_String_const_iterator@V?$_String_val@U?$_Simple_types@D@std@@@std@@@std@@@std@@P6A_NH@Z@std@@YA?AV?$reverse_iterator@V?$_String_const_iterator@V?$_String_val@U?$_Simple_types@D@std@@@std@@@std@@@0@V10@V10@P6A_NH@Z@Z 10001a72 f i ErrorHandling.obj
 0001:00000a9e       ??$use_facet@V?$ctype@G@std@@@std@@YAABV?$ctype@G@0@ABVlocale@0@@Z 10001a9e f i ErrorHandling.obj
 0001:00000b2f       ??0?$basic_ostringstream@DU?$char_traits@D@std@@V?$allocator@D@2@@std@@QAE@XZ 10001b2f f i ErrorHandling.obj
 0001:00000ba3       ??0?$basic_ostringstream@GU?$char_traits@G@std@@V?$allocator@G@2@@std@@QAE@XZ 10001ba3 f i ErrorHandling.obj
 0001:00000c17       ??0?$basic_string@DU?$char_traits@D@std@@V?$allocator@D@2@@std@@QAE@QBD@Z 10001c17 f i ErrorHandling.obj
 0001:00000c44       ??0?$basic_string@GU?$char_traits@G@std@@V?$allocator@G@2@@std@@QAE@$$QAV01@@Z 10001c44 f i ErrorHandling.obj
 0001:00000c68       ??0?$basic_string@GU?$char_traits@G@std@@V?$allocator@G@2@@std@@QAE@QBG@Z 10001c68 f i ErrorHandling.obj
 0001:00000c98       ??0?$basic_stringbuf@DU?$char_traits@D@std@@V?$allocator@D@2@@std@@QAE@H@Z 10001c98 f i ErrorHandling.obj
 0001:00000cc5       ??0?$basic_stringbuf@GU?$char_traits@G@std@@V?$allocator@G@2@@std@@QAE@H@Z 10001cc5 f i ErrorHandling.obj
 0001:00000cf2       ??0_Sentry_base@?$basic_ostream@DU?$char_traits@D@std@@@std@@QAE@AAV12@@Z 10001cf2 f i ErrorHandling.obj
 0001:00000cf2       ??0_Sentry_base@?$basic_ostream@GU?$char_traits@G@std@@@std@@QAE@AAV12@@Z 10001cf2 f i ErrorHandling.obj
 0001:00000d13       ??0any@tstrings@@QAE@ABV?$basic_string@GU?$char_traits@G@std@@V?$allocator@G@2@@std@@@Z 10001d13 f i ErrorHandling.obj
 0001:00000d44       ??0any@tstrings@@QAE@XZ    10001d44 f i ErrorHandling.obj
 0001:00000d58       ??0bad_alloc@std@@QAE@ABV01@@Z 10001d58 f i ErrorHandling.obj
 0001:00000d70       ??0bad_array_new_length@std@@QAE@ABV01@@Z 10001d70 f i ErrorHandling.obj
 0001:00000d88       ??0bad_array_new_length@std@@QAE@XZ 10001d88 f i ErrorHandling.obj
 0001:00000da0       ??0bad_cast@std@@QAE@ABV01@@Z 10001da0 f i ErrorHandling.obj
 0001:00000db8       ??0bad_cast@std@@QAE@XZ    10001db8 f i ErrorHandling.obj
 0001:00000dd0       ??0exception@std@@QAE@ABV01@@Z 10001dd0 f i ErrorHandling.obj
 0001:00000df9       ??0sentry@?$basic_ostream@DU?$char_traits@D@std@@@std@@QAE@AAV12@@Z 10001df9 f i ErrorHandling.obj
 0001:00000e52       ??0sentry@?$basic_ostream@GU?$char_traits@G@std@@@std@@QAE@AAV12@@Z 10001e52 f i ErrorHandling.obj
 0001:00000eab       ??1?$basic_ostringstream@DU?$char_traits@D@std@@V?$allocator@D@2@@std@@UAE@XZ 10001eab f i ErrorHandling.obj
 0001:00000edb       ??1?$basic_ostringstream@GU?$char_traits@G@std@@V?$allocator@G@2@@std@@UAE@XZ 10001edb f i ErrorHandling.obj
 0001:00000f0b       ??1?$basic_string@DU?$char_traits@D@std@@V?$allocator@D@2@@std@@QAE@XZ 10001f0b f i ErrorHandling.obj
 0001:00000f10       ??1?$basic_string@GU?$char_traits@G@std@@V?$allocator@G@2@@std@@QAE@XZ 10001f10 f i ErrorHandling.obj
 0001:00000f15       ??1?$basic_stringbuf@DU?$char_traits@D@std@@V?$allocator@D@2@@std@@UAE@XZ 10001f15 f i ErrorHandling.obj
 0001:00000f2c       ??1?$basic_stringbuf@GU?$char_traits@G@std@@V?$allocator@G@2@@std@@UAE@XZ 10001f2c f i ErrorHandling.obj
 0001:00000f43       ??1?$unique_ptr@V_Facet_base@std@@U?$default_delete@V_Facet_base@std@@@2@@std@@QAE@XZ 10001f43 f i ErrorHandling.obj
 0001:00000f50       ??1_Sentry_base@?$basic_ostream@DU?$char_traits@D@std@@@std@@QAE@XZ 10001f50 f i ErrorHandling.obj
 0001:00000f50       ??1_Sentry_base@?$basic_ostream@GU?$char_traits@G@std@@@std@@QAE@XZ 10001f50 f i ErrorHandling.obj
 0001:00000f98       ??1any@tstrings@@QAE@XZ    10001f98 f i ErrorHandling.obj
 0001:00000f9d       ??1SysError@@UAE@XZ        10001f9d f i MsiUtils.obj
 0001:00000f9d       ??1bad_array_new_length@std@@UAE@XZ 10001f9d f i ErrorHandling.obj
 0001:00000f9d       ??1runtime_error@std@@UAE@XZ 10001f9d f i Guid.obj
 0001:00000f9d       ??1bad_alloc@std@@UAE@XZ   10001f9d f i ErrorHandling.obj
 0001:00000f9d       ??1bad_cast@std@@UAE@XZ    10001f9d f i ErrorHandling.obj
 0001:00000f9d       ??1invalid_argument@std@@UAE@XZ 10001f9d f i tstrings.obj
 0001:00000f9d       ??1NoMoreItemsError@msi@@UAE@XZ 10001f9d f i MsiDb.obj
 0001:00000f9d       ??1Error@msi@@UAE@XZ       10001f9d f i MsiDb.obj
 0001:00000fae       ??1locale@std@@QAE@XZ      10001fae f i ErrorHandling.obj
 0001:00000fc7       ??1sentry@?$basic_ostream@DU?$char_traits@D@std@@@std@@QAE@XZ 10001fc7 f i ErrorHandling.obj
 0001:00001017       ??1sentry@?$basic_ostream@GU?$char_traits@G@std@@@std@@QAE@XZ 10002017 f i ErrorHandling.obj
 0001:00001067       ??6@YAAAV?$basic_ostream@DU?$char_traits@D@std@@@std@@AAV01@ABVany@tstrings@@@Z 10002067 f i ErrorHandling.obj
 0001:0000109f       ??_D?$basic_ostringstream@DU?$char_traits@D@std@@V?$allocator@D@2@@std@@QAEXXZ 1000209f f i ErrorHandling.obj
 0001:000010b3       ??_D?$basic_ostringstream@GU?$char_traits@G@std@@V?$allocator@G@2@@std@@QAEXXZ 100020b3 f i ErrorHandling.obj
 0001:000010c7       ??_E?$basic_ostringstream@DU?$char_traits@D@std@@V?$allocator@D@2@@std@@$4PPPPPPPM@A@AEPAXI@Z 100020c7 f i ErrorHandling.obj
 0001:000010cf       ??_E?$basic_ostringstream@GU?$char_traits@G@std@@V?$allocator@G@2@@std@@$4PPPPPPPM@A@AEPAXI@Z 100020cf f i ErrorHandling.obj
 0001:000010d7       ??_G?$basic_ostringstream@DU?$char_traits@D@std@@V?$allocator@D@2@@std@@UAEPAXI@Z 100020d7 f i ErrorHandling.obj
 0001:000010d7       ??_E?$basic_ostringstream@DU?$char_traits@D@std@@V?$allocator@D@2@@std@@UAEPAXI@Z 100020d7 f i ErrorHandling.obj
 0001:000010fc       ??_G?$basic_ostringstream@GU?$char_traits@G@std@@V?$allocator@G@2@@std@@UAEPAXI@Z 100020fc f i ErrorHandling.obj
 0001:000010fc       ??_E?$basic_ostringstream@GU?$char_traits@G@std@@V?$allocator@G@2@@std@@UAEPAXI@Z 100020fc f i ErrorHandling.obj
 0001:00001121       ??_E?$basic_stringbuf@DU?$char_traits@D@std@@V?$allocator@D@2@@std@@UAEPAXI@Z 10002121 f i ErrorHandling.obj
 0001:00001121       ??_G?$basic_stringbuf@DU?$char_traits@D@std@@V?$allocator@D@2@@std@@UAEPAXI@Z 10002121 f i ErrorHandling.obj
 0001:00001140       ??_G?$basic_stringbuf@GU?$char_traits@G@std@@V?$allocator@G@2@@std@@UAEPAXI@Z 10002140 f i ErrorHandling.obj
 0001:00001140       ??_E?$basic_stringbuf@GU?$char_traits@G@std@@V?$allocator@G@2@@std@@UAEPAXI@Z 10002140 f i ErrorHandling.obj
 0001:0000115f       ??_GSysError@@UAEPAXI@Z    1000215f f i MsiUtils.obj
 0001:0000115f       ??_Gexception@std@@UAEPAXI@Z 1000215f f i ErrorHandling.obj
 0001:0000115f       ??_Ebad_array_new_length@std@@UAEPAXI@Z 1000215f f i ErrorHandling.obj
 0001:0000115f       ??_Eruntime_error@std@@UAEPAXI@Z 1000215f f i Guid.obj
 0001:0000115f       ??_Einvalid_argument@std@@UAEPAXI@Z 1000215f f i tstrings.obj
 0001:0000115f       ??_Gbad_cast@std@@UAEPAXI@Z 1000215f f i ErrorHandling.obj
 0001:0000115f       ??_Elogic_error@std@@UAEPAXI@Z 1000215f f i tstrings.obj
 0001:0000115f       ??_Ebad_cast@std@@UAEPAXI@Z 1000215f f i ErrorHandling.obj
 0001:0000115f       ??_Gbad_array_new_length@std@@UAEPAXI@Z 1000215f f i ErrorHandling.obj
 0001:0000115f       ??_Gbad_alloc@std@@UAEPAXI@Z 1000215f f i ErrorHandling.obj
 0001:0000115f       ??_Glogic_error@std@@UAEPAXI@Z 1000215f f i tstrings.obj
 0001:0000115f       ??_Ebad_alloc@std@@UAEPAXI@Z 1000215f f i ErrorHandling.obj
 0001:0000115f       ??_Ginvalid_argument@std@@UAEPAXI@Z 1000215f f i tstrings.obj
 0001:0000115f       ??_Eexception@std@@UAEPAXI@Z 1000215f f i ErrorHandling.obj
 0001:0000115f       ??_Gruntime_error@std@@UAEPAXI@Z 1000215f f i Guid.obj
 0001:0000115f       ??_ESysError@@UAEPAXI@Z    1000215f f i MsiUtils.obj
 0001:00001189       ?_Adjust_manually_vector_aligned@std@@YAXAAPAXAAI@Z 10002189 f i ErrorHandling.obj
 0001:000011ac       ?_Calculate_growth@?$basic_string@DU?$char_traits@D@std@@V?$allocator@D@2@@std@@CAIIII@Z 100021ac f i ErrorHandling.obj
 0001:000011dd       ?_Calculate_growth@?$basic_string@GU?$char_traits@G@std@@V?$allocator@G@2@@std@@CAIIII@Z 100021dd f i ErrorHandling.obj
 0001:0000120e       ?_Construct_lv_contents@?$basic_string@DU?$char_traits@D@std@@V?$allocator@D@2@@std@@AAEXABV12@@Z 1000220e f i ErrorHandling.obj
 0001:0000127c       ?_Getfacet@locale@std@@QBEPBVfacet@12@I@Z 1000227c f i ErrorHandling.obj
 0001:000012b5       ?_Getstate@?$basic_stringbuf@GU?$char_traits@G@std@@V?$allocator@G@2@@std@@CAHH@Z 100022b5 f i ErrorHandling.obj
 0001:000012b5       ?_Getstate@?$basic_stringbuf@DU?$char_traits@D@std@@V?$allocator@D@2@@std@@CAHH@Z 100022b5 f i ErrorHandling.obj
 0001:000012e9       ?_Take_contents@?$basic_string@DU?$char_traits@D@std@@V?$allocator@D@2@@std@@AAEXAAV12@U?$integral_constant@_N$00@2@@Z 100022e9 f i ErrorHandling.obj
 0001:0000130c       ?_Take_contents@?$basic_string@GU?$char_traits@G@std@@V?$allocator@G@2@@std@@AAEXAAV12@U?$integral_constant@_N$00@2@@Z 1000230c f i ErrorHandling.obj
 0001:00001331       ?__scrt_throw_std_bad_array_new_length@@YAXXZ 10002331 f i MSVCRT:throw_bad_alloc.obj
 0001:00001331       ?_Throw_bad_array_new_length@std@@YAXXZ 10002331 f i ErrorHandling.obj
 0001:0000134e       ?_Throw_bad_cast@std@@YAXXZ 1000234e f i ErrorHandling.obj
 0001:0000136b       ?_Tidy@?$basic_stringbuf@DU?$char_traits@D@std@@V?$allocator@D@2@@std@@IAEXXZ 1000236b f i ErrorHandling.obj
 0001:000013c8       ?_Tidy@?$basic_stringbuf@GU?$char_traits@G@std@@V?$allocator@G@2@@std@@IAEXXZ 100023c8 f i ErrorHandling.obj
 0001:0000142c       ?_Tidy_deallocate@?$basic_string@DU?$char_traits@D@std@@V?$allocator@D@2@@std@@AAEXXZ 1000242c f i ErrorHandling.obj
 0001:00001452       ?_Tidy_deallocate@?$basic_string@GU?$char_traits@G@std@@V?$allocator@G@2@@std@@AAEXXZ 10002452 f i ErrorHandling.obj
 0001:00001480       ?_Xlen_string@std@@YAXXZ   10002480 f i ErrorHandling.obj
 0001:0000148b       ?_Xran@?$_String_val@U?$_Simple_types@D@std@@@std@@SAXXZ 1000248b f i ErrorHandling.obj
 0001:0000148b       ?_Xran@?$_String_val@U?$_Simple_types@G@std@@@std@@SAXXZ 1000248b f i FileUtils.obj
 0001:00001496       ?allocate@?$allocator@G@std@@QAEPAGI@Z 10002496 f i ErrorHandling.obj
 0001:000014b3       ?assign@?$basic_string@DU?$char_traits@D@std@@V?$allocator@D@2@@std@@QAEAAV12@ABV12@II@Z 100024b3 f i ErrorHandling.obj
 0001:000014ef       ?assign@?$basic_string@DU?$char_traits@D@std@@V?$allocator@D@2@@std@@QAEAAV12@QBDI@Z 100024ef f i ErrorHandling.obj
 0001:00001538       ?assign@?$basic_string@GU?$char_traits@G@std@@V?$allocator@G@2@@std@@QAEAAV12@QBGI@Z 10002538 f i ErrorHandling.obj
 0001:00001583       ?find@?$basic_string@DU?$char_traits@D@std@@V?$allocator@D@2@@std@@QBEIDI@Z 10002583 f i ErrorHandling.obj
 0001:000015a4       ?find_last_of@?$basic_string@DU?$char_traits@D@std@@V?$allocator@D@2@@std@@QBEIQBDI@Z 100025a4 f i ErrorHandling.obj
 0001:000016ac       ?joinErrorMessages@@YA?AV?$basic_string@DU?$char_traits@D@std@@V?$allocator@D@2@@std@@ABV12@0@Z 100026ac f   ErrorHandling.obj
 0001:0000186c       ?makeMessage@@YA?AV?$basic_string@DU?$char_traits@D@std@@V?$allocator@D@2@@std@@ABVruntime_error@2@ABUSourceCodePos@@@Z 1000286c f   ErrorHandling.obj
 0001:00001956       ?overflow@?$basic_stringbuf@DU?$char_traits@D@std@@V?$allocator@D@2@@std@@MAEHH@Z 10002956 f i ErrorHandling.obj
 0001:00001a7d       ?overflow@?$basic_stringbuf@GU?$char_traits@G@std@@V?$allocator@G@2@@std@@MAEGG@Z 10002a7d f i ErrorHandling.obj
 0001:00001bdd       ?pbackfail@?$basic_stringbuf@DU?$char_traits@D@std@@V?$allocator@D@2@@std@@MAEHH@Z 10002bdd f i ErrorHandling.obj
 0001:00001c2d       ?pbackfail@?$basic_stringbuf@GU?$char_traits@G@std@@V?$allocator@G@2@@std@@MAEGG@Z 10002c2d f i ErrorHandling.obj
 0001:00001dbd       ?reportError@@YAXABUSourceCodePos@@ABVruntime_error@std@@@Z 10002dbd f   ErrorHandling.obj
 0001:00001e56       ?reportUnknownError@@YAXABUSourceCodePos@@@Z 10002e56 f   ErrorHandling.obj
 0001:00001e90       ?seekoff@?$basic_stringbuf@DU?$char_traits@D@std@@V?$allocator@D@2@@std@@MAE?AV?$fpos@U_Mbstatet@@@2@_JHH@Z 10002e90 f i ErrorHandling.obj
 0001:00001fe9       ?seekoff@?$basic_stringbuf@GU?$char_traits@G@std@@V?$allocator@G@2@@std@@MAE?AV?$fpos@U_Mbstatet@@@2@_JHH@Z 10002fe9 f i ErrorHandling.obj
 0001:0000217a       ?seekpos@?$basic_stringbuf@DU?$char_traits@D@std@@V?$allocator@D@2@@std@@MAE?AV?$fpos@U_Mbstatet@@@2@V32@H@Z 1000317a f i ErrorHandling.obj
 0001:00002264       ?seekpos@?$basic_stringbuf@GU?$char_traits@G@std@@V?$allocator@G@2@@std@@MAE?AV?$fpos@U_Mbstatet@@@2@V32@H@Z 10003264 f i ErrorHandling.obj
 0001:0000235a       ?str@?$basic_stringbuf@DU?$char_traits@D@std@@V?$allocator@D@2@@std@@QBE?AV?$basic_string@DU?$char_traits@D@std@@V?$allocator@D@2@@2@XZ 1000335a f i ErrorHandling.obj
 0001:000023d1       ?str@?$basic_stringbuf@GU?$char_traits@G@std@@V?$allocator@G@2@@std@@QBE?AV?$basic_string@GU?$char_traits@G@std@@V?$allocator@G@2@@2@XZ 100033d1 f i ErrorHandling.obj
 0001:00002456       ?str@any@tstrings@@QBE?AV?$basic_string@DU?$char_traits@D@std@@V?$allocator@D@2@@std@@XZ 10003456 f i ErrorHandling.obj
 0001:00002496       ?underflow@?$basic_stringbuf@DU?$char_traits@D@std@@V?$allocator@D@2@@std@@MAEHXZ 10003496 f i ErrorHandling.obj
 0001:000024e9       ?underflow@?$basic_stringbuf@GU?$char_traits@G@std@@V?$allocator@G@2@@std@@MAEGXZ 100034e9 f i ErrorHandling.obj
 0001:00002543       ?what@exception@std@@UBEPBDXZ 10003543 f i ErrorHandling.obj
 0001:00002551       _wmemcpy                   10003551 f i ErrorHandling.obj
 0001:00002569       _wmemmove                  10003569 f i ErrorHandling.obj
 0001:00002581       ??$_Reallocate_grow_by@V<lambda_2b70dce17ee1239412236ff821cd936e>@@IG@?$basic_string@GU?$char_traits@G@std@@V?$allocator@G@2@@std@@AAEAAV01@IV<lambda_2b70dce17ee1239412236ff821cd936e>@@IG@Z 10003581 f i FileUtils.obj
 0001:00002616       ??$_Reallocate_grow_by@V<lambda_68b8a09d57a0de6c0cf526835bc8b658>@@PBGI@?$basic_string@GU?$char_traits@G@std@@V?$allocator@G@2@@std@@AAEAAV01@IV<lambda_68b8a09d57a0de6c0cf526835bc8b658>@@PBGI@Z 10003616 f i FileUtils.obj
 0001:000026ab       ??$_Traits_find_last_of@U?$char_traits@G@std@@@std@@YAIQBGII0IU?$integral_constant@_N$00@0@@Z 100036ab f i FileUtils.obj
 0001:00002784       ??$_Traits_find_last_of@U?$char_traits@G@std@@@std@@YAIQBGII0IU?$integral_constant@_N$0A@@0@@Z 10003784 f i FileUtils.obj
 0001:000027d3       ??R<lambda_2b70dce17ee1239412236ff821cd936e>@@QBEXQAGQBGIIG@Z 100037d3 f i FileUtils.obj
 0001:0000280c       ??R<lambda_68b8a09d57a0de6c0cf526835bc8b658>@@QBEXQAGQBGI1I@Z 1000380c f i FileUtils.obj
 0001:00002845       ?_Construct_lv_contents@?$basic_string@GU?$char_traits@G@std@@V?$allocator@G@2@@std@@AAEXABV12@@Z 10003845 f i FileUtils.obj
 0001:000028a5       ?_Mark@?$_String_bitmap@G$0A@@std@@QAE_NPBGQBG@Z 100038a5 f i FileUtils.obj
 0001:000028d3       ?_Match@?$_String_bitmap@G$0A@@std@@QBE_NG@Z 100038d3 f i FileUtils.obj
 0001:000028f4       ?append@?$basic_string@GU?$char_traits@G@std@@V?$allocator@G@2@@std@@QAEAAV12@IG@Z 100038f4 f i FileUtils.obj
 0001:0000294f       ?append@?$basic_string@GU?$char_traits@G@std@@V?$allocator@G@2@@std@@QAEAAV12@QBGI@Z 1000394f f i FileUtils.obj
 0001:000029aa       ?assign@?$basic_string@GU?$char_traits@G@std@@V?$allocator@G@2@@std@@QAEAAV12@ABV12@II@Z 100039aa f i FileUtils.obj
 0001:000029e7       ?basename@FileUtils@@YA?AV?$basic_string@GU?$char_traits@G@std@@V?$allocator@G@2@@std@@ABV23@@Z 100039e7 f   FileUtils.obj
 0001:00002a37       ?combinePath@FileUtils@@YA?AV?$basic_string@GU?$char_traits@G@std@@V?$allocator@G@2@@std@@ABV23@0@Z 10003a37 f   FileUtils.obj
 0001:00002c2d       ?find_last_of@?$basic_string@GU?$char_traits@G@std@@V?$allocator@G@2@@std@@QBEIQBGI@Z 10003c2d f i FileUtils.obj
 0001:00002c62       ?isDirSeparator@FileUtils@@YA_NG@Z 10003c62 f   FileUtils.obj
 0001:00002c78       ?removeTrailingSlash@FileUtils@@YA?AV?$basic_string@GU?$char_traits@G@std@@V?$allocator@G@2@@std@@ABV23@@Z 10003c78 f   FileUtils.obj
 0001:00002cfa       _wmemchr                   10003cfa f i FileUtils.obj
 0001:00002d1b       _wmemset                   10003d1b f i FileUtils.obj
 0001:00002d45       ??$?HGU?$char_traits@G@std@@V?$allocator@G@1@@std@@YA?AV?$basic_string@GU?$char_traits@G@std@@V?$allocator@G@2@@0@$$QAV10@QBG@Z 10003d45 f i Guid.obj
 0001:00002d6c       ??$?HGU?$char_traits@G@std@@V?$allocator@G@1@@std@@YA?AV?$basic_string@GU?$char_traits@G@std@@V?$allocator@G@2@@0@QBGABV10@@Z 10003d6c f i Guid.obj
 0001:00002db5       ??$_Find_unchecked1@PAGG@std@@YAPAGPAGQAGABGU?$integral_constant@_N$0A@@0@@Z 10003db5 f i Guid.obj
 0001:00002dd7       ??$_Reallocate_grow_by@V<lambda_3e20e6c7e29fb350de04c962bd5a58e9>@@IIG@?$basic_string@GU?$char_traits@G@std@@V?$allocator@G@2@@std@@AAEAAV01@IV<lambda_3e20e6c7e29fb350de04c962bd5a58e9>@@IIG@Z 10003dd7 f i Guid.obj
 0001:00002e70       ??$_Traits_compare@U?$char_traits@G@std@@@std@@YAHQBGI0I@Z 10003e70 f i Guid.obj
 0001:00002ea3       ??$_Traits_find_ch@U?$char_traits@G@std@@@std@@YAIQBGIIG@Z 10003ea3 f i Guid.obj
 0001:00002ed6       ??$remove@V?$_String_iterator@V?$_String_val@U?$_Simple_types@G@std@@@std@@@std@@G@std@@YA?AV?$_String_iterator@V?$_String_val@U?$_Simple_types@G@std@@@std@@@0@V10@V10@ABG@Z 10003ed6 f i Guid.obj
 0001:00002f1c       ??0?$JpError@Vruntime_error@std@@@@QAE@ABV0@@Z 10003f1c f i Guid.obj
 0001:00002f77       ??0?$JpError@Vruntime_error@std@@@@QAE@ABVruntime_error@std@@ABUSourceCodePos@@@Z 10003f77 f i Guid.obj
 0001:00002fcd       ??0?$basic_string@GU?$char_traits@G@std@@V?$allocator@G@2@@std@@QAE@U_String_constructor_concat_tag@1@ABV01@QBGI2I@Z 10003fcd f i Guid.obj
 0001:00003044       ??0Guid@@QAE@ABV?$basic_string@GU?$char_traits@G@std@@V?$allocator@G@2@@std@@@Z 10004044 f   Guid.obj
 0001:000031d0       ??0JpErrorBase@@QAE@ABV0@@Z 100041d0 f i Guid.obj
 0001:000031db       ??0SourceCodePos@@QAE@PBD0H@Z 100041db f i Guid.obj
 0001:000031f4       ??0exception@std@@QAE@QBD@Z 100041f4 f i Guid.obj
 0001:00003229       ??0runtime_error@std@@QAE@ABV01@@Z 10004229 f i Guid.obj
 0001:00003241       ??0runtime_error@std@@QAE@ABV?$basic_string@DU?$char_traits@D@std@@V?$allocator@D@2@@1@@Z 10004241 f i Guid.obj
 0001:00003269       ??1?$JpError@Vruntime_error@std@@@@UAE@XZ 10004269 f i Guid.obj
 0001:00003294       ??4?$basic_string@GU?$char_traits@G@std@@V?$allocator@G@2@@std@@QAEAAV01@$$QAV01@@Z 10004294 f i Guid.obj
 0001:000032b6       ??4?$basic_string@GU?$char_traits@G@std@@V?$allocator@G@2@@std@@QAEAAV01@ABV01@@Z 100042b6 f i Guid.obj
 0001:000032d8       ??6any@tstrings@@QAEAAV01@ABV?$basic_string@GU?$char_traits@G@std@@V?$allocator@G@2@@std@@@Z 100042d8 f i Guid.obj
 0001:000032ed       ??R<lambda_3e20e6c7e29fb350de04c962bd5a58e9>@@QBEXQAGQBGIIIG@Z 100042ed f i Guid.obj
 0001:00003339       ??_E?$JpError@Vruntime_error@std@@@@W3AEPAXI@Z 10004339 f i Guid.obj
 0001:00003341       ??_E?$JpError@Vruntime_error@std@@@@UAEPAXI@Z 10004341 f i Guid.obj
 0001:00003341       ??_G?$JpError@Vruntime_error@std@@@@UAEPAXI@Z 10004341 f i Guid.obj
 0001:00003360       ?_Construct@?$basic_string@GU?$char_traits@G@std@@V?$allocator@G@2@@std@@QAEXQAG0Urandom_access_iterator_tag@2@@Z 10004360 f i Guid.obj
 0001:0000337d       ?_Copy_assign@?$basic_string@GU?$char_traits@G@std@@V?$allocator@G@2@@std@@AAEXABV12@U?$integral_constant@_N$0A@@2@@Z 1000437d f i Guid.obj
 0001:00003397       ?_Move_assign@?$basic_string@GU?$char_traits@G@std@@V?$allocator@G@2@@std@@AAEXAAV12@U_Equal_allocators@2@@Z 10004397 f i Guid.obj
 0001:000033b9       ?compare@?$basic_string@GU?$char_traits@G@std@@V?$allocator@G@2@@std@@QBEHABV12@@Z 100043b9 f i Guid.obj
 0001:000033e6       ?find@?$basic_string@GU?$char_traits@G@std@@V?$allocator@G@2@@std@@QBEIGI@Z 100043e6 f i Guid.obj
 0001:00003407       ?winStringToUtf16@tstrings@@YA?AV?$basic_string@GU?$char_traits@G@std@@V?$allocator@G@2@@std@@ABV23@@Z 10004407 f i tstrings.obj
 0001:00003407       ?fromUtf16@tstrings@@YA?AV?$basic_string@GU?$char_traits@G@std@@V?$allocator@G@2@@std@@ABV23@@Z 10004407 f i Guid.obj
 0001:000034b6       ?insert@?$basic_string@GU?$char_traits@G@std@@V?$allocator@G@2@@std@@QAEAAV12@IIG@Z 100044b6 f i Guid.obj
 0001:00003527       ?makeException@@YA?AV?$JpError@Vruntime_error@std@@@@ABV?$basic_string@DU?$char_traits@D@std@@V?$allocator@D@2@@std@@ABUSourceCodePos@@@Z 10004527 f i Guid.obj
 0001:0000357b       ?makeException@@YA?AV?$JpError@Vruntime_error@std@@@@ABVany@tstrings@@ABUSourceCodePos@@@Z 1000457b f i Guid.obj
 0001:000035bb       ?makeException@@YA?AV?$JpError@Vruntime_error@std@@@@PBDABUSourceCodePos@@@Z 100045bb f i Guid.obj
 0001:000035fb       ?rawMessage@?$JpError@VError@msi@@@@UBEPBDXZ 100045fb f i MsiDb.obj
 0001:000035fb       ?rawMessage@?$JpError@VSysError@@@@UBEPBDXZ 100045fb f i MsiUtils.obj
 0001:000035fb       ?rawMessage@?$JpError@Vruntime_error@std@@@@UBEPBDXZ 100045fb f i Guid.obj
 0001:000035fb       ?rawMessage@?$JpError@VNoMoreItemsError@msi@@@@UBEPBDXZ 100045fb f i MsiDb.obj
 0001:00003609       ?toString@Guid@@QBE?AV?$basic_string@GU?$char_traits@G@std@@V?$allocator@G@2@@std@@H@Z 10004609 f   Guid.obj
 0001:00003840       ?what@?$JpError@Vruntime_error@std@@@@UBEPBDXZ 10004840 f i Guid.obj
 0001:00003840       ?what@?$JpError@VSysError@@@@UBEPBDXZ 10004840 f i MsiUtils.obj
 0001:0000384c       _wmemcmp                   1000484c f i Guid.obj
 0001:00003881       ?ChangeIcon@@YA_NPAXABV?$basic_string@GU?$char_traits@G@std@@V?$allocator@G@2@@std@@@Z 10004881 f   IconSwap.obj
 0001:00003ae1       ?PrintError@@YAXXZ         10004ae1 f   IconSwap.obj
 0001:00003b28       ___local_stdio_printf_options 10004b28 f i IconSwap.obj
 0001:00003b2e       __vfprintf_l               10004b2e f i IconSwap.obj
 0001:00003b52       _printf                    10004b52 f i IconSwap.obj
 0001:00003b70       ??$_Destroy_range@V?$allocator@V?$basic_string@GU?$char_traits@G@std@@V?$allocator@G@2@@std@@@std@@@std@@YAXPAV?$basic_string@GU?$char_traits@G@std@@V?$allocator@G@2@@0@QAV10@AAV?$allocator@V?$basic_string@GU?$char_traits@G@std@@V?$allocator@G@2@@std@@@0@@Z 10004b70 f i JniUtils.obj
 0001:00003b89       ??$_Emplace_reallocate@V?$basic_string@GU?$char_traits@G@std@@V?$allocator@G@2@@std@@@?$vector@V?$basic_string@GU?$char_traits@G@std@@V?$allocator@G@2@@std@@V?$allocator@V?$basic_string@GU?$char_traits@G@std@@V?$allocator@G@2@@std@@@2@@std@@QAEPAV?$basic_string@GU?$char_traits@G@std@@V?$allocator@G@2@@1@QAV21@$$QAV21@@Z 10004b89 f i JniUtils.obj
 0001:00003c33       ??$_Uninitialized_move@PAV?$basic_string@GU?$char_traits@G@std@@V?$allocator@G@2@@std@@V?$allocator@V?$basic_string@GU?$char_traits@G@std@@V?$allocator@G@2@@std@@@2@@std@@YAPAV?$basic_string@GU?$char_traits@G@std@@V?$allocator@G@2@@0@QAV10@0PAV10@AAV?$allocator@V?$basic_string@GU?$char_traits@G@std@@V?$allocator@G@2@@std@@@0@@Z 10004c33 f i JniUtils.obj
 0001:00003c66       ??0?$basic_string@GU?$char_traits@G@std@@V?$allocator@G@2@@std@@QAE@QBGI@Z 10004c66 f i JniUtils.obj
 0001:00003d37       ??1?$unique_ptr@UJniObjWithEnv@jni@@ULocalRefDeleter@12@@std@@QAE@XZ 10004d37 f i JniUtils.obj
 0001:00003d80       ??1?$vector@V?$basic_string@GU?$char_traits@G@std@@V?$allocator@G@2@@std@@V?$allocator@V?$basic_string@GU?$char_traits@G@std@@V?$allocator@G@2@@std@@@2@@std@@QAE@XZ 10004d80 f i JniUtils.obj
 0001:00003d85       ??RLocalRefDeleter@JniObjWithEnv@jni@@QAEXU12@@Z 10004d85 f   JniUtils.obj
 0001:00003da1       ?_Calculate_growth@?$vector@V?$basic_string@GU?$char_traits@G@std@@V?$allocator@G@2@@std@@V?$allocator@V?$basic_string@GU?$char_traits@G@std@@V?$allocator@G@2@@std@@@2@@std@@ABEII@Z 10004da1 f i JniUtils.obj
 0001:00003dca       ?_Change_array@?$vector@V?$basic_string@GU?$char_traits@G@std@@V?$allocator@G@2@@std@@V?$allocator@V?$basic_string@GU?$char_traits@G@std@@V?$allocator@G@2@@std@@@2@@std@@AAEXQAV?$basic_string@GU?$char_traits@G@std@@V?$allocator@G@2@@2@II@Z 10004dca f i JniUtils.obj
 0001:00003e14       ?_Tidy@?$vector@V?$basic_string@GU?$char_traits@G@std@@V?$allocator@G@2@@std@@V?$allocator@V?$basic_string@GU?$char_traits@G@std@@V?$allocator@G@2@@std@@@2@@std@@AAEXXZ 10004e14 f i JniUtils.obj
 0001:00003e4c       ?_Xlength@?$vector@EV?$allocator@E@std@@@std@@CAXXZ 10004e4c f i ResourceEditor.obj
 0001:00003e4c       ?_Xlength@?$vector@V?$basic_string@GU?$char_traits@G@std@@V?$allocator@G@2@@std@@V?$allocator@V?$basic_string@GU?$char_traits@G@std@@V?$allocator@G@2@@std@@@2@@std@@CAXXZ 10004e4c f i JniUtils.obj
 0001:00003e4c       ?_Xlength@?$vector@GV?$allocator@G@std@@@std@@CAXXZ 10004e4c f i MsiUtils.obj
 0001:00003e57       ?allocate@?$allocator@V?$basic_string@GU?$char_traits@G@std@@V?$allocator@G@2@@std@@@std@@QAEPAV?$basic_string@GU?$char_traits@G@std@@V?$allocator@G@2@@2@I@Z 10004e57 f i JniUtils.obj
 0001:00003e75       ?toJString@jni@@YAPAV_jstring@@PAUJNIEnv_@@ABV?$basic_string@GU?$char_traits@G@std@@V?$allocator@G@2@@std@@@Z 10004e75 f   JniUtils.obj
 0001:00003ee9       ?toUnicodeString@jni@@YA?AV?$basic_string@GU?$char_traits@G@std@@V?$allocator@G@2@@std@@PAUJNIEnv_@@PAV_jstring@@@Z 10004ee9 f   JniUtils.obj
 0001:00003f7f       ?toUnicodeStringArray@jni@@YA?AV?$vector@V?$basic_string@GU?$char_traits@G@std@@V?$allocator@G@2@@std@@V?$allocator@V?$basic_string@GU?$char_traits@G@std@@V?$allocator@G@2@@std@@@2@@std@@PAUJNIEnv_@@PAV_jobjectArray@@@Z 10004f7f f   JniUtils.obj
 0001:0000403f       ??$endl@DU?$char_traits@D@std@@@std@@YAAAV?$basic_ostream@DU?$char_traits@D@std@@@0@AAV10@@Z 1000503f f i Log.obj
 0001:0000406b       ??0LogEvent@@QAE@XZ        1000506b f   Log.obj
 0001:0000425b       ??1LogEvent@@QAE@XZ        1000525b f i Log.obj
 0001:0000427f       ??6?$basic_ostream@GU?$char_traits@G@std@@@std@@QAEAAV01@G@Z 1000527f f i Log.obj
 0001:00004408       ??_ENopLogAppender@@UAEPAXI@Z 10005408 f i app.obj
 0001:00004408       ??_GLogAppender@@UAEPAXI@Z 10005408 f i Log.obj
 0001:00004408       ??_GNopLogAppender@@UAEPAXI@Z 10005408 f i app.obj
 0001:00004408       ??_ELogAppender@@UAEPAXI@Z 10005408 f i Log.obj
 0001:00004428       ??_EStreamLogAppender@@UAEPAXI@Z 10005428 f i Log.obj
 0001:00004428       ??_GStreamLogAppender@@UAEPAXI@Z 10005428 f i Log.obj
 0001:00004448       ?append@StreamLogAppender@@UAEXABULogEvent@@@Z 10005448 f   Log.obj
 0001:000045d2       ?defaultLogger@Logger@@SAAAV1@XZ 100055d2 f   Log.obj
 0001:0000462b       ?isLoggable@Logger@@QBE_NW4LogLevel@1@@Z 1000562b f   Log.obj
 0001:00004637       ?log@Logger@@QBEXW4LogLevel@1@PBGH1ABV?$basic_string@GU?$char_traits@G@std@@V?$allocator@G@2@@std@@@Z 10005637 f   Log.obj
 0001:000047a8       ?log@Logger@@QBEXW4LogLevel@1@PBGH1ABVany@tstrings@@@Z 100057a8 f i Log.obj
 0001:000047f2       ??$?6I@any@tstrings@@QAEAAV01@I@Z 100057f2 f i MsiDb.obj
 0001:00004805       ??$?6K@any@tstrings@@QAEAAV01@K@Z 10005805 f i MsiDb.obj
 0001:00004818       ??$_Fgetc@D@std@@YA_NAADPAU_iobuf@@@Z 10005818 f i MsiDb.obj
 0001:00004836       ??$_Fputc@D@std@@YA_NDPAU_iobuf@@@Z 10005836 f i MsiDb.obj
 0001:0000484f       ??$_Reallocate_grow_by@V<lambda_15711c68e099a15a58f4d77303cb286d>@@D@?$basic_string@DU?$char_traits@D@std@@V?$allocator@D@2@@std@@AAEAAV01@IV<lambda_15711c68e099a15a58f4d77303cb286d>@@D@Z 1000584f f i MsiDb.obj
 0001:000048da       ??$_Ungetc@D@std@@YA_NABDPAU_iobuf@@@Z 100058da f i MsiDb.obj
 0001:000048f5       ??$makeException@VError@msi@@@@YA?AV?$JpError@VError@msi@@@@ABVError@msi@@ABUSourceCodePos@@@Z 100058f5 f i MsiDb.obj
 0001:0000490b       ??$makeException@VNoMoreItemsError@msi@@@@YA?AV?$JpError@VNoMoreItemsError@msi@@@@ABVNoMoreItemsError@msi@@ABUSourceCodePos@@@Z 1000590b f i MsiDb.obj
 0001:00004921       ??$use_facet@V?$codecvt@DDU_Mbstatet@@@std@@@std@@YAABV?$codecvt@DDU_Mbstatet@@@0@ABVlocale@0@@Z 10005921 f i MsiDb.obj
 0001:000049b2       ??0?$JpError@VError@msi@@@@QAE@ABV0@@Z 100059b2 f i MsiDb.obj
 0001:00004a06       ??0?$JpError@VError@msi@@@@QAE@ABVError@msi@@ABUSourceCodePos@@@Z 10005a06 f i MsiDb.obj
 0001:00004a55       ??0?$JpError@VNoMoreItemsError@msi@@@@QAE@ABV0@@Z 10005a55 f i MsiDb.obj
 0001:00004ab0       ??0?$JpError@VNoMoreItemsError@msi@@@@QAE@ABVNoMoreItemsError@msi@@ABUSourceCodePos@@@Z 10005ab0 f i MsiDb.obj
 0001:00004b06       ??0?$fpos@U_Mbstatet@@@std@@QAE@U_Mbstatet@@_J@Z 10005b06 f i MsiDb.obj
 0001:00004b2e       ??0Database@msi@@QAE@ABV?$basic_string@GU?$char_traits@G@std@@V?$allocator@G@2@@std@@@Z 10005b2e f   MsiDb.obj
 0001:00004b69       ??0DatabaseView@msi@@QAE@ABVDatabase@1@ABV?$basic_string@GU?$char_traits@G@std@@V?$allocator@G@2@@std@@ABVDatabaseRecord@1@@Z 10005b69 f   MsiDb.obj
 0001:00004ca7       ??0Error@msi@@QAE@ABV01@@Z 10005ca7 f i MsiDb.obj
 0001:00004cc8       ??0NoMoreItemsError@msi@@QAE@ABV01@@Z 10005cc8 f i MsiDb.obj
 0001:00004ce0       ??0NoMoreItemsError@msi@@QAE@ABVany@tstrings@@@Z 10005ce0 f i MsiDb.obj
 0001:00004d04       ??1?$JpError@VError@msi@@@@UAE@XZ 10005d04 f i MsiDb.obj
 0001:00004d2f       ??1?$JpError@VNoMoreItemsError@msi@@@@UAE@XZ 10005d2f f i MsiDb.obj
 0001:00004d5a       ??1?$basic_filebuf@DU?$char_traits@D@std@@@std@@UAE@XZ 10005d5a f i MsiDb.obj
 0001:00004db8       ??1DatabaseRecord@msi@@QAE@XZ 10005db8 f i MsiDb.obj
 0001:00004df9       ??1DatabaseView@msi@@QAE@XZ 10005df9 f i MsiDb.obj
 0001:00004e47       ??4DatabaseRecord@msi@@QAEAAV01@ABV01@@Z 10005e47 f   MsiDb.obj
 0001:00004e7f       ??R<lambda_15711c68e099a15a58f4d77303cb286d>@@QBEXQADQBDID@Z 10005e7f f i MsiDb.obj
 0001:00004ea8       ??_E?$JpError@VError@msi@@@@W3AEPAXI@Z 10005ea8 f i MsiDb.obj
 0001:00004eb0       ??_E?$JpError@VNoMoreItemsError@msi@@@@W3AEPAXI@Z 10005eb0 f i MsiDb.obj
 0001:00004eb8       ??_G?$JpError@VError@msi@@@@UAEPAXI@Z 10005eb8 f i MsiDb.obj
 0001:00004eb8       ??_E?$JpError@VError@msi@@@@UAEPAXI@Z 10005eb8 f i MsiDb.obj
 0001:00004ed7       ??_G?$JpError@VNoMoreItemsError@msi@@@@UAEPAXI@Z 10005ed7 f i MsiDb.obj
 0001:00004ed7       ??_E?$JpError@VNoMoreItemsError@msi@@@@UAEPAXI@Z 10005ed7 f i MsiDb.obj
 0001:00004ef6       ??_E?$basic_filebuf@DU?$char_traits@D@std@@@std@@UAEPAXI@Z 10005ef6 f i MsiDb.obj
 0001:00004ef6       ??_G?$basic_filebuf@DU?$char_traits@D@std@@@std@@UAEPAXI@Z 10005ef6 f i MsiDb.obj
 0001:00004f15       ??_ENoMoreItemsError@msi@@UAEPAXI@Z 10005f15 f i MsiDb.obj
 0001:00004f15       ??_GNoMoreItemsError@msi@@UAEPAXI@Z 10005f15 f i MsiDb.obj
 0001:00004f15       ??_EError@msi@@UAEPAXI@Z   10005f15 f i MsiDb.obj
 0001:00004f15       ??_GError@msi@@UAEPAXI@Z   10005f15 f i MsiDb.obj
 0001:00004f3f       ?_Endwrite@?$basic_filebuf@DU?$char_traits@D@std@@@std@@IAE_NXZ 10005f3f f i MsiDb.obj
 0001:00004fd5       ?_Init@?$basic_filebuf@DU?$char_traits@D@std@@@std@@IAEXPAU_iobuf@@W4_Initfl@12@@Z 10005fd5 f i MsiDb.obj
 0001:00005051       ?_Initcvt@?$basic_filebuf@DU?$char_traits@D@std@@@std@@IAEXABV?$codecvt@DDU_Mbstatet@@@2@@Z 10006051 f i MsiDb.obj
 0001:0000507b       ?_Lock@?$basic_filebuf@DU?$char_traits@D@std@@@std@@UAEXXZ 1000607b f i MsiDb.obj
 0001:0000508c       ?_Reset_back@?$basic_filebuf@DU?$char_traits@D@std@@@std@@AAEXXZ 1000608c f i MsiDb.obj
 0001:000050af       ?_Set_back@?$basic_filebuf@DU?$char_traits@D@std@@@std@@AAEXXZ 100060af f i MsiDb.obj
 0001:000050e2       ?_Unlock@?$basic_filebuf@DU?$char_traits@D@std@@@std@@UAEXXZ 100060e2 f i MsiDb.obj
 0001:000050f3       ?close@?$basic_filebuf@DU?$char_traits@D@std@@@std@@QAEPAV12@XZ 100060f3 f i MsiDb.obj
 0001:00005149       ?erase@?$basic_string@DU?$char_traits@D@std@@V?$allocator@D@2@@std@@QAEAAV12@II@Z 10006149 f i MsiDb.obj
 0001:00005197       ?fetch@DatabaseRecord@msi@@QAEAAV12@AAVDatabaseView@2@@Z 10006197 f   MsiDb.obj
 0001:000051dd       ?fetch@DatabaseView@msi@@QAE?AVDatabaseRecord@2@XZ 100061dd f   MsiDb.obj
 0001:0000528f       ?getFieldCount@DatabaseRecord@msi@@QBEIXZ 1000628f f   MsiDb.obj
 0001:00005305       ?getProperty@Database@msi@@QBE?AV?$basic_string@GU?$char_traits@G@std@@V?$allocator@G@2@@std@@ABV34@@Z 10006305 f   MsiDb.obj
 0001:000054c5       ?imbue@?$basic_filebuf@DU?$char_traits@D@std@@@std@@MAEXABVlocale@2@@Z 100064c5 f i MsiDb.obj
 0001:00005589       ?overflow@?$basic_filebuf@DU?$char_traits@D@std@@@std@@MAEHH@Z 10006589 f i MsiDb.obj
 0001:00005685       ?pbackfail@?$basic_filebuf@DU?$char_traits@D@std@@@std@@MAEHH@Z 10006685 f i MsiDb.obj
 0001:00005704       ?push_back@?$basic_string@DU?$char_traits@D@std@@V?$allocator@D@2@@std@@QAEXD@Z 10006704 f i MsiDb.obj
 0001:00005740       ?seekoff@?$basic_filebuf@DU?$char_traits@D@std@@@std@@MAE?AV?$fpos@U_Mbstatet@@@2@_JHH@Z 10006740 f i MsiDb.obj
 0001:000057fd       ?seekpos@?$basic_filebuf@DU?$char_traits@D@std@@@std@@MAE?AV?$fpos@U_Mbstatet@@@2@V32@H@Z 100067fd f i MsiDb.obj
 0001:00005883       ?setbuf@?$basic_filebuf@DU?$char_traits@D@std@@@std@@MAEPAV?$basic_streambuf@DU?$char_traits@D@std@@@2@PAD_J@Z 10006883 f i MsiDb.obj
 0001:000058d2       ?sync@?$basic_filebuf@DU?$char_traits@D@std@@@std@@MAEHXZ 100068d2 f i MsiDb.obj
 0001:000058fe       ?tryFetch@DatabaseView@msi@@QAE?AVDatabaseRecord@2@XZ 100068fe f   MsiDb.obj
 0001:000059ba       ?uflow@?$basic_filebuf@DU?$char_traits@D@std@@@std@@MAEHXZ 100069ba f i MsiDb.obj
 0001:00005b4f       ?underflow@?$basic_filebuf@DU?$char_traits@D@std@@@std@@MAEHXZ 10006b4f f i MsiDb.obj
 0001:00005b89       ?what@?$JpError@VError@msi@@@@UBEPBDXZ 10006b89 f i MsiDb.obj
 0001:00005b89       ?what@?$JpError@VNoMoreItemsError@msi@@@@UBEPBDXZ 10006b89 f i MsiDb.obj
 0001:00005b95       ?xsgetn@?$basic_filebuf@DU?$char_traits@D@std@@@std@@MAE_JPAD_J@Z 10006b95 f i MsiDb.obj
 0001:00005cad       ?xsputn@?$basic_filebuf@DU?$char_traits@D@std@@@std@@MAE_JPBD_J@Z 10006cad f i MsiDb.obj
 0001:00005d85       ??$?0ABUpiecewise_construct_t@std@@V?$tuple@ABV?$basic_string@GU?$char_traits@G@std@@V?$allocator@G@2@@std@@@1@V?$tuple@$$V@1@@?$_Tree_temp_node@V?$allocator@U?$_Tree_node@U?$pair@$$CBV?$basic_string@GU?$char_traits@G@std@@V?$allocator@G@2@@std@@V12@@std@@PAX@std@@@std@@@std@@QAE@AAV?$allocator@U?$_Tree_node@U?$pair@$$CBV?$basic_string@GU?$char_traits@G@std@@V?$allocator@G@2@@std@@V12@@std@@PAX@std@@@1@PAU?$_Tree_node@U?$pair@$$CBV?$basic_string@GU?$char_traits@G@std@@V?$allocator@G@2@@std@@V12@@std@@PAX@1@ABUpiecewise_construct_t@1@$$QAV?$tuple@ABV?$basic_string@GU?$char_traits@G@std@@V?$allocator@G@2@@std@@@1@$$QAV?$tuple@$$V@1@@Z 10006d85 f i MsiUtils.obj
 0001:00005de8       ??$?0ABV?$basic_string@GU?$char_traits@G@std@@V?$allocator@G@2@@std@@$$Z$$V@?$pair@$$CBV?$basic_string@GU?$char_traits@G@std@@V?$allocator@G@2@@std@@V12@@std@@QAE@Upiecewise_construct_t@1@V?$tuple@ABV?$basic_string@GU?$char_traits@G@std@@V?$allocator@G@2@@std@@@1@V?$tuple@$$V@1@@Z 10006de8 f i MsiUtils.obj
 0001:00005e15       ??$?0V?$_Vector_iterator@V?$_Vector_val@U?$_Simple_types@G@std@@@std@@@std@@$0A@@?$basic_string@GU?$char_traits@G@std@@V?$allocator@G@2@@std@@QAE@V?$_Vector_iterator@V?$_Vector_val@U?$_Simple_types@G@std@@@std@@@1@0ABV?$allocator@G@1@@Z 10006e15 f i MsiUtils.obj
 0001:00005e40       ??$?0V?$tuple@ABV?$basic_string@GU?$char_traits@G@std@@V?$allocator@G@2@@std@@@std@@V?$tuple@$$V@1@$0A@$$Z$S@?$pair@$$CBV?$basic_string@GU?$char_traits@G@std@@V?$allocator@G@2@@std@@V12@@std@@QAE@AAV?$tuple@ABV?$basic_string@GU?$char_traits@G@std@@V?$allocator@G@2@@std@@@1@AAV?$tuple@$$V@1@U?$integer_sequence@I$0A@@1@U?$integer_sequence@I$S@1@@Z 10006e40 f i MsiUtils.obj
 0001:00005e75       ??$_Buyheadnode@V?$allocator@U?$_Tree_node@U?$pair@$$CBV?$basic_string@GU?$char_traits@G@std@@V?$allocator@G@2@@std@@V12@@std@@PAX@std@@@std@@@?$_Tree_node@U?$pair@$$CBV?$basic_string@GU?$char_traits@G@std@@V?$allocator@G@2@@std@@V12@@std@@PAX@std@@SAPAU01@AAV?$allocator@U?$_Tree_node@U?$pair@$$CBV?$basic_string@GU?$char_traits@G@std@@V?$allocator@G@2@@std@@V12@@std@@PAX@std@@@1@@Z 10006e75 f i MsiUtils.obj
 0001:00005e8c       ??$_Copy_memmove@PAGPAG@std@@YAPAGPAG00@Z 10006e8c f i MsiUtils.obj
 0001:00005e8c       ??$_Copy_memmove@PAEPAE@std@@YAPAEPAE00@Z 10006e8c f i ResourceEditor.obj
 0001:00005eae       ??$_Erase_head@V?$allocator@U?$_Tree_node@U?$pair@$$CBV?$basic_string@GU?$char_traits@G@std@@V?$allocator@G@2@@std@@V12@@std@@PAX@std@@@std@@@?$_Tree_val@U?$_Tree_simple_types@U?$pair@$$CBV?$basic_string@GU?$char_traits@G@std@@V?$allocator@G@2@@std@@V12@@std@@@std@@@std@@QAEXAAV?$allocator@U?$_Tree_node@U?$pair@$$CBV?$basic_string@GU?$char_traits@G@std@@V?$allocator@G@2@@std@@V12@@std@@PAX@std@@@1@@Z 10006eae f i MsiUtils.obj
 0001:00005ece       ??$_Erase_tree@V?$allocator@U?$_Tree_node@U?$pair@$$CBV?$basic_string@GU?$char_traits@G@std@@V?$allocator@G@2@@std@@V12@@std@@PAX@std@@@std@@@?$_Tree_val@U?$_Tree_simple_types@U?$pair@$$CBV?$basic_string@GU?$char_traits@G@std@@V?$allocator@G@2@@std@@V12@@std@@@std@@@std@@QAEXAAV?$allocator@U?$_Tree_node@U?$pair@$$CBV?$basic_string@GU?$char_traits@G@std@@V?$allocator@G@2@@std@@V12@@std@@PAX@std@@@1@PAU?$_Tree_node@U?$pair@$$CBV?$basic_string@GU?$char_traits@G@std@@V?$allocator@G@2@@std@@V12@@std@@PAX@1@@Z 10006ece f i MsiUtils.obj
 0001:00005eff       ??$_Find_lower_bound@V?$basic_string@GU?$char_traits@G@std@@V?$allocator@G@2@@std@@@?$_Tree@V?$_Tmap_traits@V?$basic_string@GU?$char_traits@G@std@@V?$allocator@G@2@@std@@V12@U?$less@V?$basic_string@GU?$char_traits@G@std@@V?$allocator@G@2@@std@@@2@V?$allocator@U?$pair@$$CBV?$basic_string@GU?$char_traits@G@std@@V?$allocator@G@2@@std@@V12@@std@@@2@$0A@@std@@@std@@IBE?AU?$_Tree_find_result@PAU?$_Tree_node@U?$pair@$$CBV?$basic_string@GU?$char_traits@G@std@@V?$allocator@G@2@@std@@V12@@std@@PAX@std@@@1@ABV?$basic_string@GU?$char_traits@G@std@@V?$allocator@G@2@@1@@Z 10006eff f i MsiUtils.obj
 0001:00005f4d       ??$_Freenode@V?$allocator@U?$_Tree_node@U?$pair@$$CBV?$basic_string@GU?$char_traits@G@std@@V?$allocator@G@2@@std@@V12@@std@@PAX@std@@@std@@@?$_Tree_node@U?$pair@$$CBV?$basic_string@GU?$char_traits@G@std@@V?$allocator@G@2@@std@@V12@@std@@PAX@std@@SAXAAV?$allocator@U?$_Tree_node@U?$pair@$$CBV?$basic_string@GU?$char_traits@G@std@@V?$allocator@G@2@@std@@V12@@std@@PAX@std@@@1@PAU01@@Z 10006f4d f i MsiUtils.obj
 0001:00005f68       ??$_Lower_bound_duplicate@V?$basic_string@GU?$char_traits@G@std@@V?$allocator@G@2@@std@@@?$_Tree@V?$_Tmap_traits@V?$basic_string@GU?$char_traits@G@std@@V?$allocator@G@2@@std@@V12@U?$less@V?$basic_string@GU?$char_traits@G@std@@V?$allocator@G@2@@std@@@2@V?$allocator@U?$pair@$$CBV?$basic_string@GU?$char_traits@G@std@@V?$allocator@G@2@@std@@V12@@std@@@2@$0A@@std@@@std@@IBE_NQAU?$_Tree_node@U?$pair@$$CBV?$basic_string@GU?$char_traits@G@std@@V?$allocator@G@2@@std@@V12@@std@@PAX@1@ABV?$basic_string@GU?$char_traits@G@std@@V?$allocator@G@2@@1@@Z 10006f68 f i MsiUtils.obj
 0001:00005f8c       ??$_Resize@U_Value_init_tag@std@@@?$vector@GV?$allocator@G@std@@@std@@AAEXIABU_Value_init_tag@1@@Z 10006f8c f i MsiUtils.obj
 0001:00005fde       ??$_Resize_reallocate@U_Value_init_tag@std@@@?$vector@GV?$allocator@G@std@@@std@@AAEXIABU_Value_init_tag@1@@Z 10006fde f i MsiUtils.obj
 0001:00006048       ??$_Try_emplace@ABV?$basic_string@GU?$char_traits@G@std@@V?$allocator@G@2@@std@@$$V@?$map@V?$basic_string@GU?$char_traits@G@std@@V?$allocator@G@2@@std@@V12@U?$less@V?$basic_string@GU?$char_traits@G@std@@V?$allocator@G@2@@std@@@2@V?$allocator@U?$pair@$$CBV?$basic_string@GU?$char_traits@G@std@@V?$allocator@G@2@@std@@V12@@std@@@2@@std@@AAE?AU?$pair@PAU?$_Tree_node@U?$pair@$$CBV?$basic_string@GU?$char_traits@G@std@@V?$allocator@G@2@@std@@V12@@std@@PAX@std@@_N@1@ABV?$basic_string@GU?$char_traits@G@std@@V?$allocator@G@2@@1@@Z 10007048 f i MsiUtils.obj
 0001:000060d4       ??$_Uninitialized_move@PAGV?$allocator@G@std@@@std@@YAPAGQAG0PAGAAV?$allocator@G@0@@Z 100070d4 f i MsiUtils.obj
 0001:000060f8       ??$_Zero_range@PAG@std@@YAPAGQAG0@Z 100070f8 f i MsiUtils.obj
 0001:000060f8       ??$_Zero_range@PAE@std@@YAPAEQAE0@Z 100070f8 f i ResourceEditor.obj
 0001:00006114       ??$construct@U?$pair@$$CBV?$basic_string@GU?$char_traits@G@std@@V?$allocator@G@2@@std@@V12@@std@@ABUpiecewise_construct_t@2@V?$tuple@ABV?$basic_string@GU?$char_traits@G@std@@V?$allocator@G@2@@std@@@2@V?$tuple@$$V@2@@?$_Default_allocator_traits@V?$allocator@U?$_Tree_node@U?$pair@$$CBV?$basic_string@GU?$char_traits@G@std@@V?$allocator@G@2@@std@@V12@@std@@PAX@std@@@std@@@std@@SAXAAV?$allocator@U?$_Tree_node@U?$pair@$$CBV?$basic_string@GU?$char_traits@G@std@@V?$allocator@G@2@@std@@V12@@std@@PAX@std@@@1@QAU?$pair@$$CBV?$basic_string@GU?$char_traits@G@std@@V?$allocator@G@2@@std@@V12@@1@ABUpiecewise_construct_t@1@$$QAV?$tuple@ABV?$basic_string@GU?$char_traits@G@std@@V?$allocator@G@2@@std@@@1@$$QAV?$tuple@$$V@1@@Z 10007114 f i MsiUtils.obj
 0001:000062a4       ??$makeException@VSysError@@@@YA?AV?$JpError@VSysError@@@@ABVSysError@@ABUSourceCodePos@@@Z 100072a4 f i MsiUtils.obj
 0001:000062ba       ??0?$JpError@VSysError@@@@QAE@ABV0@@Z 100072ba f i MsiUtils.obj
 0001:00006315       ??0?$JpError@VSysError@@@@QAE@ABVSysError@@ABUSourceCodePos@@@Z 10007315 f i MsiUtils.obj
 0001:0000636b       ??0?$_Tree_temp_node_alloc@V?$allocator@U?$_Tree_node@U?$pair@$$CBV?$basic_string@GU?$char_traits@G@std@@V?$allocator@G@2@@std@@V12@@std@@PAX@std@@@std@@@std@@QAE@AAV?$allocator@U?$_Tree_node@U?$pair@$$CBV?$basic_string@GU?$char_traits@G@std@@V?$allocator@G@2@@std@@V12@@std@@PAX@std@@@1@@Z 1000736b f i MsiUtils.obj
 0001:0000639e       ??0Error@msi@@QAE@ABV?$basic_string@DU?$char_traits@D@std@@V?$allocator@D@2@@std@@I@Z 1000739e f   MsiUtils.obj
 0001:000063f7       ??0Error@msi@@QAE@ABVany@tstrings@@I@Z 100073f7 f   MsiUtils.obj
 0001:00006457       ??0SysError@@QAE@ABV0@@Z   10007457 f i MsiUtils.obj
 0001:0000646f       ??1?$JpError@VSysError@@@@UAE@XZ 1000746f f i MsiUtils.obj
 0001:0000649a       ??1?$_Tree_temp_node_alloc@V?$allocator@U?$_Tree_node@U?$pair@$$CBV?$basic_string@GU?$char_traits@G@std@@V?$allocator@G@2@@std@@V12@@std@@PAX@std@@@std@@@std@@QAE@XZ 1000749a f i MsiUtils.obj
 0001:0000649a       ??1?$_Alloc_construct_ptr@V?$allocator@U?$_Tree_node@U?$pair@$$CBV?$basic_string@GU?$char_traits@G@std@@V?$allocator@G@2@@std@@V12@@std@@PAX@std@@@std@@@std@@QAE@XZ 1000749a f i MsiUtils.obj
 0001:000064ad       ??1?$_Tree_temp_node@V?$allocator@U?$_Tree_node@U?$pair@$$CBV?$basic_string@GU?$char_traits@G@std@@V?$allocator@G@2@@std@@V12@@std@@PAX@std@@@std@@@std@@QAE@XZ 100074ad f i MsiUtils.obj
 0001:000064d4       ??1?$unique_ptr@PAUHINSTANCE__@@ULibraryReleaser@Dll@@@std@@QAE@XZ 100074d4 f i MsiUtils.obj
 0001:00006515       ??1?$vector@GV?$allocator@G@std@@@std@@QAE@XZ 10007515 f i MsiUtils.obj
 0001:0000651a       ??1StringResource@@QAE@XZ  1000751a f i MsiUtils.obj
 0001:0000652d       ??E?$_Tree_unchecked_const_iterator@V?$_Tree_val@U?$_Tree_simple_types@U?$pair@$$CBV?$basic_string@GU?$char_traits@G@std@@V?$allocator@G@2@@std@@V12@@std@@@std@@@std@@U_Iterator_base0@2@@std@@QAEAAV01@XZ 1000752d f i MsiUtils.obj
 0001:00006561       ??_E?$JpError@VSysError@@@@W3AEPAXI@Z 10007561 f i MsiUtils.obj
 0001:00006569       ??_G?$JpError@VSysError@@@@UAEPAXI@Z 10007569 f i MsiUtils.obj
 0001:00006569       ??_E?$JpError@VSysError@@@@UAEPAXI@Z 10007569 f i MsiUtils.obj
 0001:00006588       ??_G?$pair@$$CBV?$basic_string@GU?$char_traits@G@std@@V?$allocator@G@2@@std@@V12@@std@@QAEPAXI@Z 10007588 f i MsiUtils.obj
 0001:000065b1       ?_Calculate_growth@?$vector@GV?$allocator@G@std@@@std@@ABEII@Z 100075b1 f i MsiUtils.obj
 0001:000065d7       ?_Change_array@?$vector@GV?$allocator@G@std@@@std@@AAEXQAGII@Z 100075d7 f i MsiUtils.obj
 0001:0000660f       ?_Insert_node@?$_Tree_val@U?$_Tree_simple_types@U?$pair@$$CBV?$basic_string@GU?$char_traits@G@std@@V?$allocator@G@2@@std@@V12@@std@@@std@@@std@@QAEPAU?$_Tree_node@U?$pair@$$CBV?$basic_string@GU?$char_traits@G@std@@V?$allocator@G@2@@std@@V12@@std@@PAX@2@U?$_Tree_id@PAU?$_Tree_node@U?$pair@$$CBV?$basic_string@GU?$char_traits@G@std@@V?$allocator@G@2@@std@@V12@@std@@PAX@std@@@2@QAU32@@Z 1000760f f i MsiUtils.obj
 0001:0000670e       ?_Lrotate@?$_Tree_val@U?$_Tree_simple_types@U?$pair@$$CBV?$basic_string@GU?$char_traits@G@std@@V?$allocator@G@2@@std@@V12@@std@@@std@@@std@@QAEXPAU?$_Tree_node@U?$pair@$$CBV?$basic_string@GU?$char_traits@G@std@@V?$allocator@G@2@@std@@V12@@std@@PAX@2@@Z 1000770e f i MsiUtils.obj
 0001:0000674f       ?_Min@?$_Tree_val@U?$_Tree_simple_types@U?$pair@$$CBV?$basic_string@GU?$char_traits@G@std@@V?$allocator@G@2@@std@@V12@@std@@@std@@@std@@SAPAU?$_Tree_node@U?$pair@$$CBV?$basic_string@GU?$char_traits@G@std@@V?$allocator@G@2@@std@@V12@@std@@PAX@2@PAU32@@Z 1000774f f i MsiUtils.obj
 0001:00006768       ?_Rrotate@?$_Tree_val@U?$_Tree_simple_types@U?$pair@$$CBV?$basic_string@GU?$char_traits@G@std@@V?$allocator@G@2@@std@@V12@@std@@@std@@@std@@QAEXPAU?$_Tree_node@U?$pair@$$CBV?$basic_string@GU?$char_traits@G@std@@V?$allocator@G@2@@std@@V12@@std@@PAX@2@@Z 10007768 f i MsiUtils.obj
 0001:000067ab       ?_Throw_tree_length_error@std@@YAXXZ 100077ab f i MsiUtils.obj
 0001:000067b6       ?_Tidy@?$vector@GV?$allocator@G@std@@@std@@AAEXXZ 100077b6 f i MsiUtils.obj
 0001:000067dc       ?closeMSIHANDLE@msi@@YAXK@Z 100077dc f   MsiUtils.obj
 0001:000068a5       ?getString@DatabaseRecord@msi@@QBE?AV?$basic_string@GU?$char_traits@G@std@@V?$allocator@G@2@@std@@I@Z 100078a5 f   MsiUtils.obj
 0001:00006c01       ??0PlatformLogEvent@@QAE@XZ 10007c01 f   PlatformLogEvent.obj
 0001:00006c15       ?_Eos@?$basic_string@GU?$char_traits@G@std@@V?$allocator@G@2@@std@@AAEXI@Z 10007c15 f i PlatformLogEvent.obj
 0001:00006c2d       ?appendFormatted@LogEvent@@CAXABUPlatformLogEvent@@AAV?$basic_string@GU?$char_traits@G@std@@V?$allocator@G@2@@std@@@Z 10007c2d f   PlatformLogEvent.obj
 0001:00006ca3       ?init@LogEvent@@CAXAAUPlatformLogEvent@@@Z 10007ca3 f   PlatformLogEvent.obj
 0001:00006cca       ?initializeLogging@Logger@@CAXXZ 10007cca f   PlatformLogEvent.obj
 0001:00006d5a       ?initializingLogging@Logger@@CAXXZ 10007d5a f   PlatformLogEvent.obj
 0001:00006d63       ?resize@?$basic_string@GU?$char_traits@G@std@@V?$allocator@G@2@@std@@QAEXIG@Z 10007d63 f i PlatformLogEvent.obj
 0001:00006dd9       ??$?0V?$istreambuf_iterator@DU?$char_traits@D@std@@@std@@$0A@@?$vector@EV?$allocator@E@std@@@std@@QAE@V?$istreambuf_iterator@DU?$char_traits@D@std@@@1@0ABV?$allocator@E@1@@Z 10007dd9 f i ResourceEditor.obj
 0001:00006e08       ??$?6PAX@any@tstrings@@QAEAAV01@PAX@Z 10007e08 f i ResourceEditor.obj
 0001:00006e1b       ??$_Emplace_reallocate@D@?$vector@EV?$allocator@E@std@@@std@@QAEPAEQAE$$QAD@Z 10007e1b f i ResourceEditor.obj
 0001:00006ea6       ??$_Range_construct_or_tidy@V?$istreambuf_iterator@DU?$char_traits@D@std@@@std@@@?$vector@EV?$allocator@E@std@@@std@@AAEXV?$istreambuf_iterator@DU?$char_traits@D@std@@@1@0Uinput_iterator_tag@1@@Z 10007ea6 f i ResourceEditor.obj
 0001:00006efc       ??$_Resize@U_Value_init_tag@std@@@?$vector@EV?$allocator@E@std@@@std@@AAEXIABU_Value_init_tag@1@@Z 10007efc f i ResourceEditor.obj
 0001:00006f44       ??$_Resize_reallocate@U_Value_init_tag@std@@@?$vector@EV?$allocator@E@std@@@std@@AAEXIABU_Value_init_tag@1@@Z 10007f44 f i ResourceEditor.obj
 0001:00006fa8       ??$_Uninitialized_move@PAEV?$allocator@E@std@@@std@@YAPAEQAE0PAEAAV?$allocator@E@0@@Z 10007fa8 f i ResourceEditor.obj
 0001:00006fc9       ??$_Uninitialized_value_construct_n@V?$allocator@E@std@@@std@@YAPAEPAEIAAV?$allocator@E@0@@Z 10007fc9 f i ResourceEditor.obj
 0001:00006fe1       ??$emplace_back@D@?$vector@EV?$allocator@E@std@@@std@@QAEX$$QAD@Z 10007fe1 f i ResourceEditor.obj
 0001:00007003       ??0?$basic_filebuf@DU?$char_traits@D@std@@@std@@QAE@XZ 10008003 f i ResourceEditor.obj
 0001:00007051       ??0?$basic_ifstream@DU?$char_traits@D@std@@@std@@QAE@ABV?$basic_string@GU?$char_traits@G@std@@V?$allocator@G@2@@1@HH@Z 10008051 f i ResourceEditor.obj
 0001:00007094       ??0?$basic_ifstream@DU?$char_traits@D@std@@@std@@QAE@PBGHH@Z 10008094 f i ResourceEditor.obj
 0001:00007132       ??0FileLock@ResourceEditor@@QAE@ABV?$basic_string@GU?$char_traits@G@std@@V?$allocator@G@2@@std@@@Z 10008132 f   ResourceEditor.obj
 0001:000071f2       ??0FileLock@ResourceEditor@@QAE@PAX@Z 100081f2 f   ResourceEditor.obj
 0001:00007203       ??0ResourceEditor@@QAE@XZ  10008203 f   ResourceEditor.obj
 0001:00007250       ??0any@tstrings@@QAE@PBD@Z 10008250 f i ResourceEditor.obj
 0001:000072b7       ??1?$_Tidy_guard@V?$vector@EV?$allocator@E@std@@@std@@@std@@QAE@XZ 100082b7 f i ResourceEditor.obj
 0001:000072c2       ??1?$basic_ifstream@DU?$char_traits@D@std@@@std@@UAE@XZ 100082c2 f i ResourceEditor.obj
 0001:000072f2       ??1?$vector@EV?$allocator@E@std@@@std@@QAE@XZ 100082f2 f i ResourceEditor.obj
 0001:000072f7       ??1FileLock@ResourceEditor@@QAE@XZ 100082f7 f   ResourceEditor.obj
 0001:00007433       ??_D?$basic_ifstream@DU?$char_traits@D@std@@@std@@QAEXXZ 10008433 f i ResourceEditor.obj
 0001:00007447       ??_E?$basic_ifstream@DU?$char_traits@D@std@@@std@@$4PPPPPPPM@A@AEPAXI@Z 10008447 f i ResourceEditor.obj
 0001:0000744f       ??_G?$basic_ifstream@DU?$char_traits@D@std@@@std@@UAEPAXI@Z 1000844f f i ResourceEditor.obj
 0001:0000744f       ??_E?$basic_ifstream@DU?$char_traits@D@std@@@std@@UAEPAXI@Z 1000844f f i ResourceEditor.obj
 0001:00007474       ?_Calculate_growth@?$vector@EV?$allocator@E@std@@@std@@ABEII@Z 10008474 f i ResourceEditor.obj
 0001:00007498       ?_Change_array@?$vector@EV?$allocator@E@std@@@std@@AAEXQAEII@Z 10008498 f i ResourceEditor.obj
 0001:000074cb       ?_Inc@?$istreambuf_iterator@DU?$char_traits@D@std@@@std@@AAEXXZ 100084cb f i ResourceEditor.obj
 0001:000074ed       ?_Move_assign@?$vector@EV?$allocator@E@std@@@std@@AAEXAAV12@U_Equal_allocators@2@@Z 100084ed f i ResourceEditor.obj
 0001:00007517       ?_Peek@?$istreambuf_iterator@DU?$char_traits@D@std@@@std@@ABEDXZ 10008517 f i ResourceEditor.obj
 0001:0000753c       ?_Tidy@?$vector@EV?$allocator@E@std@@@std@@AAEXXZ 1000853c f i ResourceEditor.obj
 0001:0000755f       ?apply@ResourceEditor@@QAEAAV1@ABVFileLock@1@AAV?$basic_istream@DU?$char_traits@D@std@@@std@@_J@Z 1000855f f   ResourceEditor.obj
 0001:000076c7       ?apply@ResourceEditor@@QAEAAV1@ABVFileLock@1@ABV?$basic_string@GU?$char_traits@G@std@@V?$allocator@G@2@@std@@@Z 100086c7 f   ResourceEditor.obj
 0001:0000773b       ?equal@?$istreambuf_iterator@DU?$char_traits@D@std@@@std@@QBE_NABV12@@Z 1000873b f i ResourceEditor.obj
 0001:00007772       ?id@ResourceEditor@@QAEAAV1@PBG@Z 10008772 f   ResourceEditor.obj
 0001:00007810       ?open@?$basic_filebuf@DU?$char_traits@D@std@@@std@@QAEPAV12@PBGHH@Z 10008810 f i ResourceEditor.obj
 0001:00007878       ?type@ResourceEditor@@QAEAAV1@PBG@Z 10008878 f   ResourceEditor.obj
 0001:00007925       ??$?6V?$basic_string@DU?$char_traits@D@std@@V?$allocator@D@2@@std@@@any@tstrings@@QAEAAV01@V?$basic_string@DU?$char_traits@D@std@@V?$allocator@D@2@@std@@@Z 10008925 f i Resources.obj
 0001:00007979       ??0Resource@@QAE@IPBGPAUHINSTANCE__@@@Z 10008979 f   Resources.obj
 0001:000079c7       ??0any@tstrings@@QAE@ABV?$basic_string@DU?$char_traits@D@std@@V?$allocator@D@2@@std@@@Z 100089c7 f i Resources.obj
 0001:00007a16       ??6@YAAAV?$basic_ostream@GU?$char_traits@G@std@@@std@@AAV01@ABVany@tstrings@@@Z 10008a16 f i Resources.obj
 0001:00007a54       ?findResource@Resource@@ABEPAUHRSRC__@@XZ 10008a54 f   Resources.obj
 0001:00007a72       ?getErrMsg@Resource@@ABE?AV?$basic_string@DU?$char_traits@D@std@@V?$allocator@D@2@@std@@ABV23@@Z 10008a72 f   Resources.obj
 0001:00007b15       ?getPtr@Resource@@ABEPAXAAK@Z 10008b15 f   Resources.obj
 0001:00007c94       ?init@Resource@@AAEXPBG0PAUHINSTANCE__@@@Z 10008c94 f   Resources.obj
 0001:00007ddf       ?string@StringResource@@QBE?AV?$basic_string@GU?$char_traits@G@std@@V?$allocator@G@2@@std@@XZ 10008ddf f   Resources.obj
 0001:00007e2e       ??$?6GU?$char_traits@G@std@@_J@std@@YAAAV?$basic_ostream@GU?$char_traits@G@std@@@0@AAV10@ABU?$_Smanip@_J@0@@Z 10008e2e f i VersionInfo.obj
 0001:00007e4e       ??$_Find@V?$basic_string@GU?$char_traits@G@std@@V?$allocator@G@2@@std@@@?$_Tree@V?$_Tmap_traits@V?$basic_string@GU?$char_traits@G@std@@V?$allocator@G@2@@std@@V12@U?$less@V?$basic_string@GU?$char_traits@G@std@@V?$allocator@G@2@@std@@@2@V?$allocator@U?$pair@$$CBV?$basic_string@GU?$char_traits@G@std@@V?$allocator@G@2@@std@@V12@@std@@@2@$0A@@std@@@std@@ABEPAU?$_Tree_node@U?$pair@$$CBV?$basic_string@GU?$char_traits@G@std@@V?$allocator@G@2@@std@@V12@@std@@PAX@1@ABV?$basic_string@GU?$char_traits@G@std@@V?$allocator@G@2@@1@@Z 10008e4e f i VersionInfo.obj
 0001:00007e7e       ??$_Traits_equal@U?$char_traits@G@std@@@std@@YA_NQBGI0I@Z 10008e7e f i VersionInfo.obj
 0001:00007ea3       ??$_Traits_rfind@U?$char_traits@G@std@@@std@@YAIQBGII0I@Z 10008ea3 f i VersionInfo.obj
 0001:00007fb2       ??0?$basic_stringstream@DU?$char_traits@D@std@@V?$allocator@D@2@@std@@QAE@H@Z 10008fb2 f i VersionInfo.obj
 0001:0000802f       ??0?$basic_stringstream@GU?$char_traits@G@std@@V?$allocator@G@2@@std@@QAE@XZ 1000902f f i VersionInfo.obj
 0001:00008179       ??0VersionInfo@@QAE@XZ     10009179 f   VersionInfo.obj
 0001:00008198       ??1?$basic_stringstream@DU?$char_traits@D@std@@V?$allocator@D@2@@std@@UAE@XZ 10009198 f i VersionInfo.obj
 0001:000081c8       ??1?$basic_stringstream@GU?$char_traits@G@std@@V?$allocator@G@2@@std@@UAE@XZ 100091c8 f i VersionInfo.obj
 0001:000081f8       ??1ResourceEditor@@QAE@XZ  100091f8 f i VersionInfo.obj
 0001:0000836d       ??_D?$basic_stringstream@DU?$char_traits@D@std@@V?$allocator@D@2@@std@@QAEXXZ 1000936d f i VersionInfo.obj
 0001:00008381       ??_D?$basic_stringstream@GU?$char_traits@G@std@@V?$allocator@G@2@@std@@QAEXXZ 10009381 f i VersionInfo.obj
 0001:00008395       ??_E?$basic_stringstream@DU?$char_traits@D@std@@V?$allocator@D@2@@std@@$4PPPPPPPM@A@AEPAXI@Z 10009395 f i VersionInfo.obj
 0001:0000839d       ??_E?$basic_stringstream@GU?$char_traits@G@std@@V?$allocator@G@2@@std@@$4PPPPPPPM@A@AEPAXI@Z 1000939d f i VersionInfo.obj
 0001:000083a5       ??_G?$basic_stringstream@DU?$char_traits@D@std@@V?$allocator@D@2@@std@@UAEPAXI@Z 100093a5 f i VersionInfo.obj
 0001:000083a5       ??_E?$basic_stringstream@DU?$char_traits@D@std@@V?$allocator@D@2@@std@@UAEPAXI@Z 100093a5 f i VersionInfo.obj
 0001:000083ca       ??_G?$basic_stringstream@GU?$char_traits@G@std@@V?$allocator@G@2@@std@@UAEPAXI@Z 100093ca f i VersionInfo.obj
 0001:000083ca       ??_E?$basic_stringstream@GU?$char_traits@G@std@@V?$allocator@G@2@@std@@UAEPAXI@Z 100093ca f i VersionInfo.obj
 0001:000083ef       ?_Equal@?$basic_string@GU?$char_traits@G@std@@V?$allocator@G@2@@std@@QBE_NQBG@Z 100093ef f i VersionInfo.obj
 0001:000084d3       ?apply@VersionInfo@@QBEABV1@ABVFileLock@ResourceEditor@@@Z 100094d3 f   VersionInfo.obj
 0001:00008648       ?createFIXEDFILEINFO@VersionInfo@@ABE?AUtagVS_FIXEDFILEINFO@@XZ 10009648 f   VersionInfo.obj
 0001:00008783       ?fillBuffer@VersionInfo@@ABEXAAV?$basic_ostream@DU?$char_traits@D@std@@@std@@@Z 10009783 f   VersionInfo.obj
 0001:00008a52       ?hex@std@@YAAAVios_base@1@AAV21@@Z 10009a52 f i VersionInfo.obj
 0001:00008a69       ?rfind@?$basic_string@GU?$char_traits@G@std@@V?$allocator@G@2@@std@@QBEIQBGI@Z 10009a69 f i VersionInfo.obj
 0001:00008a9a       ?setProperty@VersionInfo@@QAEAAV1@ABV?$basic_string@GU?$char_traits@G@std@@V?$allocator@G@2@@std@@0@Z 10009a9a f   VersionInfo.obj
 0001:00008af6       ?uppercase@std@@YAAAVios_base@1@AAV21@@Z 10009af6 f i VersionInfo.obj
 0001:00008b91       ___local_stdio_scanf_options 10009b91 f i VersionInfo.obj
 0001:00008b97       __vswscanf_s_l             10009b97 f i VersionInfo.obj
 0001:00008bc1       _swscanf_s                 10009bc1 f i VersionInfo.obj
 0001:00008bd9       ?freeLibrary@Dll@@SAXPAUHINSTANCE__@@@Z 10009bd9 f   WinDll.obj
 0001:00008beb       ??0SysError@@QAE@ABVany@tstrings@@PBXKPBD@Z 10009beb f   WinErrorHandling.obj
 0001:00008c56       ?getSysErrorMessage@SysError@@SA?AV?$basic_string@GU?$char_traits@G@std@@V?$allocator@G@2@@std@@KPAUHINSTANCE__@@@Z 10009c56 f   WinErrorHandling.obj
 0001:00008fd1       ?_Equal@?$basic_string@GU?$char_traits@G@std@@V?$allocator@G@2@@std@@QBE_NABV12@@Z 10009fd1 f i WinFileUtils.obj
 0001:00008ffe       ??$?HDU?$char_traits@D@std@@V?$allocator@D@1@@std@@YA?AV?$basic_string@DU?$char_traits@D@std@@V?$allocator@D@2@@0@ABV10@QBD@Z 10009ffe f i WinSysInfo.obj
 0001:00009048       ??$?HDU?$char_traits@D@std@@V?$allocator@D@1@@std@@YA?AV?$basic_string@DU?$char_traits@D@std@@V?$allocator@D@2@@0@QBDABV10@@Z 1000a048 f i WinSysInfo.obj
 0001:0000924e       ??0?$basic_string@DU?$char_traits@D@std@@V?$allocator@D@2@@std@@QAE@U_String_constructor_concat_tag@1@ABV01@QBDI2I@Z 1000a24e f i WinSysInfo.obj
 0001:000092c1       ?getCurrentModuleHandle@SysInfo@@YAPAUHINSTANCE__@@XZ 1000a2c1 f   WinSysInfo.obj
 0001:00009361       ?getCurrentModulePath@SysInfo@@YA?AV?$basic_string@GU?$char_traits@G@std@@V?$allocator@G@2@@std@@XZ 1000a361 f   WinSysInfo.obj
 0001:000094a2       ?getSystem32Dir@SysInfo@@YA?AV?$basic_string@GU?$char_traits@G@std@@V?$allocator@G@2@@std@@XZ 1000a4a2 f   WinSysInfo.obj
 0001:00009654       ?StringCchLengthW@@YGJPBGIPAI@Z 1000a654 f i WindowsRegistry.obj
 0001:000096d3       _Java_jdk_jpackage_internal_WindowsRegistry_closeRegistryKey@16 1000a6d3 f   WindowsRegistry.obj
 0001:000096e0       _Java_jdk_jpackage_internal_WindowsRegistry_comparePaths@16 1000a6e0 f   WindowsRegistry.obj
 0001:00009814       _Java_jdk_jpackage_internal_WindowsRegistry_enumRegistryValue@20 1000a814 f   WindowsRegistry.obj
 0001:000099ab       _Java_jdk_jpackage_internal_WindowsRegistry_openRegistryKey@16 1000a9ab f   WindowsRegistry.obj
 0001:00009ab1       _Java_jdk_jpackage_internal_WindowsRegistry_readDwordValue@24 1000aab1 f   WindowsRegistry.obj
 0001:00009c16       ?append@NopLogAppender@@UAEXABULogEvent@@@Z 1000ac16 f i app.obj
 0001:00009d51       ?lastErrorMsg@app@@YA?AV?$basic_string@DU?$char_traits@D@std@@V?$allocator@D@2@@std@@XZ 1000ad51 f   app.obj
 0001:00009d86       ??0?$basic_istringstream@DU?$char_traits@D@std@@V?$allocator@D@2@@std@@QAE@ABV?$basic_string@DU?$char_traits@D@std@@V?$allocator@D@2@@1@H@Z 1000ad86 f i jpackage.obj
 0001:00009e00       ??0?$basic_stringbuf@DU?$char_traits@D@std@@V?$allocator@D@2@@std@@QAE@ABV?$basic_string@DU?$char_traits@D@std@@V?$allocator@D@2@@1@H@Z 1000ae00 f i jpackage.obj
 0001:00009e4d       ??1?$basic_istringstream@DU?$char_traits@D@std@@V?$allocator@D@2@@std@@UAE@XZ 1000ae4d f i jpackage.obj
 0001:00009e7d       ??1Database@msi@@QAE@XZ    1000ae7d f i jpackage.obj
 0001:00009ecb       ??1VersionInfo@@QAE@XZ     1000aecb f i jpackage.obj
 0001:00009ed2       ??_D?$basic_istringstream@DU?$char_traits@D@std@@V?$allocator@D@2@@std@@QAEXXZ 1000aed2 f i jpackage.obj
 0001:00009ee6       ??_E?$basic_istringstream@DU?$char_traits@D@std@@V?$allocator@D@2@@std@@$4PPPPPPPM@A@AEPAXI@Z 1000aee6 f i jpackage.obj
 0001:00009eee       ??_G?$basic_istringstream@DU?$char_traits@D@std@@V?$allocator@D@2@@std@@UAEPAXI@Z 1000aeee f i jpackage.obj
 0001:00009eee       ??_E?$basic_istringstream@DU?$char_traits@D@std@@V?$allocator@D@2@@std@@UAEPAXI@Z 1000aeee f i jpackage.obj
 0001:00009f13       ?_Init@?$basic_stringbuf@DU?$char_traits@D@std@@V?$allocator@D@2@@std@@IAEXPBDIH@Z 1000af13 f i jpackage.obj
 0001:00009fc1       _Java_jdk_jpackage_internal_ExecutableRebrander_iconSwap@20 1000afc1 f   jpackage.obj
 0001:0000a08b       _Java_jdk_jpackage_internal_ExecutableRebrander_lockResource@12 1000b08b f   jpackage.obj
 0001:0000a13a       _Java_jdk_jpackage_internal_ExecutableRebrander_unlockResource@16 1000b13a f   jpackage.obj
 0001:0000a1bc       _Java_jdk_jpackage_internal_ExecutableRebrander_versionSwap@20 1000b1bc f   jpackage.obj
 0001:0000a36c       _Java_jdk_jpackage_internal_WinExeBundler_embedMSI@20 1000b36c f   jpackage.obj
 0001:0000a58f       ??$_Reallocate_grow_by@V<lambda_c1b8c41cb4019640539cfd828748c4d4>@@ID@?$basic_string@DU?$char_traits@D@std@@V?$allocator@D@2@@std@@AAEAAV01@IV<lambda_c1b8c41cb4019640539cfd828748c4d4>@@ID@Z 1000b58f f i tstrings.obj
 0001:0000a61e       ??$transform@V?$_String_iterator@V?$_String_val@U?$_Simple_types@G@std@@@std@@@std@@V12@P6AHH@Z@std@@YA?AV?$_String_iterator@V?$_String_val@U?$_Simple_types@G@std@@@std@@@0@V10@0V10@P6AHH@Z@Z 1000b61e f i tstrings.obj
 0001:0000a64e       ??0invalid_argument@std@@QAE@ABV01@@Z 1000b64e f i tstrings.obj
 0001:0000a666       ??0invalid_argument@std@@QAE@PBD@Z 1000b666 f i tstrings.obj
 0001:0000a685       ??0logic_error@std@@QAE@ABV01@@Z 1000b685 f i tstrings.obj
 0001:0000a69d       ??R<lambda_c1b8c41cb4019640539cfd828748c4d4>@@QBEXQADQBDIID@Z 1000b69d f i tstrings.obj
 0001:0000a6d0       ?append@?$basic_string@DU?$char_traits@D@std@@V?$allocator@D@2@@std@@QAEAAV12@ID@Z 1000b6d0 f i tstrings.obj
 0001:0000a72b       ?equals@tstrings@@YA_NABV?$basic_string@GU?$char_traits@G@std@@V?$allocator@G@2@@std@@0W4CompareType@1@@Z 1000b72b f   tstrings.obj
 0001:0000a90e       ?resize@?$basic_string@DU?$char_traits@D@std@@V?$allocator@D@2@@std@@QAEXID@Z 1000b90e f i tstrings.obj
 0001:0000a938       ?toLower@tstrings@@YA?AV?$basic_string@GU?$char_traits@G@std@@V?$allocator@G@2@@std@@ABV23@@Z 1000b938 f   tstrings.obj
 0001:0000ab41       ?toUtf16@tstrings@@YA?AV?$basic_string@GU?$char_traits@G@std@@V?$allocator@G@2@@std@@ABV?$basic_string@DU?$char_traits@D@std@@V?$allocator@D@2@@3@@Z 1000bb41 f   tstrings.obj
 0001:0000ab5b       ?toUtf8@tstrings@@YA?AV?$basic_string@DU?$char_traits@D@std@@V?$allocator@D@2@@std@@ABV?$basic_string@GU?$char_traits@G@std@@V?$allocator@G@2@@3@@Z 1000bb5b f   tstrings.obj
 0001:0000ab75       ?unsafe_format@tstrings@@YA?AV?$basic_string@GU?$char_traits@G@std@@V?$allocator@G@2@@std@@PBGZZ 1000bb75 f   tstrings.obj
 0001:0000ac0d       __vsnwprintf_s_l           1000bc0d f i tstrings.obj
 0001:0000ac3f       ?uncaught_exception@std@@YA_NXZ 1000bc3f f   msvcprt:MSVCP140.dll
 0001:0000ac45       ?_Xlength_error@std@@YAXPBD@Z 1000bc45 f   msvcprt:MSVCP140.dll
 0001:0000ac4b       ?_Xout_of_range@std@@YAXPBD@Z 1000bc4b f   msvcprt:MSVCP140.dll
 0001:0000ac51       ??1_Fac_node@std@@QAE@XZ   1000bc51 f i msvcprt:locale0_implib.obj
 0001:0000ac82       ??1_Fac_tidy_reg_t@std@@QAE@XZ 1000bc82 f i msvcprt:locale0_implib.obj
 0001:0000aca9       ?_Facet_Register@std@@YAXPAV_Facet_base@1@@Z 1000bca9 f   msvcprt:locale0_implib.obj
 0001:0000acd5       ?_Getgloballocale@locale@std@@CAPAV_Locimp@12@XZ 1000bcd5 f   msvcprt:MSVCP140.dll
 0001:0000acdb       ?_Lock@?$basic_streambuf@DU?$char_traits@D@std@@@std@@UAEXXZ 1000bcdb f   msvcprt:MSVCP140.dll
 0001:0000ace1       ?_Lock@?$basic_streambuf@GU?$char_traits@G@std@@@std@@UAEXXZ 1000bce1 f   msvcprt:MSVCP140.dll
 0001:0000ace7       ?_Unlock@?$basic_streambuf@DU?$char_traits@D@std@@@std@@UAEXXZ 1000bce7 f   msvcprt:MSVCP140.dll
 0001:0000aced       ?_Unlock@?$basic_streambuf@GU?$char_traits@G@std@@@std@@UAEXXZ 1000bced f   msvcprt:MSVCP140.dll
 0001:0000acf3       ?imbue@?$basic_streambuf@DU?$char_traits@D@std@@@std@@MAEXABVlocale@2@@Z 1000bcf3 f   msvcprt:MSVCP140.dll
 0001:0000acf9       ?imbue@?$basic_streambuf@GU?$char_traits@G@std@@@std@@MAEXABVlocale@2@@Z 1000bcf9 f   msvcprt:MSVCP140.dll
 0001:0000acff       ?setbuf@?$basic_streambuf@DU?$char_traits@D@std@@@std@@MAEPAV12@PAD_J@Z 1000bcff f   msvcprt:MSVCP140.dll
 0001:0000ad05       ?setbuf@?$basic_streambuf@GU?$char_traits@G@std@@@std@@MAEPAV12@PAG_J@Z 1000bd05 f   msvcprt:MSVCP140.dll
 0001:0000ad0b       ?showmanyc@?$basic_streambuf@DU?$char_traits@D@std@@@std@@MAE_JXZ 1000bd0b f   msvcprt:MSVCP140.dll
 0001:0000ad11       ?showmanyc@?$basic_streambuf@GU?$char_traits@G@std@@@std@@MAE_JXZ 1000bd11 f   msvcprt:MSVCP140.dll
 0001:0000ad17       ?sync@?$basic_streambuf@DU?$char_traits@D@std@@@std@@MAEHXZ 1000bd17 f   msvcprt:MSVCP140.dll
 0001:0000ad1d       ?sync@?$basic_streambuf@GU?$char_traits@G@std@@@std@@MAEHXZ 1000bd1d f   msvcprt:MSVCP140.dll
 0001:0000ad23       ?uflow@?$basic_streambuf@DU?$char_traits@D@std@@@std@@MAEHXZ 1000bd23 f   msvcprt:MSVCP140.dll
 0001:0000ad29       ?uflow@?$basic_streambuf@GU?$char_traits@G@std@@@std@@MAEGXZ 1000bd29 f   msvcprt:MSVCP140.dll
 0001:0000ad2f       ?xsgetn@?$basic_streambuf@DU?$char_traits@D@std@@@std@@MAE_JPAD_J@Z 1000bd2f f   msvcprt:MSVCP140.dll
 0001:0000ad35       ?xsgetn@?$basic_streambuf@GU?$char_traits@G@std@@@std@@MAE_JPAG_J@Z 1000bd35 f   msvcprt:MSVCP140.dll
 0001:0000ad3b       ?xsputn@?$basic_streambuf@DU?$char_traits@D@std@@@std@@MAE_JPBD_J@Z 1000bd3b f   msvcprt:MSVCP140.dll
 0001:0000ad41       ?xsputn@?$basic_streambuf@GU?$char_traits@G@std@@@std@@MAE_JPBG_J@Z 1000bd41 f   msvcprt:MSVCP140.dll
 0001:0000ad47       ?_Fiopen@std@@YAPAU_iobuf@@PBGHH@Z 1000bd47 f   msvcprt:MSVCP140.dll
 0001:0000ad4d       ?_Xbad_alloc@std@@YAXXZ    1000bd4d f   msvcprt:MSVCP140.dll
 0001:0000ad53       ?setw@std@@YA?AU?$_Smanip@_J@1@_J@Z 1000bd53 f   msvcprt:MSVCP140.dll
 0001:0000ad59       ??2@YAPAXI@Z               1000bd59 f   MSVCRT:new_scalar.obj
 0001:0000ad89       ??3@YAXPAXI@Z              1000bd89 f   MSVCRT:delete_scalar_size.obj
 0001:0000ad97       @__security_check_cookie@4 1000bd97 f   MSVCRT:secchk.obj
 0001:0000ada8       __EH_epilog3               1000bda8 f   MSVCRT:ehprolg3.obj
 0001:0000adbd       __EH_epilog3_GS            1000bdbd f   MSVCRT:ehprolg3.obj
 0001:0000adce       __EH_epilog3_catch_GS      1000bdce f   MSVCRT:ehprolg3.obj
 0001:0000addf       __EH_prolog3               1000bddf f   MSVCRT:ehprolg3.obj
 0001:0000ae13       __EH_prolog3_GS            1000be13 f   MSVCRT:ehprolg3.obj
 0001:0000ae4a       __EH_prolog3_catch         1000be4a f   MSVCRT:ehprolg3.obj
 0001:0000ae81       __EH_prolog3_catch_GS      1000be81 f   MSVCRT:ehprolg3.obj
 0001:0000aec0       __alloca_probe             1000bec0 f   MSVCRT:chkstk.obj
 0001:0000aec0       __chkstk                   1000bec0 f   MSVCRT:chkstk.obj
 0001:0000aeed       ??_Gtype_info@@UAEPAXI@Z   1000beed f i MSVCRT:std_type_info_static.obj
 0001:0000aeed       ??_Etype_info@@UAEPAXI@Z   1000beed f i MSVCRT:std_type_info_static.obj
 0001:0000af10       ___raise_securityfailure   1000bf10 f   MSVCRT:gs_report.obj
 0001:0000af3b       ___report_gsfailure        1000bf3b f   MSVCRT:gs_report.obj
 0001:0000b034       ___report_rangecheckfailure 1000c034 f   MSVCRT:gs_report.obj
 0001:0000b040       ___report_securityfailure  1000c040 f   MSVCRT:gs_report.obj
 0001:0000b110       __alldiv                   1000c110 f   MSVCRT:lldiv.obj
 0001:0000b1c0       __allrem                   1000c1c0 f   MSVCRT:llrem.obj
 0001:0000b272       ??3@YAXPAX@Z               1000c272 f   MSVCRT:delete_scalar.obj
 0001:0000b277       ??_U@YAPAXI@Z              1000c277 f   MSVCRT:new_array.obj
 0001:0000b280       ??_V@YAXPAX@Z              1000c280 f   MSVCRT:delete_array.obj
 0001:0000b2c9       ___scrt_acquire_startup_lock 1000c2c9 f   MSVCRT:utility.obj
 0001:0000b2fb       ___scrt_dllmain_after_initialize_c 1000c2fb f   MSVCRT:utility.obj
 0001:0000b326       ___scrt_dllmain_before_initialize_c 1000c326 f   MSVCRT:utility.obj
 0001:0000b334       ___scrt_dllmain_crt_thread_attach 1000c334 f   MSVCRT:utility.obj
 0001:0000b353       ___scrt_dllmain_crt_thread_detach 1000c353 f   MSVCRT:utility.obj
 0001:0000b360       ___scrt_dllmain_exception_filter 1000c360 f   MSVCRT:utility.obj
 0001:0000b394       ___scrt_dllmain_uninitialize_c 1000c394 f   MSVCRT:utility.obj
 0001:0000b3b7       ___scrt_dllmain_uninitialize_critical 1000c3b7 f   MSVCRT:utility.obj
 0001:0000b3c4       ___scrt_initialize_crt     1000c3c4 f   MSVCRT:utility.obj
 0001:0000b3fd       ___scrt_initialize_onexit_tables 1000c3fd f   MSVCRT:utility.obj
 0001:0000b484       ___scrt_is_nonwritable_in_current_image 1000c484 f   MSVCRT:utility.obj
 0001:0000b518       ___scrt_release_startup_lock 1000c518 f   MSVCRT:utility.obj
 0001:0000b535       ___scrt_uninitialize_crt   1000c535 f   MSVCRT:utility.obj
 0001:0000b55d       __onexit                   1000c55d f   MSVCRT:utility.obj
 0001:0000b58a       _atexit                    1000c58a f   MSVCRT:utility.obj
 0001:0000b8df       __DllMainCRTStartup@12     1000c8df f   MSVCRT:dll_dllmain.obj
 0001:0000b902       @_guard_check_icall_nop@4  1000c902 f i MSVCRT:guard_support.obj
 0001:0000b905       ??0bad_alloc@std@@QAE@XZ   1000c905 f i MSVCRT:throw_bad_alloc.obj
 0001:0000b91d       ?__scrt_throw_std_bad_alloc@@YAXXZ 1000c91d f   MSVCRT:throw_bad_alloc.obj
 0001:0000b93a       ___isa_available_init      1000c93a f   MSVCRT:cpu_disp.obj
 0001:0000bb0a       __get_startup_argv_mode    1000cb0a f   MSVCRT:argv_mode.obj
 0001:0000bb0e       ___scrt_is_ucrt_dll_in_use 1000cb0e f   MSVCRT:ucrt_detection.obj
 0001:0000bb1a       ___scrt_fastfail           1000cb1a f   MSVCRT:utility_desktop.obj
 0001:0000bc34       __crt_debugger_hook        1000cc34 f   MSVCRT:utility_desktop.obj
 0001:0000bc40       __SEH_prolog4              1000cc40 f   MSVCRT:sehprolg4.obj
 0001:0000bc84       __SEH_epilog4              1000cc84 f   MSVCRT:sehprolg4.obj
 0001:0000bc98       __except_handler4          1000cc98 f   MSVCRT:chandler4gs.obj
 0001:0000bd14       ___security_init_cookie    1000cd14 f   MSVCRT:gs_support.obj
 0001:0000bd5f       _DllMain@12                1000cd5f f   MSVCRT:dll_dllmain_stub.obj
 0001:0000bd81       ?__scrt_initialize_type_info@@YAXXZ 1000cd81 f   MSVCRT:tncleanup.obj
 0001:0000bd8d       ?__scrt_uninitialize_type_info@@YAXXZ 1000cd8d f   MSVCRT:tncleanup.obj
 0001:0000bd99       ___scrt_initialize_default_local_stdio_options 1000cd99 f   MSVCRT:default_local_stdio_options.obj
 0001:0000bdb6       ___scrt_get_dyn_tls_init_callback 1000cdb6 f   MSVCRT:dyn_tls_init.obj
 0001:0000bdbc       __RTC_Initialize           1000cdbc f   MSVCRT:initsect.obj
 0001:0000bde8       __RTC_Terminate            1000cde8 f   MSVCRT:initsect.obj
 0001:0000be14       _MsiDatabaseOpenViewW@12   1000ce14 f   msi:msi.dll
 0001:0000be1a       _MsiViewExecute@8          1000ce1a f   msi:msi.dll
 0001:0000be20       _MsiViewFetch@8            1000ce20 f   msi:msi.dll
 0001:0000be26       _MsiOpenDatabaseW@12       1000ce26 f   msi:msi.dll
 0001:0000be2c       _MsiRecordGetFieldCount@4  1000ce2c f   msi:msi.dll
 0001:0000be32       _MsiCloseHandle@4          1000ce32 f   msi:msi.dll
 0001:0000be38       _MsiRecordGetStringW@16    1000ce38 f   msi:msi.dll
 0001:0000be3e       _IsProcessorFeaturePresent@4 1000ce3e f   kernel32:KERNEL32.dll
 0001:0000be44       _memchr                    1000ce44 f   vcruntime:VCRUNTIME140.dll
 0001:0000be4a       _memcpy                    1000ce4a f   vcruntime:VCRUNTIME140.dll
 0001:0000be50       _memmove                   1000ce50 f   vcruntime:VCRUNTIME140.dll
 0001:0000be56       ___std_exception_copy      1000ce56 f   vcruntime:VCRUNTIME140.dll
 0001:0000be5c       ___std_exception_destroy   1000ce5c f   vcruntime:VCRUNTIME140.dll
 0001:0000be62       __CxxThrowException@8      1000ce62 f   vcruntime:VCRUNTIME140.dll
 0001:0000be68       ___CxxFrameHandler3        1000ce68 f   vcruntime:VCRUNTIME140.dll
 0001:0000be6e       _memset                    1000ce6e f   vcruntime:VCRUNTIME140.dll
 0001:0000be74       __purecall                 1000ce74 f   vcruntime:VCRUNTIME140.dll
 0001:0000be7a       ___std_terminate           1000ce7a f   vcruntime:VCRUNTIME140.dll
 0001:0000be80       __except_handler4_common   1000ce80 f   vcruntime:VCRUNTIME140.dll
 0001:0000be86       ___std_type_info_destroy_list 1000ce86 f   vcruntime:VCRUNTIME140.dll
 0001:0000be8c       _strlen                    1000ce8c f   ucrt:api-ms-win-crt-string-l1-1-0.dll
 0001:0000be92       _free                      1000ce92 f   ucrt:api-ms-win-crt-heap-l1-1-0.dll
 0001:0000be98       _malloc                    1000ce98 f   ucrt:api-ms-win-crt-heap-l1-1-0.dll
 0001:0000be9e       __callnewh                 1000ce9e f   ucrt:api-ms-win-crt-heap-l1-1-0.dll
 0001:0000bea4       __seh_filter_dll           1000cea4 f   ucrt:api-ms-win-crt-runtime-l1-1-0.dll
 0001:0000beaa       __configure_narrow_argv    1000ceaa f   ucrt:api-ms-win-crt-runtime-l1-1-0.dll
 0001:0000beb0       __initialize_narrow_environment 1000ceb0 f   ucrt:api-ms-win-crt-runtime-l1-1-0.dll
 0001:0000beb6       __initialize_onexit_table  1000ceb6 f   ucrt:api-ms-win-crt-runtime-l1-1-0.dll
 0001:0000bebc       __register_onexit_function 1000cebc f   ucrt:api-ms-win-crt-runtime-l1-1-0.dll
 0001:0000bec2       __execute_onexit_table     1000cec2 f   ucrt:api-ms-win-crt-runtime-l1-1-0.dll
 0001:0000bec8       __crt_atexit               1000cec8 f   ucrt:api-ms-win-crt-runtime-l1-1-0.dll
 0001:0000bece       __cexit                    1000cece f   ucrt:api-ms-win-crt-runtime-l1-1-0.dll
 0001:0000bed4       __initterm                 1000ced4 f   ucrt:api-ms-win-crt-runtime-l1-1-0.dll
 0001:0000beda       __initterm_e               1000ceda f   ucrt:api-ms-win-crt-runtime-l1-1-0.dll
 0001:0000bee0       ___vcrt_uninitialize       1000cee0 f   MSVCRT:ucrt_stubs.obj
 0001:0000bee0       ___acrt_initialize         1000cee0 f   MSVCRT:ucrt_stubs.obj
 0001:0000bee0       ___acrt_uninitialize_critical 1000cee0 f   MSVCRT:ucrt_stubs.obj
 0001:0000bee0       ___scrt_stub_for_acrt_initialize 1000cee0 f   MSVCRT:ucrt_stubs.obj
 0001:0000bee0       ___vcrt_initialize         1000cee0 f   MSVCRT:ucrt_stubs.obj
 0001:0000bee0       ___acrt_thread_detach      1000cee0 f   MSVCRT:ucrt_stubs.obj
 0001:0000bee0       ___acrt_uninitialize       1000cee0 f   MSVCRT:ucrt_stubs.obj
 0001:0000bee0       ___scrt_stub_for_acrt_uninitialize 1000cee0 f   MSVCRT:ucrt_stubs.obj
 0001:0000bee0       ___scrt_stub_for_acrt_uninitialize_critical 1000cee0 f   MSVCRT:ucrt_stubs.obj
 0001:0000bee0       ___vcrt_uninitialize_critical 1000cee0 f   MSVCRT:ucrt_stubs.obj
 0001:0000bee0       ___vcrt_thread_detach      1000cee0 f   MSVCRT:ucrt_stubs.obj
 0001:0000bee0       ___acrt_thread_attach      1000cee0 f   MSVCRT:ucrt_stubs.obj
 0001:0000bee0       ___scrt_stub_for_acrt_thread_detach 1000cee0 f   MSVCRT:ucrt_stubs.obj
 0001:0000bee0       ___vcrt_thread_attach      1000cee0 f   MSVCRT:ucrt_stubs.obj
 0001:0000bee0       ___scrt_stub_for_acrt_thread_attach 1000cee0 f   MSVCRT:ucrt_stubs.obj
 0001:0000bee3       __is_c_termination_complete 1000cee3 f   MSVCRT:ucrt_stubs.obj
 0001:0000bee3       ___scrt_stub_for_is_c_termination_complete 1000cee3 f   MSVCRT:ucrt_stubs.obj
 0001:0000bee6       __filter_x86_sse2_floating_point_exception 1000cee6 f   MSVCRT:x86_exception_filter.obj
 0001:0000bee6       __filter_x86_sse2_floating_point_exception_default 1000cee6 f   MSVCRT:x86_exception_filter.obj
 0002:00000000       __imp__RegCloseKey@4       1000f000     advapi32:ADVAPI32.dll
 0002:00000004       __imp__RegOpenKeyExW@20    1000f004     advapi32:ADVAPI32.dll
 0002:00000008       __imp__RegQueryValueExW@24 1000f008     advapi32:ADVAPI32.dll
 0002:0000000c       __imp__RegEnumValueW@32    1000f00c     advapi32:ADVAPI32.dll
 0002:00000010       \177ADVAPI32_NULL_THUNK_DATA 1000f010     advapi32:ADVAPI32.dll
 0002:00000014       __imp__FindResourceW@12    1000f014     kernel32:KERNEL32.dll
 0002:00000018       __imp__SizeofResource@8    1000f018     kernel32:KERNEL32.dll
 0002:0000001c       __imp__LockResource@4      1000f01c     kernel32:KERNEL32.dll
 0002:00000020       __imp__LoadResource@8      1000f020     kernel32:KERNEL32.dll
 0002:00000024       __imp__EndUpdateResourceW@8 1000f024     kernel32:KERNEL32.dll
 0002:00000028       __imp__BeginUpdateResourceW@8 1000f028     kernel32:KERNEL32.dll
 0002:0000002c       __imp__GetLocalTime@4      1000f02c     kernel32:KERNEL32.dll
 0002:00000030       __imp__GetCurrentThreadId@0 1000f030     kernel32:KERNEL32.dll
 0002:00000034       __imp__GetCurrentProcessId@0 1000f034     kernel32:KERNEL32.dll
 0002:00000038       __imp__UpdateResourceW@24  1000f038     kernel32:KERNEL32.dll
 0002:0000003c       __imp__FormatMessageW@28   1000f03c     kernel32:KERNEL32.dll
 0002:00000040       __imp__LocalFree@4         1000f040     kernel32:KERNEL32.dll
 0002:00000044       __imp__GetLastError@0      1000f044     kernel32:KERNEL32.dll
 0002:00000048       __imp__CloseHandle@4       1000f048     kernel32:KERNEL32.dll
 0002:0000004c       __imp__SetFilePointer@16   1000f04c     kernel32:KERNEL32.dll
 0002:00000050       __imp__ReadFile@20         1000f050     kernel32:KERNEL32.dll
 0002:00000054       __imp__CreateFileW@28      1000f054     kernel32:KERNEL32.dll
 0002:00000058       __imp__FreeLibrary@4       1000f058     kernel32:KERNEL32.dll
 0002:0000005c       __imp__GetModuleHandleExW@12 1000f05c     kernel32:KERNEL32.dll
 0002:00000060       __imp__LoadLibraryExW@12   1000f060     kernel32:KERNEL32.dll
 0002:00000064       __imp__GetSystemDirectoryW@8 1000f064     kernel32:KERNEL32.dll
 0002:00000068       __imp__GetModuleFileNameW@12 1000f068     kernel32:KERNEL32.dll
 0002:0000006c       __imp__GetLongPathNameW@12 1000f06c     kernel32:KERNEL32.dll
 0002:00000070       __imp__MultiByteToWideChar@24 1000f070     kernel32:KERNEL32.dll
 0002:00000074       __imp__WideCharToMultiByte@32 1000f074     kernel32:KERNEL32.dll
 0002:00000078       __imp__UnhandledExceptionFilter@4 1000f078     kernel32:KERNEL32.dll
 0002:0000007c       __imp__SetUnhandledExceptionFilter@4 1000f07c     kernel32:KERNEL32.dll
 0002:00000080       __imp__GetCurrentProcess@0 1000f080     kernel32:KERNEL32.dll
 0002:00000084       __imp__TerminateProcess@8  1000f084     kernel32:KERNEL32.dll
 0002:00000088       __imp__IsProcessorFeaturePresent@4 1000f088     kernel32:KERNEL32.dll
 0002:0000008c       __imp__IsDebuggerPresent@0 1000f08c     kernel32:KERNEL32.dll
 0002:00000090       __imp__QueryPerformanceCounter@4 1000f090     kernel32:KERNEL32.dll
 0002:00000094       __imp__GetSystemTimeAsFileTime@4 1000f094     kernel32:KERNEL32.dll
 0002:00000098       __imp__DisableThreadLibraryCalls@4 1000f098     kernel32:KERNEL32.dll
 0002:0000009c       __imp__InitializeSListHead@4 1000f09c     kernel32:KERNEL32.dll
 0002:000000a0       \177KERNEL32_NULL_THUNK_DATA 1000f0a0     kernel32:KERNEL32.dll
 0002:000000a4       __imp_?unshift@?$codecvt@DDU_Mbstatet@@@std@@QBEHAAU_Mbstatet@@PAD1AAPAD@Z 1000f0a4     msvcprt:MSVCP140.dll
 0002:000000a8       __imp_?_Getcat@?$codecvt@DDU_Mbstatet@@@std@@SAIPAPBVfacet@locale@2@PBV42@@Z 1000f0a8     msvcprt:MSVCP140.dll
 0002:000000ac       __imp_?_Gndec@?$basic_streambuf@DU?$char_traits@D@std@@@std@@IAEPADXZ 1000f0ac     msvcprt:MSVCP140.dll
 0002:000000b0       __imp_?_Init@?$basic_streambuf@DU?$char_traits@D@std@@@std@@IAEXXZ 1000f0b0     msvcprt:MSVCP140.dll
 0002:000000b4       __imp_??6?$basic_ostream@GU?$char_traits@G@std@@@std@@QAEAAV01@I@Z 1000f0b4     msvcprt:MSVCP140.dll
 0002:000000b8       __imp_??6?$basic_ostream@GU?$char_traits@G@std@@@std@@QAEAAV01@K@Z 1000f0b8     msvcprt:MSVCP140.dll
 0002:000000bc       __imp_?id@?$codecvt@DDU_Mbstatet@@@std@@2V0locale@2@A 1000f0bc     msvcprt:MSVCP140.dll
 0002:000000c0       __imp_??6?$basic_ostream@DU?$char_traits@D@std@@@std@@QAEAAV01@I@Z 1000f0c0     msvcprt:MSVCP140.dll
 0002:000000c4       __imp_?getloc@?$basic_streambuf@DU?$char_traits@D@std@@@std@@QBE?AVlocale@2@XZ 1000f0c4     msvcprt:MSVCP140.dll
 0002:000000c8       __imp_?sbumpc@?$basic_streambuf@DU?$char_traits@D@std@@@std@@QAEHXZ 1000f0c8     msvcprt:MSVCP140.dll
 0002:000000cc       __imp_?sgetc@?$basic_streambuf@DU?$char_traits@D@std@@@std@@QAEHXZ 1000f0cc     msvcprt:MSVCP140.dll
 0002:000000d0       __imp_??6?$basic_ostream@GU?$char_traits@G@std@@@std@@QAEAAV01@PBX@Z 1000f0d0     msvcprt:MSVCP140.dll
 0002:000000d4       __imp_??0?$basic_istream@DU?$char_traits@D@std@@@std@@QAE@PAV?$basic_streambuf@DU?$char_traits@D@std@@@1@_N@Z 1000f0d4     msvcprt:MSVCP140.dll
 0002:000000d8       __imp_??1?$basic_istream@DU?$char_traits@D@std@@@std@@UAE@XZ 1000f0d8     msvcprt:MSVCP140.dll
 0002:000000dc       __imp_?read@?$basic_istream@DU?$char_traits@D@std@@@std@@QAEAAV12@PAD_J@Z 1000f0dc     msvcprt:MSVCP140.dll
 0002:000000e0       __imp_?_Fiopen@std@@YAPAU_iobuf@@PBGHH@Z 1000f0e0     msvcprt:MSVCP140.dll
 0002:000000e4       __imp_?_Xbad_alloc@std@@YAXXZ 1000f0e4     msvcprt:MSVCP140.dll
 0002:000000e8       __imp_?in@?$codecvt@DDU_Mbstatet@@@std@@QBEHAAU_Mbstatet@@PBD1AAPBDPAD3AAPAD@Z 1000f0e8     msvcprt:MSVCP140.dll
 0002:000000ec       __imp_??6?$basic_ostream@GU?$char_traits@G@std@@@std@@QAEAAV01@P6AAAVios_base@1@AAV21@@Z@Z 1000f0ec     msvcprt:MSVCP140.dll
 0002:000000f0       __imp_?seekp@?$basic_ostream@DU?$char_traits@D@std@@@std@@QAEAAV12@V?$fpos@U_Mbstatet@@@2@@Z 1000f0f0     msvcprt:MSVCP140.dll
 0002:000000f4       __imp_?tellp@?$basic_ostream@DU?$char_traits@D@std@@@std@@QAE?AV?$fpos@U_Mbstatet@@@2@XZ 1000f0f4     msvcprt:MSVCP140.dll
 0002:000000f8       __imp_?seekg@?$basic_istream@DU?$char_traits@D@std@@@std@@QAEAAV12@V?$fpos@U_Mbstatet@@@2@@Z 1000f0f8     msvcprt:MSVCP140.dll
 0002:000000fc       __imp_??0?$basic_iostream@DU?$char_traits@D@std@@@std@@QAE@PAV?$basic_streambuf@DU?$char_traits@D@std@@@1@@Z 1000f0fc     msvcprt:MSVCP140.dll
 0002:00000100       __imp_??1?$basic_iostream@DU?$char_traits@D@std@@@std@@UAE@XZ 1000f100     msvcprt:MSVCP140.dll
 0002:00000104       __imp_??0?$basic_iostream@GU?$char_traits@G@std@@@std@@QAE@PAV?$basic_streambuf@GU?$char_traits@G@std@@@1@@Z 1000f104     msvcprt:MSVCP140.dll
 0002:00000108       __imp_??1?$basic_iostream@GU?$char_traits@G@std@@@std@@UAE@XZ 1000f108     msvcprt:MSVCP140.dll
 0002:0000010c       __imp_?setw@std@@YA?AU?$_Smanip@_J@1@_J@Z 1000f10c     msvcprt:MSVCP140.dll
 0002:00000110       __imp_??6?$basic_ostream@DU?$char_traits@D@std@@@std@@QAEAAV01@K@Z 1000f110     msvcprt:MSVCP140.dll
 0002:00000114       __imp_?cerr@std@@3V?$basic_ostream@DU?$char_traits@D@std@@@1@A 1000f114     msvcprt:MSVCP140.dll
 0002:00000118       __imp_?always_noconv@codecvt_base@std@@QBE_NXZ 1000f118     msvcprt:MSVCP140.dll
 0002:0000011c       __imp_?out@?$codecvt@DDU_Mbstatet@@@std@@QBEHAAU_Mbstatet@@PBD1AAPBDPAD3AAPAD@Z 1000f11c     msvcprt:MSVCP140.dll
 0002:00000120       __imp_?cout@std@@3V?$basic_ostream@DU?$char_traits@D@std@@@1@A 1000f120     msvcprt:MSVCP140.dll
 0002:00000124       __imp_?put@?$basic_ostream@DU?$char_traits@D@std@@@std@@QAEAAV12@D@Z 1000f124     msvcprt:MSVCP140.dll
 0002:00000128       __imp_??6?$basic_ostream@DU?$char_traits@D@std@@@std@@QAEAAV01@P6AAAV01@AAV01@@Z@Z 1000f128     msvcprt:MSVCP140.dll
 0002:0000012c       __imp_??6?$basic_ostream@GU?$char_traits@G@std@@@std@@QAEAAV01@H@Z 1000f12c     msvcprt:MSVCP140.dll
 0002:00000130       __imp_?widen@?$basic_ios@DU?$char_traits@D@std@@@std@@QBEDD@Z 1000f130     msvcprt:MSVCP140.dll
 0002:00000134       __imp_?id@?$ctype@G@std@@2V0locale@2@A 1000f134     msvcprt:MSVCP140.dll
 0002:00000138       __imp_?xsputn@?$basic_streambuf@GU?$char_traits@G@std@@@std@@MAE_JPBG_J@Z 1000f138     msvcprt:MSVCP140.dll
 0002:0000013c       __imp_?xsputn@?$basic_streambuf@DU?$char_traits@D@std@@@std@@MAE_JPBD_J@Z 1000f13c     msvcprt:MSVCP140.dll
 0002:00000140       __imp_?xsgetn@?$basic_streambuf@GU?$char_traits@G@std@@@std@@MAE_JPAG_J@Z 1000f140     msvcprt:MSVCP140.dll
 0002:00000144       __imp_?xsgetn@?$basic_streambuf@DU?$char_traits@D@std@@@std@@MAE_JPAD_J@Z 1000f144     msvcprt:MSVCP140.dll
 0002:00000148       __imp_?uflow@?$basic_streambuf@GU?$char_traits@G@std@@@std@@MAEGXZ 1000f148     msvcprt:MSVCP140.dll
 0002:0000014c       __imp_?uflow@?$basic_streambuf@DU?$char_traits@D@std@@@std@@MAEHXZ 1000f14c     msvcprt:MSVCP140.dll
 0002:00000150       __imp_?sync@?$basic_streambuf@GU?$char_traits@G@std@@@std@@MAEHXZ 1000f150     msvcprt:MSVCP140.dll
 0002:00000154       __imp_?sync@?$basic_streambuf@DU?$char_traits@D@std@@@std@@MAEHXZ 1000f154     msvcprt:MSVCP140.dll
 0002:00000158       __imp_?showmanyc@?$basic_streambuf@GU?$char_traits@G@std@@@std@@MAE_JXZ 1000f158     msvcprt:MSVCP140.dll
 0002:0000015c       __imp_?showmanyc@?$basic_streambuf@DU?$char_traits@D@std@@@std@@MAE_JXZ 1000f15c     msvcprt:MSVCP140.dll
 0002:00000160       __imp_?setbuf@?$basic_streambuf@GU?$char_traits@G@std@@@std@@MAEPAV12@PAG_J@Z 1000f160     msvcprt:MSVCP140.dll
 0002:00000164       __imp_?setbuf@?$basic_streambuf@DU?$char_traits@D@std@@@std@@MAEPAV12@PAD_J@Z 1000f164     msvcprt:MSVCP140.dll
 0002:00000168       __imp_?imbue@?$basic_streambuf@GU?$char_traits@G@std@@@std@@MAEXABVlocale@2@@Z 1000f168     msvcprt:MSVCP140.dll
 0002:0000016c       __imp_?imbue@?$basic_streambuf@DU?$char_traits@D@std@@@std@@MAEXABVlocale@2@@Z 1000f16c     msvcprt:MSVCP140.dll
 0002:00000170       __imp_?_Unlock@?$basic_streambuf@GU?$char_traits@G@std@@@std@@UAEXXZ 1000f170     msvcprt:MSVCP140.dll
 0002:00000174       __imp_?_Unlock@?$basic_streambuf@DU?$char_traits@D@std@@@std@@UAEXXZ 1000f174     msvcprt:MSVCP140.dll
 0002:00000178       __imp_?_Lock@?$basic_streambuf@GU?$char_traits@G@std@@@std@@UAEXXZ 1000f178     msvcprt:MSVCP140.dll
 0002:0000017c       __imp_?_Lock@?$basic_streambuf@DU?$char_traits@D@std@@@std@@UAEXXZ 1000f17c     msvcprt:MSVCP140.dll
 0002:00000180       __imp_?flush@?$basic_ostream@DU?$char_traits@D@std@@@std@@QAEAAV12@XZ 1000f180     msvcprt:MSVCP140.dll
 0002:00000184       __imp_?write@?$basic_ostream@DU?$char_traits@D@std@@@std@@QAEAAV12@PBD_J@Z 1000f184     msvcprt:MSVCP140.dll
 0002:00000188       __imp_??6?$basic_ostream@DU?$char_traits@D@std@@@std@@QAEAAV01@H@Z 1000f188     msvcprt:MSVCP140.dll
 0002:0000018c       __imp_?_Osfx@?$basic_ostream@DU?$char_traits@D@std@@@std@@QAEXXZ 1000f18c     msvcprt:MSVCP140.dll
 0002:00000190       __imp_??1?$basic_ostream@DU?$char_traits@D@std@@@std@@UAE@XZ 1000f190     msvcprt:MSVCP140.dll
 0002:00000194       __imp_??0?$basic_ostream@DU?$char_traits@D@std@@@std@@QAE@PAV?$basic_streambuf@DU?$char_traits@D@std@@@1@_N@Z 1000f194     msvcprt:MSVCP140.dll
 0002:00000198       __imp_?flush@?$basic_ostream@GU?$char_traits@G@std@@@std@@QAEAAV12@XZ 1000f198     msvcprt:MSVCP140.dll
 0002:0000019c       __imp_?_Osfx@?$basic_ostream@GU?$char_traits@G@std@@@std@@QAEXXZ 1000f19c     msvcprt:MSVCP140.dll
 0002:000001a0       __imp_??1?$basic_ostream@GU?$char_traits@G@std@@@std@@UAE@XZ 1000f1a0     msvcprt:MSVCP140.dll
 0002:000001a4       __imp_??0?$basic_ostream@GU?$char_traits@G@std@@@std@@QAE@PAV?$basic_streambuf@GU?$char_traits@G@std@@@1@_N@Z 1000f1a4     msvcprt:MSVCP140.dll
 0002:000001a8       __imp_??0?$basic_ios@GU?$char_traits@G@std@@@std@@IAE@XZ 1000f1a8     msvcprt:MSVCP140.dll
 0002:000001ac       __imp_?setstate@?$basic_ios@GU?$char_traits@G@std@@@std@@QAEXH_N@Z 1000f1ac     msvcprt:MSVCP140.dll
 0002:000001b0       __imp_??1?$basic_ios@GU?$char_traits@G@std@@@std@@UAE@XZ 1000f1b0     msvcprt:MSVCP140.dll
 0002:000001b4       __imp_??0?$basic_ios@DU?$char_traits@D@std@@@std@@IAE@XZ 1000f1b4     msvcprt:MSVCP140.dll
 0002:000001b8       __imp_?setstate@?$basic_ios@DU?$char_traits@D@std@@@std@@QAEXH_N@Z 1000f1b8     msvcprt:MSVCP140.dll
 0002:000001bc       __imp_??1?$basic_ios@DU?$char_traits@D@std@@@std@@UAE@XZ 1000f1bc     msvcprt:MSVCP140.dll
 0002:000001c0       __imp_?_Pninc@?$basic_streambuf@GU?$char_traits@G@std@@@std@@IAEPAGXZ 1000f1c0     msvcprt:MSVCP140.dll
 0002:000001c4       __imp_?gbump@?$basic_streambuf@GU?$char_traits@G@std@@@std@@IAEXH@Z 1000f1c4     msvcprt:MSVCP140.dll
 0002:000001c8       __imp_?sputn@?$basic_streambuf@GU?$char_traits@G@std@@@std@@QAE_JPBG_J@Z 1000f1c8     msvcprt:MSVCP140.dll
 0002:000001cc       __imp_?sputc@?$basic_streambuf@GU?$char_traits@G@std@@@std@@QAEGG@Z 1000f1cc     msvcprt:MSVCP140.dll
 0002:000001d0       __imp_??1?$basic_streambuf@GU?$char_traits@G@std@@@std@@UAE@XZ 1000f1d0     msvcprt:MSVCP140.dll
 0002:000001d4       __imp_??0?$basic_streambuf@GU?$char_traits@G@std@@@std@@IAE@XZ 1000f1d4     msvcprt:MSVCP140.dll
 0002:000001d8       __imp_?_Pninc@?$basic_streambuf@DU?$char_traits@D@std@@@std@@IAEPADXZ 1000f1d8     msvcprt:MSVCP140.dll
 0002:000001dc       __imp_?sputn@?$basic_streambuf@DU?$char_traits@D@std@@@std@@QAE_JPBD_J@Z 1000f1dc     msvcprt:MSVCP140.dll
 0002:000001e0       __imp_?sputc@?$basic_streambuf@DU?$char_traits@D@std@@@std@@QAEHD@Z 1000f1e0     msvcprt:MSVCP140.dll
 0002:000001e4       __imp_??1?$basic_streambuf@DU?$char_traits@D@std@@@std@@UAE@XZ 1000f1e4     msvcprt:MSVCP140.dll
 0002:000001e8       __imp_??0?$basic_streambuf@DU?$char_traits@D@std@@@std@@IAE@XZ 1000f1e8     msvcprt:MSVCP140.dll
 0002:000001ec       __imp_?getloc@ios_base@std@@QBE?AVlocale@2@XZ 1000f1ec     msvcprt:MSVCP140.dll
 0002:000001f0       __imp_?exceptions@ios_base@std@@QAEXH@Z 1000f1f0     msvcprt:MSVCP140.dll
 0002:000001f4       __imp_?_Getcat@?$ctype@G@std@@SAIPAPBVfacet@locale@2@PBV42@@Z 1000f1f4     msvcprt:MSVCP140.dll
 0002:000001f8       __imp_?widen@?$ctype@G@std@@QBEGD@Z 1000f1f8     msvcprt:MSVCP140.dll
 0002:000001fc       __imp_?_Getgloballocale@locale@std@@CAPAV_Locimp@12@XZ 1000f1fc     msvcprt:MSVCP140.dll
 0002:00000200       __imp_??Bid@locale@std@@QAEIXZ 1000f200     msvcprt:MSVCP140.dll
 0002:00000204       __imp_?_Xout_of_range@std@@YAXPBD@Z 1000f204     msvcprt:MSVCP140.dll
 0002:00000208       __imp_?_Xlength_error@std@@YAXPBD@Z 1000f208     msvcprt:MSVCP140.dll
 0002:0000020c       __imp_?uncaught_exception@std@@YA_NXZ 1000f20c     msvcprt:MSVCP140.dll
 0002:00000210       __imp_??1_Lockit@std@@QAE@XZ 1000f210     msvcprt:MSVCP140.dll
 0002:00000214       __imp_??0_Lockit@std@@QAE@H@Z 1000f214     msvcprt:MSVCP140.dll
 0002:00000218       \177MSVCP140_NULL_THUNK_DATA 1000f218     msvcprt:MSVCP140.dll
 0002:0000021c       __imp__memcpy              1000f21c     vcruntime:VCRUNTIME140.dll
 0002:00000220       __imp__memmove             1000f220     vcruntime:VCRUNTIME140.dll
 0002:00000224       __imp____std_exception_copy 1000f224     vcruntime:VCRUNTIME140.dll
 0002:00000228       __imp____std_type_info_destroy_list 1000f228     vcruntime:VCRUNTIME140.dll
 0002:0000022c       __imp___except_handler4_common 1000f22c     vcruntime:VCRUNTIME140.dll
 0002:00000230       __imp____std_terminate     1000f230     vcruntime:VCRUNTIME140.dll
 0002:00000234       __imp___purecall           1000f234     vcruntime:VCRUNTIME140.dll
 0002:00000238       __imp__memset              1000f238     vcruntime:VCRUNTIME140.dll
 0002:0000023c       __imp____CxxFrameHandler3  1000f23c     vcruntime:VCRUNTIME140.dll
 0002:00000240       __imp___CxxThrowException@8 1000f240     vcruntime:VCRUNTIME140.dll
 0002:00000244       __imp____std_exception_destroy 1000f244     vcruntime:VCRUNTIME140.dll
 0002:00000248       __imp__memchr              1000f248     vcruntime:VCRUNTIME140.dll
 0002:0000024c       \177VCRUNTIME140_NULL_THUNK_DATA 1000f24c     vcruntime:VCRUNTIME140.dll
 0002:00000250       __imp___unlock_file        1000f250     ucrt:api-ms-win-crt-filesystem-l1-1-0.dll
 0002:00000254       __imp___lock_file          1000f254     ucrt:api-ms-win-crt-filesystem-l1-1-0.dll
 0002:00000258       \177api-ms-win-crt-filesystem-l1-1-0_NULL_THUNK_DATA 1000f258     ucrt:api-ms-win-crt-filesystem-l1-1-0.dll
 0002:0000025c       __imp__free                1000f25c     ucrt:api-ms-win-crt-heap-l1-1-0.dll
 0002:00000260       __imp___callnewh           1000f260     ucrt:api-ms-win-crt-heap-l1-1-0.dll
 0002:00000264       __imp__malloc              1000f264     ucrt:api-ms-win-crt-heap-l1-1-0.dll
 0002:00000268       \177api-ms-win-crt-heap-l1-1-0_NULL_THUNK_DATA 1000f268     ucrt:api-ms-win-crt-heap-l1-1-0.dll
 0002:0000026c       __imp___crt_atexit         1000f26c     ucrt:api-ms-win-crt-runtime-l1-1-0.dll
 0002:00000270       __imp___execute_onexit_table 1000f270     ucrt:api-ms-win-crt-runtime-l1-1-0.dll
 0002:00000274       __imp___register_onexit_function 1000f274     ucrt:api-ms-win-crt-runtime-l1-1-0.dll
 0002:00000278       __imp___cexit              1000f278     ucrt:api-ms-win-crt-runtime-l1-1-0.dll
 0002:0000027c       __imp___initialize_narrow_environment 1000f27c     ucrt:api-ms-win-crt-runtime-l1-1-0.dll
 0002:00000280       __imp___configure_narrow_argv 1000f280     ucrt:api-ms-win-crt-runtime-l1-1-0.dll
 0002:00000284       __imp___seh_filter_dll     1000f284     ucrt:api-ms-win-crt-runtime-l1-1-0.dll
 0002:00000288       __imp___initterm           1000f288     ucrt:api-ms-win-crt-runtime-l1-1-0.dll
 0002:0000028c       __imp___initterm_e         1000f28c     ucrt:api-ms-win-crt-runtime-l1-1-0.dll
 0002:00000290       __imp___invalid_parameter_noinfo_noreturn 1000f290     ucrt:api-ms-win-crt-runtime-l1-1-0.dll
 0002:00000294       __imp___initialize_onexit_table 1000f294     ucrt:api-ms-win-crt-runtime-l1-1-0.dll
 0002:00000298       \177api-ms-win-crt-runtime-l1-1-0_NULL_THUNK_DATA 1000f298     ucrt:api-ms-win-crt-runtime-l1-1-0.dll
 0002:0000029c       __imp____stdio_common_vswscanf 1000f29c     ucrt:api-ms-win-crt-stdio-l1-1-0.dll
 0002:000002a0       __imp__setvbuf             1000f2a0     ucrt:api-ms-win-crt-stdio-l1-1-0.dll
 0002:000002a4       __imp__fwrite              1000f2a4     ucrt:api-ms-win-crt-stdio-l1-1-0.dll
 0002:000002a8       __imp___fseeki64           1000f2a8     ucrt:api-ms-win-crt-stdio-l1-1-0.dll
 0002:000002ac       __imp__fsetpos             1000f2ac     ucrt:api-ms-win-crt-stdio-l1-1-0.dll
 0002:000002b0       __imp____acrt_iob_func     1000f2b0     ucrt:api-ms-win-crt-stdio-l1-1-0.dll
 0002:000002b4       __imp____stdio_common_vfprintf 1000f2b4     ucrt:api-ms-win-crt-stdio-l1-1-0.dll
 0002:000002b8       __imp__ungetc              1000f2b8     ucrt:api-ms-win-crt-stdio-l1-1-0.dll
 0002:000002bc       __imp____stdio_common_vsnwprintf_s 1000f2bc     ucrt:api-ms-win-crt-stdio-l1-1-0.dll
 0002:000002c0       __imp___get_stream_buffer_pointers 1000f2c0     ucrt:api-ms-win-crt-stdio-l1-1-0.dll
 0002:000002c4       __imp__fclose              1000f2c4     ucrt:api-ms-win-crt-stdio-l1-1-0.dll
 0002:000002c8       __imp__fflush              1000f2c8     ucrt:api-ms-win-crt-stdio-l1-1-0.dll
 0002:000002cc       __imp__fgetc               1000f2cc     ucrt:api-ms-win-crt-stdio-l1-1-0.dll
 0002:000002d0       __imp__fgetpos             1000f2d0     ucrt:api-ms-win-crt-stdio-l1-1-0.dll
 0002:000002d4       __imp__fputc               1000f2d4     ucrt:api-ms-win-crt-stdio-l1-1-0.dll
 0002:000002d8       __imp__fread               1000f2d8     ucrt:api-ms-win-crt-stdio-l1-1-0.dll
 0002:000002dc       \177api-ms-win-crt-stdio-l1-1-0_NULL_THUNK_DATA 1000f2dc     ucrt:api-ms-win-crt-stdio-l1-1-0.dll
 0002:000002e0       __imp__wcslen              1000f2e0     ucrt:api-ms-win-crt-string-l1-1-0.dll
 0002:000002e4       __imp__strlen              1000f2e4     ucrt:api-ms-win-crt-string-l1-1-0.dll
 0002:000002e8       __imp__tolower             1000f2e8     ucrt:api-ms-win-crt-string-l1-1-0.dll
 0002:000002ec       __imp__isspace             1000f2ec     ucrt:api-ms-win-crt-string-l1-1-0.dll
 0002:000002f0       \177api-ms-win-crt-string-l1-1-0_NULL_THUNK_DATA 1000f2f0     ucrt:api-ms-win-crt-string-l1-1-0.dll
 0002:000002f4       __imp__MsiRecordGetStringW@16 1000f2f4     msi:msi.dll
 0002:000002f8       __imp__MsiRecordGetFieldCount@4 1000f2f8     msi:msi.dll
 0002:000002fc       __imp__MsiOpenDatabaseW@12 1000f2fc     msi:msi.dll
 0002:00000300       __imp__MsiViewFetch@8      1000f300     msi:msi.dll
 0002:00000304       __imp__MsiCloseHandle@4    1000f304     msi:msi.dll
 0002:00000308       __imp__MsiViewExecute@8    1000f308     msi:msi.dll
 0002:0000030c       __imp__MsiDatabaseOpenViewW@12 1000f30c     msi:msi.dll
 0002:00000310       \177msi_NULL_THUNK_DATA    1000f310     msi:msi.dll
 0002:00000314       __imp__IIDFromString@8     1000f314     ole32:ole32.dll
 0002:00000318       __imp__StringFromGUID2@12  1000f318     ole32:ole32.dll
 0002:0000031c       \177ole32_NULL_THUNK_DATA  1000f31c     ole32:ole32.dll
 0002:00000320       ___guard_check_icall_fptr  1000f320     MSVCRT:guard_support.obj
 0002:00000324       ___xc_a                    1000f324     MSVCRT:initializers.obj
 0002:00000338       ___xc_z                    1000f338     MSVCRT:initializers.obj
 0002:0000033c       ___xi_a                    1000f33c     MSVCRT:initializers.obj
 0002:00000340       ___xi_z                    1000f340     MSVCRT:initializers.obj
 0002:00000344       ___xp_a                    1000f344     MSVCRT:initializers.obj
 0002:00000348       ___xp_z                    1000f348     MSVCRT:initializers.obj
 0002:0000034c       ___xt_a                    1000f34c     MSVCRT:initializers.obj
 0002:00000350       ___xt_z                    1000f350     MSVCRT:initializers.obj
 0002:0000035c       ??_7exception@std@@6B@     1000f35c     ErrorHandling.obj
 0002:00000364       ??_C@_0BC@EOODALEL@Unknown?5exception@ 1000f364     ErrorHandling.obj
 0002:0000037c       ??_7bad_alloc@std@@6B@     1000f37c     ErrorHandling.obj
 0002:00000388       ??_7bad_array_new_length@std@@6B@ 1000f388     ErrorHandling.obj
 0002:00000390       ??_C@_0BF@KINCDENJ@bad?5array?5new?5length@ 1000f390     ErrorHandling.obj
 0002:000003a8       ??_C@_0BA@JFNIOLAK@string?5too?5long@ 1000f3a8     ErrorHandling.obj
 0002:000003b8       ??_C@_00CNPNBAHC@@         1000f3b8     ErrorHandling.obj
 0002:000003c0       ??_7bad_cast@std@@6B@      1000f3c0     ErrorHandling.obj
 0002:000003c8       ??_C@_08EPJLHIJG@bad?5cast@ 1000f3c8     ErrorHandling.obj
 0002:000003d8       ??_7?$basic_stringbuf@GU?$char_traits@G@std@@V?$allocator@G@2@@std@@6B@ 1000f3d8     ErrorHandling.obj
 0002:00000418       ??_7?$basic_ostringstream@GU?$char_traits@G@std@@V?$allocator@G@2@@std@@6B@ 1000f418     ErrorHandling.obj
 0002:0000041c       ??_8?$basic_ostringstream@GU?$char_traits@G@std@@V?$allocator@G@2@@std@@7B@ 1000f41c     ErrorHandling.obj
 0002:00000424       ??_C@_02HHAEMJFE@?2?1@     1000f424     ErrorHandling.obj
 0002:00000428       ??_C@_0BJ@HAJDFNON@Exception?5with?5message?5?8@ 1000f428     ErrorHandling.obj
 0002:00000444       ??_C@_08OFLCGKIF@?8?5caught@ 1000f444     ErrorHandling.obj
 0002:00000450       ??_C@_1DC@DNLNKJFM@?$AAU?$AAn?$AAk?$AAn?$AAo?$AAw?$AAn?$AA?5?$AAe?$AAx?$AAc?$AAe?$AAp?$AAt?$AAi@ 1000f450     ErrorHandling.obj
 0002:00000488       ??_7?$basic_stringbuf@DU?$char_traits@D@std@@V?$allocator@D@2@@std@@6B@ 1000f488     ErrorHandling.obj
 0002:000004c8       ??_7?$basic_ostringstream@DU?$char_traits@D@std@@V?$allocator@D@2@@std@@6B@ 1000f4c8     ErrorHandling.obj
 0002:000004cc       ??_8?$basic_ostringstream@DU?$char_traits@D@std@@V?$allocator@D@2@@std@@7B@ 1000f4cc     ErrorHandling.obj
 0002:000004d4       ??_C@_04KJCOMIHH@?$CI?$CJ?3?5@ 1000f4d4     ErrorHandling.obj
 0002:000004dc       ??_C@_05OKLJFBOO@?$CJ?5at?5@ 1000f4dc     ErrorHandling.obj
 0002:000004e4       ??_C@_01ODHLEDKK@?$CI@     1000f4e4     ErrorHandling.obj
 0002:000004e8       ??_C@_06PKHGJEE@?$DL?4?0?3?$CB?$DP@ 1000f4e8     ErrorHandling.obj
 0002:000004f0       ??_C@_01CLKCMJKC@?5@       1000f4f0     ErrorHandling.obj
 0002:000004f4       ??_C@_02KHOJGJKF@?4?5@     1000f4f4     ErrorHandling.obj
 0002:000004f8       ??_C@_0BI@CFPLBAOH@invalid?5string?5position@ 1000f4f8     ErrorHandling.obj
 0002:00000510       ?pathSeparator@FileUtils@@3GB 1000f510     FileUtils.obj
 0002:0000051c       ??_C@_15MNCACJLI@?$AA?2?$AA?1@ 1000f51c     FileUtils.obj
 0002:00000528       ??_7runtime_error@std@@6B@ 1000f528     Guid.obj
 0002:00000534       ??_7JpErrorBase@@6B@       1000f534     Guid.obj
 0002:0000053c       ??_7?$JpError@Vruntime_error@std@@@@6BJpErrorBase@@@ 1000f53c     Guid.obj
 0002:00000544       ??_7?$JpError@Vruntime_error@std@@@@6Bruntime_error@std@@@ 1000f544     Guid.obj
 0002:0000054c       ??_C@_0CA@BMPGLJJN@?$GAanonymous?9namespace?8?3?3initGuid@ 1000f54c     Guid.obj
 0002:0000056c       ??_C@_0DC@KGKIHNFD@s?2src?2jdk?4jpackage?2windows?2nati@ 1000f56c     Guid.obj
 0002:000005a0       ??_C@_0P@CINEOJHO@IIDFromString?$CI@ 1000f5a0     Guid.obj
 0002:000005b0       ??_C@_08EPEDOCDA@?$CJ?5failed@ 1000f5b0     Guid.obj
 0002:000005bc       ??_C@_13EHOOFIKC@?$AA?$HN@ 1000f5bc     Guid.obj
 0002:000005c0       ??_C@_13GCIFAHHO@?$AA?$HL@ 1000f5c0     Guid.obj
 0002:000005c4       ??_C@_0P@ILPPFPKA@Guid?3?3toString@ 1000f5c4     Guid.obj
 0002:000005d4       ??_C@_0BJ@GPEFFCPB@StringFromGUID2?$CI?$CJ?5failed@ 1000f5d4     Guid.obj
 0002:000005f0       ??_C@_02KPKOKMHB@?$CFS@    1000f5f0     IconSwap.obj
 0002:000005f4       ??_C@_0CC@PCGMLBAN@Error?3?5Failed?5to?5allocate?5memor@ 1000f5f4     IconSwap.obj
 0002:00000618       ??_C@_0BF@FFNHJCPB@jni?3?3toUnicodeString@ 1000f618     JniUtils.obj
 0002:00000630       ??_C@_0DL@OIDODNLL@s?2src?2jdk?4jpackage?2windows?2nati@ 1000f630     JniUtils.obj
 0002:0000066c       ??_C@_0BI@NCGLOMCE@GetStringChars?$CI?$CJ?5failed@ 1000f66c     JniUtils.obj
 0002:00000684       ??_C@_0P@BMIEBKCM@jni?3?3toJString@ 1000f684     JniUtils.obj
 0002:00000694       ??_C@_0BD@OGPAMFEO@NewString?$CI?$CJ?5failed@ 1000f694     JniUtils.obj
 0002:000006a8       ??_C@_0EO@PDHCJKHH@AtEndOfScope?$DMclass?5?$DMlambda_bafb@ 1000f6a8     JniUtils.obj
 0002:000006f8       ??_C@_0DB@BLDOPEOL@s?2src?2jdk?4jpackage?2share?2native@ 1000f6f8     JniUtils.obj
 0002:0000072c       ??_C@_0BA@FOIKENOD@vector?5too?5long@ 1000f72c     JniUtils.obj
 0002:00000740       ??_7LogAppender@@6B@       1000f740     Log.obj
 0002:0000074c       ??_7StreamLogAppender@@6B@ 1000f74c     Log.obj
 0002:00000754       ??_C@_1M@MGIHBMCI@?$AAT?$AAR?$AAA?$AAC?$AAE@ 1000f754     Log.obj
 0002:00000760       ??_C@_19FILLMKCG@?$AAI?$AAN?$AAF?$AAO@ 1000f760     Log.obj
 0002:0000076c       ??_C@_1BA@KPCCLDOC@?$AAW?$AAA?$AAR?$AAN?$AAI?$AAN?$AAG@ 1000f76c     Log.obj
 0002:0000077c       ??_C@_1M@BJACCECO@?$AAE?$AAR?$AAR?$AAO?$AAR@ 1000f77c     Log.obj
 0002:00000788       ??_C@_1BA@HABJOAEE@?$AAU?$AAN?$AAK?$AAN?$AAO?$AAW?$AAN@ 1000f788     Log.obj
 0002:00000798       ??_C@_15ELOONFKJ@?$AA?3?$AA?5@ 1000f798     Log.obj
 0002:000007a0       ??_C@_15CMBHNMLL@?$AA?5?$AA?$CI@ 1000f7a0     Log.obj
 0002:000007a8       ??_C@_01JLIPDDHJ@?3@       1000f7a8     Log.obj
 0002:000007ac       ??_C@_01PKGAHCOL@?$CJ@     1000f7ac     Log.obj
 0002:000007b4       ??_7Error@msi@@6B@         1000f7b4     MsiDb.obj
 0002:000007c0       ??_7NoMoreItemsError@msi@@6B@ 1000f7c0     MsiDb.obj
 0002:000007cc       ??_7?$basic_filebuf@DU?$char_traits@D@std@@@std@@6B@ 1000f7cc     MsiDb.obj
 0002:00000808       ??_C@_0BF@HECCNMNO@?$CJ?5failed?5with?5error?$DN@ 1000f808     MsiDb.obj
 0002:00000824       ??_7?$JpError@VError@msi@@@@6BJpErrorBase@@@ 1000f824     MsiDb.obj
 0002:0000082c       ??_7?$JpError@VError@msi@@@@6BError@msi@@@ 1000f82c     MsiDb.obj
 0002:00000834       ??_C@_0CJ@GCOBILED@msi?3?3?$GAanonymous?9namespace?8?3?3ope@ 1000f834     MsiDb.obj
 0002:00000860       ??_C@_0DD@OMCLKPIE@s?2src?2jdk?4jpackage?2windows?2nati@ 1000f860     MsiDb.obj
 0002:00000894       ??_C@_0BB@PGLHLGNP@MsiOpenDatabase?$CI@ 1000f894     MsiDb.obj
 0002:000008a8       ??_C@_0BN@OKIJDOFB@?0?5MSIDBOPEN_READONLY?$CJ?5failed@ 1000f8a8     MsiDb.obj
 0002:000008c8       ??_C@_0CO@LCNLDDEH@SELECT?5Value?5FROM?5Property?5WHER@ 1000f8c8     MsiDb.obj
 0002:000008f8       ??_C@_01GEODFPGF@?8@       1000f8f8     MsiDb.obj
 0002:000008fc       ??_C@_0BL@BEBKODAA@msi?3?3Database?3?3getProperty@ 1000f8fc     MsiDb.obj
 0002:00000918       ??_C@_0BG@MBCEGHCK@record?4getFieldCount?$CI@ 1000f918     MsiDb.obj
 0002:00000930       ??_C@_02KEGNLNML@?0?5@     1000f930     MsiDb.obj
 0002:00000934       ??_C@_0BM@HHAOOHHI@?$CJ?5returned?5unexpected?5value@ 1000f934     MsiDb.obj
 0002:00000950       ??_C@_0CD@IBMNDFG@msi?3?3DatabaseRecord?3?3getFieldCo@ 1000f950     MsiDb.obj
 0002:00000974       ??_C@_0CA@OEIMMPMH@MsiRecordGetFieldCount?$CI?$CJ?5failed@ 1000f974     MsiDb.obj
 0002:00000994       ??_C@_0CA@IOLDDDHB@msi?3?3DatabaseView?3?3DatabaseView@ 1000f994     MsiDb.obj
 0002:000009b4       ??_C@_0BF@NMGELMFN@MsiDatabaseOpenView?$CI@ 1000f9b4     MsiDb.obj
 0002:000009cc       ??_C@_0BA@FCCIPHNF@MsiViewExecute?$CI@ 1000f9cc     MsiDb.obj
 0002:000009e0       ??_7?$JpError@VNoMoreItemsError@msi@@@@6BJpErrorBase@@@ 1000f9e0     MsiDb.obj
 0002:000009e8       ??_7?$JpError@VNoMoreItemsError@msi@@@@6BNoMoreItemsError@msi@@@ 1000f9e8     MsiDb.obj
 0002:000009f0       ??_C@_0BJ@FJKBHIAJ@msi?3?3DatabaseView?3?3fetch@ 1000f9f0     MsiDb.obj
 0002:00000a0c       ??_C@_0BD@JIBAHKDM@No?5more?5items?5in?5?$FL@ 1000fa0c     MsiDb.obj
 0002:00000a20       ??_C@_07MPHPDHHG@?$FN?5query@ 1000fa20     MsiDb.obj
 0002:00000a28       ??_C@_0BM@HAGAJLHK@msi?3?3DatabaseView?3?3tryFetch@ 1000fa28     MsiDb.obj
 0002:00000a44       ??_C@_0O@CGOANHIE@MsiViewFetch?$CI@ 1000fa44     MsiDb.obj
 0002:00000a54       ??_C@_0BB@GCADKGJO@map?1set?5too?5long@ 1000fa54     MsiUtils.obj
 0002:00000a6c       ??_7SysError@@6B@          1000fa6c     MsiUtils.obj
 0002:00000a74       ??_C@_0DG@PCFDMKKJ@s?2src?2jdk?4jpackage?2windows?2nati@ 1000fa74     MsiUtils.obj
 0002:00000aac       ??_C@_0BA@PCHEKKD@MsiCloseHandle?$CI@ 1000faac     MsiUtils.obj
 0002:00000abc       ??_C@_1CI@KPCFIJEE@?$AAm?$AAs?$AAi?$AA?3?$AA?3?$AAc?$AAl?$AAo?$AAs?$AAe?$AAM?$AAS?$AAI?$AAH?$AAA@ 1000fabc     MsiUtils.obj
 0002:00000ae8       ??_C@_1GM@KLMFKHLE@?$AAs?$AA?2?$AAs?$AAr?$AAc?$AA?2?$AAj?$AAd?$AAk?$AA?4?$AAj?$AAp?$AAa?$AAc?$AAk@ 1000fae8     MsiUtils.obj
 0002:00000b54       ??_C@_0BD@MMKFHCJA@MsiRecordGetString@ 1000fb54     MsiUtils.obj
 0002:00000b6c       ??_7?$JpError@VSysError@@@@6BJpErrorBase@@@ 1000fb6c     MsiUtils.obj
 0002:00000b74       ??_7?$JpError@VSysError@@@@6BSysError@@@ 1000fb74     MsiUtils.obj
 0002:00000b7c       ??_C@_01LBDDMOBJ@?$FN@     1000fb7c     MsiUtils.obj
 0002:00000b80       ??_C@_0M@DFKEBDIB@MSI?5error?5?$FL@ 1000fb80     MsiUtils.obj
 0002:00000b8c       ??_C@_1BG@GJFCCOOL@?$AAm?$AAs?$AAi?$AAm?$AAs?$AAg?$AA?4?$AAd?$AAl?$AAl@ 1000fb8c     MsiUtils.obj
 0002:00000ba4       ??_C@_0CI@PIBEIPJI@msi?3?3?$GAanonymous?9namespace?8?3?3mak@ 1000fba4     MsiUtils.obj
 0002:00000bcc       ??_C@_0N@LDHCNCJC@System?5error@ 1000fbcc     MsiUtils.obj
 0002:00000bdc       ??_C@_0BA@HCMFAFI@LoadLibraryExW?$CI@ 1000fbdc     MsiUtils.obj
 0002:00000bec       ??_C@_1BO@BCJFDHGG@?$AAN?$AAo?$AA?5?$AAd?$AAe?$AAs?$AAc?$AAr?$AAi?$AAp?$AAt?$AAi?$AAo?$AAn@ 1000fbec     MsiUtils.obj
 0002:00000c0c       ??_C@_02GBLMOEJC@?5?$FL@   1000fc0c     MsiUtils.obj
 0002:00000c10       ??_C@_0CI@DLOLPNJF@msi?3?3?$GAanonymous?9namespace?8?3?3get@ 1000fc10     MsiUtils.obj
 0002:00000c40       ??_C@_1HI@LAPLFCFO@?$AA?$CF?$AA0?$AA4?$AAu?$AA?1?$AA?$CF?$AA0?$AA2?$AAu?$AA?1?$AA?$CF?$AA0?$AA2?$AAu?$AA?5@ 1000fc40     PlatformLogEvent.obj
 0002:00000cb8       ??_C@_1BA@LEPJIIOK@?$AAU?$AAn?$AAk?$AAn?$AAo?$AAw?$AAn@ 1000fcb8     PlatformLogEvent.obj
 0002:00000cc8       ??_C@_0CD@IGBKECFO@ResourceEditor?3?3FileLock?3?3FileL@ 1000fcc8     ResourceEditor.obj
 0002:00000cf0       ??_C@_0EB@PMHIEHM@s?2src?2jdk?4jpackage?2windows?2nati@ 1000fcf0     ResourceEditor.obj
 0002:00000d34       ??_C@_0BF@EEHHJMNO@BeginUpdateResource?$CI@ 1000fd34     ResourceEditor.obj
 0002:00000d4c       ??_C@_0CE@BDEPPPPO@ResourceEditor?3?3FileLock?3?3?$HOFile@ 1000fd4c     ResourceEditor.obj
 0002:00000d70       ??_C@_0BD@EKOCFJGM@EndUpdateResource?$CI@ 1000fd70     ResourceEditor.obj
 0002:00000d84       ??_C@_09CNJBHKGC@?$CJ?5failed?4@ 1000fd84     ResourceEditor.obj
 0002:00000d90       ??_C@_13GMDMCADD@?$AA?$CD@ 1000fd90     ResourceEditor.obj
 0002:00000d94       ??_C@_0BG@LIOFEBPP@ResourceEditor?3?3apply@ 1000fd94     ResourceEditor.obj
 0002:00000dac       ??_C@_0BI@OLOABBFD@UpdateResource?$CI?$CJ?5failed@ 1000fdac     ResourceEditor.obj
 0002:00000dc8       ??_7?$basic_ifstream@DU?$char_traits@D@std@@@std@@6B@ 1000fdc8     ResourceEditor.obj
 0002:00000dcc       ??_8?$basic_ifstream@DU?$char_traits@D@std@@@std@@7B@ 1000fdcc     ResourceEditor.obj
 0002:00000dd4       ??_C@_08DCJJILDN@?5?$CIname?$DN?8@ 1000fdd4     Resources.obj
 0002:00000de0       ??_C@_09BLBBBHKI@?8?0?5type?$DN?8@ 1000fde0     Resources.obj
 0002:00000dec       ??_C@_02HJPKOJGD@?8?$CJ@   1000fdec     Resources.obj
 0002:00000df0       ??_C@_0BB@IHINCNEI@Resource?3?3getPtr@ 1000fdf0     Resources.obj
 0002:00000e04       ??_C@_0DH@MGEPKFIC@s?2src?2jdk?4jpackage?2windows?2nati@ 1000fe04     Resources.obj
 0002:00000e3c       ??_C@_0BF@IIGEHKJO@cannot?5find?5resource@ 1000fe3c     Resources.obj
 0002:00000e54       ??_C@_0BF@IICCOAKJ@cannot?5load?5resource@ 1000fe54     Resources.obj
 0002:00000e6c       ??_C@_0DO@FONBEFMI@s?2src?2jdk?4jpackage?2windows?2nati@ 1000fe6c     VersionInfo.obj
 0002:00000eac       ??_C@_1BI@FCMLLAGN@?$AA?$CF?$AAd?$AA?4?$AA?$CF?$AAd?$AA?4?$AA?$CF?$AAd?$AA?4?$AA?$CF?$AAd@ 1000feac     VersionInfo.obj
 0002:00000ec4       ??_C@_0DK@CCIPDNEP@?$GAanonymous?9namespace?8?3?3FixedFil@ 1000fec4     VersionInfo.obj
 0002:00000f00       ??_C@_0CA@BBEPHEMG@Malformed?5file?5version?5value?3?5?$FL@ 1000ff00     VersionInfo.obj
 0002:00000f20       ??_C@_0CB@DNPOCCOG@?$GAanonymous?9namespace?8?3?3writeWOR@ 1000ff20     VersionInfo.obj
 0002:00000f44       ??_C@_0BD@KNFLMKLN@Invalid?5WORD?5value@ 1000ff44     VersionInfo.obj
 0002:00000f58       ??_C@_0CH@DDHGPDCC@?$GAanonymous?9namespace?8?3?3add32bit@ 1000ff58     VersionInfo.obj
 0002:00000f80       ??_C@_0CD@PIIDNOPO@Invalid?5data?5written?5in?5the?5str@ 1000ff80     VersionInfo.obj
 0002:00000fa4       ??_C@_0CP@MFBNHLMG@?$GAanonymous?9namespace?8?3?3StreamSi@ 1000ffa4     VersionInfo.obj
 0002:00000fd4       ??_C@_0BM@PFELLINL@Invalid?5negative?5size?5value@ 1000ffd4     VersionInfo.obj
 0002:00000ff0       ??_C@_1DE@HKLKJHCE@?$AAF?$AAI?$AAX?$AAE?$AAD?$AAF?$AAI?$AAL?$AAE?$AAI?$AAN?$AAF?$AAO?$AA_?$AAF@ 1000fff0     VersionInfo.obj
 0002:00001028       ??_7?$basic_stringstream@DU?$char_traits@D@std@@V?$allocator@D@2@@std@@6B@ 10010028     VersionInfo.obj
 0002:0000102c       ??_8?$basic_stringstream@DU?$char_traits@D@std@@V?$allocator@D@2@@std@@7B?$basic_istream@DU?$char_traits@D@std@@@1@@ 1001002c     VersionInfo.obj
 0002:00001034       ??_8?$basic_stringstream@DU?$char_traits@D@std@@V?$allocator@D@2@@std@@7B?$basic_ostream@DU?$char_traits@D@std@@@1@@ 10010034     VersionInfo.obj
 0002:0000103c       ??_C@_0BD@LPEGHGBH@VersionInfo?3?3apply@ 1001003c     VersionInfo.obj
 0002:00001050       ??_C@_0CH@NICCFHCM@Missing?5mandatory?5FILEVERSION?5p@ 10010050     VersionInfo.obj
 0002:0000107c       ??_7?$basic_stringstream@GU?$char_traits@G@std@@V?$allocator@G@2@@std@@6B@ 1001007c     VersionInfo.obj
 0002:00001080       ??_8?$basic_stringstream@GU?$char_traits@G@std@@V?$allocator@G@2@@std@@7B?$basic_istream@GU?$char_traits@G@std@@@1@@ 10010080     VersionInfo.obj
 0002:00001088       ??_8?$basic_stringstream@GU?$char_traits@G@std@@V?$allocator@G@2@@std@@7B?$basic_ostream@GU?$char_traits@G@std@@@1@@ 10010088     VersionInfo.obj
 0002:00001090       ??_C@_1BO@HMJELANO@?$AAF?$AAI?$AAX?$AAE?$AAD?$AAF?$AAI?$AAL?$AAE?$AAI?$AAN?$AAF?$AAO?$AA_@ 10010090     VersionInfo.obj
 0002:000010b0       ??_C@_1CA@FOECMPGO@?$AAV?$AAS?$AA_?$AAV?$AAE?$AAR?$AAS?$AAI?$AAO?$AAN?$AA_?$AAI?$AAN?$AAF?$AAO@ 100100b0     VersionInfo.obj
 0002:000010d0       ??_C@_1BO@PBBNDBNF@?$AAS?$AAt?$AAr?$AAi?$AAn?$AAg?$AAF?$AAi?$AAl?$AAe?$AAI?$AAn?$AAf?$AAo@ 100100d0     VersionInfo.obj
 0002:000010f0       ??_C@_1BI@LJHFMFCG@?$AAV?$AAa?$AAr?$AAF?$AAi?$AAl?$AAe?$AAI?$AAn?$AAf?$AAo@ 100100f0     VersionInfo.obj
 0002:00001108       ??_C@_1BI@OMFAJHAK@?$AAT?$AAr?$AAa?$AAn?$AAs?$AAl?$AAa?$AAt?$AAi?$AAo?$AAn@ 10010108     VersionInfo.obj
 0002:00001120       ??_C@_1DK@JLHDHGFK@?$AAF?$AAI?$AAX?$AAE?$AAD?$AAF?$AAI?$AAL?$AAE?$AAI?$AAN?$AAF?$AAO?$AA_?$AAP@ 10010120     VersionInfo.obj
 0002:0000115c       ??_C@_0L@OLMNIJED@Some?5error@ 1001015c     WinErrorHandling.obj
 0002:00001168       ??_C@_0CA@GCNKJPPO@GetModuleHandleEx?$CI?$CJ?5failed?5for?5@ 10010168     WinErrorHandling.obj
 0002:00001188       ??_C@_09GKEDKJ@?5address?4@ 10010188     WinErrorHandling.obj
 0002:00001198       ??_C@_1EG@ONADDMNL@?$AA?$GA?$AAa?$AAn?$AAo?$AAn?$AAy?$AAm?$AAo?$AAu?$AAs?$AA?9?$AAn?$AAa?$AAm?$AAe@ 10010198     WinErrorHandling.obj
 0002:000011e0       ??_C@_1HM@EKFPGHAD@?$AAs?$AA?2?$AAs?$AAr?$AAc?$AA?2?$AAj?$AAd?$AAk?$AA?4?$AAj?$AAp?$AAa?$AAc?$AAk@ 100101e0     WinErrorHandling.obj
 0002:0000125c       ??_C@_1DC@DBLHEFGC@?$AAN?$AAo?$AA?5?$AAd?$AAe?$AAs?$AAc?$AAr?$AAi?$AAp?$AAt?$AAi?$AAo?$AAn?$AA?5@ 1001025c     WinErrorHandling.obj
 0002:00001290       ??_C@_0O@EGFCNMMA@system?5error?5@ 10010290     WinErrorHandling.obj
 0002:000012a0       ??_C@_02GFKOMOKH@?5?$CI@   100102a0     WinErrorHandling.obj
 0002:000012a4       ??_C@_0BD@HIJECHKD@GetSystemDirectory@ 100102a4     WinSysInfo.obj
 0002:000012b8       ??_C@_0CO@MKEKIODH@SysInfo?3?3?$GAanonymous?9namespace?8?3@ 100102b8     WinSysInfo.obj
 0002:000012e8       ??_C@_0DI@GLHFKFGD@s?2src?2jdk?4jpackage?2windows?2nati@ 100102e8     WinSysInfo.obj
 0002:00001320       ??_C@_0BJ@OHFMJCIO@GetModuleFileName?5failed@ 10010320     WinSysInfo.obj
 0002:0000133c       ??_C@_0CA@LHHGDJIE@SysInfo?3?3getCurrentModuleHandle@ 1001033c     WinSysInfo.obj
 0002:0000135c       ??_C@_0BK@NEANLJHL@GetModuleHandleExW?5failed@ 1001035c     WinSysInfo.obj
 0002:00001378       ??_C@_0DB@OADGFLCE@SysInfo?3?3?$GAanonymous?9namespace?8?3@ 10010378     WinSysInfo.obj
 0002:000013ac       ??_C@_07OCDKBNAP@?5failed@ 100103ac     WinSysInfo.obj
 0002:000013b4       ??_C@_0BG@GKMJLKJB@Unexpected?5reply?5from@ 100103b4     WinSysInfo.obj
 0002:000013cc       ??_C@_0DK@LKGGAEPL@Java_jdk_jpackage_internal_Wind@ 100103cc     WindowsRegistry.obj
 0002:00001408       ??_C@_0EC@NPMOIIFN@s?2src?2jdk?4jpackage?2windows?2nati@ 10010408     WindowsRegistry.obj
 0002:0000144c       ??_C@_0CA@DJLBMGAF@Inavlid?5Windows?5registry?5key?5id@ 1001044c     WindowsRegistry.obj
 0002:0000146c       ??_C@_0DL@FEEEGFIN@Java_jdk_jpackage_internal_Wind@ 1001046c     WindowsRegistry.obj
 0002:000014a8       ??_C@_0DN@GHOAPCGH@Java_jdk_jpackage_internal_Wind@ 100104a8     WindowsRegistry.obj
 0002:000014e8       ??_C@_0DI@LNIHIHKN@Java_jdk_jpackage_internal_Wind@ 100104e8     WindowsRegistry.obj
 0002:00001524       ??_7NopLogAppender@@6B@    10010524     app.obj
 0002:00001544       ??_C@_02LMMGGCAJ@?3?5@     10010544     app.obj
 0002:00001548       ??_C@_02PBFOLPKM@?$FN?5@   10010548     app.obj
 0002:0000154c       ??_C@_01OHGJGJJP@?$FL@     1001054c     app.obj
 0002:00001550       ??_C@_0DM@HKFNBGII@Java_jdk_jpackage_internal_Exec@ 10010550     jpackage.obj
 0002:0000158c       ??_C@_0DL@BGFDHIPP@s?2src?2jdk?4jpackage?2windows?2nati@ 1001058c     jpackage.obj
 0002:000015c8       ??_C@_0DO@NDGNLHPE@Java_jdk_jpackage_internal_Exec@ 100105c8     jpackage.obj
 0002:00001608       ??_C@_0DI@JFLFLAGO@Java_jdk_jpackage_internal_Exec@ 10010608     jpackage.obj
 0002:00001640       ??_C@_0DL@KDKICCGN@Java_jdk_jpackage_internal_Exec@ 10010640     jpackage.obj
 0002:00001680       ??_7?$basic_istringstream@DU?$char_traits@D@std@@V?$allocator@D@2@@std@@6B@ 10010680     jpackage.obj
 0002:00001684       ??_8?$basic_istringstream@DU?$char_traits@D@std@@V?$allocator@D@2@@std@@7B@ 10010684     jpackage.obj
 0002:0000168c       ??_C@_17BKKLFCBK@?$AAm?$AAs?$AAi@ 1001068c     jpackage.obj
 0002:00001694       ??_C@_1BI@OOBDCHEH@?$AAP?$AAr?$AAo?$AAd?$AAu?$AAc?$AAt?$AAC?$AAo?$AAd?$AAe@ 10010694     jpackage.obj
 0002:000016ac       ??_C@_1BK@BMAHLKDK@?$AAp?$AAr?$AAo?$AAd?$AAu?$AAc?$AAt?$AA_?$AAc?$AAo?$AAd?$AAe@ 100106ac     jpackage.obj
 0002:000016c8       ??_C@_0DC@CADNMJOE@Java_jdk_jpackage_internal_WinE@ 100106c8     jpackage.obj
 0002:00001700       ??_7logic_error@std@@6B@   10010700     tstrings.obj
 0002:0000170c       ??_7invalid_argument@std@@6B@ 1001070c     tstrings.obj
 0002:00001714       ??_C@_0CB@PKEJGPPE@Destination?5buffer?5can?8t?5be?5NUL@ 10010714     tstrings.obj
 0002:00001738       ??_C@_0CN@LGHLBHHG@tstrings?3?3?$GAanonymous?9namespace?8@ 10010738     tstrings.obj
 0002:00001768       ??_C@_0DE@PAENJCPL@s?2src?2jdk?4jpackage?2share?2native@ 10010768     tstrings.obj
 0002:0000179c       ??_C@_0CM@GJHHAJJB@Unexpected?5reply?5from?5WideCharT@ 1001079c     tstrings.obj
 0002:000017c8       ??_C@_0CP@CGMDKJBF@tstrings?3?3?$GAanonymous?9namespace?8@ 100107c8     tstrings.obj
 0002:000017f8       ??_C@_0CM@HMGDIOLF@Unexpected?5reply?5from?5MultiByte@ 100107f8     tstrings.obj
 0002:00001824       ?nothrow@std@@3Unothrow_t@1@B 10010824     msvcprt:nothrow.obj
 0002:0000182c       ??_7type_info@@6B@         1001082c     MSVCRT:std_type_info_static.obj
 0002:00001838       __pDefaultRawDllMain       10010838     MSVCRT:dll_dllmain.obj
 0002:00001838       __pRawDllMain              10010838     MSVCRT:dll_dllmain.obj
 0002:0000183c       ??_C@_0P@GHFPNOJB@bad?5allocation@ 1001083c     MSVCRT:throw_bad_alloc.obj
 0002:000018c0       __load_config_used         100108c0     MSVCRT:loadcfg.obj
 0002:00001978       ??_R4exception@std@@6B@    10010978     ErrorHandling.obj
 0002:0000198c       ??_R3exception@std@@8      1001098c     ErrorHandling.obj
 0002:0000199c       ??_R2exception@std@@8      1001099c     ErrorHandling.obj
 0002:000019a4       ??_R1A@?0A@EA@exception@std@@8 100109a4     ErrorHandling.obj
 0002:000019c0       ??_R4bad_alloc@std@@6B@    100109c0     ErrorHandling.obj
 0002:000019d4       ??_R3bad_alloc@std@@8      100109d4     ErrorHandling.obj
 0002:000019e4       ??_R2bad_alloc@std@@8      100109e4     ErrorHandling.obj
 0002:000019f0       ??_R1A@?0A@EA@bad_alloc@std@@8 100109f0     ErrorHandling.obj
 0002:00001a0c       ??_R4bad_array_new_length@std@@6B@ 10010a0c     ErrorHandling.obj
 0002:00001a20       ??_R3bad_array_new_length@std@@8 10010a20     ErrorHandling.obj
 0002:00001a30       ??_R2bad_array_new_length@std@@8 10010a30     ErrorHandling.obj
 0002:00001a40       ??_R1A@?0A@EA@bad_array_new_length@std@@8 10010a40     ErrorHandling.obj
 0002:00001a5c       ??_R4?$basic_stringbuf@DU?$char_traits@D@std@@V?$allocator@D@2@@std@@6B@ 10010a5c     ErrorHandling.obj
 0002:00001a70       ??_R3?$basic_stringbuf@DU?$char_traits@D@std@@V?$allocator@D@2@@std@@8 10010a70     ErrorHandling.obj
 0002:00001a80       ??_R2?$basic_stringbuf@DU?$char_traits@D@std@@V?$allocator@D@2@@std@@8 10010a80     ErrorHandling.obj
 0002:00001a8c       ??_R1A@?0A@EA@?$basic_stringbuf@DU?$char_traits@D@std@@V?$allocator@D@2@@std@@8 10010a8c     ErrorHandling.obj
 0002:00001aa8       ??_R1A@?0A@EA@?$basic_streambuf@DU?$char_traits@D@std@@@std@@8 10010aa8     ErrorHandling.obj
 0002:00001ac4       ??_R3?$basic_streambuf@DU?$char_traits@D@std@@@std@@8 10010ac4     ErrorHandling.obj
 0002:00001ad4       ??_R2?$basic_streambuf@DU?$char_traits@D@std@@@std@@8 10010ad4     ErrorHandling.obj
 0002:00001adc       ??_R4?$basic_ostringstream@DU?$char_traits@D@std@@V?$allocator@D@2@@std@@6B@ 10010adc     ErrorHandling.obj
 0002:00001af0       ??_R3?$basic_ostringstream@DU?$char_traits@D@std@@V?$allocator@D@2@@std@@8 10010af0     ErrorHandling.obj
 0002:00001b00       ??_R2?$basic_ostringstream@DU?$char_traits@D@std@@V?$allocator@D@2@@std@@8 10010b00     ErrorHandling.obj
 0002:00001b18       ??_R1A@?0A@EA@?$basic_ostringstream@DU?$char_traits@D@std@@V?$allocator@D@2@@std@@8 10010b18     ErrorHandling.obj
 0002:00001b34       ??_R1A@?0A@EA@?$basic_ostream@DU?$char_traits@D@std@@@std@@8 10010b34     ErrorHandling.obj
 0002:00001b50       ??_R3?$basic_ostream@DU?$char_traits@D@std@@@std@@8 10010b50     ErrorHandling.obj
 0002:00001b60       ??_R2?$basic_ostream@DU?$char_traits@D@std@@@std@@8 10010b60     ErrorHandling.obj
 0002:00001b74       ??_R1A@A@3FA@?$basic_ios@DU?$char_traits@D@std@@@std@@8 10010b74     ErrorHandling.obj
 0002:00001b90       ??_R3?$basic_ios@DU?$char_traits@D@std@@@std@@8 10010b90     ErrorHandling.obj
 0002:00001ba0       ??_R2?$basic_ios@DU?$char_traits@D@std@@@std@@8 10010ba0     ErrorHandling.obj
 0002:00001bb0       ??_R1A@?0A@EA@?$basic_ios@DU?$char_traits@D@std@@@std@@8 10010bb0     ErrorHandling.obj
 0002:00001bcc       ??_R1A@?0A@EA@ios_base@std@@8 10010bcc     ErrorHandling.obj
 0002:00001be8       ??_R3ios_base@std@@8       10010be8     ErrorHandling.obj
 0002:00001bf8       ??_R2ios_base@std@@8       10010bf8     ErrorHandling.obj
 0002:00001c04       ??_R17?0A@EA@?$_Iosb@H@std@@8 10010c04     ErrorHandling.obj
 0002:00001c20       ??_R3?$_Iosb@H@std@@8      10010c20     ErrorHandling.obj
 0002:00001c30       ??_R2?$_Iosb@H@std@@8      10010c30     ErrorHandling.obj
 0002:00001c38       ??_R1A@?0A@EA@?$_Iosb@H@std@@8 10010c38     ErrorHandling.obj
 0002:00001c54       ??_R1A@A@3EA@ios_base@std@@8 10010c54     ErrorHandling.obj
 0002:00001c70       ??_R17A@3EA@?$_Iosb@H@std@@8 10010c70     ErrorHandling.obj
 0002:00001c8c       ??_R4?$basic_stringbuf@GU?$char_traits@G@std@@V?$allocator@G@2@@std@@6B@ 10010c8c     ErrorHandling.obj
 0002:00001ca0       ??_R3?$basic_stringbuf@GU?$char_traits@G@std@@V?$allocator@G@2@@std@@8 10010ca0     ErrorHandling.obj
 0002:00001cb0       ??_R2?$basic_stringbuf@GU?$char_traits@G@std@@V?$allocator@G@2@@std@@8 10010cb0     ErrorHandling.obj
 0002:00001cbc       ??_R1A@?0A@EA@?$basic_stringbuf@GU?$char_traits@G@std@@V?$allocator@G@2@@std@@8 10010cbc     ErrorHandling.obj
 0002:00001cd8       ??_R1A@?0A@EA@?$basic_streambuf@GU?$char_traits@G@std@@@std@@8 10010cd8     ErrorHandling.obj
 0002:00001cf4       ??_R3?$basic_streambuf@GU?$char_traits@G@std@@@std@@8 10010cf4     ErrorHandling.obj
 0002:00001d04       ??_R2?$basic_streambuf@GU?$char_traits@G@std@@@std@@8 10010d04     ErrorHandling.obj
 0002:00001d0c       ??_R4?$basic_ostringstream@GU?$char_traits@G@std@@V?$allocator@G@2@@std@@6B@ 10010d0c     ErrorHandling.obj
 0002:00001d20       ??_R3?$basic_ostringstream@GU?$char_traits@G@std@@V?$allocator@G@2@@std@@8 10010d20     ErrorHandling.obj
 0002:00001d30       ??_R2?$basic_ostringstream@GU?$char_traits@G@std@@V?$allocator@G@2@@std@@8 10010d30     ErrorHandling.obj
 0002:00001d48       ??_R1A@?0A@EA@?$basic_ostringstream@GU?$char_traits@G@std@@V?$allocator@G@2@@std@@8 10010d48     ErrorHandling.obj
 0002:00001d64       ??_R1A@?0A@EA@?$basic_ostream@GU?$char_traits@G@std@@@std@@8 10010d64     ErrorHandling.obj
 0002:00001d80       ??_R3?$basic_ostream@GU?$char_traits@G@std@@@std@@8 10010d80     ErrorHandling.obj
 0002:00001d90       ??_R2?$basic_ostream@GU?$char_traits@G@std@@@std@@8 10010d90     ErrorHandling.obj
 0002:00001da4       ??_R1A@A@3FA@?$basic_ios@GU?$char_traits@G@std@@@std@@8 10010da4     ErrorHandling.obj
 0002:00001dc0       ??_R3?$basic_ios@GU?$char_traits@G@std@@@std@@8 10010dc0     ErrorHandling.obj
 0002:00001dd0       ??_R2?$basic_ios@GU?$char_traits@G@std@@@std@@8 10010dd0     ErrorHandling.obj
 0002:00001de0       ??_R1A@?0A@EA@?$basic_ios@GU?$char_traits@G@std@@@std@@8 10010de0     ErrorHandling.obj
 0002:00001dfc       ??_R4bad_cast@std@@6B@     10010dfc     ErrorHandling.obj
 0002:00001e10       ??_R3bad_cast@std@@8       10010e10     ErrorHandling.obj
 0002:00001e20       ??_R2bad_cast@std@@8       10010e20     ErrorHandling.obj
 0002:00001e2c       ??_R1A@?0A@EA@bad_cast@std@@8 10010e2c     ErrorHandling.obj
 0002:00001e48       ??_R4runtime_error@std@@6B@ 10010e48     Guid.obj
 0002:00001e5c       ??_R3runtime_error@std@@8  10010e5c     Guid.obj
 0002:00001e6c       ??_R2runtime_error@std@@8  10010e6c     Guid.obj
 0002:00001e78       ??_R1A@?0A@EA@runtime_error@std@@8 10010e78     Guid.obj
 0002:00001e94       ??_R4JpErrorBase@@6B@      10010e94     Guid.obj
 0002:00001ea8       ??_R3JpErrorBase@@8        10010ea8     Guid.obj
 0002:00001eb8       ??_R2JpErrorBase@@8        10010eb8     Guid.obj
 0002:00001ec0       ??_R1A@?0A@EA@JpErrorBase@@8 10010ec0     Guid.obj
 0002:00001edc       ??_R4?$JpError@Vruntime_error@std@@@@6BJpErrorBase@@@ 10010edc     Guid.obj
 0002:00001ef0       ??_R3?$JpError@Vruntime_error@std@@@@8 10010ef0     Guid.obj
 0002:00001f00       ??_R2?$JpError@Vruntime_error@std@@@@8 10010f00     Guid.obj
 0002:00001f14       ??_R1A@?0A@EA@?$JpError@Vruntime_error@std@@@@8 10010f14     Guid.obj
 0002:00001f30       ??_R13?0A@EA@runtime_error@std@@8 10010f30     Guid.obj
 0002:00001f4c       ??_R13?0A@EA@exception@std@@8 10010f4c     Guid.obj
 0002:00001f68       ??_R4?$JpError@Vruntime_error@std@@@@6Bruntime_error@std@@@ 10010f68     Guid.obj
 0002:00001f7c       ??_R4StreamLogAppender@@6B@ 10010f7c     Log.obj
 0002:00001f90       ??_R3StreamLogAppender@@8  10010f90     Log.obj
 0002:00001fa0       ??_R2StreamLogAppender@@8  10010fa0     Log.obj
 0002:00001fac       ??_R1A@?0A@EA@StreamLogAppender@@8 10010fac     Log.obj
 0002:00001fc8       ??_R1A@?0A@EA@LogAppender@@8 10010fc8     Log.obj
 0002:00001fe4       ??_R3LogAppender@@8        10010fe4     Log.obj
 0002:00001ff4       ??_R2LogAppender@@8        10010ff4     Log.obj
 0002:00001ffc       ??_R4LogAppender@@6B@      10010ffc     Log.obj
 0002:00002010       ??_R4?$basic_filebuf@DU?$char_traits@D@std@@@std@@6B@ 10011010     MsiDb.obj
 0002:00002024       ??_R3?$basic_filebuf@DU?$char_traits@D@std@@@std@@8 10011024     MsiDb.obj
 0002:00002034       ??_R2?$basic_filebuf@DU?$char_traits@D@std@@@std@@8 10011034     MsiDb.obj
 0002:00002040       ??_R1A@?0A@EA@?$basic_filebuf@DU?$char_traits@D@std@@@std@@8 10011040     MsiDb.obj
 0002:0000205c       ??_R4Error@msi@@6B@        1001105c     MsiDb.obj
 0002:00002070       ??_R3Error@msi@@8          10011070     MsiDb.obj
 0002:00002080       ??_R2Error@msi@@8          10011080     MsiDb.obj
 0002:00002090       ??_R1A@?0A@EA@Error@msi@@8 10011090     MsiDb.obj
 0002:000020ac       ??_R4NoMoreItemsError@msi@@6B@ 100110ac     MsiDb.obj
 0002:000020c0       ??_R3NoMoreItemsError@msi@@8 100110c0     MsiDb.obj
 0002:000020d0       ??_R2NoMoreItemsError@msi@@8 100110d0     MsiDb.obj
 0002:000020e4       ??_R1A@?0A@EA@NoMoreItemsError@msi@@8 100110e4     MsiDb.obj
 0002:00002100       ??_R4?$JpError@VError@msi@@@@6BJpErrorBase@@@ 10011100     MsiDb.obj
 0002:00002114       ??_R3?$JpError@VError@msi@@@@8 10011114     MsiDb.obj
 0002:00002124       ??_R2?$JpError@VError@msi@@@@8 10011124     MsiDb.obj
 0002:0000213c       ??_R1A@?0A@EA@?$JpError@VError@msi@@@@8 1001113c     MsiDb.obj
 0002:00002158       ??_R13?0A@EA@Error@msi@@8  10011158     MsiDb.obj
 0002:00002174       ??_R4?$JpError@VError@msi@@@@6BError@msi@@@ 10011174     MsiDb.obj
 0002:00002188       ??_R4?$JpError@VNoMoreItemsError@msi@@@@6BJpErrorBase@@@ 10011188     MsiDb.obj
 0002:0000219c       ??_R3?$JpError@VNoMoreItemsError@msi@@@@8 1001119c     MsiDb.obj
 0002:000021ac       ??_R2?$JpError@VNoMoreItemsError@msi@@@@8 100111ac     MsiDb.obj
 0002:000021c8       ??_R1A@?0A@EA@?$JpError@VNoMoreItemsError@msi@@@@8 100111c8     MsiDb.obj
 0002:000021e4       ??_R13?0A@EA@NoMoreItemsError@msi@@8 100111e4     MsiDb.obj
 0002:00002200       ??_R4?$JpError@VNoMoreItemsError@msi@@@@6BNoMoreItemsError@msi@@@ 10011200     MsiDb.obj
 0002:00002214       ??_R4SysError@@6B@         10011214     MsiUtils.obj
 0002:00002228       ??_R3SysError@@8           10011228     MsiUtils.obj
 0002:00002238       ??_R2SysError@@8           10011238     MsiUtils.obj
 0002:00002248       ??_R1A@?0A@EA@SysError@@8  10011248     MsiUtils.obj
 0002:00002264       ??_R4?$JpError@VSysError@@@@6BJpErrorBase@@@ 10011264     MsiUtils.obj
 0002:00002278       ??_R3?$JpError@VSysError@@@@8 10011278     MsiUtils.obj
 0002:00002288       ??_R2?$JpError@VSysError@@@@8 10011288     MsiUtils.obj
 0002:000022a0       ??_R1A@?0A@EA@?$JpError@VSysError@@@@8 100112a0     MsiUtils.obj
 0002:000022bc       ??_R13?0A@EA@SysError@@8   100112bc     MsiUtils.obj
 0002:000022d8       ??_R4?$JpError@VSysError@@@@6BSysError@@@ 100112d8     MsiUtils.obj
 0002:000022ec       ??_R4?$basic_ifstream@DU?$char_traits@D@std@@@std@@6B@ 100112ec     ResourceEditor.obj
 0002:00002300       ??_R3?$basic_ifstream@DU?$char_traits@D@std@@@std@@8 10011300     ResourceEditor.obj
 0002:00002310       ??_R2?$basic_ifstream@DU?$char_traits@D@std@@@std@@8 10011310     ResourceEditor.obj
 0002:00002328       ??_R1A@?0A@EA@?$basic_ifstream@DU?$char_traits@D@std@@@std@@8 10011328     ResourceEditor.obj
 0002:00002344       ??_R1A@?0A@EA@?$basic_istream@DU?$char_traits@D@std@@@std@@8 10011344     ResourceEditor.obj
 0002:00002360       ??_R3?$basic_istream@DU?$char_traits@D@std@@@std@@8 10011360     ResourceEditor.obj
 0002:00002370       ??_R2?$basic_istream@DU?$char_traits@D@std@@@std@@8 10011370     ResourceEditor.obj
 0002:00002384       ??_R4?$basic_stringstream@DU?$char_traits@D@std@@V?$allocator@D@2@@std@@6B@ 10011384     VersionInfo.obj
 0002:00002398       ??_R3?$basic_stringstream@DU?$char_traits@D@std@@V?$allocator@D@2@@std@@8 10011398     VersionInfo.obj
 0002:000023a8       ??_R2?$basic_stringstream@DU?$char_traits@D@std@@V?$allocator@D@2@@std@@8 100113a8     VersionInfo.obj
 0002:000023d4       ??_R1A@?0A@EA@?$basic_stringstream@DU?$char_traits@D@std@@V?$allocator@D@2@@std@@8 100113d4     VersionInfo.obj
 0002:000023f0       ??_R1A@?0A@EA@?$basic_iostream@DU?$char_traits@D@std@@@std@@8 100113f0     VersionInfo.obj
 0002:0000240c       ??_R3?$basic_iostream@DU?$char_traits@D@std@@@std@@8 1001140c     VersionInfo.obj
 0002:0000241c       ??_R2?$basic_iostream@DU?$char_traits@D@std@@@std@@8 1001141c     VersionInfo.obj
 0002:00002444       ??_R1BA@?0A@EA@?$basic_ostream@DU?$char_traits@D@std@@@std@@8 10011444     VersionInfo.obj
 0002:00002460       ??_R4?$basic_stringstream@GU?$char_traits@G@std@@V?$allocator@G@2@@std@@6B@ 10011460     VersionInfo.obj
 0002:00002474       ??_R3?$basic_stringstream@GU?$char_traits@G@std@@V?$allocator@G@2@@std@@8 10011474     VersionInfo.obj
 0002:00002484       ??_R2?$basic_stringstream@GU?$char_traits@G@std@@V?$allocator@G@2@@std@@8 10011484     VersionInfo.obj
 0002:000024b0       ??_R1A@?0A@EA@?$basic_stringstream@GU?$char_traits@G@std@@V?$allocator@G@2@@std@@8 100114b0     VersionInfo.obj
 0002:000024cc       ??_R1A@?0A@EA@?$basic_iostream@GU?$char_traits@G@std@@@std@@8 100114cc     VersionInfo.obj
 0002:000024e8       ??_R3?$basic_iostream@GU?$char_traits@G@std@@@std@@8 100114e8     VersionInfo.obj
 0002:000024f8       ??_R2?$basic_iostream@GU?$char_traits@G@std@@@std@@8 100114f8     VersionInfo.obj
 0002:00002520       ??_R1A@?0A@EA@?$basic_istream@GU?$char_traits@G@std@@@std@@8 10011520     VersionInfo.obj
 0002:0000253c       ??_R3?$basic_istream@GU?$char_traits@G@std@@@std@@8 1001153c     VersionInfo.obj
 0002:0000254c       ??_R2?$basic_istream@GU?$char_traits@G@std@@@std@@8 1001154c     VersionInfo.obj
 0002:00002560       ??_R1BA@?0A@EA@?$basic_ostream@GU?$char_traits@G@std@@@std@@8 10011560     VersionInfo.obj
 0002:0000257c       ??_R4NopLogAppender@@6B@   1001157c     app.obj
 0002:00002590       ??_R3NopLogAppender@@8     10011590     app.obj
 0002:000025a0       ??_R2NopLogAppender@@8     100115a0     app.obj
 0002:000025ac       ??_R1A@?0A@EA@NopLogAppender@@8 100115ac     app.obj
 0002:00002660       ??_R4?$basic_istringstream@DU?$char_traits@D@std@@V?$allocator@D@2@@std@@6B@ 10011660     jpackage.obj
 0002:00002674       ??_R3?$basic_istringstream@DU?$char_traits@D@std@@V?$allocator@D@2@@std@@8 10011674     jpackage.obj
 0002:00002684       ??_R2?$basic_istringstream@DU?$char_traits@D@std@@V?$allocator@D@2@@std@@8 10011684     jpackage.obj
 0002:0000269c       ??_R1A@?0A@EA@?$basic_istringstream@DU?$char_traits@D@std@@V?$allocator@D@2@@std@@8 1001169c     jpackage.obj
 0002:000026b8       ??_R4logic_error@std@@6B@  100116b8     tstrings.obj
 0002:000026cc       ??_R3logic_error@std@@8    100116cc     tstrings.obj
 0002:000026dc       ??_R2logic_error@std@@8    100116dc     tstrings.obj
 0002:000026e8       ??_R1A@?0A@EA@logic_error@std@@8 100116e8     tstrings.obj
 0002:00002704       ??_R4invalid_argument@std@@6B@ 10011704     tstrings.obj
 0002:00002718       ??_R3invalid_argument@std@@8 10011718     tstrings.obj
 0002:00002728       ??_R2invalid_argument@std@@8 10011728     tstrings.obj
 0002:00002738       ??_R1A@?0A@EA@invalid_argument@std@@8 10011738     tstrings.obj
 0002:00002754       ??_R4type_info@@6B@        10011754     MSVCRT:std_type_info_static.obj
 0002:00002768       ??_R3type_info@@8          10011768     MSVCRT:std_type_info_static.obj
 0002:00002778       ??_R2type_info@@8          10011778     MSVCRT:std_type_info_static.obj
 0002:00002780       ??_R1A@?0A@EA@type_info@@8 10011780     MSVCRT:std_type_info_static.obj
 0002:0000279c       ___safe_se_handler_table   1001179c     <linker-defined>
 0002:00002c34       ___rtc_iaa                 10011c34     MSVCRT:initsect.obj
 0002:00002c38       ___rtc_izz                 10011c38     MSVCRT:initsect.obj
 0002:00002c3c       ___rtc_taa                 10011c3c     MSVCRT:initsect.obj
 0002:00002c40       ___rtc_tzz                 10011c40     MSVCRT:initsect.obj
 0002:00003150       __TI3?AVbad_array_new_length@std@@ 10012150     ErrorHandling.obj
 0002:00003160       __CTA3?AVbad_array_new_length@std@@ 10012160     ErrorHandling.obj
 0002:00003170       __CT??_R0?AVbad_array_new_length@std@@@8??0bad_array_new_length@std@@QAE@ABV01@@Z12 10012170     ErrorHandling.obj
 0002:0000318c       __CT??_R0?AVbad_alloc@std@@@8??0bad_alloc@std@@QAE@ABV01@@Z12 1001218c     ErrorHandling.obj
 0002:000031a8       __CT??_R0?AVexception@std@@@8??0exception@std@@QAE@ABV01@@Z12 100121a8     ErrorHandling.obj
 0002:000031c4       __TI2?AVbad_cast@std@@     100121c4     ErrorHandling.obj
 0002:000031d4       __CTA2?AVbad_cast@std@@    100121d4     ErrorHandling.obj
 0002:000031e0       __CT??_R0?AVbad_cast@std@@@8??0bad_cast@std@@QAE@ABV01@@Z12 100121e0     ErrorHandling.obj
 0002:00003358       __TI4?AV?$JpError@Vruntime_error@std@@@@ 10012358     Guid.obj
 0002:00003368       __CTA4?AV?$JpError@Vruntime_error@std@@@@ 10012368     Guid.obj
 0002:0000337c       __CT??_R0?AV?$JpError@Vruntime_error@std@@@@@8??0?$JpError@Vruntime_error@std@@@@QAE@ABV0@@Z40 1001237c     Guid.obj
 0002:00003398       __CT??_R0?AVJpErrorBase@@@8??0JpErrorBase@@QAE@ABV0@@Z4 10012398     Guid.obj
 0002:000033b4       __CT??_R0?AVruntime_error@std@@@8??0runtime_error@std@@QAE@ABV01@@Z124 100123b4     Guid.obj
 0002:000033d0       __CT??_R0?AVexception@std@@@8??0exception@std@@QAE@ABV01@@Z124 100123d0     Guid.obj
 0002:000037fc       __TI5?AV?$JpError@VError@msi@@@@ 100127fc     MsiDb.obj
 0002:0000380c       __CTA5?AV?$JpError@VError@msi@@@@ 1001280c     MsiDb.obj
 0002:00003824       __CT??_R0?AV?$JpError@VError@msi@@@@@8??0?$JpError@VError@msi@@@@QAE@ABV0@@Z44 10012824     MsiDb.obj
 0002:00003840       __CT??_R0?AVError@msi@@@8??0Error@msi@@QAE@ABV01@@Z164 10012840     MsiDb.obj
 0002:0000385c       __TI6?AV?$JpError@VNoMoreItemsError@msi@@@@ 1001285c     MsiDb.obj
 0002:0000386c       __CTA6?AV?$JpError@VNoMoreItemsError@msi@@@@ 1001286c     MsiDb.obj
 0002:00003888       __CT??_R0?AV?$JpError@VNoMoreItemsError@msi@@@@@8??0?$JpError@VNoMoreItemsError@msi@@@@QAE@ABV0@@Z44 10012888     MsiDb.obj
 0002:000038a4       __CT??_R0?AVNoMoreItemsError@msi@@@8??0NoMoreItemsError@msi@@QAE@ABV01@@Z164 100128a4     MsiDb.obj
 0002:00003a60       __TI5?AV?$JpError@VSysError@@@@ 10012a60     MsiUtils.obj
 0002:00003a70       __CTA5?AV?$JpError@VSysError@@@@ 10012a70     MsiUtils.obj
 0002:00003a88       __CT??_R0?AV?$JpError@VSysError@@@@@8??0?$JpError@VSysError@@@@QAE@ABV0@@Z40 10012a88     MsiUtils.obj
 0002:00003aa4       __CT??_R0?AVSysError@@@8??0SysError@@QAE@ABV0@@Z124 10012aa4     MsiUtils.obj
 0002:00004884       __TI3?AVinvalid_argument@std@@ 10013884     tstrings.obj
 0002:00004894       __CTA3?AVinvalid_argument@std@@ 10013894     tstrings.obj
 0002:000048a4       __CT??_R0?AVinvalid_argument@std@@@8??0invalid_argument@std@@QAE@ABV01@@Z12 100138a4     tstrings.obj
 0002:000048c0       __CT??_R0?AVlogic_error@std@@@8??0logic_error@std@@QAE@ABV01@@Z12 100138c0     tstrings.obj
 0002:00004964       __TI2?AVbad_alloc@std@@    10013964     MSVCRT:throw_bad_alloc.obj
 0002:00004974       __CTA2?AVbad_alloc@std@@   10013974     MSVCRT:throw_bad_alloc.obj
 0002:00004c88       __IMPORT_DESCRIPTOR_MSVCP140 10013c88     msvcprt:MSVCP140.dll
 0002:00004c9c       __IMPORT_DESCRIPTOR_ole32  10013c9c     ole32:ole32.dll
 0002:00004cb0       __IMPORT_DESCRIPTOR_msi    10013cb0     msi:msi.dll
 0002:00004cc4       __IMPORT_DESCRIPTOR_ADVAPI32 10013cc4     advapi32:ADVAPI32.dll
 0002:00004cd8       __IMPORT_DESCRIPTOR_KERNEL32 10013cd8     kernel32:KERNEL32.dll
 0002:00004cec       __IMPORT_DESCRIPTOR_VCRUNTIME140 10013cec     vcruntime:VCRUNTIME140.dll
 0002:00004d00       __IMPORT_DESCRIPTOR_api-ms-win-crt-runtime-l1-1-0 10013d00     ucrt:api-ms-win-crt-runtime-l1-1-0.dll
 0002:00004d14       __IMPORT_DESCRIPTOR_api-ms-win-crt-string-l1-1-0 10013d14     ucrt:api-ms-win-crt-string-l1-1-0.dll
 0002:00004d28       __IMPORT_DESCRIPTOR_api-ms-win-crt-stdio-l1-1-0 10013d28     ucrt:api-ms-win-crt-stdio-l1-1-0.dll
 0002:00004d3c       __IMPORT_DESCRIPTOR_api-ms-win-crt-heap-l1-1-0 10013d3c     ucrt:api-ms-win-crt-heap-l1-1-0.dll
 0002:00004d50       __IMPORT_DESCRIPTOR_api-ms-win-crt-filesystem-l1-1-0 10013d50     ucrt:api-ms-win-crt-filesystem-l1-1-0.dll
 0002:00004d64       __NULL_IMPORT_DESCRIPTOR   10013d64     msvcprt:MSVCP140.dll
 0003:00000220       ___security_cookie_complement 10016220     MSVCRT:gs_cookie.obj
 0003:00000224       ___security_cookie         10016224     MSVCRT:gs_cookie.obj
 0003:00000230       ___scrt_native_dllmain_reason 10016230     MSVCRT:utility.obj
 0003:00000234       ___isa_enabled             10016234     MSVCRT:cpu_disp.obj
 0003:00000240       ___scrt_ucrt_dll_is_in_use 10016240     MSVCRT:ucrt_stubs.obj
 0003:00000248       ??_R0?AVbad_array_new_length@std@@@8 10016248     ErrorHandling.obj
 0003:00000270       ??_R0?AVbad_alloc@std@@@8  10016270     ErrorHandling.obj
 0003:0000028c       ??_R0?AVexception@std@@@8  1001628c     ErrorHandling.obj
 0003:000002a8       ??_R0?AVbad_cast@std@@@8   100162a8     ErrorHandling.obj
 0003:000002c8       ??_R0?AV?$basic_stringbuf@DU?$char_traits@D@std@@V?$allocator@D@2@@std@@@8 100162c8     ErrorHandling.obj
 0003:00000318       ??_R0?AV?$basic_streambuf@DU?$char_traits@D@std@@@std@@@8 10016318     ErrorHandling.obj
 0003:00000358       ??_R0?AV?$basic_ostringstream@DU?$char_traits@D@std@@V?$allocator@D@2@@std@@@8 10016358     ErrorHandling.obj
 0003:000003ac       ??_R0?AV?$basic_ostream@DU?$char_traits@D@std@@@std@@@8 100163ac     ErrorHandling.obj
 0003:000003e8       ??_R0?AV?$basic_ios@DU?$char_traits@D@std@@@std@@@8 100163e8     ErrorHandling.obj
 0003:00000420       ??_R0?AVios_base@std@@@8   10016420     ErrorHandling.obj
 0003:0000043c       ??_R0?AV?$_Iosb@H@std@@@8  1001643c     ErrorHandling.obj
 0003:00000458       ??_R0?AV?$basic_stringbuf@GU?$char_traits@G@std@@V?$allocator@G@2@@std@@@8 10016458     ErrorHandling.obj
 0003:000004a8       ??_R0?AV?$basic_streambuf@GU?$char_traits@G@std@@@std@@@8 100164a8     ErrorHandling.obj
 0003:000004e8       ??_R0?AV?$basic_ostringstream@GU?$char_traits@G@std@@V?$allocator@G@2@@std@@@8 100164e8     ErrorHandling.obj
 0003:0000053c       ??_R0?AV?$basic_ostream@GU?$char_traits@G@std@@@std@@@8 1001653c     ErrorHandling.obj
 0003:00000578       ??_R0?AV?$basic_ios@GU?$char_traits@G@std@@@std@@@8 10016578     ErrorHandling.obj
 0003:000005b0       ??_R0?AVruntime_error@std@@@8 100165b0     Guid.obj
 0003:000005d0       ??_R0?AV?$JpError@Vruntime_error@std@@@@@8 100165d0     Guid.obj
 0003:00000600       ??_R0?AVJpErrorBase@@@8    10016600     Guid.obj
 0003:0000061c       ??_R0?AVStreamLogAppender@@@8 1001661c     Log.obj
 0003:0000063c       ??_R0?AVLogAppender@@@8    1001663c     Log.obj
 0003:00000658       ??_R0?AV?$JpError@VError@msi@@@@@8 10016658     MsiDb.obj
 0003:00000680       ??_R0?AVError@msi@@@8      10016680     MsiDb.obj
 0003:00000698       ??_R0?AVNoMoreItemsError@msi@@@8 10016698     MsiDb.obj
 0003:000006bc       ??_R0?AV?$JpError@VNoMoreItemsError@msi@@@@@8 100166bc     MsiDb.obj
 0003:000006ec       ??_R0?AV?$basic_filebuf@DU?$char_traits@D@std@@@std@@@8 100166ec     MsiDb.obj
 0003:00000728       ??_R0?AV?$JpError@VSysError@@@@@8 10016728     MsiUtils.obj
 0003:0000074c       ??_R0?AVSysError@@@8       1001674c     MsiUtils.obj
 0003:00000764       ??_R0?AV?$basic_ifstream@DU?$char_traits@D@std@@@std@@@8 10016764     ResourceEditor.obj
 0003:000007a0       ??_R0?AV?$basic_istream@DU?$char_traits@D@std@@@std@@@8 100167a0     ResourceEditor.obj
 0003:000007e0       ??_R0?AV?$basic_stringstream@DU?$char_traits@D@std@@V?$allocator@D@2@@std@@@8 100167e0     VersionInfo.obj
 0003:00000830       ??_R0?AV?$basic_iostream@DU?$char_traits@D@std@@@std@@@8 10016830     VersionInfo.obj
 0003:00000870       ??_R0?AV?$basic_stringstream@GU?$char_traits@G@std@@V?$allocator@G@2@@std@@@8 10016870     VersionInfo.obj
 0003:000008c0       ??_R0?AV?$basic_iostream@GU?$char_traits@G@std@@@std@@@8 100168c0     VersionInfo.obj
 0003:000008fc       ??_R0?AV?$basic_istream@GU?$char_traits@G@std@@@std@@@8 100168fc     VersionInfo.obj
 0003:00000938       ??_R0?AVNopLogAppender@@@8 10016938     app.obj
 0003:000009b8       ??_R0?AV?$basic_istringstream@DU?$char_traits@D@std@@V?$allocator@D@2@@std@@@8 100169b8     jpackage.obj
 0003:00000a0c       ??_R0?AVinvalid_argument@std@@@8 10016a0c     tstrings.obj
 0003:00000a30       ??_R0?AVlogic_error@std@@@8 10016a30     tstrings.obj
 0003:00000a50       ??_R0?AVtype_info@@@8      10016a50     MSVCRT:std_type_info_static.obj
 0003:00000a68       ?_Psave@?$_Facetptr@V?$ctype@G@std@@@std@@2PBVfacet@locale@2@B 10016a68     ErrorHandling.obj
 0003:00000a70       ?_OptionsStorage@?1??__local_stdio_printf_options@@9@4_KA 10016a70     IconSwap.obj
 0003:00000a8c       ?_Stinit@?1??_Init@?$basic_filebuf@DU?$char_traits@D@std@@@std@@IAEXPAU_iobuf@@W4_Initfl@23@@Z@4U_Mbstatet@@A 10016a8c     MsiDb.obj
 0003:00000a94       ?_Psave@?$_Facetptr@V?$codecvt@DDU_Mbstatet@@@std@@@std@@2PBVfacet@locale@2@B 10016a94     MsiDb.obj
 0003:00000a98       ?_OptionsStorage@?1??__local_stdio_scanf_options@@9@4_KA 10016a98     VersionInfo.obj
 0003:00000dcc       ___scrt_current_native_startup_state 10016dcc     MSVCRT:utility.obj
 0003:00000dd0       ___scrt_native_startup_lock 10016dd0     MSVCRT:utility.obj
 0003:00000df4       ___isa_available           10016df4     MSVCRT:cpu_disp.obj
 0003:00000df8       ___favor                   10016df8     MSVCRT:cpu_disp.obj
 0003:00000dfc       ___scrt_debugger_hook_flag 10016dfc     MSVCRT:utility_desktop.obj
 0003:00000e00       ?__type_info_root_node@@3U__type_info_node@@A 10016e00     MSVCRT:tncleanup.obj
 0003:00000e08       ___dyn_tls_init_callback   10016e08     <common>

 entry point at        0001:0000b8df

 Static symbols

 0000:fffe6000       .debug$S                   10000000     jpackage.exp
 0000:fffe6000       .debug$S                   10000000     msvcprt:MSVCP140.dll
 0000:fffe6000       .debug$S                   10000000     msvcprt:MSVCP140.dll
 0000:fffe6000       .debug$S                   10000000     msvcprt:MSVCP140.dll
 0000:fffe6000       .debug$S                   10000000     msvcprt:MSVCP140.dll
 0000:fffe6000       .debug$S                   10000000     msvcprt:MSVCP140.dll
 0000:fffe6000       .debug$S                   10000000     msvcprt:MSVCP140.dll
 0000:fffe6000       .debug$S                   10000000     msvcprt:MSVCP140.dll
 0000:fffe6000       .debug$S                   10000000     msvcprt:MSVCP140.dll
 0000:fffe6000       .debug$S                   10000000     msvcprt:MSVCP140.dll
 0000:fffe6000       .debug$S                   10000000     msvcprt:MSVCP140.dll
 0000:fffe6000       .debug$S                   10000000     msvcprt:MSVCP140.dll
 0000:fffe6000       .debug$S                   10000000     msvcprt:MSVCP140.dll
 0000:fffe6000       .debug$S                   10000000     msvcprt:MSVCP140.dll
 0000:fffe6000       .debug$S                   10000000     msvcprt:MSVCP140.dll
 0000:fffe6000       .debug$S                   10000000     msvcprt:MSVCP140.dll
 0000:fffe6000       .debug$S                   10000000     msvcprt:MSVCP140.dll
 0000:fffe6000       .debug$S                   10000000     msvcprt:MSVCP140.dll
 0000:fffe6000       .debug$S                   10000000     msvcprt:MSVCP140.dll
 0000:fffe6000       .debug$S                   10000000     msvcprt:MSVCP140.dll
 0000:fffe6000       .debug$S                   10000000     msvcprt:MSVCP140.dll
 0000:fffe6000       .debug$S                   10000000     msvcprt:MSVCP140.dll
 0000:fffe6000       .debug$S                   10000000     msvcprt:MSVCP140.dll
 0000:fffe6000       .debug$S                   10000000     msvcprt:MSVCP140.dll
 0000:fffe6000       .debug$S                   10000000     msvcprt:MSVCP140.dll
 0000:fffe6000       .debug$S                   10000000     msvcprt:MSVCP140.dll
 0000:fffe6000       .debug$S                   10000000     msvcprt:MSVCP140.dll
 0000:fffe6000       .debug$S                   10000000     msvcprt:MSVCP140.dll
 0000:fffe6000       .debug$S                   10000000     msvcprt:MSVCP140.dll
 0000:fffe6000       .debug$S                   10000000     msvcprt:MSVCP140.dll
 0000:fffe6000       .debug$S                   10000000     msvcprt:MSVCP140.dll
 0000:fffe6000       .debug$S                   10000000     msvcprt:MSVCP140.dll
 0000:fffe6000       .debug$S                   10000000     msvcprt:MSVCP140.dll
 0000:fffe6000       .debug$S                   10000000     msvcprt:MSVCP140.dll
 0000:fffe6000       .debug$S                   10000000     msvcprt:MSVCP140.dll
 0000:fffe6000       .debug$S                   10000000     msvcprt:MSVCP140.dll
 0000:fffe6000       .debug$S                   10000000     msvcprt:MSVCP140.dll
 0000:fffe6000       .debug$S                   10000000     msvcprt:MSVCP140.dll
 0000:fffe6000       .debug$S                   10000000     msvcprt:MSVCP140.dll
 0000:fffe6000       .debug$S                   10000000     msvcprt:MSVCP140.dll
 0000:fffe6000       .debug$S                   10000000     msvcprt:MSVCP140.dll
 0000:fffe6000       .debug$S                   10000000     msvcprt:MSVCP140.dll
 0000:fffe6000       .debug$S                   10000000     msvcprt:MSVCP140.dll
 0000:fffe6000       .debug$S                   10000000     msvcprt:MSVCP140.dll
 0000:fffe6000       .debug$S                   10000000     msvcprt:MSVCP140.dll
 0000:fffe6000       .debug$S                   10000000     msvcprt:MSVCP140.dll
 0000:fffe6000       .debug$S                   10000000     msvcprt:MSVCP140.dll
 0000:fffe6000       .debug$S                   10000000     msvcprt:MSVCP140.dll
 0000:fffe6000       .debug$S                   10000000     msvcprt:MSVCP140.dll
 0000:fffe6000       .debug$S                   10000000     msvcprt:MSVCP140.dll
 0000:fffe6000       .debug$S                   10000000     msvcprt:MSVCP140.dll
 0000:fffe6000       .debug$S                   10000000     msvcprt:MSVCP140.dll
 0000:fffe6000       .debug$S                   10000000     msvcprt:MSVCP140.dll
 0000:fffe6000       .debug$S                   10000000     msvcprt:MSVCP140.dll
 0000:fffe6000       .debug$S                   10000000     msvcprt:MSVCP140.dll
 0000:fffe6000       .debug$S                   10000000     msvcprt:MSVCP140.dll
 0000:fffe6000       .debug$S                   10000000     msvcprt:MSVCP140.dll
 0000:fffe6000       .debug$S                   10000000     msvcprt:MSVCP140.dll
 0000:fffe6000       .debug$S                   10000000     msvcprt:MSVCP140.dll
 0000:fffe6000       .debug$S                   10000000     msvcprt:MSVCP140.dll
 0000:fffe6000       .debug$S                   10000000     msvcprt:MSVCP140.dll
 0000:fffe6000       .debug$S                   10000000     msvcprt:MSVCP140.dll
 0000:fffe6000       .debug$S                   10000000     msvcprt:MSVCP140.dll
 0000:fffe6000       .debug$S                   10000000     msvcprt:MSVCP140.dll
 0000:fffe6000       .debug$S                   10000000     msvcprt:MSVCP140.dll
 0000:fffe6000       .debug$S                   10000000     msvcprt:MSVCP140.dll
 0000:fffe6000       .debug$S                   10000000     msvcprt:MSVCP140.dll
 0000:fffe6000       .debug$S                   10000000     msvcprt:MSVCP140.dll
 0000:fffe6000       .debug$S                   10000000     msvcprt:MSVCP140.dll
 0000:fffe6000       .debug$S                   10000000     msvcprt:MSVCP140.dll
 0000:fffe6000       .debug$S                   10000000     msvcprt:MSVCP140.dll
 0000:fffe6000       .debug$S                   10000000     msvcprt:MSVCP140.dll
 0000:fffe6000       .debug$S                   10000000     msvcprt:MSVCP140.dll
 0000:fffe6000       .debug$S                   10000000     msvcprt:MSVCP140.dll
 0000:fffe6000       .debug$S                   10000000     msvcprt:MSVCP140.dll
 0000:fffe6000       .debug$S                   10000000     msvcprt:MSVCP140.dll
 0000:fffe6000       .debug$S                   10000000     msvcprt:MSVCP140.dll
 0000:fffe6000       .debug$S                   10000000     msvcprt:MSVCP140.dll
 0000:fffe6000       .debug$S                   10000000     msvcprt:MSVCP140.dll
 0000:fffe6000       .debug$S                   10000000     msvcprt:MSVCP140.dll
 0000:fffe6000       .debug$S                   10000000     msvcprt:MSVCP140.dll
 0000:fffe6000       .debug$S                   10000000     msvcprt:MSVCP140.dll
 0000:fffe6000       .debug$S                   10000000     msvcprt:MSVCP140.dll
 0000:fffe6000       .debug$S                   10000000     msvcprt:MSVCP140.dll
 0000:fffe6000       .debug$S                   10000000     msvcprt:MSVCP140.dll
 0000:fffe6000       .debug$S                   10000000     msvcprt:MSVCP140.dll
 0000:fffe6000       .debug$S                   10000000     msvcprt:MSVCP140.dll
 0000:fffe6000       .debug$S                   10000000     msvcprt:MSVCP140.dll
 0000:fffe6000       .debug$S                   10000000     msvcprt:MSVCP140.dll
 0000:fffe6000       .debug$S                   10000000     msvcprt:MSVCP140.dll
 0000:fffe6000       .debug$S                   10000000     msvcprt:MSVCP140.dll
 0000:fffe6000       .debug$S                   10000000     msvcprt:MSVCP140.dll
 0000:fffe6000       .debug$S                   10000000     msvcprt:MSVCP140.dll
 0000:fffe6000       .debug$S                   10000000     msvcprt:MSVCP140.dll
 0000:fffe6000       .debug$S                   10000000     msvcprt:MSVCP140.dll
 0000:fffe6000       .debug$S                   10000000     msvcprt:MSVCP140.dll
 0000:fffe6000       .debug$S                   10000000     msvcprt:MSVCP140.dll
 0000:fffe6000       .debug$S                   10000000     msvcprt:MSVCP140.dll
 0000:fffe6000       .debug$S                   10000000     msvcprt:MSVCP140.dll
 0000:fffe6000       .debug$S                   10000000     msvcprt:MSVCP140.dll
 0000:fffe6000       .debug$S                   10000000     msvcprt:MSVCP140.dll
 0000:fffe6000       .debug$S                   10000000     vcruntime:VCRUNTIME140.dll
 0000:fffe6000       .debug$S                   10000000     vcruntime:VCRUNTIME140.dll
 0000:fffe6000       .debug$S                   10000000     vcruntime:VCRUNTIME140.dll
 0000:fffe6000       .debug$S                   10000000     vcruntime:VCRUNTIME140.dll
 0000:fffe6000       .debug$S                   10000000     vcruntime:VCRUNTIME140.dll
 0000:fffe6000       .debug$S                   10000000     vcruntime:VCRUNTIME140.dll
 0000:fffe6000       .debug$S                   10000000     vcruntime:VCRUNTIME140.dll
 0000:fffe6000       .debug$S                   10000000     vcruntime:VCRUNTIME140.dll
 0000:fffe6000       .debug$S                   10000000     vcruntime:VCRUNTIME140.dll
 0000:fffe6000       .debug$S                   10000000     vcruntime:VCRUNTIME140.dll
 0000:fffe6000       .debug$S                   10000000     vcruntime:VCRUNTIME140.dll
 0000:fffe6000       .debug$S                   10000000     vcruntime:VCRUNTIME140.dll
 0000:fffe6000       .debug$S                   10000000     vcruntime:VCRUNTIME140.dll
 0000:fffe6000       .debug$S                   10000000     vcruntime:VCRUNTIME140.dll
 0000:fffe6000       .debug$S                   10000000     vcruntime:VCRUNTIME140.dll
 0000:fffe6000       .debug$S                   10000000     ucrt:api-ms-win-crt-environment-l1-1-0.dll
 0002:ffff1000       .idata$6                   10000000     ucrt:api-ms-win-crt-environment-l1-1-0.dll
 0000:fffe6000       .debug$S                   10000000     ucrt:api-ms-win-crt-filesystem-l1-1-0.dll
 0000:fffe6000       .debug$S                   10000000     ucrt:api-ms-win-crt-filesystem-l1-1-0.dll
 0000:fffe6000       .debug$S                   10000000     ucrt:api-ms-win-crt-filesystem-l1-1-0.dll
 0000:fffe6000       .debug$S                   10000000     ucrt:api-ms-win-crt-heap-l1-1-0.dll
 0000:fffe6000       .debug$S                   10000000     ucrt:api-ms-win-crt-heap-l1-1-0.dll
 0000:fffe6000       .debug$S                   10000000     ucrt:api-ms-win-crt-heap-l1-1-0.dll
 0000:fffe6000       .debug$S                   10000000     ucrt:api-ms-win-crt-heap-l1-1-0.dll
 0000:fffe6000       .debug$S                   10000000     ucrt:api-ms-win-crt-runtime-l1-1-0.dll
 0000:fffe6000       .debug$S                   10000000     ucrt:api-ms-win-crt-runtime-l1-1-0.dll
 0000:fffe6000       .debug$S                   10000000     ucrt:api-ms-win-crt-runtime-l1-1-0.dll
 0000:fffe6000       .debug$S                   10000000     ucrt:api-ms-win-crt-runtime-l1-1-0.dll
 0000:fffe6000       .debug$S                   10000000     ucrt:api-ms-win-crt-runtime-l1-1-0.dll
 0000:fffe6000       .debug$S                   10000000     ucrt:api-ms-win-crt-runtime-l1-1-0.dll
 0000:fffe6000       .debug$S                   10000000     ucrt:api-ms-win-crt-runtime-l1-1-0.dll
 0000:fffe6000       .debug$S                   10000000     ucrt:api-ms-win-crt-runtime-l1-1-0.dll
 0000:fffe6000       .debug$S                   10000000     ucrt:api-ms-win-crt-runtime-l1-1-0.dll
 0000:fffe6000       .debug$S                   10000000     ucrt:api-ms-win-crt-runtime-l1-1-0.dll
 0000:fffe6000       .debug$S                   10000000     ucrt:api-ms-win-crt-runtime-l1-1-0.dll
 0000:fffe6000       .debug$S                   10000000     ucrt:api-ms-win-crt-runtime-l1-1-0.dll
 0000:fffe6000       .debug$S                   10000000     ucrt:api-ms-win-crt-runtime-l1-1-0.dll
 0000:fffe6000       .debug$S                   10000000     ucrt:api-ms-win-crt-runtime-l1-1-0.dll
 0000:fffe6000       .debug$S                   10000000     ucrt:api-ms-win-crt-runtime-l1-1-0.dll
 0000:fffe6000       .debug$S                   10000000     ucrt:api-ms-win-crt-stdio-l1-1-0.dll
 0000:fffe6000       .debug$S                   10000000     ucrt:api-ms-win-crt-stdio-l1-1-0.dll
 0000:fffe6000       .debug$S                   10000000     ucrt:api-ms-win-crt-stdio-l1-1-0.dll
 0000:fffe6000       .debug$S                   10000000     ucrt:api-ms-win-crt-stdio-l1-1-0.dll
 0000:fffe6000       .debug$S                   10000000     ucrt:api-ms-win-crt-stdio-l1-1-0.dll
 0000:fffe6000       .debug$S                   10000000     ucrt:api-ms-win-crt-stdio-l1-1-0.dll
 0000:fffe6000       .debug$S                   10000000     ucrt:api-ms-win-crt-stdio-l1-1-0.dll
 0000:fffe6000       .debug$S                   10000000     ucrt:api-ms-win-crt-stdio-l1-1-0.dll
 0000:fffe6000       .debug$S                   10000000     ucrt:api-ms-win-crt-stdio-l1-1-0.dll
 0000:fffe6000       .debug$S                   10000000     ucrt:api-ms-win-crt-stdio-l1-1-0.dll
 0000:fffe6000       .debug$S                   10000000     ucrt:api-ms-win-crt-stdio-l1-1-0.dll
 0000:fffe6000       .debug$S                   10000000     ucrt:api-ms-win-crt-stdio-l1-1-0.dll
 0000:fffe6000       .debug$S                   10000000     ucrt:api-ms-win-crt-stdio-l1-1-0.dll
 0000:fffe6000       .debug$S                   10000000     ucrt:api-ms-win-crt-stdio-l1-1-0.dll
 0000:fffe6000       .debug$S                   10000000     ucrt:api-ms-win-crt-stdio-l1-1-0.dll
 0000:fffe6000       .debug$S                   10000000     ucrt:api-ms-win-crt-stdio-l1-1-0.dll
 0000:fffe6000       .debug$S                   10000000     ucrt:api-ms-win-crt-stdio-l1-1-0.dll
 0000:fffe6000       .debug$S                   10000000     ucrt:api-ms-win-crt-string-l1-1-0.dll
 0000:fffe6000       .debug$S                   10000000     ucrt:api-ms-win-crt-string-l1-1-0.dll
 0000:fffe6000       .debug$S                   10000000     ucrt:api-ms-win-crt-string-l1-1-0.dll
 0000:fffe6000       .debug$S                   10000000     ucrt:api-ms-win-crt-string-l1-1-0.dll
 0000:fffe6000       .debug$S                   10000000     Shell32:SHELL32.dll
 0002:ffff1000       .idata$6                   10000000     Shell32:SHELL32.dll
 0000:fffe6000       .debug$S                   10000000     advapi32:ADVAPI32.dll
 0000:fffe6000       .debug$S                   10000000     advapi32:ADVAPI32.dll
 0000:fffe6000       .debug$S                   10000000     advapi32:ADVAPI32.dll
 0000:fffe6000       .debug$S                   10000000     advapi32:ADVAPI32.dll
 0000:fffe6000       .debug$S                   10000000     kernel32:KERNEL32.dll
 0000:fffe6000       .debug$S                   10000000     kernel32:KERNEL32.dll
 0000:fffe6000       .debug$S                   10000000     kernel32:KERNEL32.dll
 0000:fffe6000       .debug$S                   10000000     kernel32:KERNEL32.dll
 0000:fffe6000       .debug$S                   10000000     kernel32:KERNEL32.dll
 0000:fffe6000       .debug$S                   10000000     kernel32:KERNEL32.dll
 0000:fffe6000       .debug$S                   10000000     kernel32:KERNEL32.dll
 0000:fffe6000       .debug$S                   10000000     kernel32:KERNEL32.dll
 0000:fffe6000       .debug$S                   10000000     kernel32:KERNEL32.dll
 0000:fffe6000       .debug$S                   10000000     kernel32:KERNEL32.dll
 0000:fffe6000       .debug$S                   10000000     kernel32:KERNEL32.dll
 0000:fffe6000       .debug$S                   10000000     kernel32:KERNEL32.dll
 0000:fffe6000       .debug$S                   10000000     kernel32:KERNEL32.dll
 0000:fffe6000       .debug$S                   10000000     kernel32:KERNEL32.dll
 0000:fffe6000       .debug$S                   10000000     kernel32:KERNEL32.dll
 0000:fffe6000       .debug$S                   10000000     kernel32:KERNEL32.dll
 0000:fffe6000       .debug$S                   10000000     kernel32:KERNEL32.dll
 0000:fffe6000       .debug$S                   10000000     kernel32:KERNEL32.dll
 0000:fffe6000       .debug$S                   10000000     kernel32:KERNEL32.dll
 0000:fffe6000       .debug$S                   10000000     kernel32:KERNEL32.dll
 0000:fffe6000       .debug$S                   10000000     kernel32:KERNEL32.dll
 0000:fffe6000       .debug$S                   10000000     kernel32:KERNEL32.dll
 0000:fffe6000       .debug$S                   10000000     kernel32:KERNEL32.dll
 0000:fffe6000       .debug$S                   10000000     kernel32:KERNEL32.dll
 0000:fffe6000       .debug$S                   10000000     kernel32:KERNEL32.dll
 0000:fffe6000       .debug$S                   10000000     kernel32:KERNEL32.dll
 0000:fffe6000       .debug$S                   10000000     kernel32:KERNEL32.dll
 0000:fffe6000       .debug$S                   10000000     kernel32:KERNEL32.dll
 0000:fffe6000       .debug$S                   10000000     kernel32:KERNEL32.dll
 0000:fffe6000       .debug$S                   10000000     kernel32:KERNEL32.dll
 0000:fffe6000       .debug$S                   10000000     kernel32:KERNEL32.dll
 0000:fffe6000       .debug$S                   10000000     kernel32:KERNEL32.dll
 0000:fffe6000       .debug$S                   10000000     kernel32:KERNEL32.dll
 0000:fffe6000       .debug$S                   10000000     kernel32:KERNEL32.dll
 0000:fffe6000       .debug$S                   10000000     kernel32:KERNEL32.dll
 0000:fffe6000       .debug$S                   10000000     kernel32:KERNEL32.dll
 0000:fffe6000       .debug$S                   10000000     kernel32:KERNEL32.dll
 0000:fffe6000       .debug$S                   10000000     kernel32:KERNEL32.dll
 0000:fffe6000       .debug$S                   10000000     kernel32:KERNEL32.dll
 0000:fffe6000       .debug$S                   10000000     kernel32:KERNEL32.dll
 0000:fffe6000       .debug$S                   10000000     kernel32:KERNEL32.dll
 0000:fffe6000       .debug$S                   10000000     kernel32:KERNEL32.dll
 0000:fffe6000       .debug$S                   10000000     kernel32:KERNEL32.dll
 0000:fffe6000       .debug$S                   10000000     kernel32:KERNEL32.dll
 0000:fffe6000       .debug$S                   10000000     kernel32:KERNEL32.dll
 0000:fffe6000       .debug$S                   10000000     kernel32:KERNEL32.dll
 0000:fffe6000       .debug$S                   10000000     kernel32:KERNEL32.dll
 0000:fffe6000       .debug$S                   10000000     kernel32:KERNEL32.dll
 0000:fffe6000       .debug$S                   10000000     kernel32:KERNEL32.dll
 0000:fffe6000       .debug$S                   10000000     kernel32:KERNEL32.dll
 0000:fffe6000       .debug$S                   10000000     kernel32:KERNEL32.dll
 0000:fffe6000       .debug$S                   10000000     kernel32:KERNEL32.dll
 0000:fffe6000       .debug$S                   10000000     kernel32:KERNEL32.dll
 0000:fffe6000       .debug$S                   10000000     kernel32:KERNEL32.dll
 0000:fffe6000       .debug$S                   10000000     kernel32:KERNEL32.dll
 0000:fffe6000       .debug$S                   10000000     kernel32:KERNEL32.dll
 0000:fffe6000       .debug$S                   10000000     kernel32:KERNEL32.dll
 0000:fffe6000       .debug$S                   10000000     kernel32:KERNEL32.dll
 0000:fffe6000       .debug$S                   10000000     kernel32:KERNEL32.dll
 0000:fffe6000       .debug$S                   10000000     msi:msi.dll
 0000:fffe6000       .debug$S                   10000000     msi:msi.dll
 0000:fffe6000       .debug$S                   10000000     msi:msi.dll
 0000:fffe6000       .debug$S                   10000000     msi:msi.dll
 0000:fffe6000       .debug$S                   10000000     msi:msi.dll
 0000:fffe6000       .debug$S                   10000000     msi:msi.dll
 0000:fffe6000       .debug$S                   10000000     msi:msi.dll
 0000:fffe6000       .debug$S                   10000000     msi:msi.dll
 0000:fffe6000       .debug$S                   10000000     msi:msi.dll
 0000:fffe6000       .debug$S                   10000000     msi:msi.dll
 0000:fffe6000       .debug$S                   10000000     msi:msi.dll
 0000:fffe6000       .debug$S                   10000000     msi:msi.dll
 0000:fffe6000       .debug$S                   10000000     msi:msi.dll
 0000:fffe6000       .debug$S                   10000000     msi:msi.dll
 0000:fffe6000       .debug$S                   10000000     msi:msi.dll
 0000:fffe6000       .debug$S                   10000000     msi:msi.dll
 0000:fffe6000       .debug$S                   10000000     msi:msi.dll
 0000:fffe6000       .debug$S                   10000000     msi:msi.dll
 0000:fffe6000       .debug$S                   10000000     msi:msi.dll
 0000:fffe6000       .debug$S                   10000000     msi:msi.dll
 0000:fffe6000       .debug$S                   10000000     msi:msi.dll
 0000:fffe6000       .debug$S                   10000000     msi:msi.dll
 0000:fffe6000       .debug$S                   10000000     ole32:ole32.dll
 0000:fffe6000       .debug$S                   10000000     ole32:ole32.dll
 0000:fffe6000       .debug$S                   10000000     ole32:ole32.dll
 0000:fffe6000       .debug$S                   10000000     shlwapi:SHLWAPI.dll
 0002:ffff1000       .idata$6                   10000000     shlwapi:SHLWAPI.dll
 0000:fffe6000       .debug$S                   10000000     user32:USER32.dll
 0002:ffff1000       .idata$6                   10000000     user32:USER32.dll
 0001:00000000       ??__FlastErrorLogAppender@?A0xd3578678@@YAXXZ 10001000 f   app.obj
 0001:0000000c       ??__FnopLogAppender@?A0xd3578678@@YAXXZ 1000100c f   app.obj
 0001:00000018       ??__FstandardLogAppender@?A0xd3578678@@YAXXZ 10001018 f   app.obj
 0001:00000024       ??__F_Fac_tidy_reg@std@@YAXXZ 10001024 f   msvcprt:locale0_implib.obj
 0001:00000227       __catch$??$?6GU?$char_traits@G@std@@@std@@YAAAV?$basic_ostream@GU?$char_traits@G@std@@@0@AAV10@PBD@Z$0 10001227 f i ErrorHandling.obj
 0001:000003a3       __catch$??$?6GU?$char_traits@G@std@@@std@@YAAAV?$basic_ostream@GU?$char_traits@G@std@@@0@AAV10@PBG@Z$0 100013a3 f i ErrorHandling.obj
 0001:00000549       __catch$??$?6U?$char_traits@D@std@@@std@@YAAAV?$basic_ostream@DU?$char_traits@D@std@@@0@AAV10@PBD@Z$0 10001549 f i ErrorHandling.obj
 0001:000006fd       __catch$??$_Insert_string@DU?$char_traits@D@std@@I@std@@YAAAV?$basic_ostream@DU?$char_traits@D@std@@@0@AAV10@QBDI@Z$0 100016fd f i ErrorHandling.obj
 0001:00000840       __catch$??$_Insert_string@GU?$char_traits@G@std@@I@std@@YAAAV?$basic_ostream@GU?$char_traits@G@std@@@0@AAV10@QBGI@Z$0 10001840 f i ErrorHandling.obj
 0001:000015d8       ?getFilename@?A0xd1a094c7@@YA?AV?$basic_string@GU?$char_traits@G@std@@V?$allocator@G@2@@std@@ABUSourceCodePos@@@Z 100025d8 f   ErrorHandling.obj
 0001:0000169a       ?isNotSpace@?A0xd1a094c7@@YA_NH@Z 1000269a f   ErrorHandling.obj
 0001:00001c8a       ?printWithoutWhitespaces@?A0xd1a094c7@@YAIAAV?$basic_ostream@DU?$char_traits@D@std@@@std@@ABV?$basic_string@DU?$char_traits@D@std@@V?$allocator@D@2@@3@W4TrimMode@1@@Z 10002c8a f   ErrorHandling.obj
 0001:00001d35       ?reportError@?A0xd1a094c7@@YAXABUSourceCodePos@@ABV?$basic_string@GU?$char_traits@G@std@@V?$allocator@G@2@@std@@@Z 10002d35 f   ErrorHandling.obj
 0001:00003423       ?initGuid@?A0x2459fff0@@YAXABV?$basic_string@GU?$char_traits@G@std@@V?$allocator@G@2@@std@@AAU_GUID@@@Z 10004423 f   Guid.obj
 0001:00003c8c       ??1?$AtEndOfScope@V<lambda_bafb2a7f1406751b8a75ac1ff6dad7d1>@@@@QAE@XZ 10004c8c f   JniUtils.obj
 0001:00003ce4       __catch$??1?$AtEndOfScope@V<lambda_bafb2a7f1406751b8a75ac1ff6dad7d1>@@@@QAE@XZ$0 10004ce4 f   JniUtils.obj
 0001:00003d0d       __catch$??1?$AtEndOfScope@V<lambda_bafb2a7f1406751b8a75ac1ff6dad7d1>@@@@QAE@XZ$1 10004d0d f   JniUtils.obj
 0001:000043b5       __catch$??6?$basic_ostream@GU?$char_traits@G@std@@@std@@QAEAAV01@G@Z$0 100053b5 f i Log.obj
 0001:00004408       ??_GLastErrorLogAppender@?A0xd3578678@@UAEPAXI@Z 10005408 f i app.obj
 0001:00004408       ??_GStandardLogAppender@?A0xd3578678@@UAEPAXI@Z 10005408 f i app.obj
 0001:000054de       ?openDatabase@?A0x6ccb95c8@msi@@YAKABV?$basic_string@GU?$char_traits@G@std@@V?$allocator@G@2@@std@@@Z 100064de f   MsiDb.obj
 0001:00006132       ??$getProperty@P6GIKIPAGPAK@ZKI@?A0x0e70828c@msi@@YA?AV?$basic_string@GU?$char_traits@G@std@@V?$allocator@G@2@@std@@P6GIKIPAGPAK@ZQBDKI@Z 10007132 f   MsiUtils.obj
 0001:000068c8       ?makeMessage@?A0x0e70828c@msi@@YA?AV?$basic_string@DU?$char_traits@D@std@@V?$allocator@D@2@@std@@ABV34@I@Z 100078c8 f   MsiUtils.obj
 0001:00006a2d       __catch$?makeMessage@?A0x0e70828c@msi@@YA?AV?$basic_string@DU?$char_traits@D@std@@V?$allocator@D@2@@std@@ABV34@I@Z$0 10007a2d f   MsiUtils.obj
 0001:00006d84       ?retrieveModuleName@?A0x40e1fcfd@@YA?AV?$basic_string@GU?$char_traits@G@std@@V?$allocator@G@2@@std@@XZ 10007d84 f   PlatformLogEvent.obj
 0001:00006dbd       __catch$?retrieveModuleName@?A0x40e1fcfd@@YA?AV?$basic_string@GU?$char_traits@G@std@@V?$allocator@G@2@@std@@XZ$0 10007dbd f   PlatformLogEvent.obj
 0001:00007343       __catch$??1FileLock@ResourceEditor@@QAE@XZ$0 10008343 f   ResourceEditor.obj
 0001:0000736c       __catch$??1FileLock@ResourceEditor@@QAE@XZ$1 1000836c f   ResourceEditor.obj
 0001:00007f11       ??$for_each@V?$_Tree_const_iterator@V?$_Tree_val@U?$_Tree_simple_types@U?$pair@$$CBV?$basic_string@GU?$char_traits@G@std@@V?$allocator@G@2@@std@@V12@@std@@@std@@@std@@@std@@V<lambda_fa730d0a4b0afd944df9b292ec615b4b>@@@std@@YA?AV<lambda_fa730d0a4b0afd944df9b292ec615b4b>@@V?$_Tree_const_iterator@V?$_Tree_val@U?$_Tree_simple_types@U?$pair@$$CBV?$basic_string@GU?$char_traits@G@std@@V?$allocator@G@2@@std@@V12@@std@@@std@@@std@@@0@0V1@@Z 10008f11 f   VersionInfo.obj
 0001:000080ab       ??0FixedFileVersion@?A0xcb1fbc16@@QAE@ABV?$basic_string@GU?$char_traits@G@std@@V?$allocator@G@2@@std@@@Z 100090ab f   VersionInfo.obj
 0001:00008155       ??0StreamSize@?A0xcb1fbc16@@QAE@AAV?$basic_ostream@DU?$char_traits@D@std@@@std@@@Z 10009155 f   VersionInfo.obj
 0001:0000820c       ??1StreamSize@?A0xcb1fbc16@@QAE@XZ 1000920c f   VersionInfo.obj
 0001:000082e5       __catch$??1StreamSize@?A0xcb1fbc16@@QAE@XZ$0 100092e5 f   VersionInfo.obj
 0001:0000830e       __catch$??1StreamSize@?A0xcb1fbc16@@QAE@XZ$1 1000930e f   VersionInfo.obj
 0001:0000841c       ?add32bitPadding@?A0xcb1fbc16@@YAXAAV?$basic_ostream@DU?$char_traits@D@std@@@std@@@Z 1000941c f   VersionInfo.obj
 0001:0000874d       __catch$?createFIXEDFILEINFO@VersionInfo@@ABE?AUtagVS_FIXEDFILEINFO@@XZ$0 1000974d f   VersionInfo.obj
 0001:00008aff       ?write@?A0xcb1fbc16@@YAAAV?$basic_ostream@DU?$char_traits@D@std@@@std@@AAV23@ABV?$basic_string@GU?$char_traits@G@std@@V?$allocator@G@2@@3@@Z 10009aff f   VersionInfo.obj
 0001:00008b26       ?writeWORD@?A0xcb1fbc16@@YAAAV?$basic_ostream@DU?$char_traits@D@std@@@std@@AAV23@I@Z 10009b26 f   VersionInfo.obj
 0001:00008d11       ?getSystemMessageDescription@?A0xd5983087@@YA?AV?$basic_string@GU?$char_traits@G@std@@V?$allocator@G@2@@std@@KPAUHINSTANCE__@@@Z 10009d11 f   WinErrorHandling.obj
 0001:00008df5       ?makeMessage@?A0xd5983087@@YA?AV?$basic_string@DU?$char_traits@D@std@@V?$allocator@D@2@@std@@ABV23@PBDPBXK@Z 10009df5 f   WinErrorHandling.obj
 0001:00009090       ??$getSystemDirImpl@P6GIPAGI@Z@?A0x7970c2a6@SysInfo@@YA?AV?$basic_string@GU?$char_traits@G@std@@V?$allocator@G@2@@std@@P6GIPAGI@ZABV?$basic_string@DU?$char_traits@D@std@@V?$allocator@D@2@@3@@Z 1000a090 f   WinSysInfo.obj
 0001:00009377       ?getModulePath@?A0x7970c2a6@SysInfo@@YA?AV?$basic_string@GU?$char_traits@G@std@@V?$allocator@G@2@@std@@PAUHINSTANCE__@@@Z 1000a377 f   WinSysInfo.obj
 0001:000094e8       ?GetLongPath@?A0x764c93a3@@YA?AV?$basic_string@GU?$char_traits@G@std@@V?$allocator@G@2@@std@@ABV23@@Z 1000a4e8 f   WindowsRegistry.obj
 0001:0000968d       ?StringLengthWorkerW@@YGJPBGIPAI@Z 1000a68d f   WindowsRegistry.obj
 0001:000097c6       __catch$_Java_jdk_jpackage_internal_WindowsRegistry_comparePaths@16$0 1000a7c6 f   WindowsRegistry.obj
 0001:000097ef       __catch$_Java_jdk_jpackage_internal_WindowsRegistry_comparePaths@16$1 1000a7ef f   WindowsRegistry.obj
 0001:00009936       __catch$_Java_jdk_jpackage_internal_WindowsRegistry_enumRegistryValue@20$0 1000a936 f   WindowsRegistry.obj
 0001:0000995f       __catch$_Java_jdk_jpackage_internal_WindowsRegistry_enumRegistryValue@20$1 1000a95f f   WindowsRegistry.obj
 0001:00009a26       __catch$_Java_jdk_jpackage_internal_WindowsRegistry_openRegistryKey@16$0 1000aa26 f   WindowsRegistry.obj
 0001:00009a4f       __catch$_Java_jdk_jpackage_internal_WindowsRegistry_openRegistryKey@16$1 1000aa4f f   WindowsRegistry.obj
 0001:00009b6e       __catch$_Java_jdk_jpackage_internal_WindowsRegistry_readDwordValue@24$0 1000ab6e f   WindowsRegistry.obj
 0001:00009ba0       __catch$_Java_jdk_jpackage_internal_WindowsRegistry_readDwordValue@24$1 1000aba0 f   WindowsRegistry.obj
 0001:00009c19       ?append@StandardLogAppender@?A0xd3578678@@UAEXABULogEvent@@@Z 1000ac19 f   app.obj
 0001:00009d0b       ?append@LastErrorLogAppender@?A0xd3578678@@UAEXABULogEvent@@@Z 1000ad0b f   app.obj
 0001:0000a03d       __catch$_Java_jdk_jpackage_internal_ExecutableRebrander_iconSwap@20$0 1000b03d f   jpackage.obj
 0001:0000a066       __catch$_Java_jdk_jpackage_internal_ExecutableRebrander_iconSwap@20$1 1000b066 f   jpackage.obj
 0001:0000a0e0       __catch$_Java_jdk_jpackage_internal_ExecutableRebrander_lockResource@12$0 1000b0e0 f   jpackage.obj
 0001:0000a109       __catch$_Java_jdk_jpackage_internal_ExecutableRebrander_lockResource@12$1 1000b109 f   jpackage.obj
 0001:0000a169       __catch$_Java_jdk_jpackage_internal_ExecutableRebrander_unlockResource@16$0 1000b169 f   jpackage.obj
 0001:0000a192       __catch$_Java_jdk_jpackage_internal_ExecutableRebrander_unlockResource@16$1 1000b192 f   jpackage.obj
 0001:0000a313       __catch$_Java_jdk_jpackage_internal_ExecutableRebrander_versionSwap@20$0 1000b313 f   jpackage.obj
 0001:0000a33c       __catch$_Java_jdk_jpackage_internal_ExecutableRebrander_versionSwap@20$1 1000b33c f   jpackage.obj
 0001:0000a527       __catch$_Java_jdk_jpackage_internal_WinExeBundler_embedMSI@20$0 1000b527 f   jpackage.obj
 0001:0000a55f       __catch$_Java_jdk_jpackage_internal_WinExeBundler_embedMSI@20$1 1000b55f f   jpackage.obj
 0001:0000a78b       ?fromMultiByte@?A0xf04d92fb@tstrings@@YA?AV?$basic_string@GU?$char_traits@G@std@@V?$allocator@G@2@@std@@ABV?$basic_string@DU?$char_traits@D@std@@V?$allocator@D@2@@4@H@Z 1000b78b f   tstrings.obj
 0001:0000a9ca       ?toMultiByte@?A0xf04d92fb@tstrings@@YA?AV?$basic_string@DU?$char_traits@D@std@@V?$allocator@D@2@@std@@ABV?$basic_string@GU?$char_traits@G@std@@V?$allocator@G@2@@4@H@Z 1000b9ca f   tstrings.obj
 0001:0000aec0       $$000000                   1000bec0     MSVCRT:chkstk.obj
 0001:0000b110       $$000000                   1000c110     MSVCRT:lldiv.obj
 0001:0000b1c0       $$000000                   1000c1c0     MSVCRT:llrem.obj
 0001:0000b285       ?find_pe_section@@YAPAU_IMAGE_SECTION_HEADER@@QAEI@Z 1000c285 f   MSVCRT:utility.obj
 0001:0000b59f       ?dllmain_crt_dispatch@@YGHQAUHINSTANCE__@@KQAX@Z 1000c59f f   MSVCRT:dll_dllmain.obj
 0001:0000b5f2       ?dllmain_crt_process_attach@@YAHQAUHINSTANCE__@@QAX@Z 1000c5f2 f   MSVCRT:dll_dllmain.obj
 0001:0000b6f9       ?dllmain_crt_process_detach@@YAH_N@Z 1000c6f9 f   MSVCRT:dll_dllmain.obj
 0001:0000b7a9       ?dllmain_dispatch@@YAHQAUHINSTANCE__@@KQAX@Z 1000c7a9 f   MSVCRT:dll_dllmain.obj
 0001:0000b8b4       ?dllmain_raw@@YGHQAUHINSTANCE__@@KQAX@Z 1000c8b4 f   MSVCRT:dll_dllmain.obj
 0001:0000bc40       $$000000                   1000cc40     MSVCRT:sehprolg4.obj
 0001:0000bcc7       ___get_entropy             1000ccc7 f   MSVCRT:gs_support.obj
 0001:0000bf5e       __unwindfunclet$??$?6GU?$char_traits@G@std@@@std@@YAAAV?$basic_ostream@GU?$char_traits@G@std@@@0@AAV10@PBD@Z$2 1000cf5e f   ErrorHandling.obj
 0001:0000bf66       __unwindfunclet$??$?6GU?$char_traits@G@std@@@std@@YAAAV?$basic_ostream@GU?$char_traits@G@std@@@0@AAV10@PBD@Z$3 1000cf66 f   ErrorHandling.obj
 0001:0000bf73       __ehhandler$??$?6GU?$char_traits@G@std@@@std@@YAAAV?$basic_ostream@GU?$char_traits@G@std@@@0@AAV10@PBD@Z 1000cf73 f   ErrorHandling.obj
 0001:0000bf90       __unwindfunclet$??$?6GU?$char_traits@G@std@@@std@@YAAAV?$basic_ostream@GU?$char_traits@G@std@@@0@AAV10@PBG@Z$2 1000cf90 f   ErrorHandling.obj
 0001:0000bf9d       __ehhandler$??$?6GU?$char_traits@G@std@@@std@@YAAAV?$basic_ostream@GU?$char_traits@G@std@@@0@AAV10@PBG@Z 1000cf9d f   ErrorHandling.obj
 0001:0000bfba       __unwindfunclet$??$?6U?$char_traits@D@std@@@std@@YAAAV?$basic_ostream@DU?$char_traits@D@std@@@0@AAV10@PBD@Z$2 1000cfba f   ErrorHandling.obj
 0001:0000bfc7       __ehhandler$??$?6U?$char_traits@D@std@@@std@@YAAAV?$basic_ostream@DU?$char_traits@D@std@@@0@AAV10@PBD@Z 1000cfc7 f   ErrorHandling.obj
 0001:0000bfe4       __unwindfunclet$??$_Insert_string@DU?$char_traits@D@std@@I@std@@YAAAV?$basic_ostream@DU?$char_traits@D@std@@@0@AAV10@QBDI@Z$2 1000cfe4 f   ErrorHandling.obj
 0001:0000bff1       __ehhandler$??$_Insert_string@DU?$char_traits@D@std@@I@std@@YAAAV?$basic_ostream@DU?$char_traits@D@std@@@0@AAV10@QBDI@Z 1000cff1 f   ErrorHandling.obj
 0001:0000c00e       __unwindfunclet$??$_Insert_string@GU?$char_traits@G@std@@I@std@@YAAAV?$basic_ostream@GU?$char_traits@G@std@@@0@AAV10@QBGI@Z$2 1000d00e f   ErrorHandling.obj
 0001:0000c01b       __ehhandler$??$_Insert_string@GU?$char_traits@G@std@@I@std@@YAAAV?$basic_ostream@GU?$char_traits@G@std@@@0@AAV10@QBGI@Z 1000d01b f   ErrorHandling.obj
 0001:0000c038       __unwindfunclet$??$use_facet@V?$ctype@G@std@@@std@@YAABV?$ctype@G@0@ABVlocale@0@@Z$0 1000d038 f   ErrorHandling.obj
 0001:0000c038       __unwindfunclet$??$use_facet@V?$codecvt@DDU_Mbstatet@@@std@@@std@@YAABV?$codecvt@DDU_Mbstatet@@@0@ABVlocale@0@@Z$0 1000d038 f   MsiDb.obj
 0001:0000c041       __unwindfunclet$??$use_facet@V?$ctype@G@std@@@std@@YAABV?$ctype@G@0@ABVlocale@0@@Z$1 1000d041 f   ErrorHandling.obj
 0001:0000c041       __unwindfunclet$??$use_facet@V?$codecvt@DDU_Mbstatet@@@std@@@std@@YAABV?$codecvt@DDU_Mbstatet@@@0@ABVlocale@0@@Z$1 1000d041 f   MsiDb.obj
 0001:0000c04e       __ehhandler$??$use_facet@V?$ctype@G@std@@@std@@YAABV?$ctype@G@0@ABVlocale@0@@Z 1000d04e f   ErrorHandling.obj
 0001:0000c04e       __ehhandler$??$use_facet@V?$codecvt@DDU_Mbstatet@@@std@@@std@@YAABV?$codecvt@DDU_Mbstatet@@@0@ABVlocale@0@@Z 1000d04e f   MsiDb.obj
 0001:0000c06b       __unwindfunclet$??0?$basic_ostringstream@DU?$char_traits@D@std@@V?$allocator@D@2@@std@@QAE@XZ$0 1000d06b f   ErrorHandling.obj
 0001:0000c088       __unwindfunclet$??0?$basic_ostringstream@DU?$char_traits@D@std@@V?$allocator@D@2@@std@@QAE@XZ$1 1000d088 f   ErrorHandling.obj
 0001:0000c099       __ehhandler$??0?$basic_ostringstream@DU?$char_traits@D@std@@V?$allocator@D@2@@std@@QAE@XZ 1000d099 f   ErrorHandling.obj
 0001:0000c0b6       __unwindfunclet$??0?$basic_ostringstream@GU?$char_traits@G@std@@V?$allocator@G@2@@std@@QAE@XZ$0 1000d0b6 f   ErrorHandling.obj
 0001:0000c0d3       __unwindfunclet$??0?$basic_ostringstream@GU?$char_traits@G@std@@V?$allocator@G@2@@std@@QAE@XZ$1 1000d0d3 f   ErrorHandling.obj
 0001:0000c0e4       __ehhandler$??0?$basic_ostringstream@GU?$char_traits@G@std@@V?$allocator@G@2@@std@@QAE@XZ 1000d0e4 f   ErrorHandling.obj
 0001:0000c101       __unwindfunclet$??0any@tstrings@@QAE@ABV?$basic_string@GU?$char_traits@G@std@@V?$allocator@G@2@@std@@@Z$0 1000d101 f   ErrorHandling.obj
 0001:0000c10e       __ehhandler$??0any@tstrings@@QAE@ABV?$basic_string@GU?$char_traits@G@std@@V?$allocator@G@2@@std@@@Z 1000d10e f   ErrorHandling.obj
 0001:0000c12b       __unwindfunclet$??0sentry@?$basic_ostream@DU?$char_traits@D@std@@@std@@QAE@AAV12@@Z$0 1000d12b f   ErrorHandling.obj
 0001:0000c12b       __unwindfunclet$??0sentry@?$basic_ostream@GU?$char_traits@G@std@@@std@@QAE@AAV12@@Z$0 1000d12b f   ErrorHandling.obj
 0001:0000c138       __ehhandler$??0sentry@?$basic_ostream@DU?$char_traits@D@std@@@std@@QAE@AAV12@@Z 1000d138 f   ErrorHandling.obj
 0001:0000c138       __ehhandler$??0sentry@?$basic_ostream@GU?$char_traits@G@std@@@std@@QAE@AAV12@@Z 1000d138 f   ErrorHandling.obj
 0001:0000c155       __ehhandler$??1_Sentry_base@?$basic_ostream@DU?$char_traits@D@std@@@std@@QAE@XZ 1000d155 f   ErrorHandling.obj
 0001:0000c155       __ehhandler$??1_Sentry_base@?$basic_ostream@GU?$char_traits@G@std@@@std@@QAE@XZ 1000d155 f   ErrorHandling.obj
 0001:0000c155       __ehhandler$??1?$unique_ptr@UJniObjWithEnv@jni@@ULocalRefDeleter@12@@std@@QAE@XZ 1000d155 f   JniUtils.obj
 0001:0000c155       __ehhandler$??1DatabaseRecord@msi@@QAE@XZ 1000d155 f   MsiDb.obj
 0001:0000c155       __ehhandler$??1?$unique_ptr@PAUHINSTANCE__@@ULibraryReleaser@Dll@@@std@@QAE@XZ 1000d155 f   MsiUtils.obj
 0001:0000c172       __ehhandler$??1sentry@?$basic_ostream@DU?$char_traits@D@std@@@std@@QAE@XZ 1000d172 f   ErrorHandling.obj
 0001:0000c172       __ehhandler$??1sentry@?$basic_ostream@GU?$char_traits@G@std@@@std@@QAE@XZ 1000d172 f   ErrorHandling.obj
 0001:0000c172       __ehhandler$??1?$basic_filebuf@DU?$char_traits@D@std@@@std@@UAE@XZ 1000d172 f   MsiDb.obj
 0001:0000c172       __ehhandler$??1DatabaseView@msi@@QAE@XZ 1000d172 f   MsiDb.obj
 0001:0000c172       __ehhandler$??1Database@msi@@QAE@XZ 1000d172 f   jpackage.obj
 0001:0000c18f       __unwindfunclet$??6@YAAAV?$basic_ostream@DU?$char_traits@D@std@@@std@@AAV01@ABVany@tstrings@@@Z$0 1000d18f f   ErrorHandling.obj
 0001:0000c18f       __unwindfunclet$?append@LastErrorLogAppender@?A0xd3578678@@UAEXABULogEvent@@@Z$0 1000d18f f   app.obj
 0001:0000c19c       __ehhandler$??6@YAAAV?$basic_ostream@DU?$char_traits@D@std@@@std@@AAV01@ABVany@tstrings@@@Z 1000d19c f   ErrorHandling.obj
 0001:0000c19c       __ehhandler$?append@LastErrorLogAppender@?A0xd3578678@@UAEXABULogEvent@@@Z 1000d19c f   app.obj
 0001:0000c1c3       __unwindfunclet$?getFilename@?A0xd1a094c7@@YA?AV?$basic_string@GU?$char_traits@G@std@@V?$allocator@G@2@@std@@ABUSourceCodePos@@@Z$0 1000d1c3 f   ErrorHandling.obj
 0001:0000c1cb       __unwindfunclet$?getFilename@?A0xd1a094c7@@YA?AV?$basic_string@GU?$char_traits@G@std@@V?$allocator@G@2@@std@@ABUSourceCodePos@@@Z$2 1000d1cb f   ErrorHandling.obj
 0001:0000c1d8       __ehhandler$?getFilename@?A0xd1a094c7@@YA?AV?$basic_string@GU?$char_traits@G@std@@V?$allocator@G@2@@std@@ABUSourceCodePos@@@Z 1000d1d8 f   ErrorHandling.obj
 0001:0000c1ff       __unwindfunclet$?joinErrorMessages@@YA?AV?$basic_string@DU?$char_traits@D@std@@V?$allocator@D@2@@std@@ABV12@0@Z$0 1000d1ff f   ErrorHandling.obj
 0001:0000c207       __unwindfunclet$?joinErrorMessages@@YA?AV?$basic_string@DU?$char_traits@D@std@@V?$allocator@D@2@@std@@ABV12@0@Z$1 1000d207 f   ErrorHandling.obj
 0001:0000c20f       __unwindfunclet$?joinErrorMessages@@YA?AV?$basic_string@DU?$char_traits@D@std@@V?$allocator@D@2@@std@@ABV12@0@Z$2 1000d20f f   ErrorHandling.obj
 0001:0000c217       __unwindfunclet$?joinErrorMessages@@YA?AV?$basic_string@DU?$char_traits@D@std@@V?$allocator@D@2@@std@@ABV12@0@Z$3 1000d217 f   ErrorHandling.obj
 0001:0000c222       __unwindfunclet$?joinErrorMessages@@YA?AV?$basic_string@DU?$char_traits@D@std@@V?$allocator@D@2@@std@@ABV12@0@Z$4 1000d222 f   ErrorHandling.obj
 0001:0000c22f       __ehhandler$?joinErrorMessages@@YA?AV?$basic_string@DU?$char_traits@D@std@@V?$allocator@D@2@@std@@ABV12@0@Z 1000d22f f   ErrorHandling.obj
 0001:0000c259       __unwindfunclet$?makeMessage@@YA?AV?$basic_string@DU?$char_traits@D@std@@V?$allocator@D@2@@std@@ABVruntime_error@2@ABUSourceCodePos@@@Z$0 1000d259 f   ErrorHandling.obj
 0001:0000c264       __unwindfunclet$?makeMessage@@YA?AV?$basic_string@DU?$char_traits@D@std@@V?$allocator@D@2@@std@@ABVruntime_error@2@ABUSourceCodePos@@@Z$1 1000d264 f   ErrorHandling.obj
 0001:0000c26c       __unwindfunclet$?makeMessage@@YA?AV?$basic_string@DU?$char_traits@D@std@@V?$allocator@D@2@@std@@ABVruntime_error@2@ABUSourceCodePos@@@Z$2 1000d26c f   ErrorHandling.obj
 0001:0000c27c       __ehhandler$?makeMessage@@YA?AV?$basic_string@DU?$char_traits@D@std@@V?$allocator@D@2@@std@@ABVruntime_error@2@ABUSourceCodePos@@@Z 1000d27c f   ErrorHandling.obj
 0001:0000c2a6       __unwindfunclet$?reportError@?A0xd1a094c7@@YAXABUSourceCodePos@@ABV?$basic_string@GU?$char_traits@G@std@@V?$allocator@G@2@@std@@@Z$0 1000d2a6 f   ErrorHandling.obj
 0001:0000c2ae       __unwindfunclet$?reportError@?A0xd1a094c7@@YAXABUSourceCodePos@@ABV?$basic_string@GU?$char_traits@G@std@@V?$allocator@G@2@@std@@@Z$1 1000d2ae f   ErrorHandling.obj
 0001:0000c2b6       __unwindfunclet$?reportError@?A0xd1a094c7@@YAXABUSourceCodePos@@ABV?$basic_string@GU?$char_traits@G@std@@V?$allocator@G@2@@std@@@Z$2 1000d2b6 f   ErrorHandling.obj
 0001:0000c2c3       __ehhandler$?reportError@?A0xd1a094c7@@YAXABUSourceCodePos@@ABV?$basic_string@GU?$char_traits@G@std@@V?$allocator@G@2@@std@@@Z 1000d2c3 f   ErrorHandling.obj
 0001:0000c2ea       __unwindfunclet$?reportError@@YAXABUSourceCodePos@@ABVruntime_error@std@@@Z$0 1000d2ea f   ErrorHandling.obj
 0001:0000c2f5       __unwindfunclet$?reportError@@YAXABUSourceCodePos@@ABVruntime_error@std@@@Z$1 1000d2f5 f   ErrorHandling.obj
 0001:0000c302       __ehhandler$?reportError@@YAXABUSourceCodePos@@ABVruntime_error@std@@@Z 1000d302 f   ErrorHandling.obj
 0001:0000c32c       __unwindfunclet$?reportUnknownError@@YAXABUSourceCodePos@@@Z$0 1000d32c f   ErrorHandling.obj
 0001:0000c32c       __unwindfunclet$?log@Logger@@QBEXW4LogLevel@1@PBGH1ABVany@tstrings@@@Z$0 1000d32c f   Log.obj
 0001:0000c32c       __unwindfunclet$?appendFormatted@LogEvent@@CAXABUPlatformLogEvent@@AAV?$basic_string@GU?$char_traits@G@std@@V?$allocator@G@2@@std@@@Z$0 1000d32c f   PlatformLogEvent.obj
 0001:0000c32c       __unwindfunclet$?initializeLogging@Logger@@CAXXZ$0 1000d32c f   PlatformLogEvent.obj
 0001:0000c32c       __unwindfunclet$??6@YAAAV?$basic_ostream@GU?$char_traits@G@std@@@std@@AAV01@ABVany@tstrings@@@Z$0 1000d32c f   Resources.obj
 0001:0000c339       __ehhandler$?reportUnknownError@@YAXABUSourceCodePos@@@Z 1000d339 f   ErrorHandling.obj
 0001:0000c339       __ehhandler$?log@Logger@@QBEXW4LogLevel@1@PBGH1ABVany@tstrings@@@Z 1000d339 f   Log.obj
 0001:0000c339       __ehhandler$?appendFormatted@LogEvent@@CAXABUPlatformLogEvent@@AAV?$basic_string@GU?$char_traits@G@std@@V?$allocator@G@2@@std@@@Z 1000d339 f   PlatformLogEvent.obj
 0001:0000c339       __ehhandler$?initializeLogging@Logger@@CAXXZ 1000d339 f   PlatformLogEvent.obj
 0001:0000c339       __ehhandler$??6@YAAAV?$basic_ostream@GU?$char_traits@G@std@@@std@@AAV01@ABVany@tstrings@@@Z 1000d339 f   Resources.obj
 0001:0000c360       __unwindfunclet$?str@?$basic_stringbuf@DU?$char_traits@D@std@@V?$allocator@D@2@@std@@QBE?AV?$basic_string@DU?$char_traits@D@std@@V?$allocator@D@2@@2@XZ$0 1000d360 f   ErrorHandling.obj
 0001:0000c37e       __ehhandler$?str@?$basic_stringbuf@DU?$char_traits@D@std@@V?$allocator@D@2@@std@@QBE?AV?$basic_string@DU?$char_traits@D@std@@V?$allocator@D@2@@2@XZ 1000d37e f   ErrorHandling.obj
 0001:0000c39b       __unwindfunclet$?str@?$basic_stringbuf@GU?$char_traits@G@std@@V?$allocator@G@2@@std@@QBE?AV?$basic_string@GU?$char_traits@G@std@@V?$allocator@G@2@@2@XZ$0 1000d39b f   ErrorHandling.obj
 0001:0000c39b       __unwindfunclet$?getSystemMessageDescription@?A0xd5983087@@YA?AV?$basic_string@GU?$char_traits@G@std@@V?$allocator@G@2@@std@@KPAUHINSTANCE__@@@Z$0 1000d39b f   WinErrorHandling.obj
 0001:0000c3b9       __ehhandler$?str@?$basic_stringbuf@GU?$char_traits@G@std@@V?$allocator@G@2@@std@@QBE?AV?$basic_string@GU?$char_traits@G@std@@V?$allocator@G@2@@2@XZ 1000d3b9 f   ErrorHandling.obj
 0001:0000c3b9       __ehhandler$?getSystemMessageDescription@?A0xd5983087@@YA?AV?$basic_string@GU?$char_traits@G@std@@V?$allocator@G@2@@std@@KPAUHINSTANCE__@@@Z 1000d3b9 f   WinErrorHandling.obj
 0001:0000c3d6       __unwindfunclet$?str@any@tstrings@@QBE?AV?$basic_string@DU?$char_traits@D@std@@V?$allocator@D@2@@std@@XZ$0 1000d3d6 f   ErrorHandling.obj
 0001:0000c3d6       __unwindfunclet$?string@StringResource@@QBE?AV?$basic_string@GU?$char_traits@G@std@@V?$allocator@G@2@@std@@XZ$0 1000d3d6 f   Resources.obj
 0001:0000c3e3       __ehhandler$?str@any@tstrings@@QBE?AV?$basic_string@DU?$char_traits@D@std@@V?$allocator@D@2@@std@@XZ 1000d3e3 f   ErrorHandling.obj
 0001:0000c3e3       __ehhandler$?string@StringResource@@QBE?AV?$basic_string@GU?$char_traits@G@std@@V?$allocator@G@2@@std@@XZ 1000d3e3 f   Resources.obj
 0001:0000c40a       __unwindfunclet$?combinePath@FileUtils@@YA?AV?$basic_string@GU?$char_traits@G@std@@V?$allocator@G@2@@std@@ABV23@0@Z$1 1000d40a f   FileUtils.obj
 0001:0000c412       __unwindfunclet$?combinePath@FileUtils@@YA?AV?$basic_string@GU?$char_traits@G@std@@V?$allocator@G@2@@std@@ABV23@0@Z$2 1000d412 f   FileUtils.obj
 0001:0000c42b       __unwindfunclet$?combinePath@FileUtils@@YA?AV?$basic_string@GU?$char_traits@G@std@@V?$allocator@G@2@@std@@ABV23@0@Z$4 1000d42b f   FileUtils.obj
 0001:0000c438       __ehhandler$?combinePath@FileUtils@@YA?AV?$basic_string@GU?$char_traits@G@std@@V?$allocator@G@2@@std@@ABV23@0@Z 1000d438 f   FileUtils.obj
 0001:0000c45f       __unwindfunclet$??0?$JpError@Vruntime_error@std@@@@QAE@ABV0@@Z$0 1000d45f f   Guid.obj
 0001:0000c45f       __unwindfunclet$??0?$JpError@Vruntime_error@std@@@@QAE@ABVruntime_error@std@@ABUSourceCodePos@@@Z$0 1000d45f f   Guid.obj
 0001:0000c45f       __unwindfunclet$??0?$JpError@VError@msi@@@@QAE@ABV0@@Z$0 1000d45f f   MsiDb.obj
 0001:0000c45f       __unwindfunclet$??0?$JpError@VError@msi@@@@QAE@ABVError@msi@@ABUSourceCodePos@@@Z$0 1000d45f f   MsiDb.obj
 0001:0000c45f       __unwindfunclet$??0?$JpError@VNoMoreItemsError@msi@@@@QAE@ABV0@@Z$0 1000d45f f   MsiDb.obj
 0001:0000c45f       __unwindfunclet$??0?$JpError@VNoMoreItemsError@msi@@@@QAE@ABVNoMoreItemsError@msi@@ABUSourceCodePos@@@Z$0 1000d45f f   MsiDb.obj
 0001:0000c45f       __unwindfunclet$??0?$JpError@VSysError@@@@QAE@ABV0@@Z$0 1000d45f f   MsiUtils.obj
 0001:0000c45f       __unwindfunclet$??0?$JpError@VSysError@@@@QAE@ABVSysError@@ABUSourceCodePos@@@Z$0 1000d45f f   MsiUtils.obj
 0001:0000c46f       __ehhandler$??0?$JpError@Vruntime_error@std@@@@QAE@ABV0@@Z 1000d46f f   Guid.obj
 0001:0000c46f       __ehhandler$??0?$JpError@Vruntime_error@std@@@@QAE@ABVruntime_error@std@@ABUSourceCodePos@@@Z 1000d46f f   Guid.obj
 0001:0000c46f       __ehhandler$??0?$JpError@VError@msi@@@@QAE@ABV0@@Z 1000d46f f   MsiDb.obj
 0001:0000c46f       __ehhandler$??0?$JpError@VError@msi@@@@QAE@ABVError@msi@@ABUSourceCodePos@@@Z 1000d46f f   MsiDb.obj
 0001:0000c46f       __ehhandler$??0?$JpError@VNoMoreItemsError@msi@@@@QAE@ABV0@@Z 1000d46f f   MsiDb.obj
 0001:0000c46f       __ehhandler$??0?$JpError@VNoMoreItemsError@msi@@@@QAE@ABVNoMoreItemsError@msi@@ABUSourceCodePos@@@Z 1000d46f f   MsiDb.obj
 0001:0000c46f       __ehhandler$??0?$JpError@VSysError@@@@QAE@ABV0@@Z 1000d46f f   MsiUtils.obj
 0001:0000c46f       __ehhandler$??0?$JpError@VSysError@@@@QAE@ABVSysError@@ABUSourceCodePos@@@Z 1000d46f f   MsiUtils.obj
 0001:0000c48c       __unwindfunclet$??0Guid@@QAE@ABV?$basic_string@GU?$char_traits@G@std@@V?$allocator@G@2@@std@@@Z$0 1000d48c f   Guid.obj
 0001:0000c494       __unwindfunclet$??0Guid@@QAE@ABV?$basic_string@GU?$char_traits@G@std@@V?$allocator@G@2@@std@@@Z$1 1000d494 f   Guid.obj
 0001:0000c4a1       __ehhandler$??0Guid@@QAE@ABV?$basic_string@GU?$char_traits@G@std@@V?$allocator@G@2@@std@@@Z 1000d4a1 f   Guid.obj
 0001:0000c4c8       __unwindfunclet$?initGuid@?A0x2459fff0@@YAXABV?$basic_string@GU?$char_traits@G@std@@V?$allocator@G@2@@std@@AAU_GUID@@@Z$0 1000d4c8 f   Guid.obj
 0001:0000c4c8       __unwindfunclet$??0FixedFileVersion@?A0xcb1fbc16@@QAE@ABV?$basic_string@GU?$char_traits@G@std@@V?$allocator@G@2@@std@@@Z$0 1000d4c8 f   VersionInfo.obj
 0001:0000c4d8       __ehhandler$?initGuid@?A0x2459fff0@@YAXABV?$basic_string@GU?$char_traits@G@std@@V?$allocator@G@2@@std@@AAU_GUID@@@Z 1000d4d8 f   Guid.obj
 0001:0000c4d8       __ehhandler$??0FixedFileVersion@?A0xcb1fbc16@@QAE@ABV?$basic_string@GU?$char_traits@G@std@@V?$allocator@G@2@@std@@@Z 1000d4d8 f   VersionInfo.obj
 0001:0000c502       __unwindfunclet$?makeException@@YA?AV?$JpError@Vruntime_error@std@@@@ABV?$basic_string@DU?$char_traits@D@std@@V?$allocator@D@2@@std@@ABUSourceCodePos@@@Z$0 1000d502 f   Guid.obj
 0001:0000c50f       __ehhandler$?makeException@@YA?AV?$JpError@Vruntime_error@std@@@@ABV?$basic_string@DU?$char_traits@D@std@@V?$allocator@D@2@@std@@ABUSourceCodePos@@@Z 1000d50f f   Guid.obj
 0001:0000c52c       __unwindfunclet$?makeException@@YA?AV?$JpError@Vruntime_error@std@@@@ABVany@tstrings@@ABUSourceCodePos@@@Z$0 1000d52c f   Guid.obj
 0001:0000c52c       __unwindfunclet$?makeException@@YA?AV?$JpError@Vruntime_error@std@@@@PBDABUSourceCodePos@@@Z$0 1000d52c f   Guid.obj
 0001:0000c52c       __unwindfunclet$?getSystem32Dir@SysInfo@@YA?AV?$basic_string@GU?$char_traits@G@std@@V?$allocator@G@2@@std@@XZ$0 1000d52c f   WinSysInfo.obj
 0001:0000c539       __ehhandler$?makeException@@YA?AV?$JpError@Vruntime_error@std@@@@ABVany@tstrings@@ABUSourceCodePos@@@Z 1000d539 f   Guid.obj
 0001:0000c539       __ehhandler$?makeException@@YA?AV?$JpError@Vruntime_error@std@@@@PBDABUSourceCodePos@@@Z 1000d539 f   Guid.obj
 0001:0000c539       __ehhandler$?getSystem32Dir@SysInfo@@YA?AV?$basic_string@GU?$char_traits@G@std@@V?$allocator@G@2@@std@@XZ 1000d539 f   WinSysInfo.obj
 0001:0000c560       __unwindfunclet$?toString@Guid@@QBE?AV?$basic_string@GU?$char_traits@G@std@@V?$allocator@G@2@@std@@H@Z$0 1000d560 f   Guid.obj
 0001:0000c568       __unwindfunclet$?toString@Guid@@QBE?AV?$basic_string@GU?$char_traits@G@std@@V?$allocator@G@2@@std@@H@Z$1 1000d568 f   Guid.obj
 0001:0000c586       __ehhandler$?toString@Guid@@QBE?AV?$basic_string@GU?$char_traits@G@std@@V?$allocator@G@2@@std@@H@Z 1000d586 f   Guid.obj
 0001:0000c5b0       __ehhandler$??1?$AtEndOfScope@V<lambda_bafb2a7f1406751b8a75ac1ff6dad7d1>@@@@QAE@XZ 1000d5b0 f   JniUtils.obj
 0001:0000c5cd       __unwindfunclet$?toUnicodeString@jni@@YA?AV?$basic_string@GU?$char_traits@G@std@@V?$allocator@G@2@@std@@PAUJNIEnv_@@PAV_jstring@@@Z$0 1000d5cd f   JniUtils.obj
 0001:0000c5da       __ehhandler$?toUnicodeString@jni@@YA?AV?$basic_string@GU?$char_traits@G@std@@V?$allocator@G@2@@std@@PAUJNIEnv_@@PAV_jstring@@@Z 1000d5da f   JniUtils.obj
 0001:0000c601       __unwindfunclet$?toUnicodeStringArray@jni@@YA?AV?$vector@V?$basic_string@GU?$char_traits@G@std@@V?$allocator@G@2@@std@@V?$allocator@V?$basic_string@GU?$char_traits@G@std@@V?$allocator@G@2@@std@@@2@@std@@PAUJNIEnv_@@PAV_jobjectArray@@@Z$0 1000d601 f   JniUtils.obj
 0001:0000c61a       __unwindfunclet$?toUnicodeStringArray@jni@@YA?AV?$vector@V?$basic_string@GU?$char_traits@G@std@@V?$allocator@G@2@@std@@V?$allocator@V?$basic_string@GU?$char_traits@G@std@@V?$allocator@G@2@@std@@@2@@std@@PAUJNIEnv_@@PAV_jobjectArray@@@Z$1 1000d61a f   JniUtils.obj
 0001:0000c622       __unwindfunclet$?toUnicodeStringArray@jni@@YA?AV?$vector@V?$basic_string@GU?$char_traits@G@std@@V?$allocator@G@2@@std@@V?$allocator@V?$basic_string@GU?$char_traits@G@std@@V?$allocator@G@2@@std@@@2@@std@@PAUJNIEnv_@@PAV_jobjectArray@@@Z$2 1000d622 f   JniUtils.obj
 0001:0000c62f       __ehhandler$?toUnicodeStringArray@jni@@YA?AV?$vector@V?$basic_string@GU?$char_traits@G@std@@V?$allocator@G@2@@std@@V?$allocator@V?$basic_string@GU?$char_traits@G@std@@V?$allocator@G@2@@std@@@2@@std@@PAUJNIEnv_@@PAV_jobjectArray@@@Z 1000d62f f   JniUtils.obj
 0001:0000c656       __unwindfunclet$??6?$basic_ostream@GU?$char_traits@G@std@@@std@@QAEAAV01@G@Z$2 1000d656 f   Log.obj
 0001:0000c663       __ehhandler$??6?$basic_ostream@GU?$char_traits@G@std@@@std@@QAEAAV01@G@Z 1000d663 f   Log.obj
 0001:0000c680       __unwindfunclet$?append@StreamLogAppender@@UAEXABULogEvent@@@Z$0 1000d680 f   Log.obj
 0001:0000c688       __unwindfunclet$?append@StreamLogAppender@@UAEXABULogEvent@@@Z$1 1000d688 f   Log.obj
 0001:0000c693       __unwindfunclet$?append@StreamLogAppender@@UAEXABULogEvent@@@Z$2 1000d693 f   Log.obj
 0001:0000c69b       __unwindfunclet$?append@StreamLogAppender@@UAEXABULogEvent@@@Z$3 1000d69b f   Log.obj
 0001:0000c6a8       __ehhandler$?append@StreamLogAppender@@UAEXABULogEvent@@@Z 1000d6a8 f   Log.obj
 0001:0000c6d2       __unwindfunclet$?log@Logger@@QBEXW4LogLevel@1@PBGH1ABV?$basic_string@GU?$char_traits@G@std@@V?$allocator@G@2@@std@@@Z$0 1000d6d2 f   Log.obj
 0001:0000c6da       __unwindfunclet$?log@Logger@@QBEXW4LogLevel@1@PBGH1ABV?$basic_string@GU?$char_traits@G@std@@V?$allocator@G@2@@std@@@Z$1 1000d6da f   Log.obj
 0001:0000c6ea       __ehhandler$?log@Logger@@QBEXW4LogLevel@1@PBGH1ABV?$basic_string@GU?$char_traits@G@std@@V?$allocator@G@2@@std@@@Z 1000d6ea f   Log.obj
 0001:0000c714       __unwindfunclet$??0Database@msi@@QAE@ABV?$basic_string@GU?$char_traits@G@std@@V?$allocator@G@2@@std@@@Z$0 1000d714 f   MsiDb.obj
 0001:0000c721       __ehhandler$??0Database@msi@@QAE@ABV?$basic_string@GU?$char_traits@G@std@@V?$allocator@G@2@@std@@@Z 1000d721 f   MsiDb.obj
 0001:0000c73e       __unwindfunclet$??0DatabaseView@msi@@QAE@ABVDatabase@1@ABV?$basic_string@GU?$char_traits@G@std@@V?$allocator@G@2@@std@@ABVDatabaseRecord@1@@Z$0 1000d73e f   MsiDb.obj
 0001:0000c746       __unwindfunclet$??0DatabaseView@msi@@QAE@ABVDatabase@1@ABV?$basic_string@GU?$char_traits@G@std@@V?$allocator@G@2@@std@@ABVDatabaseRecord@1@@Z$3 1000d746 f   MsiDb.obj
 0001:0000c751       __unwindfunclet$??0DatabaseView@msi@@QAE@ABVDatabase@1@ABV?$basic_string@GU?$char_traits@G@std@@V?$allocator@G@2@@std@@ABVDatabaseRecord@1@@Z$4 1000d751 f   MsiDb.obj
 0001:0000c759       __unwindfunclet$??0DatabaseView@msi@@QAE@ABVDatabase@1@ABV?$basic_string@GU?$char_traits@G@std@@V?$allocator@G@2@@std@@ABVDatabaseRecord@1@@Z$1 1000d759 f   MsiDb.obj
 0001:0000c764       __unwindfunclet$??0DatabaseView@msi@@QAE@ABVDatabase@1@ABV?$basic_string@GU?$char_traits@G@std@@V?$allocator@G@2@@std@@ABVDatabaseRecord@1@@Z$2 1000d764 f   MsiDb.obj
 0001:0000c771       __ehhandler$??0DatabaseView@msi@@QAE@ABVDatabase@1@ABV?$basic_string@GU?$char_traits@G@std@@V?$allocator@G@2@@std@@ABVDatabaseRecord@1@@Z 1000d771 f   MsiDb.obj
 0001:0000c79b       __ehhandler$??4DatabaseRecord@msi@@QAEAAV01@ABV01@@Z 1000d79b f   MsiDb.obj
 0001:0000c7b8       __unwindfunclet$?fetch@DatabaseRecord@msi@@QAEAAV12@AAVDatabaseView@2@@Z$0 1000d7b8 f   MsiDb.obj
 0001:0000c7c5       __ehhandler$?fetch@DatabaseRecord@msi@@QAEAAV12@AAVDatabaseView@2@@Z 1000d7c5 f   MsiDb.obj
 0001:0000c7e2       __unwindfunclet$?fetch@DatabaseView@msi@@QAE?AVDatabaseRecord@2@XZ$0 1000d7e2 f   MsiDb.obj
 0001:0000c7fb       __unwindfunclet$?fetch@DatabaseView@msi@@QAE?AVDatabaseRecord@2@XZ$1 1000d7fb f   MsiDb.obj
 0001:0000c806       __unwindfunclet$?fetch@DatabaseView@msi@@QAE?AVDatabaseRecord@2@XZ$2 1000d806 f   MsiDb.obj
 0001:0000c813       __ehhandler$?fetch@DatabaseView@msi@@QAE?AVDatabaseRecord@2@XZ 1000d813 f   MsiDb.obj
 0001:0000c83d       __unwindfunclet$?getFieldCount@DatabaseRecord@msi@@QBEIXZ$0 1000d83d f   MsiDb.obj
 0001:0000c845       __unwindfunclet$?getFieldCount@DatabaseRecord@msi@@QBEIXZ$1 1000d845 f   MsiDb.obj
 0001:0000c852       __ehhandler$?getFieldCount@DatabaseRecord@msi@@QBEIXZ 1000d852 f   MsiDb.obj
 0001:0000c879       __unwindfunclet$?getProperty@Database@msi@@QBE?AV?$basic_string@GU?$char_traits@G@std@@V?$allocator@G@2@@std@@ABV34@@Z$0 1000d879 f   MsiDb.obj
 0001:0000c884       __unwindfunclet$?getProperty@Database@msi@@QBE?AV?$basic_string@GU?$char_traits@G@std@@V?$allocator@G@2@@std@@ABV34@@Z$1 1000d884 f   MsiDb.obj
 0001:0000c88c       __unwindfunclet$?getProperty@Database@msi@@QBE?AV?$basic_string@GU?$char_traits@G@std@@V?$allocator@G@2@@std@@ABV34@@Z$2 1000d88c f   MsiDb.obj
 0001:0000c894       __unwindfunclet$?getProperty@Database@msi@@QBE?AV?$basic_string@GU?$char_traits@G@std@@V?$allocator@G@2@@std@@ABV34@@Z$3 1000d894 f   MsiDb.obj
 0001:0000c89c       __unwindfunclet$?getProperty@Database@msi@@QBE?AV?$basic_string@GU?$char_traits@G@std@@V?$allocator@G@2@@std@@ABV34@@Z$4 1000d89c f   MsiDb.obj
 0001:0000c8a4       __unwindfunclet$?getProperty@Database@msi@@QBE?AV?$basic_string@GU?$char_traits@G@std@@V?$allocator@G@2@@std@@ABV34@@Z$5 1000d8a4 f   MsiDb.obj
 0001:0000c8af       __unwindfunclet$?getProperty@Database@msi@@QBE?AV?$basic_string@GU?$char_traits@G@std@@V?$allocator@G@2@@std@@ABV34@@Z$6 1000d8af f   MsiDb.obj
 0001:0000c8bc       __ehhandler$?getProperty@Database@msi@@QBE?AV?$basic_string@GU?$char_traits@G@std@@V?$allocator@G@2@@std@@ABV34@@Z 1000d8bc f   MsiDb.obj
 0001:0000c8e6       __unwindfunclet$?openDatabase@?A0x6ccb95c8@msi@@YAKABV?$basic_string@GU?$char_traits@G@std@@V?$allocator@G@2@@std@@@Z$0 1000d8e6 f   MsiDb.obj
 0001:0000c8f1       __unwindfunclet$?openDatabase@?A0x6ccb95c8@msi@@YAKABV?$basic_string@GU?$char_traits@G@std@@V?$allocator@G@2@@std@@@Z$1 1000d8f1 f   MsiDb.obj
 0001:0000c8fe       __ehhandler$?openDatabase@?A0x6ccb95c8@msi@@YAKABV?$basic_string@GU?$char_traits@G@std@@V?$allocator@G@2@@std@@@Z 1000d8fe f   MsiDb.obj
 0001:0000c928       __unwindfunclet$?tryFetch@DatabaseView@msi@@QAE?AVDatabaseRecord@2@XZ$1 1000d928 f   MsiDb.obj
 0001:0000c933       __unwindfunclet$?tryFetch@DatabaseView@msi@@QAE?AVDatabaseRecord@2@XZ$2 1000d933 f   MsiDb.obj
 0001:0000c940       __ehhandler$?tryFetch@DatabaseView@msi@@QAE?AVDatabaseRecord@2@XZ 1000d940 f   MsiDb.obj
 0001:0000c96a       __unwindfunclet$?uflow@?$basic_filebuf@DU?$char_traits@D@std@@@std@@MAEHXZ$0 1000d96a f   MsiDb.obj
 0001:0000c977       __ehhandler$?uflow@?$basic_filebuf@DU?$char_traits@D@std@@@std@@MAEHXZ 1000d977 f   MsiDb.obj
 0001:0000c99e       __unwindfunclet$??$?0ABUpiecewise_construct_t@std@@V?$tuple@ABV?$basic_string@GU?$char_traits@G@std@@V?$allocator@G@2@@std@@@1@V?$tuple@$$V@1@@?$_Tree_temp_node@V?$allocator@U?$_Tree_node@U?$pair@$$CBV?$basic_string@GU?$char_traits@G@std@@V?$allocator@G@2@@std@@V12@@std@@PAX@std@@@std@@@std@@QAE@AAV?$allocator@U?$_Tree_node@U?$pair@$$CBV?$basic_string@GU?$char_traits@G@std@@V?$allocator@G@2@@std@@V12@@std@@PAX@std@@@1@PAU?$_Tree_node@U?$pair@$$CBV?$basic_string@GU?$char_traits@G@std@@V?$allocator@G@2@@std@@V12@@std@@PAX@1@ABUpiecewise_construct_t@1@$$QAV?$tuple@ABV?$basic_string@GU?$char_traits@G@std@@V?$allocator@G@2@@std@@@1@$$QAV?$tuple@$$V@1@@Z$0 1000d99e f   MsiUtils.obj
 0001:0000c99e       __unwindfunclet$??0?$_Tree_temp_node_alloc@V?$allocator@U?$_Tree_node@U?$pair@$$CBV?$basic_string@GU?$char_traits@G@std@@V?$allocator@G@2@@std@@V12@@std@@PAX@std@@@std@@@std@@QAE@AAV?$allocator@U?$_Tree_node@U?$pair@$$CBV?$basic_string@GU?$char_traits@G@std@@V?$allocator@G@2@@std@@V12@@std@@PAX@std@@@1@@Z$0 1000d99e f   MsiUtils.obj
 0001:0000c9ab       __ehhandler$??$?0ABUpiecewise_construct_t@std@@V?$tuple@ABV?$basic_string@GU?$char_traits@G@std@@V?$allocator@G@2@@std@@@1@V?$tuple@$$V@1@@?$_Tree_temp_node@V?$allocator@U?$_Tree_node@U?$pair@$$CBV?$basic_string@GU?$char_traits@G@std@@V?$allocator@G@2@@std@@V12@@std@@PAX@std@@@std@@@std@@QAE@AAV?$allocator@U?$_Tree_node@U?$pair@$$CBV?$basic_string@GU?$char_traits@G@std@@V?$allocator@G@2@@std@@V12@@std@@PAX@std@@@1@PAU?$_Tree_node@U?$pair@$$CBV?$basic_string@GU?$char_traits@G@std@@V?$allocator@G@2@@std@@V12@@std@@PAX@1@ABUpiecewise_construct_t@1@$$QAV?$tuple@ABV?$basic_string@GU?$char_traits@G@std@@V?$allocator@G@2@@std@@@1@$$QAV?$tuple@$$V@1@@Z 1000d9ab f   MsiUtils.obj
 0001:0000c9ab       __ehhandler$??0?$_Tree_temp_node_alloc@V?$allocator@U?$_Tree_node@U?$pair@$$CBV?$basic_string@GU?$char_traits@G@std@@V?$allocator@G@2@@std@@V12@@std@@PAX@std@@@std@@@std@@QAE@AAV?$allocator@U?$_Tree_node@U?$pair@$$CBV?$basic_string@GU?$char_traits@G@std@@V?$allocator@G@2@@std@@V12@@std@@PAX@std@@@1@@Z 1000d9ab f   MsiUtils.obj
 0001:0000c9c8       __unwindfunclet$??$getProperty@P6GIKIPAGPAK@ZKI@?A0x0e70828c@msi@@YA?AV?$basic_string@GU?$char_traits@G@std@@V?$allocator@G@2@@std@@P6GIKIPAGPAK@ZQBDKI@Z$0 1000d9c8 f   MsiUtils.obj
 0001:0000c9d0       __unwindfunclet$??$getProperty@P6GIKIPAGPAK@ZKI@?A0x0e70828c@msi@@YA?AV?$basic_string@GU?$char_traits@G@std@@V?$allocator@G@2@@std@@P6GIKIPAGPAK@ZQBDKI@Z$1 1000d9d0 f   MsiUtils.obj
 0001:0000c9db       __unwindfunclet$??$getProperty@P6GIKIPAGPAK@ZKI@?A0x0e70828c@msi@@YA?AV?$basic_string@GU?$char_traits@G@std@@V?$allocator@G@2@@std@@P6GIKIPAGPAK@ZQBDKI@Z$2 1000d9db f   MsiUtils.obj
 0001:0000c9e8       __ehhandler$??$getProperty@P6GIKIPAGPAK@ZKI@?A0x0e70828c@msi@@YA?AV?$basic_string@GU?$char_traits@G@std@@V?$allocator@G@2@@std@@P6GIKIPAGPAK@ZQBDKI@Z 1000d9e8 f   MsiUtils.obj
 0001:0000ca12       __unwindfunclet$??0Error@msi@@QAE@ABVany@tstrings@@I@Z$0 1000da12 f   MsiUtils.obj
 0001:0000ca1f       __ehhandler$??0Error@msi@@QAE@ABVany@tstrings@@I@Z 1000da1f f   MsiUtils.obj
 0001:0000ca46       __unwindfunclet$?closeMSIHANDLE@msi@@YAXK@Z$0 1000da46 f   MsiUtils.obj
 0001:0000ca56       __ehhandler$?closeMSIHANDLE@msi@@YAXK@Z 1000da56 f   MsiUtils.obj
 0001:0000ca76       __unwindfunclet$?makeMessage@?A0x0e70828c@msi@@YA?AV?$basic_string@DU?$char_traits@D@std@@V?$allocator@D@2@@std@@ABV34@I@Z$2 1000da76 f   MsiUtils.obj
 0001:0000ca81       __unwindfunclet$?makeMessage@?A0x0e70828c@msi@@YA?AV?$basic_string@DU?$char_traits@D@std@@V?$allocator@D@2@@std@@ABV34@I@Z$3 1000da81 f   MsiUtils.obj
 0001:0000ca89       __unwindfunclet$?makeMessage@?A0x0e70828c@msi@@YA?AV?$basic_string@DU?$char_traits@D@std@@V?$allocator@D@2@@std@@ABV34@I@Z$4 1000da89 f   MsiUtils.obj
 0001:0000ca91       __unwindfunclet$?makeMessage@?A0x0e70828c@msi@@YA?AV?$basic_string@DU?$char_traits@D@std@@V?$allocator@D@2@@std@@ABV34@I@Z$5 1000da91 f   MsiUtils.obj
 0001:0000ca9c       __unwindfunclet$?makeMessage@?A0x0e70828c@msi@@YA?AV?$basic_string@DU?$char_traits@D@std@@V?$allocator@D@2@@std@@ABV34@I@Z$6 1000da9c f   MsiUtils.obj
 0001:0000caa4       __unwindfunclet$?makeMessage@?A0x0e70828c@msi@@YA?AV?$basic_string@DU?$char_traits@D@std@@V?$allocator@D@2@@std@@ABV34@I@Z$7 1000daa4 f   MsiUtils.obj
 0001:0000caaf       __unwindfunclet$?makeMessage@?A0x0e70828c@msi@@YA?AV?$basic_string@DU?$char_traits@D@std@@V?$allocator@D@2@@std@@ABV34@I@Z$10 1000daaf f   MsiUtils.obj
 0001:0000cab7       __unwindfunclet$?makeMessage@?A0x0e70828c@msi@@YA?AV?$basic_string@DU?$char_traits@D@std@@V?$allocator@D@2@@std@@ABV34@I@Z$11 1000dab7 f   MsiUtils.obj
 0001:0000cac2       __unwindfunclet$?makeMessage@?A0x0e70828c@msi@@YA?AV?$basic_string@DU?$char_traits@D@std@@V?$allocator@D@2@@std@@ABV34@I@Z$29 1000dac2 f   MsiUtils.obj
 0001:0000cacd       __unwindfunclet$?makeMessage@?A0x0e70828c@msi@@YA?AV?$basic_string@DU?$char_traits@D@std@@V?$allocator@D@2@@std@@ABV34@I@Z$13 1000dacd f   MsiUtils.obj
 0001:0000cad8       __unwindfunclet$?makeMessage@?A0x0e70828c@msi@@YA?AV?$basic_string@DU?$char_traits@D@std@@V?$allocator@D@2@@std@@ABV34@I@Z$14 1000dad8 f   MsiUtils.obj
 0001:0000cae0       __unwindfunclet$?makeMessage@?A0x0e70828c@msi@@YA?AV?$basic_string@DU?$char_traits@D@std@@V?$allocator@D@2@@std@@ABV34@I@Z$8 1000dae0 f   MsiUtils.obj
 0001:0000caeb       __unwindfunclet$?makeMessage@?A0x0e70828c@msi@@YA?AV?$basic_string@DU?$char_traits@D@std@@V?$allocator@D@2@@std@@ABV34@I@Z$9 1000daeb f   MsiUtils.obj
 0001:0000caf8       __ehhandler$?makeMessage@?A0x0e70828c@msi@@YA?AV?$basic_string@DU?$char_traits@D@std@@V?$allocator@D@2@@std@@ABV34@I@Z 1000daf8 f   MsiUtils.obj
 0001:0000cb22       __unwindfunclet$?retrieveModuleName@?A0x40e1fcfd@@YA?AV?$basic_string@GU?$char_traits@G@std@@V?$allocator@G@2@@std@@XZ$2 1000db22 f   PlatformLogEvent.obj
 0001:0000cb2f       __ehhandler$?retrieveModuleName@?A0x40e1fcfd@@YA?AV?$basic_string@GU?$char_traits@G@std@@V?$allocator@G@2@@std@@XZ 1000db2f f   PlatformLogEvent.obj
 0001:0000cb56       __unwindfunclet$??$_Range_construct_or_tidy@V?$istreambuf_iterator@DU?$char_traits@D@std@@@std@@@?$vector@EV?$allocator@E@std@@@std@@AAEXV?$istreambuf_iterator@DU?$char_traits@D@std@@@1@0Uinput_iterator_tag@1@@Z$0 1000db56 f   ResourceEditor.obj
 0001:0000cb63       __ehhandler$??$_Range_construct_or_tidy@V?$istreambuf_iterator@DU?$char_traits@D@std@@@std@@@?$vector@EV?$allocator@E@std@@@std@@AAEXV?$istreambuf_iterator@DU?$char_traits@D@std@@@1@0Uinput_iterator_tag@1@@Z 1000db63 f   ResourceEditor.obj
 0001:0000cb80       __unwindfunclet$??0?$basic_filebuf@DU?$char_traits@D@std@@@std@@QAE@XZ$0 1000db80 f   ResourceEditor.obj
 0001:0000cb80       __unwindfunclet$??0?$basic_stringbuf@DU?$char_traits@D@std@@V?$allocator@D@2@@std@@QAE@ABV?$basic_string@DU?$char_traits@D@std@@V?$allocator@D@2@@1@H@Z$0 1000db80 f   jpackage.obj
 0001:0000cb8e       __ehhandler$??0?$basic_filebuf@DU?$char_traits@D@std@@@std@@QAE@XZ 1000db8e f   ResourceEditor.obj
 0001:0000cb8e       __ehhandler$??0?$basic_stringbuf@DU?$char_traits@D@std@@V?$allocator@D@2@@std@@QAE@ABV?$basic_string@DU?$char_traits@D@std@@V?$allocator@D@2@@1@H@Z 1000db8e f   jpackage.obj
 0001:0000cbab       __unwindfunclet$??0?$basic_ifstream@DU?$char_traits@D@std@@@std@@QAE@PBGHH@Z$0 1000dbab f   ResourceEditor.obj
 0001:0000cbc8       __unwindfunclet$??0?$basic_ifstream@DU?$char_traits@D@std@@@std@@QAE@PBGHH@Z$1 1000dbc8 f   ResourceEditor.obj
 0001:0000cbd4       __unwindfunclet$??0?$basic_ifstream@DU?$char_traits@D@std@@@std@@QAE@PBGHH@Z$2 1000dbd4 f   ResourceEditor.obj
 0001:0000cbe4       __ehhandler$??0?$basic_ifstream@DU?$char_traits@D@std@@@std@@QAE@PBGHH@Z 1000dbe4 f   ResourceEditor.obj
 0001:0000cc01       __unwindfunclet$??0FileLock@ResourceEditor@@QAE@ABV?$basic_string@GU?$char_traits@G@std@@V?$allocator@G@2@@std@@@Z$0 1000dc01 f   ResourceEditor.obj
 0001:0000cc0c       __unwindfunclet$??0FileLock@ResourceEditor@@QAE@ABV?$basic_string@GU?$char_traits@G@std@@V?$allocator@G@2@@std@@@Z$1 1000dc0c f   ResourceEditor.obj
 0001:0000cc19       __ehhandler$??0FileLock@ResourceEditor@@QAE@ABV?$basic_string@GU?$char_traits@G@std@@V?$allocator@G@2@@std@@@Z 1000dc19 f   ResourceEditor.obj
 0001:0000cc43       __unwindfunclet$??0ResourceEditor@@QAE@XZ$0 1000dc43 f   ResourceEditor.obj
 0001:0000cc4e       __unwindfunclet$??0ResourceEditor@@QAE@XZ$1 1000dc4e f   ResourceEditor.obj
 0001:0000cc5e       __ehhandler$??0ResourceEditor@@QAE@XZ 1000dc5e f   ResourceEditor.obj
 0001:0000cc7b       __unwindfunclet$??0any@tstrings@@QAE@PBD@Z$0 1000dc7b f   ResourceEditor.obj
 0001:0000cc83       __unwindfunclet$??0any@tstrings@@QAE@PBD@Z$1 1000dc83 f   ResourceEditor.obj
 0001:0000cc8b       __unwindfunclet$??0any@tstrings@@QAE@PBD@Z$2 1000dc8b f   ResourceEditor.obj
 0001:0000cc98       __ehhandler$??0any@tstrings@@QAE@PBD@Z 1000dc98 f   ResourceEditor.obj
 0001:0000ccbf       __unwindfunclet$??1FileLock@ResourceEditor@@QAE@XZ$3 1000dcbf f   ResourceEditor.obj
 0001:0000ccca       __unwindfunclet$??1FileLock@ResourceEditor@@QAE@XZ$4 1000dcca f   ResourceEditor.obj
 0001:0000ccd7       __ehhandler$??1FileLock@ResourceEditor@@QAE@XZ 1000dcd7 f   ResourceEditor.obj
 0001:0000cd01       __unwindfunclet$?apply@ResourceEditor@@QAEAAV1@ABVFileLock@1@AAV?$basic_istream@DU?$char_traits@D@std@@@std@@_J@Z$0 1000dd01 f   ResourceEditor.obj
 0001:0000cd09       __unwindfunclet$?apply@ResourceEditor@@QAEAAV1@ABVFileLock@1@AAV?$basic_istream@DU?$char_traits@D@std@@@std@@_J@Z$2 1000dd09 f   ResourceEditor.obj
 0001:0000cd14       __unwindfunclet$?apply@ResourceEditor@@QAEAAV1@ABVFileLock@1@AAV?$basic_istream@DU?$char_traits@D@std@@@std@@_J@Z$3 1000dd14 f   ResourceEditor.obj
 0001:0000cd21       __ehhandler$?apply@ResourceEditor@@QAEAAV1@ABVFileLock@1@AAV?$basic_istream@DU?$char_traits@D@std@@@std@@_J@Z 1000dd21 f   ResourceEditor.obj
 0001:0000cd4b       __unwindfunclet$?apply@ResourceEditor@@QAEAAV1@ABVFileLock@1@ABV?$basic_string@GU?$char_traits@G@std@@V?$allocator@G@2@@std@@@Z$0 1000dd4b f   ResourceEditor.obj
 0001:0000cd5b       __ehhandler$?apply@ResourceEditor@@QAEAAV1@ABVFileLock@1@ABV?$basic_string@GU?$char_traits@G@std@@V?$allocator@G@2@@std@@@Z 1000dd5b f   ResourceEditor.obj
 0001:0000cd7b       __unwindfunclet$?id@ResourceEditor@@QAEAAV1@PBG@Z$0 1000dd7b f   ResourceEditor.obj
 0001:0000cd7b       __unwindfunclet$?type@ResourceEditor@@QAEAAV1@PBG@Z$0 1000dd7b f   ResourceEditor.obj
 0001:0000cd8b       __ehhandler$?id@ResourceEditor@@QAEAAV1@PBG@Z 1000dd8b f   ResourceEditor.obj
 0001:0000cd8b       __ehhandler$?type@ResourceEditor@@QAEAAV1@PBG@Z 1000dd8b f   ResourceEditor.obj
 0001:0000cdb5       __unwindfunclet$?open@?$basic_filebuf@DU?$char_traits@D@std@@@std@@QAEPAV12@PBGHH@Z$0 1000ddb5 f   ResourceEditor.obj
 0001:0000cdc2       __ehhandler$?open@?$basic_filebuf@DU?$char_traits@D@std@@@std@@QAEPAV12@PBGHH@Z 1000ddc2 f   ResourceEditor.obj
 0001:0000cddf       __unwindfunclet$??$?6V?$basic_string@DU?$char_traits@D@std@@V?$allocator@D@2@@std@@@any@tstrings@@QAEAAV01@V?$basic_string@DU?$char_traits@D@std@@V?$allocator@D@2@@std@@@Z$0 1000dddf f   Resources.obj
 0001:0000cde7       __unwindfunclet$??$?6V?$basic_string@DU?$char_traits@D@std@@V?$allocator@D@2@@std@@@any@tstrings@@QAEAAV01@V?$basic_string@DU?$char_traits@D@std@@V?$allocator@D@2@@std@@@Z$1 1000dde7 f   Resources.obj
 0001:0000cdf7       __ehhandler$??$?6V?$basic_string@DU?$char_traits@D@std@@V?$allocator@D@2@@std@@@any@tstrings@@QAEAAV01@V?$basic_string@DU?$char_traits@D@std@@V?$allocator@D@2@@std@@@Z 1000ddf7 f   Resources.obj
 0001:0000ce17       __unwindfunclet$??0Resource@@QAE@IPBGPAUHINSTANCE__@@@Z$0 1000de17 f   Resources.obj
 0001:0000ce1f       __unwindfunclet$??0Resource@@QAE@IPBGPAUHINSTANCE__@@@Z$1 1000de1f f   Resources.obj
 0001:0000ce2f       __ehhandler$??0Resource@@QAE@IPBGPAUHINSTANCE__@@@Z 1000de2f f   Resources.obj
 0001:0000ce4c       __unwindfunclet$??0any@tstrings@@QAE@ABV?$basic_string@DU?$char_traits@D@std@@V?$allocator@D@2@@std@@@Z$0 1000de4c f   Resources.obj
 0001:0000ce54       __unwindfunclet$??0any@tstrings@@QAE@ABV?$basic_string@DU?$char_traits@D@std@@V?$allocator@D@2@@std@@@Z$1 1000de54 f   Resources.obj
 0001:0000ce61       __ehhandler$??0any@tstrings@@QAE@ABV?$basic_string@DU?$char_traits@D@std@@V?$allocator@D@2@@std@@@Z 1000de61 f   Resources.obj
 0001:0000ce88       __unwindfunclet$?getErrMsg@Resource@@ABE?AV?$basic_string@DU?$char_traits@D@std@@V?$allocator@D@2@@std@@ABV23@@Z$0 1000de88 f   Resources.obj
 0001:0000ce90       __unwindfunclet$?getErrMsg@Resource@@ABE?AV?$basic_string@DU?$char_traits@D@std@@V?$allocator@D@2@@std@@ABV23@@Z$1 1000de90 f   Resources.obj
 0001:0000cea0       __ehhandler$?getErrMsg@Resource@@ABE?AV?$basic_string@DU?$char_traits@D@std@@V?$allocator@D@2@@std@@ABV23@@Z 1000dea0 f   Resources.obj
 0001:0000cec0       __unwindfunclet$?getPtr@Resource@@ABEPAXAAK@Z$4 1000dec0 f   Resources.obj
 0001:0000cec8       __unwindfunclet$?getPtr@Resource@@ABEPAXAAK@Z$5 1000dec8 f   Resources.obj
 0001:0000ced0       __unwindfunclet$?getPtr@Resource@@ABEPAXAAK@Z$6 1000ded0 f   Resources.obj
 0001:0000cedb       __unwindfunclet$?getPtr@Resource@@ABEPAXAAK@Z$7 1000dedb f   Resources.obj
 0001:0000cee6       __unwindfunclet$?getPtr@Resource@@ABEPAXAAK@Z$0 1000dee6 f   Resources.obj
 0001:0000ceee       __unwindfunclet$?getPtr@Resource@@ABEPAXAAK@Z$1 1000deee f   Resources.obj
 0001:0000cef6       __unwindfunclet$?getPtr@Resource@@ABEPAXAAK@Z$2 1000def6 f   Resources.obj
 0001:0000cf01       __unwindfunclet$?getPtr@Resource@@ABEPAXAAK@Z$3 1000df01 f   Resources.obj
 0001:0000cf0e       __ehhandler$?getPtr@Resource@@ABEPAXAAK@Z 1000df0e f   Resources.obj
 0001:0000cf38       __unwindfunclet$?init@Resource@@AAEXPBG0PAUHINSTANCE__@@@Z$0 1000df38 f   Resources.obj
 0001:0000cf43       __unwindfunclet$?init@Resource@@AAEXPBG0PAUHINSTANCE__@@@Z$2 1000df43 f   Resources.obj
 0001:0000cf53       __ehhandler$?init@Resource@@AAEXPBG0PAUHINSTANCE__@@@Z 1000df53 f   Resources.obj
 0001:0000cf7d       __unwindfunclet$??$for_each@V?$_Tree_const_iterator@V?$_Tree_val@U?$_Tree_simple_types@U?$pair@$$CBV?$basic_string@GU?$char_traits@G@std@@V?$allocator@G@2@@std@@V12@@std@@@std@@@std@@@std@@V<lambda_fa730d0a4b0afd944df9b292ec615b4b>@@@std@@YA?AV<lambda_fa730d0a4b0afd944df9b292ec615b4b>@@V?$_Tree_const_iterator@V?$_Tree_val@U?$_Tree_simple_types@U?$pair@$$CBV?$basic_string@GU?$char_traits@G@std@@V?$allocator@G@2@@std@@V12@@std@@@std@@@std@@@0@0V1@@Z$0 1000df7d f   VersionInfo.obj
 0001:0000cf8a       __ehhandler$??$for_each@V?$_Tree_const_iterator@V?$_Tree_val@U?$_Tree_simple_types@U?$pair@$$CBV?$basic_string@GU?$char_traits@G@std@@V?$allocator@G@2@@std@@V12@@std@@@std@@@std@@@std@@V<lambda_fa730d0a4b0afd944df9b292ec615b4b>@@@std@@YA?AV<lambda_fa730d0a4b0afd944df9b292ec615b4b>@@V?$_Tree_const_iterator@V?$_Tree_val@U?$_Tree_simple_types@U?$pair@$$CBV?$basic_string@GU?$char_traits@G@std@@V?$allocator@G@2@@std@@V12@@std@@@std@@@std@@@0@0V1@@Z 1000df8a f   VersionInfo.obj
 0001:0000cfa7       __unwindfunclet$??0?$basic_stringstream@DU?$char_traits@D@std@@V?$allocator@D@2@@std@@QAE@H@Z$0 1000dfa7 f   VersionInfo.obj
 0001:0000cfc4       __unwindfunclet$??0?$basic_stringstream@DU?$char_traits@D@std@@V?$allocator@D@2@@std@@QAE@H@Z$1 1000dfc4 f   VersionInfo.obj
 0001:0000cfd5       __ehhandler$??0?$basic_stringstream@DU?$char_traits@D@std@@V?$allocator@D@2@@std@@QAE@H@Z 1000dfd5 f   VersionInfo.obj
 0001:0000cff2       __unwindfunclet$??0?$basic_stringstream@GU?$char_traits@G@std@@V?$allocator@G@2@@std@@QAE@XZ$0 1000dff2 f   VersionInfo.obj
 0001:0000d00f       __unwindfunclet$??0?$basic_stringstream@GU?$char_traits@G@std@@V?$allocator@G@2@@std@@QAE@XZ$1 1000e00f f   VersionInfo.obj
 0001:0000d020       __ehhandler$??0?$basic_stringstream@GU?$char_traits@G@std@@V?$allocator@G@2@@std@@QAE@XZ 1000e020 f   VersionInfo.obj
 0001:0000d03d       __ehhandler$??1StreamSize@?A0xcb1fbc16@@QAE@XZ 1000e03d f   VersionInfo.obj
 0001:0000d064       __unwindfunclet$?apply@VersionInfo@@QBEABV1@ABVFileLock@ResourceEditor@@@Z$1 1000e064 f   VersionInfo.obj
 0001:0000d06f       __unwindfunclet$?apply@VersionInfo@@QBEABV1@ABVFileLock@ResourceEditor@@@Z$2 1000e06f f   VersionInfo.obj
 0001:0000d07c       __ehhandler$?apply@VersionInfo@@QBEABV1@ABVFileLock@ResourceEditor@@@Z 1000e07c f   VersionInfo.obj
 0001:0000d0a9       __unwindfunclet$?createFIXEDFILEINFO@VersionInfo@@ABE?AUtagVS_FIXEDFILEINFO@@XZ$2 1000e0a9 f   VersionInfo.obj
 0001:0000d0b6       __ehhandler$?createFIXEDFILEINFO@VersionInfo@@ABE?AUtagVS_FIXEDFILEINFO@@XZ 1000e0b6 f   VersionInfo.obj
 0001:0000d0dd       __unwindfunclet$?fillBuffer@VersionInfo@@ABEXAAV?$basic_ostream@DU?$char_traits@D@std@@@std@@@Z$0 1000e0dd f   VersionInfo.obj
 0001:0000d0e8       __unwindfunclet$?fillBuffer@VersionInfo@@ABEXAAV?$basic_ostream@DU?$char_traits@D@std@@@std@@@Z$1 1000e0e8 f   VersionInfo.obj
 0001:0000d0f0       __unwindfunclet$?fillBuffer@VersionInfo@@ABEXAAV?$basic_ostream@DU?$char_traits@D@std@@@std@@@Z$2 1000e0f0 f   VersionInfo.obj
 0001:0000d0f8       __unwindfunclet$?fillBuffer@VersionInfo@@ABEXAAV?$basic_ostream@DU?$char_traits@D@std@@@std@@@Z$3 1000e0f8 f   VersionInfo.obj
 0001:0000d100       __unwindfunclet$?fillBuffer@VersionInfo@@ABEXAAV?$basic_ostream@DU?$char_traits@D@std@@@std@@@Z$4 1000e100 f   VersionInfo.obj
 0001:0000d108       __unwindfunclet$?fillBuffer@VersionInfo@@ABEXAAV?$basic_ostream@DU?$char_traits@D@std@@@std@@@Z$5 1000e108 f   VersionInfo.obj
 0001:0000d113       __unwindfunclet$?fillBuffer@VersionInfo@@ABEXAAV?$basic_ostream@DU?$char_traits@D@std@@@std@@@Z$6 1000e113 f   VersionInfo.obj
 0001:0000d11b       __unwindfunclet$?fillBuffer@VersionInfo@@ABEXAAV?$basic_ostream@DU?$char_traits@D@std@@@std@@@Z$7 1000e11b f   VersionInfo.obj
 0001:0000d123       __unwindfunclet$?fillBuffer@VersionInfo@@ABEXAAV?$basic_ostream@DU?$char_traits@D@std@@@std@@@Z$8 1000e123 f   VersionInfo.obj
 0001:0000d12b       __unwindfunclet$?fillBuffer@VersionInfo@@ABEXAAV?$basic_ostream@DU?$char_traits@D@std@@@std@@@Z$9 1000e12b f   VersionInfo.obj
 0001:0000d133       __unwindfunclet$?fillBuffer@VersionInfo@@ABEXAAV?$basic_ostream@DU?$char_traits@D@std@@@std@@@Z$10 1000e133 f   VersionInfo.obj
 0001:0000d140       __ehhandler$?fillBuffer@VersionInfo@@ABEXAAV?$basic_ostream@DU?$char_traits@D@std@@@std@@@Z 1000e140 f   VersionInfo.obj
 0001:0000d16a       __unwindfunclet$??0SysError@@QAE@ABVany@tstrings@@PBXKPBD@Z$0 1000e16a f   WinErrorHandling.obj
 0001:0000d177       __ehhandler$??0SysError@@QAE@ABVany@tstrings@@PBXKPBD@Z 1000e177 f   WinErrorHandling.obj
 0001:0000d19e       __unwindfunclet$?getSysErrorMessage@SysError@@SA?AV?$basic_string@GU?$char_traits@G@std@@V?$allocator@G@2@@std@@KPAUHINSTANCE__@@@Z$0 1000e19e f   WinErrorHandling.obj
 0001:0000d1a9       __unwindfunclet$?getSysErrorMessage@SysError@@SA?AV?$basic_string@GU?$char_traits@G@std@@V?$allocator@G@2@@std@@KPAUHINSTANCE__@@@Z$1 1000e1a9 f   WinErrorHandling.obj
 0001:0000d1b6       __ehhandler$?getSysErrorMessage@SysError@@SA?AV?$basic_string@GU?$char_traits@G@std@@V?$allocator@G@2@@std@@KPAUHINSTANCE__@@@Z 1000e1b6 f   WinErrorHandling.obj
 0001:0000d1e0       __unwindfunclet$?makeMessage@?A0xd5983087@@YA?AV?$basic_string@DU?$char_traits@D@std@@V?$allocator@D@2@@std@@ABV23@PBDPBXK@Z$0 1000e1e0 f   WinErrorHandling.obj
 0001:0000d1eb       __unwindfunclet$?makeMessage@?A0xd5983087@@YA?AV?$basic_string@DU?$char_traits@D@std@@V?$allocator@D@2@@std@@ABV23@PBDPBXK@Z$1 1000e1eb f   WinErrorHandling.obj
 0001:0000d1f6       __unwindfunclet$?makeMessage@?A0xd5983087@@YA?AV?$basic_string@DU?$char_traits@D@std@@V?$allocator@D@2@@std@@ABV23@PBDPBXK@Z$2 1000e1f6 f   WinErrorHandling.obj
 0001:0000d1fe       __unwindfunclet$?makeMessage@?A0xd5983087@@YA?AV?$basic_string@DU?$char_traits@D@std@@V?$allocator@D@2@@std@@ABV23@PBDPBXK@Z$3 1000e1fe f   WinErrorHandling.obj
 0001:0000d209       __unwindfunclet$?makeMessage@?A0xd5983087@@YA?AV?$basic_string@DU?$char_traits@D@std@@V?$allocator@D@2@@std@@ABV23@PBDPBXK@Z$4 1000e209 f   WinErrorHandling.obj
 0001:0000d216       __ehhandler$?makeMessage@?A0xd5983087@@YA?AV?$basic_string@DU?$char_traits@D@std@@V?$allocator@D@2@@std@@ABV23@PBDPBXK@Z 1000e216 f   WinErrorHandling.obj
 0001:0000d240       __unwindfunclet$??$getSystemDirImpl@P6GIPAGI@Z@?A0x7970c2a6@SysInfo@@YA?AV?$basic_string@GU?$char_traits@G@std@@V?$allocator@G@2@@std@@P6GIPAGI@ZABV?$basic_string@DU?$char_traits@D@std@@V?$allocator@D@2@@3@@Z$0 1000e240 f   WinSysInfo.obj
 0001:0000d248       __unwindfunclet$??$getSystemDirImpl@P6GIPAGI@Z@?A0x7970c2a6@SysInfo@@YA?AV?$basic_string@GU?$char_traits@G@std@@V?$allocator@G@2@@std@@P6GIPAGI@ZABV?$basic_string@DU?$char_traits@D@std@@V?$allocator@D@2@@3@@Z$4 1000e248 f   WinSysInfo.obj
 0001:0000d250       __unwindfunclet$??$getSystemDirImpl@P6GIPAGI@Z@?A0x7970c2a6@SysInfo@@YA?AV?$basic_string@GU?$char_traits@G@std@@V?$allocator@G@2@@std@@P6GIPAGI@ZABV?$basic_string@DU?$char_traits@D@std@@V?$allocator@D@2@@3@@Z$1 1000e250 f   WinSysInfo.obj
 0001:0000d258       __unwindfunclet$??$getSystemDirImpl@P6GIPAGI@Z@?A0x7970c2a6@SysInfo@@YA?AV?$basic_string@GU?$char_traits@G@std@@V?$allocator@G@2@@std@@P6GIPAGI@ZABV?$basic_string@DU?$char_traits@D@std@@V?$allocator@D@2@@3@@Z$2 1000e258 f   WinSysInfo.obj
 0001:0000d263       __unwindfunclet$??$getSystemDirImpl@P6GIPAGI@Z@?A0x7970c2a6@SysInfo@@YA?AV?$basic_string@GU?$char_traits@G@std@@V?$allocator@G@2@@std@@P6GIPAGI@ZABV?$basic_string@DU?$char_traits@D@std@@V?$allocator@D@2@@3@@Z$3 1000e263 f   WinSysInfo.obj
 0001:0000d26b       __unwindfunclet$??$getSystemDirImpl@P6GIPAGI@Z@?A0x7970c2a6@SysInfo@@YA?AV?$basic_string@GU?$char_traits@G@std@@V?$allocator@G@2@@std@@P6GIPAGI@ZABV?$basic_string@DU?$char_traits@D@std@@V?$allocator@D@2@@3@@Z$6 1000e26b f   WinSysInfo.obj
 0001:0000d278       __ehhandler$??$getSystemDirImpl@P6GIPAGI@Z@?A0x7970c2a6@SysInfo@@YA?AV?$basic_string@GU?$char_traits@G@std@@V?$allocator@G@2@@std@@P6GIPAGI@ZABV?$basic_string@DU?$char_traits@D@std@@V?$allocator@D@2@@3@@Z 1000e278 f   WinSysInfo.obj
 0001:0000d2a2       __unwindfunclet$?getCurrentModuleHandle@SysInfo@@YAPAUHINSTANCE__@@XZ$0 1000e2a2 f   WinSysInfo.obj
 0001:0000d2ad       __unwindfunclet$?getCurrentModuleHandle@SysInfo@@YAPAUHINSTANCE__@@XZ$1 1000e2ad f   WinSysInfo.obj
 0001:0000d2ba       __ehhandler$?getCurrentModuleHandle@SysInfo@@YAPAUHINSTANCE__@@XZ 1000e2ba f   WinSysInfo.obj
 0001:0000d2e4       __unwindfunclet$?getModulePath@?A0x7970c2a6@SysInfo@@YA?AV?$basic_string@GU?$char_traits@G@std@@V?$allocator@G@2@@std@@PAUHINSTANCE__@@@Z$0 1000e2e4 f   WinSysInfo.obj
 0001:0000d2ec       __unwindfunclet$?getModulePath@?A0x7970c2a6@SysInfo@@YA?AV?$basic_string@GU?$char_traits@G@std@@V?$allocator@G@2@@std@@PAUHINSTANCE__@@@Z$1 1000e2ec f   WinSysInfo.obj
 0001:0000d2f7       __unwindfunclet$?getModulePath@?A0x7970c2a6@SysInfo@@YA?AV?$basic_string@GU?$char_traits@G@std@@V?$allocator@G@2@@std@@PAUHINSTANCE__@@@Z$2 1000e2f7 f   WinSysInfo.obj
 0001:0000d304       __ehhandler$?getModulePath@?A0x7970c2a6@SysInfo@@YA?AV?$basic_string@GU?$char_traits@G@std@@V?$allocator@G@2@@std@@PAUHINSTANCE__@@@Z 1000e304 f   WinSysInfo.obj
 0001:0000d32e       __unwindfunclet$?GetLongPath@?A0x764c93a3@@YA?AV?$basic_string@GU?$char_traits@G@std@@V?$allocator@G@2@@std@@ABV23@@Z$0 1000e32e f   WindowsRegistry.obj
 0001:0000d336       __unwindfunclet$?GetLongPath@?A0x764c93a3@@YA?AV?$basic_string@GU?$char_traits@G@std@@V?$allocator@G@2@@std@@ABV23@@Z$2 1000e336 f   WindowsRegistry.obj
 0001:0000d343       __ehhandler$?GetLongPath@?A0x764c93a3@@YA?AV?$basic_string@GU?$char_traits@G@std@@V?$allocator@G@2@@std@@ABV23@@Z 1000e343 f   WindowsRegistry.obj
 0001:0000d36a       __unwindfunclet$_Java_jdk_jpackage_internal_WindowsRegistry_comparePaths@16$3 1000e36a f   WindowsRegistry.obj
 0001:0000d372       __unwindfunclet$_Java_jdk_jpackage_internal_WindowsRegistry_comparePaths@16$4 1000e372 f   WindowsRegistry.obj
 0001:0000d37f       __ehhandler$_Java_jdk_jpackage_internal_WindowsRegistry_comparePaths@16 1000e37f f   WindowsRegistry.obj
 0001:0000d3a6       __unwindfunclet$_Java_jdk_jpackage_internal_WindowsRegistry_enumRegistryValue@20$3 1000e3a6 f   WindowsRegistry.obj
 0001:0000d3b3       __ehhandler$_Java_jdk_jpackage_internal_WindowsRegistry_enumRegistryValue@20 1000e3b3 f   WindowsRegistry.obj
 0001:0000d3dd       __ehhandler$_Java_jdk_jpackage_internal_WindowsRegistry_openRegistryKey@16 1000e3dd f   WindowsRegistry.obj
 0001:0000d404       __unwindfunclet$_Java_jdk_jpackage_internal_WindowsRegistry_readDwordValue@24$3 1000e404 f   WindowsRegistry.obj
 0001:0000d411       __ehhandler$_Java_jdk_jpackage_internal_WindowsRegistry_readDwordValue@24 1000e411 f   WindowsRegistry.obj
 0001:0000d43b       __unwindfunclet$?append@StandardLogAppender@?A0xd3578678@@UAEXABULogEvent@@@Z$0 1000e43b f   app.obj
 0001:0000d446       __unwindfunclet$?append@StandardLogAppender@?A0xd3578678@@UAEXABULogEvent@@@Z$1 1000e446 f   app.obj
 0001:0000d451       __unwindfunclet$?append@StandardLogAppender@?A0xd3578678@@UAEXABULogEvent@@@Z$2 1000e451 f   app.obj
 0001:0000d461       __ehhandler$?append@StandardLogAppender@?A0xd3578678@@UAEXABULogEvent@@@Z 1000e461 f   app.obj
 0001:0000d481       __unwindfunclet$??0?$basic_istringstream@DU?$char_traits@D@std@@V?$allocator@D@2@@std@@QAE@ABV?$basic_string@DU?$char_traits@D@std@@V?$allocator@D@2@@1@H@Z$0 1000e481 f   jpackage.obj
 0001:0000d49e       __unwindfunclet$??0?$basic_istringstream@DU?$char_traits@D@std@@V?$allocator@D@2@@std@@QAE@ABV?$basic_string@DU?$char_traits@D@std@@V?$allocator@D@2@@1@H@Z$1 1000e49e f   jpackage.obj
 0001:0000d4af       __ehhandler$??0?$basic_istringstream@DU?$char_traits@D@std@@V?$allocator@D@2@@std@@QAE@ABV?$basic_string@DU?$char_traits@D@std@@V?$allocator@D@2@@1@H@Z 1000e4af f   jpackage.obj
 0001:0000d4cc       __unwindfunclet$_Java_jdk_jpackage_internal_ExecutableRebrander_iconSwap@20$3 1000e4cc f   jpackage.obj
 0001:0000d4d4       __unwindfunclet$_Java_jdk_jpackage_internal_ExecutableRebrander_iconSwap@20$4 1000e4d4 f   jpackage.obj
 0001:0000d4e1       __ehhandler$_Java_jdk_jpackage_internal_ExecutableRebrander_iconSwap@20 1000e4e1 f   jpackage.obj
 0001:0000d508       __unwindfunclet$_Java_jdk_jpackage_internal_ExecutableRebrander_lockResource@12$3 1000e508 f   jpackage.obj
 0001:0000d515       __ehhandler$_Java_jdk_jpackage_internal_ExecutableRebrander_lockResource@12 1000e515 f   jpackage.obj
 0001:0000d53c       __ehhandler$_Java_jdk_jpackage_internal_ExecutableRebrander_unlockResource@16 1000e53c f   jpackage.obj
 0001:0000d559       __unwindfunclet$_Java_jdk_jpackage_internal_ExecutableRebrander_versionSwap@20$3 1000e559 f   jpackage.obj
 0001:0000d561       __unwindfunclet$_Java_jdk_jpackage_internal_ExecutableRebrander_versionSwap@20$4 1000e561 f   jpackage.obj
 0001:0000d569       __unwindfunclet$_Java_jdk_jpackage_internal_ExecutableRebrander_versionSwap@20$5 1000e569 f   jpackage.obj
 0001:0000d571       __unwindfunclet$_Java_jdk_jpackage_internal_ExecutableRebrander_versionSwap@20$6 1000e571 f   jpackage.obj
 0001:0000d579       __unwindfunclet$_Java_jdk_jpackage_internal_ExecutableRebrander_versionSwap@20$7 1000e579 f   jpackage.obj
 0001:0000d586       __ehhandler$_Java_jdk_jpackage_internal_ExecutableRebrander_versionSwap@20 1000e586 f   jpackage.obj
 0001:0000d5ad       __unwindfunclet$_Java_jdk_jpackage_internal_WinExeBundler_embedMSI@20$3 1000e5ad f   jpackage.obj
 0001:0000d5b5       __unwindfunclet$_Java_jdk_jpackage_internal_WinExeBundler_embedMSI@20$4 1000e5b5 f   jpackage.obj
 0001:0000d5c0       __unwindfunclet$_Java_jdk_jpackage_internal_WinExeBundler_embedMSI@20$5 1000e5c0 f   jpackage.obj
 0001:0000d5cb       __unwindfunclet$_Java_jdk_jpackage_internal_WinExeBundler_embedMSI@20$6 1000e5cb f   jpackage.obj
 0001:0000d5d3       __unwindfunclet$_Java_jdk_jpackage_internal_WinExeBundler_embedMSI@20$7 1000e5d3 f   jpackage.obj
 0001:0000d5de       __unwindfunclet$_Java_jdk_jpackage_internal_WinExeBundler_embedMSI@20$8 1000e5de f   jpackage.obj
 0001:0000d5e6       __unwindfunclet$_Java_jdk_jpackage_internal_WinExeBundler_embedMSI@20$9 1000e5e6 f   jpackage.obj
 0001:0000d5ee       __unwindfunclet$_Java_jdk_jpackage_internal_WinExeBundler_embedMSI@20$10 1000e5ee f   jpackage.obj
 0001:0000d5f6       __unwindfunclet$_Java_jdk_jpackage_internal_WinExeBundler_embedMSI@20$11 1000e5f6 f   jpackage.obj
 0001:0000d601       __unwindfunclet$_Java_jdk_jpackage_internal_WinExeBundler_embedMSI@20$12 1000e601 f   jpackage.obj
 0001:0000d611       __ehhandler$_Java_jdk_jpackage_internal_WinExeBundler_embedMSI@20 1000e611 f   jpackage.obj
 0001:0000d63b       __unwindfunclet$?equals@tstrings@@YA_NABV?$basic_string@GU?$char_traits@G@std@@V?$allocator@G@2@@std@@0W4CompareType@1@@Z$0 1000e63b f   tstrings.obj
 0001:0000d648       __ehhandler$?equals@tstrings@@YA_NABV?$basic_string@GU?$char_traits@G@std@@V?$allocator@G@2@@std@@0W4CompareType@1@@Z 1000e648 f   tstrings.obj
 0001:0000d66f       __unwindfunclet$?fromMultiByte@?A0xf04d92fb@tstrings@@YA?AV?$basic_string@GU?$char_traits@G@std@@V?$allocator@G@2@@std@@ABV?$basic_string@DU?$char_traits@D@std@@V?$allocator@D@2@@4@H@Z$0 1000e66f f   tstrings.obj
 0001:0000d67c       __ehhandler$?fromMultiByte@?A0xf04d92fb@tstrings@@YA?AV?$basic_string@GU?$char_traits@G@std@@V?$allocator@G@2@@std@@ABV?$basic_string@DU?$char_traits@D@std@@V?$allocator@D@2@@4@H@Z 1000e67c f   tstrings.obj
 0001:0000d6a3       __unwindfunclet$?toLower@tstrings@@YA?AV?$basic_string@GU?$char_traits@G@std@@V?$allocator@G@2@@std@@ABV23@@Z$0 1000e6a3 f   tstrings.obj
 0001:0000d6c1       __ehhandler$?toLower@tstrings@@YA?AV?$basic_string@GU?$char_traits@G@std@@V?$allocator@G@2@@std@@ABV23@@Z 1000e6c1 f   tstrings.obj
 0001:0000d6e8       __unwindfunclet$?toMultiByte@?A0xf04d92fb@tstrings@@YA?AV?$basic_string@DU?$char_traits@D@std@@V?$allocator@D@2@@std@@ABV?$basic_string@GU?$char_traits@G@std@@V?$allocator@G@2@@4@H@Z$0 1000e6e8 f   tstrings.obj
 0001:0000d6f5       __ehhandler$?toMultiByte@?A0xf04d92fb@tstrings@@YA?AV?$basic_string@DU?$char_traits@D@std@@V?$allocator@D@2@@std@@ABV?$basic_string@GU?$char_traits@G@std@@V?$allocator@G@2@@4@H@Z 1000e6f5 f   tstrings.obj
 0001:0000d71c       __unwindfunclet$?unsafe_format@tstrings@@YA?AV?$basic_string@GU?$char_traits@G@std@@V?$allocator@G@2@@std@@PBGZZ$0 1000e71c f   tstrings.obj
 0001:0000d73a       __ehhandler$?unsafe_format@tstrings@@YA?AV?$basic_string@GU?$char_traits@G@std@@V?$allocator@G@2@@std@@PBGZZ 1000e73a f   tstrings.obj
 0001:0000d757       ??__FlastErrorLogAppender@?A0xd3578678@@YAXXZ 1000e757 f   app.obj
 0001:0000d762       ??__FnopLogAppender@?A0xd3578678@@YAXXZ 1000e762 f   app.obj
 0001:0000d76d       ??__FstandardLogAppender@?A0xd3578678@@YAXXZ 1000e76d f   app.obj
 0001:0000d778       ??__F_Fac_tidy_reg@std@@YAXXZ 1000e778 f   msvcprt:locale0_implib.obj
 0002:00000328       ?_Fac_tidy_reg$initializer$@std@@3P6AXXZA 1000f328     msvcprt:locale0_implib.obj
 0002:0000032c       ?nopLogAppender$initializer$@?A0xd3578678@@3P6AXXZA 1000f32c     app.obj
 0002:00000330       ?standardLogAppender$initializer$@?A0xd3578678@@3P6AXXZA 1000f330     app.obj
 0002:00000334       ?lastErrorLogAppender$initializer$@?A0xd3578678@@3P6AXXZA 1000f334     app.obj
 0002:00000514       ?dirSeparator@?A0x534245bb@FileUtils@@3GB 1000f514     FileUtils.obj
 0002:00000518       ?alianDirSeparator@?A0x534245bb@FileUtils@@3GB 1000f518     FileUtils.obj
 0002:00000a52       ?piecewise_construct@std@@3Upiecewise_construct_t@1@B 1000fa52     MsiUtils.obj
 0002:00000c38       ?formatStr@?A0x40e1fcfd@@3QBGB 1000fc38     PlatformLogEvent.obj
 0002:00000e69       ?piecewise_construct@std@@3Upiecewise_construct_t@1@B 1000fe69     VersionInfo.obj
 0002:00001530       ??_7StandardLogAppender@?A0xd3578678@@6B@ 10010530     app.obj
 0002:0000153c       ??_7LastErrorLogAppender@?A0xd3578678@@6B@ 1001053c     app.obj
 0002:00001830       _GS_ExceptionPointers      10010830     MSVCRT:gs_report.obj
 0002:000025c8       ??_R4StandardLogAppender@?A0xd3578678@@6B@ 100115c8     app.obj
 0002:000025dc       ??_R3StandardLogAppender@?A0xd3578678@@8 100115dc     app.obj
 0002:000025ec       ??_R2StandardLogAppender@?A0xd3578678@@8 100115ec     app.obj
 0002:000025f8       ??_R1A@?0A@EA@StandardLogAppender@?A0xd3578678@@8 100115f8     app.obj
 0002:00002614       ??_R4LastErrorLogAppender@?A0xd3578678@@6B@ 10011614     app.obj
 0002:00002628       ??_R3LastErrorLogAppender@?A0xd3578678@@8 10011628     app.obj
 0002:00002638       ??_R2LastErrorLogAppender@?A0xd3578678@@8 10011638     app.obj
 0002:00002644       ??_R1A@?0A@EA@LastErrorLogAppender@?A0xd3578678@@8 10011644     app.obj
 0002:00002c48       __ehfuncinfo$??1_Sentry_base@?$basic_ostream@DU?$char_traits@D@std@@@std@@QAE@XZ 10011c48     ErrorHandling.obj
 0002:00002c48       __ehfuncinfo$??1_Sentry_base@?$basic_ostream@GU?$char_traits@G@std@@@std@@QAE@XZ 10011c48     ErrorHandling.obj
 0002:00002c48       __ehfuncinfo$??1sentry@?$basic_ostream@DU?$char_traits@D@std@@@std@@QAE@XZ 10011c48     ErrorHandling.obj
 0002:00002c48       __ehfuncinfo$??1sentry@?$basic_ostream@GU?$char_traits@G@std@@@std@@QAE@XZ 10011c48     ErrorHandling.obj
 0002:00002c48       __ehfuncinfo$??1?$unique_ptr@UJniObjWithEnv@jni@@ULocalRefDeleter@12@@std@@QAE@XZ 10011c48     JniUtils.obj
 0002:00002c48       __ehfuncinfo$??1?$basic_filebuf@DU?$char_traits@D@std@@@std@@UAE@XZ 10011c48     MsiDb.obj
 0002:00002c48       __ehfuncinfo$??1DatabaseRecord@msi@@QAE@XZ 10011c48     MsiDb.obj
 0002:00002c48       __ehfuncinfo$??1DatabaseView@msi@@QAE@XZ 10011c48     MsiDb.obj
 0002:00002c48       __ehfuncinfo$??1?$unique_ptr@PAUHINSTANCE__@@ULibraryReleaser@Dll@@@std@@QAE@XZ 10011c48     MsiUtils.obj
 0002:00002c48       __ehfuncinfo$??1Database@msi@@QAE@XZ 10011c48     jpackage.obj
 0002:00002c6c       __unwindtable$??0sentry@?$basic_ostream@DU?$char_traits@D@std@@@std@@QAE@AAV12@@Z 10011c6c     ErrorHandling.obj
 0002:00002c6c       __unwindtable$??0sentry@?$basic_ostream@GU?$char_traits@G@std@@@std@@QAE@AAV12@@Z 10011c6c     ErrorHandling.obj
 0002:00002c74       __ehfuncinfo$??0sentry@?$basic_ostream@DU?$char_traits@D@std@@@std@@QAE@AAV12@@Z 10011c74     ErrorHandling.obj
 0002:00002c74       __ehfuncinfo$??0sentry@?$basic_ostream@GU?$char_traits@G@std@@@std@@QAE@AAV12@@Z 10011c74     ErrorHandling.obj
 0002:00002c98       __unwindtable$??0any@tstrings@@QAE@ABV?$basic_string@GU?$char_traits@G@std@@V?$allocator@G@2@@std@@@Z 10011c98     ErrorHandling.obj
 0002:00002ca0       __ehfuncinfo$??0any@tstrings@@QAE@ABV?$basic_string@GU?$char_traits@G@std@@V?$allocator@G@2@@std@@@Z 10011ca0     ErrorHandling.obj
 0002:00002cc4       __unwindtable$?str@any@tstrings@@QBE?AV?$basic_string@DU?$char_traits@D@std@@V?$allocator@D@2@@std@@XZ 10011cc4     ErrorHandling.obj
 0002:00002cc4       __unwindtable$?string@StringResource@@QBE?AV?$basic_string@GU?$char_traits@G@std@@V?$allocator@G@2@@std@@XZ 10011cc4     Resources.obj
 0002:00002ccc       __ehfuncinfo$?str@any@tstrings@@QBE?AV?$basic_string@DU?$char_traits@D@std@@V?$allocator@D@2@@std@@XZ 10011ccc     ErrorHandling.obj
 0002:00002ccc       __ehfuncinfo$?string@StringResource@@QBE?AV?$basic_string@GU?$char_traits@G@std@@V?$allocator@G@2@@std@@XZ 10011ccc     Resources.obj
 0002:00002cf0       __unwindtable$??0?$basic_ostringstream@GU?$char_traits@G@std@@V?$allocator@G@2@@std@@QAE@XZ 10011cf0     ErrorHandling.obj
 0002:00002d00       __ehfuncinfo$??0?$basic_ostringstream@GU?$char_traits@G@std@@V?$allocator@G@2@@std@@QAE@XZ 10011d00     ErrorHandling.obj
 0002:00002d24       __unwindtable$?str@?$basic_stringbuf@GU?$char_traits@G@std@@V?$allocator@G@2@@std@@QBE?AV?$basic_string@GU?$char_traits@G@std@@V?$allocator@G@2@@2@XZ 10011d24     ErrorHandling.obj
 0002:00002d24       __unwindtable$?getSystemMessageDescription@?A0xd5983087@@YA?AV?$basic_string@GU?$char_traits@G@std@@V?$allocator@G@2@@std@@KPAUHINSTANCE__@@@Z 10011d24     WinErrorHandling.obj
 0002:00002d2c       __ehfuncinfo$?str@?$basic_stringbuf@GU?$char_traits@G@std@@V?$allocator@G@2@@std@@QBE?AV?$basic_string@GU?$char_traits@G@std@@V?$allocator@G@2@@2@XZ 10011d2c     ErrorHandling.obj
 0002:00002d2c       __ehfuncinfo$?getSystemMessageDescription@?A0xd5983087@@YA?AV?$basic_string@GU?$char_traits@G@std@@V?$allocator@G@2@@std@@KPAUHINSTANCE__@@@Z 10011d2c     WinErrorHandling.obj
 0002:00002d50       __catchsym$??$?6GU?$char_traits@G@std@@@std@@YAAAV?$basic_ostream@GU?$char_traits@G@std@@@0@AAV10@PBD@Z$4 10011d50     ErrorHandling.obj
 0002:00002d60       __tryblocktable$??$?6GU?$char_traits@G@std@@@std@@YAAAV?$basic_ostream@GU?$char_traits@G@std@@@0@AAV10@PBD@Z 10011d60     ErrorHandling.obj
 0002:00002d74       __unwindtable$??$?6GU?$char_traits@G@std@@@std@@YAAAV?$basic_ostream@GU?$char_traits@G@std@@@0@AAV10@PBD@Z 10011d74     ErrorHandling.obj
 0002:00002d94       __ehfuncinfo$??$?6GU?$char_traits@G@std@@@std@@YAAAV?$basic_ostream@GU?$char_traits@G@std@@@0@AAV10@PBD@Z 10011d94     ErrorHandling.obj
 0002:00002db8       __catchsym$??$?6GU?$char_traits@G@std@@@std@@YAAAV?$basic_ostream@GU?$char_traits@G@std@@@0@AAV10@PBG@Z$3 10011db8     ErrorHandling.obj
 0002:00002dc8       __tryblocktable$??$?6GU?$char_traits@G@std@@@std@@YAAAV?$basic_ostream@GU?$char_traits@G@std@@@0@AAV10@PBG@Z 10011dc8     ErrorHandling.obj
 0002:00002ddc       __unwindtable$??$?6GU?$char_traits@G@std@@@std@@YAAAV?$basic_ostream@GU?$char_traits@G@std@@@0@AAV10@PBG@Z 10011ddc     ErrorHandling.obj
 0002:00002df4       __ehfuncinfo$??$?6GU?$char_traits@G@std@@@std@@YAAAV?$basic_ostream@GU?$char_traits@G@std@@@0@AAV10@PBG@Z 10011df4     ErrorHandling.obj
 0002:00002e18       __unwindtable$??6@YAAAV?$basic_ostream@DU?$char_traits@D@std@@@std@@AAV01@ABVany@tstrings@@@Z 10011e18     ErrorHandling.obj
 0002:00002e18       __unwindtable$?append@LastErrorLogAppender@?A0xd3578678@@UAEXABULogEvent@@@Z 10011e18     app.obj
 0002:00002e20       __ehfuncinfo$??6@YAAAV?$basic_ostream@DU?$char_traits@D@std@@@std@@AAV01@ABVany@tstrings@@@Z 10011e20     ErrorHandling.obj
 0002:00002e20       __ehfuncinfo$?append@LastErrorLogAppender@?A0xd3578678@@UAEXABULogEvent@@@Z 10011e20     app.obj
 0002:00002e44       __catchsym$??$?6U?$char_traits@D@std@@@std@@YAAAV?$basic_ostream@DU?$char_traits@D@std@@@0@AAV10@PBD@Z$3 10011e44     ErrorHandling.obj
 0002:00002e54       __tryblocktable$??$?6U?$char_traits@D@std@@@std@@YAAAV?$basic_ostream@DU?$char_traits@D@std@@@0@AAV10@PBD@Z 10011e54     ErrorHandling.obj
 0002:00002e68       __unwindtable$??$?6U?$char_traits@D@std@@@std@@YAAAV?$basic_ostream@DU?$char_traits@D@std@@@0@AAV10@PBD@Z 10011e68     ErrorHandling.obj
 0002:00002e80       __ehfuncinfo$??$?6U?$char_traits@D@std@@@std@@YAAAV?$basic_ostream@DU?$char_traits@D@std@@@0@AAV10@PBD@Z 10011e80     ErrorHandling.obj
 0002:00002ea4       __unwindtable$?reportError@@YAXABUSourceCodePos@@ABVruntime_error@std@@@Z 10011ea4     ErrorHandling.obj
 0002:00002eb4       __ehfuncinfo$?reportError@@YAXABUSourceCodePos@@ABVruntime_error@std@@@Z 10011eb4     ErrorHandling.obj
 0002:00002ed8       __unwindtable$?reportUnknownError@@YAXABUSourceCodePos@@@Z 10011ed8     ErrorHandling.obj
 0002:00002ed8       __unwindtable$?log@Logger@@QBEXW4LogLevel@1@PBGH1ABVany@tstrings@@@Z 10011ed8     Log.obj
 0002:00002ed8       __unwindtable$?appendFormatted@LogEvent@@CAXABUPlatformLogEvent@@AAV?$basic_string@GU?$char_traits@G@std@@V?$allocator@G@2@@std@@@Z 10011ed8     PlatformLogEvent.obj
 0002:00002ed8       __unwindtable$?initializeLogging@Logger@@CAXXZ 10011ed8     PlatformLogEvent.obj
 0002:00002ed8       __unwindtable$??6@YAAAV?$basic_ostream@GU?$char_traits@G@std@@@std@@AAV01@ABVany@tstrings@@@Z 10011ed8     Resources.obj
 0002:00002ee0       __ehfuncinfo$?reportUnknownError@@YAXABUSourceCodePos@@@Z 10011ee0     ErrorHandling.obj
 0002:00002ee0       __ehfuncinfo$?log@Logger@@QBEXW4LogLevel@1@PBGH1ABVany@tstrings@@@Z 10011ee0     Log.obj
 0002:00002ee0       __ehfuncinfo$?appendFormatted@LogEvent@@CAXABUPlatformLogEvent@@AAV?$basic_string@GU?$char_traits@G@std@@V?$allocator@G@2@@std@@@Z 10011ee0     PlatformLogEvent.obj
 0002:00002ee0       __ehfuncinfo$?initializeLogging@Logger@@CAXXZ 10011ee0     PlatformLogEvent.obj
 0002:00002ee0       __ehfuncinfo$??6@YAAAV?$basic_ostream@GU?$char_traits@G@std@@@std@@AAV01@ABVany@tstrings@@@Z 10011ee0     Resources.obj
 0002:00002f04       __unwindtable$?makeMessage@@YA?AV?$basic_string@DU?$char_traits@D@std@@V?$allocator@D@2@@std@@ABVruntime_error@2@ABUSourceCodePos@@@Z 10011f04     ErrorHandling.obj
 0002:00002f1c       __ehfuncinfo$?makeMessage@@YA?AV?$basic_string@DU?$char_traits@D@std@@V?$allocator@D@2@@std@@ABVruntime_error@2@ABUSourceCodePos@@@Z 10011f1c     ErrorHandling.obj
 0002:00002f40       __ehfuncinfo$?joinErrorMessages@@YA?AV?$basic_string@DU?$char_traits@D@std@@V?$allocator@D@2@@std@@ABV12@0@Z 10011f40     ErrorHandling.obj
 0002:00002f64       __unwindtable$?joinErrorMessages@@YA?AV?$basic_string@DU?$char_traits@D@std@@V?$allocator@D@2@@std@@ABV12@0@Z 10011f64     ErrorHandling.obj
 0002:00002f8c       __unwindtable$?getFilename@?A0xd1a094c7@@YA?AV?$basic_string@GU?$char_traits@G@std@@V?$allocator@G@2@@std@@ABUSourceCodePos@@@Z 10011f8c     ErrorHandling.obj
 0002:00002f9c       __ehfuncinfo$?getFilename@?A0xd1a094c7@@YA?AV?$basic_string@GU?$char_traits@G@std@@V?$allocator@G@2@@std@@ABUSourceCodePos@@@Z 10011f9c     ErrorHandling.obj
 0002:00002fc0       __unwindtable$?reportError@?A0xd1a094c7@@YAXABUSourceCodePos@@ABV?$basic_string@GU?$char_traits@G@std@@V?$allocator@G@2@@std@@@Z 10011fc0     ErrorHandling.obj
 0002:00002fd8       __ehfuncinfo$?reportError@?A0xd1a094c7@@YAXABUSourceCodePos@@ABV?$basic_string@GU?$char_traits@G@std@@V?$allocator@G@2@@std@@@Z 10011fd8     ErrorHandling.obj
 0002:00002ffc       __unwindtable$??0?$basic_ostringstream@DU?$char_traits@D@std@@V?$allocator@D@2@@std@@QAE@XZ 10011ffc     ErrorHandling.obj
 0002:0000300c       __ehfuncinfo$??0?$basic_ostringstream@DU?$char_traits@D@std@@V?$allocator@D@2@@std@@QAE@XZ 1001200c     ErrorHandling.obj
 0002:00003030       __unwindtable$?str@?$basic_stringbuf@DU?$char_traits@D@std@@V?$allocator@D@2@@std@@QBE?AV?$basic_string@DU?$char_traits@D@std@@V?$allocator@D@2@@2@XZ 10012030     ErrorHandling.obj
 0002:00003038       __ehfuncinfo$?str@?$basic_stringbuf@DU?$char_traits@D@std@@V?$allocator@D@2@@std@@QBE?AV?$basic_string@DU?$char_traits@D@std@@V?$allocator@D@2@@2@XZ 10012038     ErrorHandling.obj
 0002:0000305c       __unwindtable$??$use_facet@V?$ctype@G@std@@@std@@YAABV?$ctype@G@0@ABVlocale@0@@Z 1001205c     ErrorHandling.obj
 0002:0000305c       __unwindtable$??$use_facet@V?$codecvt@DDU_Mbstatet@@@std@@@std@@YAABV?$codecvt@DDU_Mbstatet@@@0@ABVlocale@0@@Z 1001205c     MsiDb.obj
 0002:0000306c       __ehfuncinfo$??$use_facet@V?$ctype@G@std@@@std@@YAABV?$ctype@G@0@ABVlocale@0@@Z 1001206c     ErrorHandling.obj
 0002:0000306c       __ehfuncinfo$??$use_facet@V?$codecvt@DDU_Mbstatet@@@std@@@std@@YAABV?$codecvt@DDU_Mbstatet@@@0@ABVlocale@0@@Z 1001206c     MsiDb.obj
 0002:00003090       __catchsym$??$_Insert_string@GU?$char_traits@G@std@@I@std@@YAAAV?$basic_ostream@GU?$char_traits@G@std@@@0@AAV10@QBGI@Z$3 10012090     ErrorHandling.obj
 0002:000030a0       __tryblocktable$??$_Insert_string@GU?$char_traits@G@std@@I@std@@YAAAV?$basic_ostream@GU?$char_traits@G@std@@@0@AAV10@QBGI@Z 100120a0     ErrorHandling.obj
 0002:000030b4       __unwindtable$??$_Insert_string@GU?$char_traits@G@std@@I@std@@YAAAV?$basic_ostream@GU?$char_traits@G@std@@@0@AAV10@QBGI@Z 100120b4     ErrorHandling.obj
 0002:000030cc       __ehfuncinfo$??$_Insert_string@GU?$char_traits@G@std@@I@std@@YAAAV?$basic_ostream@GU?$char_traits@G@std@@@0@AAV10@QBGI@Z 100120cc     ErrorHandling.obj
 0002:000030f0       __catchsym$??$_Insert_string@DU?$char_traits@D@std@@I@std@@YAAAV?$basic_ostream@DU?$char_traits@D@std@@@0@AAV10@QBDI@Z$3 100120f0     ErrorHandling.obj
 0002:00003100       __tryblocktable$??$_Insert_string@DU?$char_traits@D@std@@I@std@@YAAAV?$basic_ostream@DU?$char_traits@D@std@@@0@AAV10@QBDI@Z 10012100     ErrorHandling.obj
 0002:00003114       __unwindtable$??$_Insert_string@DU?$char_traits@D@std@@I@std@@YAAAV?$basic_ostream@DU?$char_traits@D@std@@@0@AAV10@QBDI@Z 10012114     ErrorHandling.obj
 0002:0000312c       __ehfuncinfo$??$_Insert_string@DU?$char_traits@D@std@@I@std@@YAAAV?$basic_ostream@DU?$char_traits@D@std@@@0@AAV10@QBDI@Z 1001212c     ErrorHandling.obj
 0002:000031fc       __unwindtable$?combinePath@FileUtils@@YA?AV?$basic_string@GU?$char_traits@G@std@@V?$allocator@G@2@@std@@ABV23@0@Z 100121fc     FileUtils.obj
 0002:0000321c       __ehfuncinfo$?combinePath@FileUtils@@YA?AV?$basic_string@GU?$char_traits@G@std@@V?$allocator@G@2@@std@@ABV23@0@Z 1001221c     FileUtils.obj
 0002:00003240       __unwindtable$??0Guid@@QAE@ABV?$basic_string@GU?$char_traits@G@std@@V?$allocator@G@2@@std@@@Z 10012240     Guid.obj
 0002:00003250       __ehfuncinfo$??0Guid@@QAE@ABV?$basic_string@GU?$char_traits@G@std@@V?$allocator@G@2@@std@@@Z 10012250     Guid.obj
 0002:00003274       __unwindtable$?toString@Guid@@QBE?AV?$basic_string@GU?$char_traits@G@std@@V?$allocator@G@2@@std@@H@Z 10012274     Guid.obj
 0002:00003284       __ehfuncinfo$?toString@Guid@@QBE?AV?$basic_string@GU?$char_traits@G@std@@V?$allocator@G@2@@std@@H@Z 10012284     Guid.obj
 0002:000032a8       __unwindtable$?makeException@@YA?AV?$JpError@Vruntime_error@std@@@@ABV?$basic_string@DU?$char_traits@D@std@@V?$allocator@D@2@@std@@ABUSourceCodePos@@@Z 100122a8     Guid.obj
 0002:000032b0       __ehfuncinfo$?makeException@@YA?AV?$JpError@Vruntime_error@std@@@@ABV?$basic_string@DU?$char_traits@D@std@@V?$allocator@D@2@@std@@ABUSourceCodePos@@@Z 100122b0     Guid.obj
 0002:000032d4       __unwindtable$??0?$JpError@Vruntime_error@std@@@@QAE@ABV0@@Z 100122d4     Guid.obj
 0002:000032d4       __unwindtable$??0?$JpError@Vruntime_error@std@@@@QAE@ABVruntime_error@std@@ABUSourceCodePos@@@Z 100122d4     Guid.obj
 0002:000032d4       __unwindtable$??0?$JpError@VError@msi@@@@QAE@ABV0@@Z 100122d4     MsiDb.obj
 0002:000032d4       __unwindtable$??0?$JpError@VError@msi@@@@QAE@ABVError@msi@@ABUSourceCodePos@@@Z 100122d4     MsiDb.obj
 0002:000032d4       __unwindtable$??0?$JpError@VNoMoreItemsError@msi@@@@QAE@ABV0@@Z 100122d4     MsiDb.obj
 0002:000032d4       __unwindtable$??0?$JpError@VNoMoreItemsError@msi@@@@QAE@ABVNoMoreItemsError@msi@@ABUSourceCodePos@@@Z 100122d4     MsiDb.obj
 0002:000032d4       __unwindtable$??0?$JpError@VSysError@@@@QAE@ABV0@@Z 100122d4     MsiUtils.obj
 0002:000032d4       __unwindtable$??0?$JpError@VSysError@@@@QAE@ABVSysError@@ABUSourceCodePos@@@Z 100122d4     MsiUtils.obj
 0002:000032dc       __ehfuncinfo$??0?$JpError@Vruntime_error@std@@@@QAE@ABV0@@Z 100122dc     Guid.obj
 0002:000032dc       __ehfuncinfo$??0?$JpError@Vruntime_error@std@@@@QAE@ABVruntime_error@std@@ABUSourceCodePos@@@Z 100122dc     Guid.obj
 0002:000032dc       __ehfuncinfo$??0?$JpError@VError@msi@@@@QAE@ABV0@@Z 100122dc     MsiDb.obj
 0002:000032dc       __ehfuncinfo$??0?$JpError@VError@msi@@@@QAE@ABVError@msi@@ABUSourceCodePos@@@Z 100122dc     MsiDb.obj
 0002:000032dc       __ehfuncinfo$??0?$JpError@VNoMoreItemsError@msi@@@@QAE@ABV0@@Z 100122dc     MsiDb.obj
 0002:000032dc       __ehfuncinfo$??0?$JpError@VNoMoreItemsError@msi@@@@QAE@ABVNoMoreItemsError@msi@@ABUSourceCodePos@@@Z 100122dc     MsiDb.obj
 0002:000032dc       __ehfuncinfo$??0?$JpError@VSysError@@@@QAE@ABV0@@Z 100122dc     MsiUtils.obj
 0002:000032dc       __ehfuncinfo$??0?$JpError@VSysError@@@@QAE@ABVSysError@@ABUSourceCodePos@@@Z 100122dc     MsiUtils.obj
 0002:00003300       __unwindtable$?makeException@@YA?AV?$JpError@Vruntime_error@std@@@@ABVany@tstrings@@ABUSourceCodePos@@@Z 10012300     Guid.obj
 0002:00003300       __unwindtable$?makeException@@YA?AV?$JpError@Vruntime_error@std@@@@PBDABUSourceCodePos@@@Z 10012300     Guid.obj
 0002:00003300       __unwindtable$?getSystem32Dir@SysInfo@@YA?AV?$basic_string@GU?$char_traits@G@std@@V?$allocator@G@2@@std@@XZ 10012300     WinSysInfo.obj
 0002:00003308       __ehfuncinfo$?makeException@@YA?AV?$JpError@Vruntime_error@std@@@@ABVany@tstrings@@ABUSourceCodePos@@@Z 10012308     Guid.obj
 0002:00003308       __ehfuncinfo$?makeException@@YA?AV?$JpError@Vruntime_error@std@@@@PBDABUSourceCodePos@@@Z 10012308     Guid.obj
 0002:00003308       __ehfuncinfo$?getSystem32Dir@SysInfo@@YA?AV?$basic_string@GU?$char_traits@G@std@@V?$allocator@G@2@@std@@XZ 10012308     WinSysInfo.obj
 0002:0000332c       __unwindtable$?initGuid@?A0x2459fff0@@YAXABV?$basic_string@GU?$char_traits@G@std@@V?$allocator@G@2@@std@@AAU_GUID@@@Z 1001232c     Guid.obj
 0002:0000332c       __unwindtable$??0FixedFileVersion@?A0xcb1fbc16@@QAE@ABV?$basic_string@GU?$char_traits@G@std@@V?$allocator@G@2@@std@@@Z 1001232c     VersionInfo.obj
 0002:00003334       __ehfuncinfo$?initGuid@?A0x2459fff0@@YAXABV?$basic_string@GU?$char_traits@G@std@@V?$allocator@G@2@@std@@AAU_GUID@@@Z 10012334     Guid.obj
 0002:00003334       __ehfuncinfo$??0FixedFileVersion@?A0xcb1fbc16@@QAE@ABV?$basic_string@GU?$char_traits@G@std@@V?$allocator@G@2@@std@@@Z 10012334     VersionInfo.obj
 0002:000033ec       __unwindtable$?toUnicodeString@jni@@YA?AV?$basic_string@GU?$char_traits@G@std@@V?$allocator@G@2@@std@@PAUJNIEnv_@@PAV_jstring@@@Z 100123ec     JniUtils.obj
 0002:000033f4       __ehfuncinfo$?toUnicodeString@jni@@YA?AV?$basic_string@GU?$char_traits@G@std@@V?$allocator@G@2@@std@@PAUJNIEnv_@@PAV_jstring@@@Z 100123f4     JniUtils.obj
 0002:00003418       __unwindtable$?toUnicodeStringArray@jni@@YA?AV?$vector@V?$basic_string@GU?$char_traits@G@std@@V?$allocator@G@2@@std@@V?$allocator@V?$basic_string@GU?$char_traits@G@std@@V?$allocator@G@2@@std@@@2@@std@@PAUJNIEnv_@@PAV_jobjectArray@@@Z 10012418     JniUtils.obj
 0002:00003438       __ehfuncinfo$?toUnicodeStringArray@jni@@YA?AV?$vector@V?$basic_string@GU?$char_traits@G@std@@V?$allocator@G@2@@std@@V?$allocator@V?$basic_string@GU?$char_traits@G@std@@V?$allocator@G@2@@std@@@2@@std@@PAUJNIEnv_@@PAV_jobjectArray@@@Z 10012438     JniUtils.obj
 0002:0000345c       __unwindtable$??1?$AtEndOfScope@V<lambda_bafb2a7f1406751b8a75ac1ff6dad7d1>@@@@QAE@XZ 1001245c     JniUtils.obj
 0002:0000346c       __tryblocktable$??1?$AtEndOfScope@V<lambda_bafb2a7f1406751b8a75ac1ff6dad7d1>@@@@QAE@XZ 1001246c     JniUtils.obj
 0002:00003480       __catchsym$??1?$AtEndOfScope@V<lambda_bafb2a7f1406751b8a75ac1ff6dad7d1>@@@@QAE@XZ$3 10012480     JniUtils.obj
 0002:000034a0       __ehfuncinfo$??1?$AtEndOfScope@V<lambda_bafb2a7f1406751b8a75ac1ff6dad7d1>@@@@QAE@XZ 100124a0     JniUtils.obj
 0002:000034c4       __catchsym$??6?$basic_ostream@GU?$char_traits@G@std@@@std@@QAEAAV01@G@Z$3 100124c4     Log.obj
 0002:000034d4       __tryblocktable$??6?$basic_ostream@GU?$char_traits@G@std@@@std@@QAEAAV01@G@Z 100124d4     Log.obj
 0002:000034e8       __unwindtable$??6?$basic_ostream@GU?$char_traits@G@std@@@std@@QAEAAV01@G@Z 100124e8     Log.obj
 0002:00003500       __ehfuncinfo$??6?$basic_ostream@GU?$char_traits@G@std@@@std@@QAEAAV01@G@Z 10012500     Log.obj
 0002:00003524       __unwindtable$?append@StreamLogAppender@@UAEXABULogEvent@@@Z 10012524     Log.obj
 0002:00003544       __ehfuncinfo$?append@StreamLogAppender@@UAEXABULogEvent@@@Z 10012544     Log.obj
 0002:00003568       __unwindtable$?log@Logger@@QBEXW4LogLevel@1@PBGH1ABV?$basic_string@GU?$char_traits@G@std@@V?$allocator@G@2@@std@@@Z 10012568     Log.obj
 0002:00003578       __ehfuncinfo$?log@Logger@@QBEXW4LogLevel@1@PBGH1ABV?$basic_string@GU?$char_traits@G@std@@V?$allocator@G@2@@std@@@Z 10012578     Log.obj
 0002:0000359c       __unwindtable$??0Database@msi@@QAE@ABV?$basic_string@GU?$char_traits@G@std@@V?$allocator@G@2@@std@@@Z 1001259c     MsiDb.obj
 0002:000035a4       __ehfuncinfo$??0Database@msi@@QAE@ABV?$basic_string@GU?$char_traits@G@std@@V?$allocator@G@2@@std@@@Z 100125a4     MsiDb.obj
 0002:000035c8       __ehfuncinfo$?getProperty@Database@msi@@QBE?AV?$basic_string@GU?$char_traits@G@std@@V?$allocator@G@2@@std@@ABV34@@Z 100125c8     MsiDb.obj
 0002:000035ec       __unwindtable$?getProperty@Database@msi@@QBE?AV?$basic_string@GU?$char_traits@G@std@@V?$allocator@G@2@@std@@ABV34@@Z 100125ec     MsiDb.obj
 0002:00003644       __unwindtable$??4DatabaseRecord@msi@@QAEAAV01@ABV01@@Z 10012644     MsiDb.obj
 0002:0000364c       __ehfuncinfo$??4DatabaseRecord@msi@@QAEAAV01@ABV01@@Z 1001264c     MsiDb.obj
 0002:00003670       __unwindtable$?fetch@DatabaseRecord@msi@@QAEAAV12@AAVDatabaseView@2@@Z 10012670     MsiDb.obj
 0002:00003680       __ehfuncinfo$?fetch@DatabaseRecord@msi@@QAEAAV12@AAVDatabaseView@2@@Z 10012680     MsiDb.obj
 0002:000036a4       __unwindtable$?getFieldCount@DatabaseRecord@msi@@QBEIXZ 100126a4     MsiDb.obj
 0002:000036b4       __ehfuncinfo$?getFieldCount@DatabaseRecord@msi@@QBEIXZ 100126b4     MsiDb.obj
 0002:000036d8       __ehfuncinfo$??0DatabaseView@msi@@QAE@ABVDatabase@1@ABV?$basic_string@GU?$char_traits@G@std@@V?$allocator@G@2@@std@@ABVDatabaseRecord@1@@Z 100126d8     MsiDb.obj
 0002:000036fc       __unwindtable$??0DatabaseView@msi@@QAE@ABVDatabase@1@ABV?$basic_string@GU?$char_traits@G@std@@V?$allocator@G@2@@std@@ABVDatabaseRecord@1@@Z 100126fc     MsiDb.obj
 0002:00003724       __unwindtable$?fetch@DatabaseView@msi@@QAE?AVDatabaseRecord@2@XZ 10012724     MsiDb.obj
 0002:0000373c       __ehfuncinfo$?fetch@DatabaseView@msi@@QAE?AVDatabaseRecord@2@XZ 1001273c     MsiDb.obj
 0002:00003760       __unwindtable$?tryFetch@DatabaseView@msi@@QAE?AVDatabaseRecord@2@XZ 10012760     MsiDb.obj
 0002:00003778       __ehfuncinfo$?tryFetch@DatabaseView@msi@@QAE?AVDatabaseRecord@2@XZ 10012778     MsiDb.obj
 0002:0000379c       __unwindtable$?uflow@?$basic_filebuf@DU?$char_traits@D@std@@@std@@MAEHXZ 1001279c     MsiDb.obj
 0002:000037a4       __ehfuncinfo$?uflow@?$basic_filebuf@DU?$char_traits@D@std@@@std@@MAEHXZ 100127a4     MsiDb.obj
 0002:000037c8       __unwindtable$?openDatabase@?A0x6ccb95c8@msi@@YAKABV?$basic_string@GU?$char_traits@G@std@@V?$allocator@G@2@@std@@@Z 100127c8     MsiDb.obj
 0002:000037d8       __ehfuncinfo$?openDatabase@?A0x6ccb95c8@msi@@YAKABV?$basic_string@GU?$char_traits@G@std@@V?$allocator@G@2@@std@@@Z 100127d8     MsiDb.obj
 0002:000038c0       __unwindtable$?closeMSIHANDLE@msi@@YAXK@Z 100128c0     MsiUtils.obj
 0002:000038c8       __ehfuncinfo$?closeMSIHANDLE@msi@@YAXK@Z 100128c8     MsiUtils.obj
 0002:000038ec       __unwindtable$??0Error@msi@@QAE@ABVany@tstrings@@I@Z 100128ec     MsiUtils.obj
 0002:000038f4       __ehfuncinfo$??0Error@msi@@QAE@ABVany@tstrings@@I@Z 100128f4     MsiUtils.obj
 0002:00003918       __unwindtable$??$getProperty@P6GIKIPAGPAK@ZKI@?A0x0e70828c@msi@@YA?AV?$basic_string@GU?$char_traits@G@std@@V?$allocator@G@2@@std@@P6GIKIPAGPAK@ZQBDKI@Z 10012918     MsiUtils.obj
 0002:00003930       __ehfuncinfo$??$getProperty@P6GIKIPAGPAK@ZKI@?A0x0e70828c@msi@@YA?AV?$basic_string@GU?$char_traits@G@std@@V?$allocator@G@2@@std@@P6GIKIPAGPAK@ZQBDKI@Z 10012930     MsiUtils.obj
 0002:00003954       __catchsym$?makeMessage@?A0x0e70828c@msi@@YA?AV?$basic_string@DU?$char_traits@D@std@@V?$allocator@D@2@@std@@ABV34@I@Z$36 10012954     MsiUtils.obj
 0002:00003964       __tryblocktable$?makeMessage@?A0x0e70828c@msi@@YA?AV?$basic_string@DU?$char_traits@D@std@@V?$allocator@D@2@@std@@ABV34@I@Z 10012964     MsiUtils.obj
 0002:00003978       __ehfuncinfo$?makeMessage@?A0x0e70828c@msi@@YA?AV?$basic_string@DU?$char_traits@D@std@@V?$allocator@D@2@@std@@ABV34@I@Z 10012978     MsiUtils.obj
 0002:0000399c       __unwindtable$?makeMessage@?A0x0e70828c@msi@@YA?AV?$basic_string@DU?$char_traits@D@std@@V?$allocator@D@2@@std@@ABV34@I@Z 1001299c     MsiUtils.obj
 0002:00003a34       __unwindtable$??$?0ABUpiecewise_construct_t@std@@V?$tuple@ABV?$basic_string@GU?$char_traits@G@std@@V?$allocator@G@2@@std@@@1@V?$tuple@$$V@1@@?$_Tree_temp_node@V?$allocator@U?$_Tree_node@U?$pair@$$CBV?$basic_string@GU?$char_traits@G@std@@V?$allocator@G@2@@std@@V12@@std@@PAX@std@@@std@@@std@@QAE@AAV?$allocator@U?$_Tree_node@U?$pair@$$CBV?$basic_string@GU?$char_traits@G@std@@V?$allocator@G@2@@std@@V12@@std@@PAX@std@@@1@PAU?$_Tree_node@U?$pair@$$CBV?$basic_string@GU?$char_traits@G@std@@V?$allocator@G@2@@std@@V12@@std@@PAX@1@ABUpiecewise_construct_t@1@$$QAV?$tuple@ABV?$basic_string@GU?$char_traits@G@std@@V?$allocator@G@2@@std@@@1@$$QAV?$tuple@$$V@1@@Z 10012a34     MsiUtils.obj
 0002:00003a34       __unwindtable$??0?$_Tree_temp_node_alloc@V?$allocator@U?$_Tree_node@U?$pair@$$CBV?$basic_string@GU?$char_traits@G@std@@V?$allocator@G@2@@std@@V12@@std@@PAX@std@@@std@@@std@@QAE@AAV?$allocator@U?$_Tree_node@U?$pair@$$CBV?$basic_string@GU?$char_traits@G@std@@V?$allocator@G@2@@std@@V12@@std@@PAX@std@@@1@@Z 10012a34     MsiUtils.obj
 0002:00003a3c       __ehfuncinfo$??$?0ABUpiecewise_construct_t@std@@V?$tuple@ABV?$basic_string@GU?$char_traits@G@std@@V?$allocator@G@2@@std@@@1@V?$tuple@$$V@1@@?$_Tree_temp_node@V?$allocator@U?$_Tree_node@U?$pair@$$CBV?$basic_string@GU?$char_traits@G@std@@V?$allocator@G@2@@std@@V12@@std@@PAX@std@@@std@@@std@@QAE@AAV?$allocator@U?$_Tree_node@U?$pair@$$CBV?$basic_string@GU?$char_traits@G@std@@V?$allocator@G@2@@std@@V12@@std@@PAX@std@@@1@PAU?$_Tree_node@U?$pair@$$CBV?$basic_string@GU?$char_traits@G@std@@V?$allocator@G@2@@std@@V12@@std@@PAX@1@ABUpiecewise_construct_t@1@$$QAV?$tuple@ABV?$basic_string@GU?$char_traits@G@std@@V?$allocator@G@2@@std@@@1@$$QAV?$tuple@$$V@1@@Z 10012a3c     MsiUtils.obj
 0002:00003a3c       __ehfuncinfo$??0?$_Tree_temp_node_alloc@V?$allocator@U?$_Tree_node@U?$pair@$$CBV?$basic_string@GU?$char_traits@G@std@@V?$allocator@G@2@@std@@V12@@std@@PAX@std@@@std@@@std@@QAE@AAV?$allocator@U?$_Tree_node@U?$pair@$$CBV?$basic_string@GU?$char_traits@G@std@@V?$allocator@G@2@@std@@V12@@std@@PAX@std@@@1@@Z 10012a3c     MsiUtils.obj
 0002:00003ac0       __catchsym$?retrieveModuleName@?A0x40e1fcfd@@YA?AV?$basic_string@GU?$char_traits@G@std@@V?$allocator@G@2@@std@@XZ$5 10012ac0     PlatformLogEvent.obj
 0002:00003ad0       __tryblocktable$?retrieveModuleName@?A0x40e1fcfd@@YA?AV?$basic_string@GU?$char_traits@G@std@@V?$allocator@G@2@@std@@XZ 10012ad0     PlatformLogEvent.obj
 0002:00003ae4       __unwindtable$?retrieveModuleName@?A0x40e1fcfd@@YA?AV?$basic_string@GU?$char_traits@G@std@@V?$allocator@G@2@@std@@XZ 10012ae4     PlatformLogEvent.obj
 0002:00003afc       __ehfuncinfo$?retrieveModuleName@?A0x40e1fcfd@@YA?AV?$basic_string@GU?$char_traits@G@std@@V?$allocator@G@2@@std@@XZ 10012afc     PlatformLogEvent.obj
 0002:00003b20       __unwindtable$??0FileLock@ResourceEditor@@QAE@ABV?$basic_string@GU?$char_traits@G@std@@V?$allocator@G@2@@std@@@Z 10012b20     ResourceEditor.obj
 0002:00003b30       __ehfuncinfo$??0FileLock@ResourceEditor@@QAE@ABV?$basic_string@GU?$char_traits@G@std@@V?$allocator@G@2@@std@@@Z 10012b30     ResourceEditor.obj
 0002:00003b54       __tryblocktable$??1FileLock@ResourceEditor@@QAE@XZ 10012b54     ResourceEditor.obj
 0002:00003b68       __catchsym$??1FileLock@ResourceEditor@@QAE@XZ$8 10012b68     ResourceEditor.obj
 0002:00003b88       __unwindtable$??1FileLock@ResourceEditor@@QAE@XZ 10012b88     ResourceEditor.obj
 0002:00003ba8       __ehfuncinfo$??1FileLock@ResourceEditor@@QAE@XZ 10012ba8     ResourceEditor.obj
 0002:00003bcc       __unwindtable$??0ResourceEditor@@QAE@XZ 10012bcc     ResourceEditor.obj
 0002:00003bdc       __ehfuncinfo$??0ResourceEditor@@QAE@XZ 10012bdc     ResourceEditor.obj
 0002:00003c00       __unwindtable$?id@ResourceEditor@@QAEAAV1@PBG@Z 10012c00     ResourceEditor.obj
 0002:00003c00       __unwindtable$?type@ResourceEditor@@QAEAAV1@PBG@Z 10012c00     ResourceEditor.obj
 0002:00003c08       __ehfuncinfo$?id@ResourceEditor@@QAEAAV1@PBG@Z 10012c08     ResourceEditor.obj
 0002:00003c08       __ehfuncinfo$?type@ResourceEditor@@QAEAAV1@PBG@Z 10012c08     ResourceEditor.obj
 0002:00003c2c       __unwindtable$?apply@ResourceEditor@@QAEAAV1@ABVFileLock@1@AAV?$basic_istream@DU?$char_traits@D@std@@@std@@_J@Z 10012c2c     ResourceEditor.obj
 0002:00003c44       __ehfuncinfo$?apply@ResourceEditor@@QAEAAV1@ABVFileLock@1@AAV?$basic_istream@DU?$char_traits@D@std@@@std@@_J@Z 10012c44     ResourceEditor.obj
 0002:00003c68       __unwindtable$?apply@ResourceEditor@@QAEAAV1@ABVFileLock@1@ABV?$basic_string@GU?$char_traits@G@std@@V?$allocator@G@2@@std@@@Z 10012c68     ResourceEditor.obj
 0002:00003c70       __ehfuncinfo$?apply@ResourceEditor@@QAEAAV1@ABVFileLock@1@ABV?$basic_string@GU?$char_traits@G@std@@V?$allocator@G@2@@std@@@Z 10012c70     ResourceEditor.obj
 0002:00003c94       __unwindtable$??0any@tstrings@@QAE@PBD@Z 10012c94     ResourceEditor.obj
 0002:00003cac       __ehfuncinfo$??0any@tstrings@@QAE@PBD@Z 10012cac     ResourceEditor.obj
 0002:00003cd0       __unwindtable$??0?$basic_ifstream@DU?$char_traits@D@std@@@std@@QAE@PBGHH@Z 10012cd0     ResourceEditor.obj
 0002:00003ce8       __ehfuncinfo$??0?$basic_ifstream@DU?$char_traits@D@std@@@std@@QAE@PBGHH@Z 10012ce8     ResourceEditor.obj
 0002:00003d0c       __unwindtable$??0?$basic_filebuf@DU?$char_traits@D@std@@@std@@QAE@XZ 10012d0c     ResourceEditor.obj
 0002:00003d0c       __unwindtable$??0?$basic_stringbuf@DU?$char_traits@D@std@@V?$allocator@D@2@@std@@QAE@ABV?$basic_string@DU?$char_traits@D@std@@V?$allocator@D@2@@1@H@Z 10012d0c     jpackage.obj
 0002:00003d14       __ehfuncinfo$??0?$basic_filebuf@DU?$char_traits@D@std@@@std@@QAE@XZ 10012d14     ResourceEditor.obj
 0002:00003d14       __ehfuncinfo$??0?$basic_stringbuf@DU?$char_traits@D@std@@V?$allocator@D@2@@std@@QAE@ABV?$basic_string@DU?$char_traits@D@std@@V?$allocator@D@2@@1@H@Z 10012d14     jpackage.obj
 0002:00003d38       __unwindtable$?open@?$basic_filebuf@DU?$char_traits@D@std@@@std@@QAEPAV12@PBGHH@Z 10012d38     ResourceEditor.obj
 0002:00003d40       __ehfuncinfo$?open@?$basic_filebuf@DU?$char_traits@D@std@@@std@@QAEPAV12@PBGHH@Z 10012d40     ResourceEditor.obj
 0002:00003d64       __unwindtable$??$_Range_construct_or_tidy@V?$istreambuf_iterator@DU?$char_traits@D@std@@@std@@@?$vector@EV?$allocator@E@std@@@std@@AAEXV?$istreambuf_iterator@DU?$char_traits@D@std@@@1@0Uinput_iterator_tag@1@@Z 10012d64     ResourceEditor.obj
 0002:00003d6c       __ehfuncinfo$??$_Range_construct_or_tidy@V?$istreambuf_iterator@DU?$char_traits@D@std@@@std@@@?$vector@EV?$allocator@E@std@@@std@@AAEXV?$istreambuf_iterator@DU?$char_traits@D@std@@@1@0Uinput_iterator_tag@1@@Z 10012d6c     ResourceEditor.obj
 0002:00003d90       __unwindtable$??0any@tstrings@@QAE@ABV?$basic_string@DU?$char_traits@D@std@@V?$allocator@D@2@@std@@@Z 10012d90     Resources.obj
 0002:00003da0       __ehfuncinfo$??0any@tstrings@@QAE@ABV?$basic_string@DU?$char_traits@D@std@@V?$allocator@D@2@@std@@@Z 10012da0     Resources.obj
 0002:00003dc4       __unwindtable$??0Resource@@QAE@IPBGPAUHINSTANCE__@@@Z 10012dc4     Resources.obj
 0002:00003dd4       __ehfuncinfo$??0Resource@@QAE@IPBGPAUHINSTANCE__@@@Z 10012dd4     Resources.obj
 0002:00003df8       __unwindtable$?init@Resource@@AAEXPBG0PAUHINSTANCE__@@@Z 10012df8     Resources.obj
 0002:00003e08       __ehfuncinfo$?init@Resource@@AAEXPBG0PAUHINSTANCE__@@@Z 10012e08     Resources.obj
 0002:00003e2c       __unwindtable$?getErrMsg@Resource@@ABE?AV?$basic_string@DU?$char_traits@D@std@@V?$allocator@D@2@@std@@ABV23@@Z 10012e2c     Resources.obj
 0002:00003e44       __ehfuncinfo$?getErrMsg@Resource@@ABE?AV?$basic_string@DU?$char_traits@D@std@@V?$allocator@D@2@@std@@ABV23@@Z 10012e44     Resources.obj
 0002:00003e68       __ehfuncinfo$?getPtr@Resource@@ABEPAXAAK@Z 10012e68     Resources.obj
 0002:00003e8c       __unwindtable$?getPtr@Resource@@ABEPAXAAK@Z 10012e8c     Resources.obj
 0002:00003eec       __unwindtable$??$?6V?$basic_string@DU?$char_traits@D@std@@V?$allocator@D@2@@std@@@any@tstrings@@QAEAAV01@V?$basic_string@DU?$char_traits@D@std@@V?$allocator@D@2@@std@@@Z 10012eec     Resources.obj
 0002:00003efc       __ehfuncinfo$??$?6V?$basic_string@DU?$char_traits@D@std@@V?$allocator@D@2@@std@@@any@tstrings@@QAEAAV01@V?$basic_string@DU?$char_traits@D@std@@V?$allocator@D@2@@std@@@Z 10012efc     Resources.obj
 0002:00003f20       __unwindtable$?apply@VersionInfo@@QBEABV1@ABVFileLock@ResourceEditor@@@Z 10012f20     VersionInfo.obj
 0002:00003f30       __ehfuncinfo$?apply@VersionInfo@@QBEABV1@ABVFileLock@ResourceEditor@@@Z 10012f30     VersionInfo.obj
 0002:00003f54       __ehfuncinfo$?fillBuffer@VersionInfo@@ABEXAAV?$basic_ostream@DU?$char_traits@D@std@@@std@@@Z 10012f54     VersionInfo.obj
 0002:00003f78       __unwindtable$?fillBuffer@VersionInfo@@ABEXAAV?$basic_ostream@DU?$char_traits@D@std@@@std@@@Z 10012f78     VersionInfo.obj
 0002:00003fd0       __catchsym$?createFIXEDFILEINFO@VersionInfo@@ABE?AUtagVS_FIXEDFILEINFO@@XZ$6 10012fd0     VersionInfo.obj
 0002:00003fe0       __tryblocktable$?createFIXEDFILEINFO@VersionInfo@@ABE?AUtagVS_FIXEDFILEINFO@@XZ 10012fe0     VersionInfo.obj
 0002:00003ff4       __unwindtable$?createFIXEDFILEINFO@VersionInfo@@ABE?AUtagVS_FIXEDFILEINFO@@XZ 10012ff4     VersionInfo.obj
 0002:0000400c       __ehfuncinfo$?createFIXEDFILEINFO@VersionInfo@@ABE?AUtagVS_FIXEDFILEINFO@@XZ 1001300c     VersionInfo.obj
 0002:00004030       __unwindtable$??1StreamSize@?A0xcb1fbc16@@QAE@XZ 10013030     VersionInfo.obj
 0002:00004040       __tryblocktable$??1StreamSize@?A0xcb1fbc16@@QAE@XZ 10013040     VersionInfo.obj
 0002:00004054       __catchsym$??1StreamSize@?A0xcb1fbc16@@QAE@XZ$3 10013054     VersionInfo.obj
 0002:00004074       __ehfuncinfo$??1StreamSize@?A0xcb1fbc16@@QAE@XZ 10013074     VersionInfo.obj
 0002:00004098       __unwindtable$??0?$basic_stringstream@DU?$char_traits@D@std@@V?$allocator@D@2@@std@@QAE@H@Z 10013098     VersionInfo.obj
 0002:000040a8       __ehfuncinfo$??0?$basic_stringstream@DU?$char_traits@D@std@@V?$allocator@D@2@@std@@QAE@H@Z 100130a8     VersionInfo.obj
 0002:000040cc       __unwindtable$??0?$basic_stringstream@GU?$char_traits@G@std@@V?$allocator@G@2@@std@@QAE@XZ 100130cc     VersionInfo.obj
 0002:000040dc       __ehfuncinfo$??0?$basic_stringstream@GU?$char_traits@G@std@@V?$allocator@G@2@@std@@QAE@XZ 100130dc     VersionInfo.obj
 0002:00004100       __unwindtable$??$for_each@V?$_Tree_const_iterator@V?$_Tree_val@U?$_Tree_simple_types@U?$pair@$$CBV?$basic_string@GU?$char_traits@G@std@@V?$allocator@G@2@@std@@V12@@std@@@std@@@std@@@std@@V<lambda_fa730d0a4b0afd944df9b292ec615b4b>@@@std@@YA?AV<lambda_fa730d0a4b0afd944df9b292ec615b4b>@@V?$_Tree_const_iterator@V?$_Tree_val@U?$_Tree_simple_types@U?$pair@$$CBV?$basic_string@GU?$char_traits@G@std@@V?$allocator@G@2@@std@@V12@@std@@@std@@@std@@@0@0V1@@Z 10013100     VersionInfo.obj
 0002:00004108       __ehfuncinfo$??$for_each@V?$_Tree_const_iterator@V?$_Tree_val@U?$_Tree_simple_types@U?$pair@$$CBV?$basic_string@GU?$char_traits@G@std@@V?$allocator@G@2@@std@@V12@@std@@@std@@@std@@@std@@V<lambda_fa730d0a4b0afd944df9b292ec615b4b>@@@std@@YA?AV<lambda_fa730d0a4b0afd944df9b292ec615b4b>@@V?$_Tree_const_iterator@V?$_Tree_val@U?$_Tree_simple_types@U?$pair@$$CBV?$basic_string@GU?$char_traits@G@std@@V?$allocator@G@2@@std@@V12@@std@@@std@@@std@@@0@0V1@@Z 10013108     VersionInfo.obj
 0002:0000412c       __unwindtable$??0SysError@@QAE@ABVany@tstrings@@PBXKPBD@Z 1001312c     WinErrorHandling.obj
 0002:00004134       __ehfuncinfo$??0SysError@@QAE@ABVany@tstrings@@PBXKPBD@Z 10013134     WinErrorHandling.obj
 0002:00004158       __unwindtable$?getSysErrorMessage@SysError@@SA?AV?$basic_string@GU?$char_traits@G@std@@V?$allocator@G@2@@std@@KPAUHINSTANCE__@@@Z 10013158     WinErrorHandling.obj
 0002:00004168       __ehfuncinfo$?getSysErrorMessage@SysError@@SA?AV?$basic_string@GU?$char_traits@G@std@@V?$allocator@G@2@@std@@KPAUHINSTANCE__@@@Z 10013168     WinErrorHandling.obj
 0002:0000418c       __ehfuncinfo$?makeMessage@?A0xd5983087@@YA?AV?$basic_string@DU?$char_traits@D@std@@V?$allocator@D@2@@std@@ABV23@PBDPBXK@Z 1001318c     WinErrorHandling.obj
 0002:000041b0       __unwindtable$?makeMessage@?A0xd5983087@@YA?AV?$basic_string@DU?$char_traits@D@std@@V?$allocator@D@2@@std@@ABV23@PBDPBXK@Z 100131b0     WinErrorHandling.obj
 0002:000041d8       __unwindtable$?getCurrentModuleHandle@SysInfo@@YAPAUHINSTANCE__@@XZ 100131d8     WinSysInfo.obj
 0002:000041e8       __ehfuncinfo$?getCurrentModuleHandle@SysInfo@@YAPAUHINSTANCE__@@XZ 100131e8     WinSysInfo.obj
 0002:0000420c       __ehfuncinfo$??$getSystemDirImpl@P6GIPAGI@Z@?A0x7970c2a6@SysInfo@@YA?AV?$basic_string@GU?$char_traits@G@std@@V?$allocator@G@2@@std@@P6GIPAGI@ZABV?$basic_string@DU?$char_traits@D@std@@V?$allocator@D@2@@3@@Z 1001320c     WinSysInfo.obj
 0002:00004230       __unwindtable$??$getSystemDirImpl@P6GIPAGI@Z@?A0x7970c2a6@SysInfo@@YA?AV?$basic_string@GU?$char_traits@G@std@@V?$allocator@G@2@@std@@P6GIPAGI@ZABV?$basic_string@DU?$char_traits@D@std@@V?$allocator@D@2@@3@@Z 10013230     WinSysInfo.obj
 0002:00004260       __unwindtable$?getModulePath@?A0x7970c2a6@SysInfo@@YA?AV?$basic_string@GU?$char_traits@G@std@@V?$allocator@G@2@@std@@PAUHINSTANCE__@@@Z 10013260     WinSysInfo.obj
 0002:00004278       __ehfuncinfo$?getModulePath@?A0x7970c2a6@SysInfo@@YA?AV?$basic_string@GU?$char_traits@G@std@@V?$allocator@G@2@@std@@PAUHINSTANCE__@@@Z 10013278     WinSysInfo.obj
 0002:0000429c       __unwindtable$?GetLongPath@?A0x764c93a3@@YA?AV?$basic_string@GU?$char_traits@G@std@@V?$allocator@G@2@@std@@ABV23@@Z 1001329c     WindowsRegistry.obj
 0002:000042ac       __ehfuncinfo$?GetLongPath@?A0x764c93a3@@YA?AV?$basic_string@GU?$char_traits@G@std@@V?$allocator@G@2@@std@@ABV23@@Z 100132ac     WindowsRegistry.obj
 0002:000042d0       __tryblocktable$_Java_jdk_jpackage_internal_WindowsRegistry_readDwordValue@24 100132d0     WindowsRegistry.obj
 0002:000042e4       __unwindtable$_Java_jdk_jpackage_internal_WindowsRegistry_readDwordValue@24 100132e4     WindowsRegistry.obj
 0002:000042fc       __catchsym$_Java_jdk_jpackage_internal_WindowsRegistry_readDwordValue@24$7 100132fc     WindowsRegistry.obj
 0002:0000431c       __ehfuncinfo$_Java_jdk_jpackage_internal_WindowsRegistry_readDwordValue@24 1001331c     WindowsRegistry.obj
 0002:00004340       __unwindtable$_Java_jdk_jpackage_internal_WindowsRegistry_openRegistryKey@16 10013340     WindowsRegistry.obj
 0002:00004350       __tryblocktable$_Java_jdk_jpackage_internal_WindowsRegistry_openRegistryKey@16 10013350     WindowsRegistry.obj
 0002:00004364       __catchsym$_Java_jdk_jpackage_internal_WindowsRegistry_openRegistryKey@16$6 10013364     WindowsRegistry.obj
 0002:00004384       __ehfuncinfo$_Java_jdk_jpackage_internal_WindowsRegistry_openRegistryKey@16 10013384     WindowsRegistry.obj
 0002:000043a8       __tryblocktable$_Java_jdk_jpackage_internal_WindowsRegistry_enumRegistryValue@20 100133a8     WindowsRegistry.obj
 0002:000043bc       __unwindtable$_Java_jdk_jpackage_internal_WindowsRegistry_enumRegistryValue@20 100133bc     WindowsRegistry.obj
 0002:000043d4       __catchsym$_Java_jdk_jpackage_internal_WindowsRegistry_enumRegistryValue@20$5 100133d4     WindowsRegistry.obj
 0002:000043f4       __ehfuncinfo$_Java_jdk_jpackage_internal_WindowsRegistry_enumRegistryValue@20 100133f4     WindowsRegistry.obj
 0002:00004418       __tryblocktable$_Java_jdk_jpackage_internal_WindowsRegistry_comparePaths@16 10013418     WindowsRegistry.obj
 0002:0000442c       __catchsym$_Java_jdk_jpackage_internal_WindowsRegistry_comparePaths@16$15 1001342c     WindowsRegistry.obj
 0002:0000444c       __unwindtable$_Java_jdk_jpackage_internal_WindowsRegistry_comparePaths@16 1001344c     WindowsRegistry.obj
 0002:0000446c       __ehfuncinfo$_Java_jdk_jpackage_internal_WindowsRegistry_comparePaths@16 1001346c     WindowsRegistry.obj
 0002:00004490       __unwindtable$?append@StandardLogAppender@?A0xd3578678@@UAEXABULogEvent@@@Z 10013490     app.obj
 0002:000044a8       __ehfuncinfo$?append@StandardLogAppender@?A0xd3578678@@UAEXABULogEvent@@@Z 100134a8     app.obj
 0002:000044cc       __tryblocktable$_Java_jdk_jpackage_internal_ExecutableRebrander_lockResource@12 100134cc     jpackage.obj
 0002:000044e0       __unwindtable$_Java_jdk_jpackage_internal_ExecutableRebrander_lockResource@12 100134e0     jpackage.obj
 0002:000044f8       __catchsym$_Java_jdk_jpackage_internal_ExecutableRebrander_lockResource@12$6 100134f8     jpackage.obj
 0002:00004518       __ehfuncinfo$_Java_jdk_jpackage_internal_ExecutableRebrander_lockResource@12 10013518     jpackage.obj
 0002:0000453c       __unwindtable$_Java_jdk_jpackage_internal_ExecutableRebrander_unlockResource@16 1001353c     jpackage.obj
 0002:0000454c       __tryblocktable$_Java_jdk_jpackage_internal_ExecutableRebrander_unlockResource@16 1001354c     jpackage.obj
 0002:00004560       __catchsym$_Java_jdk_jpackage_internal_ExecutableRebrander_unlockResource@16$4 10013560     jpackage.obj
 0002:00004580       __ehfuncinfo$_Java_jdk_jpackage_internal_ExecutableRebrander_unlockResource@16 10013580     jpackage.obj
 0002:000045a4       __tryblocktable$_Java_jdk_jpackage_internal_ExecutableRebrander_iconSwap@20 100135a4     jpackage.obj
 0002:000045b8       __catchsym$_Java_jdk_jpackage_internal_ExecutableRebrander_iconSwap@20$7 100135b8     jpackage.obj
 0002:000045d8       __unwindtable$_Java_jdk_jpackage_internal_ExecutableRebrander_iconSwap@20 100135d8     jpackage.obj
 0002:000045f8       __ehfuncinfo$_Java_jdk_jpackage_internal_ExecutableRebrander_iconSwap@20 100135f8     jpackage.obj
 0002:0000461c       __tryblocktable$_Java_jdk_jpackage_internal_ExecutableRebrander_versionSwap@20 1001361c     jpackage.obj
 0002:00004630       __catchsym$_Java_jdk_jpackage_internal_ExecutableRebrander_versionSwap@20$12 10013630     jpackage.obj
 0002:00004650       __ehfuncinfo$_Java_jdk_jpackage_internal_ExecutableRebrander_versionSwap@20 10013650     jpackage.obj
 0002:00004674       __unwindtable$_Java_jdk_jpackage_internal_ExecutableRebrander_versionSwap@20 10013674     jpackage.obj
 0002:000046ac       __tryblocktable$_Java_jdk_jpackage_internal_WinExeBundler_embedMSI@20 100136ac     jpackage.obj
 0002:000046c0       __catchsym$_Java_jdk_jpackage_internal_WinExeBundler_embedMSI@20$24 100136c0     jpackage.obj
 0002:000046e0       __ehfuncinfo$_Java_jdk_jpackage_internal_WinExeBundler_embedMSI@20 100136e0     jpackage.obj
 0002:00004704       __unwindtable$_Java_jdk_jpackage_internal_WinExeBundler_embedMSI@20 10013704     jpackage.obj
 0002:00004774       __unwindtable$??0?$basic_istringstream@DU?$char_traits@D@std@@V?$allocator@D@2@@std@@QAE@ABV?$basic_string@DU?$char_traits@D@std@@V?$allocator@D@2@@1@H@Z 10013774     jpackage.obj
 0002:00004784       __ehfuncinfo$??0?$basic_istringstream@DU?$char_traits@D@std@@V?$allocator@D@2@@std@@QAE@ABV?$basic_string@DU?$char_traits@D@std@@V?$allocator@D@2@@1@H@Z 10013784     jpackage.obj
 0002:000047a8       __unwindtable$?unsafe_format@tstrings@@YA?AV?$basic_string@GU?$char_traits@G@std@@V?$allocator@G@2@@std@@PBGZZ 100137a8     tstrings.obj
 0002:000047b0       __ehfuncinfo$?unsafe_format@tstrings@@YA?AV?$basic_string@GU?$char_traits@G@std@@V?$allocator@G@2@@std@@PBGZZ 100137b0     tstrings.obj
 0002:000047d4       __unwindtable$?equals@tstrings@@YA_NABV?$basic_string@GU?$char_traits@G@std@@V?$allocator@G@2@@std@@0W4CompareType@1@@Z 100137d4     tstrings.obj
 0002:000047dc       __ehfuncinfo$?equals@tstrings@@YA_NABV?$basic_string@GU?$char_traits@G@std@@V?$allocator@G@2@@std@@0W4CompareType@1@@Z 100137dc     tstrings.obj
 0002:00004800       __unwindtable$?toLower@tstrings@@YA?AV?$basic_string@GU?$char_traits@G@std@@V?$allocator@G@2@@std@@ABV23@@Z 10013800     tstrings.obj
 0002:00004808       __ehfuncinfo$?toLower@tstrings@@YA?AV?$basic_string@GU?$char_traits@G@std@@V?$allocator@G@2@@std@@ABV23@@Z 10013808     tstrings.obj
 0002:0000482c       __unwindtable$?toMultiByte@?A0xf04d92fb@tstrings@@YA?AV?$basic_string@DU?$char_traits@D@std@@V?$allocator@D@2@@std@@ABV?$basic_string@GU?$char_traits@G@std@@V?$allocator@G@2@@4@H@Z 1001382c     tstrings.obj
 0002:00004834       __ehfuncinfo$?toMultiByte@?A0xf04d92fb@tstrings@@YA?AV?$basic_string@DU?$char_traits@D@std@@V?$allocator@D@2@@std@@ABV?$basic_string@GU?$char_traits@G@std@@V?$allocator@G@2@@4@H@Z 10013834     tstrings.obj
 0002:00004858       __unwindtable$?fromMultiByte@?A0xf04d92fb@tstrings@@YA?AV?$basic_string@GU?$char_traits@G@std@@V?$allocator@G@2@@std@@ABV?$basic_string@DU?$char_traits@D@std@@V?$allocator@D@2@@4@H@Z 10013858     tstrings.obj
 0002:00004860       __ehfuncinfo$?fromMultiByte@?A0xf04d92fb@tstrings@@YA?AV?$basic_string@GU?$char_traits@G@std@@V?$allocator@G@2@@std@@ABV?$basic_string@DU?$char_traits@D@std@@V?$allocator@D@2@@4@H@Z 10013860     tstrings.obj
 0002:000048e0       __sehtable$___scrt_is_nonwritable_in_current_image 100138e0     MSVCRT:utility.obj
 0002:00004900       __sehtable$?dllmain_crt_process_attach@@YAHQAUHINSTANCE__@@QAX@Z 10013900     MSVCRT:dll_dllmain.obj
 0002:00004920       __sehtable$?dllmain_crt_process_detach@@YAH_N@Z 10013920     MSVCRT:dll_dllmain.obj
 0002:00004948       __sehtable$?dllmain_dispatch@@YAHQAUHINSTANCE__@@KQAX@Z 10013948     MSVCRT:dll_dllmain.obj
 0002:00004980       .edata                     10013980     jpackage.exp
 0002:000049a8       rgpv                       100139a8     jpackage.exp
 0002:000049d0       rgszName                   100139d0     jpackage.exp
 0002:000049f8       rgwOrd                     100139f8     jpackage.exp
 0002:00004a0c       szName                     10013a0c     jpackage.exp
 0002:00004a19       $N00001                    10013a19     jpackage.exp
 0002:00004a55       $N00002                    10013a55     jpackage.exp
 0002:00004a95       $N00003                    10013a95     jpackage.exp
 0002:00004ad7       $N00004                    10013ad7     jpackage.exp
 0002:00004b16       $N00005                    10013b16     jpackage.exp
 0002:00004b4c       $N00006                    10013b4c     jpackage.exp
 0002:00004b8c       $N00007                    10013b8c     jpackage.exp
 0002:00004bc8       $N00008                    10013bc8     jpackage.exp
 0002:00004c09       $N00009                    10013c09     jpackage.exp
 0002:00004c48       $N00010                    10013c48     jpackage.exp
 0002:00006794       .idata$6                   10015794     msvcprt:MSVCP140.dll
 0002:000067c4       .idata$6                   100157c4     ole32:ole32.dll
 0002:000067ce       .idata$6                   100157ce     msi:msi.dll
 0002:00006818       .idata$6                   10015818     advapi32:ADVAPI32.dll
 0002:00006ae6       .idata$6                   10015ae6     kernel32:KERNEL32.dll
 0002:00006bd2       .idata$6                   10015bd2     vcruntime:VCRUNTIME140.dll
 0002:00006e2a       .idata$6                   10015e2a     ucrt:api-ms-win-crt-runtime-l1-1-0.dll
 0002:00006e4c       .idata$6                   10015e4c     ucrt:api-ms-win-crt-string-l1-1-0.dll
 0002:00006e6e       .idata$6                   10015e6e     ucrt:api-ms-win-crt-stdio-l1-1-0.dll
 0002:00006e8e       .idata$6                   10015e8e     ucrt:api-ms-win-crt-heap-l1-1-0.dll
 0002:00006eae       .idata$6                   10015eae     ucrt:api-ms-win-crt-filesystem-l1-1-0.dll
 0003:00000000       ?moduleName@?A0x40e1fcfd@@3PAGA 10016000     PlatformLogEvent.obj
 0003:00000208       ?nopLogAppender@?A0xd3578678@@3VNopLogAppender@@A 10016208     app.obj
 0003:0000020c       ?standardLogAppender@?A0xd3578678@@3VStandardLogAppender@1@A 1001620c     app.obj
 0003:00000210       ?lastErrorLogAppender@?A0xd3578678@@3VLastErrorLogAppender@1@A 10016210     app.obj
 0003:00000958       ??_R0?AVStandardLogAppender@?A0xd3578678@@@8 10016958     app.obj
 0003:00000988       ??_R0?AVLastErrorLogAppender@?A0xd3578678@@@8 10016988     app.obj
 0003:00000a78       ?defaultLogAppenderMemory@?A0xc7174dad@@3PADA 10016a78     Log.obj
 0003:00000a80       ?defaultLoggerMemory@?A0xc7174dad@@3PADA 10016a80     Log.obj
 0003:00000a88       ?state@?A0xc7174dad@@3W4State@1@A 10016a88     Log.obj
 0003:00000aa0       ?theLastErrorMsg@?A0xd3578678@@3PBV?$basic_string@DU?$char_traits@D@std@@V?$allocator@D@2@@std@@B 10016aa0     app.obj
 0003:00000aa4       ?_Fac_head@std@@3PAU_Fac_node@1@A 10016aa4     msvcprt:locale0_implib.obj
 0003:00000aa8       ?_Fac_tidy_reg@std@@3U_Fac_tidy_reg_t@1@B 10016aa8     msvcprt:locale0_implib.obj
 0003:00000ab0       _GS_ExceptionRecord        10016ab0     MSVCRT:gs_report.obj
 0003:00000b00       _GS_ContextRecord          10016b00     MSVCRT:gs_report.obj
 0003:00000dd4       ?is_initialized_as_dll@@3_NA 10016dd4     MSVCRT:utility.obj
 0003:00000dd5       ?module_local_atexit_table_initialized@@3_NA 10016dd5     MSVCRT:utility.obj
 0003:00000dd8       ?module_local_atexit_table@@3U_onexit_table_t@@A 10016dd8     MSVCRT:utility.obj
 0003:00000de4       ?module_local_at_quick_exit_table@@3U_onexit_table_t@@A 10016de4     MSVCRT:utility.obj
 0003:00000df0       ?__proc_attached@@3HA      10016df0     MSVCRT:dll_dllmain.obj
 0004:00000060       $R000000                   10017060     jpackage.dll.res
